** EXPERIMENTAL (HLL) ** Open Watcom Linker Version 1.6beta1 Limited Availability
Portions Copyright (c) 1985-2002 Sybase, Inc. All Rights Reserved.
Created on:       11/04/07 09:03:48
Executable Image: .libs/php5.dll
creating an OS/2 EMX dynamic link library


                        +------------+
                        |   Groups   |
                        +------------+

Group                           Address              Size
=====                           =======              ====

CGROUP                          0001:00000000        007a6440
DGROUP                          0002:00000000        000244e0



                        +--------------+
                        |   Segments   |
                        +--------------+

Segment                Class          Group          Address         Size
=======                =====          =====          =======         ====

TEXT32                 CODE           CGROUP         0001:00000000   007a6440
________TEXT           CODE           CGROUP         0001:007a6440   00000000
DATA32                 DATA           DGROUP         0002:00000000   0000b090
SET1__os2dll           DATA           DGROUP         0002:0000b090   00000004
SET2__os2dll           DATA           DGROUP         0002:0000b094   00000000
SET3__os2dll           DATA           DGROUP         0002:0000b094   00000004
SET1___CTOR_LIST__     DATA           DGROUP         0002:0000b098   00000004
SET2___CTOR_LIST__     DATA           DGROUP         0002:0000b09c   00000000
SET3___CTOR_LIST__     DATA           DGROUP         0002:0000b09c   00000004
SET1___DTOR_LIST__     DATA           DGROUP         0002:0000b0a0   00000004
SET2___DTOR_LIST__     DATA           DGROUP         0002:0000b0a4   00000000
SET3___DTOR_LIST__     DATA           DGROUP         0002:0000b0a4   00000004
SET1___crtinit1__      DATA           DGROUP         0002:0000b0a8   00000004
SET2___crtinit1__      DATA           DGROUP         0002:0000b0ac   00000000
SET3___crtinit1__      DATA           DGROUP         0002:0000b0ac   00000004
SET1___crtexit1__      DATA           DGROUP         0002:0000b0b0   00000004
SET2___crtexit1__      DATA           DGROUP         0002:0000b0b4   00000000
SET3___crtexit1__      DATA           DGROUP         0002:0000b0b4   00000004
SET1___eh_frame__      DATA           DGROUP         0002:0000b0b8   00000004
SET2___eh_frame__      DATA           DGROUP         0002:0000b0bc   00000010
SET3___eh_frame__      DATA           DGROUP         0002:0000b0cc   00000004
SET1___eh_init__       DATA           DGROUP         0002:0000b0d0   00000004
SET2___eh_init__       DATA           DGROUP         0002:0000b0d4   00000004
SET3___eh_init__       DATA           DGROUP         0002:0000b0d8   00000004
SET1___eh_term__       DATA           DGROUP         0002:0000b0dc   00000004
SET2___eh_term__       DATA           DGROUP         0002:0000b0e0   00000004
SET3___eh_term__       DATA           DGROUP         0002:0000b0e4   00000004
SET1___fork_parent1__  DATA           DGROUP         0002:0000b0e8   00000004
SET2___fork_parent1__  DATA           DGROUP         0002:0000b0ec   00000000
SET3___fork_parent1__  DATA           DGROUP         0002:0000b0ec   00000004
SET1___fork_child1__   DATA           DGROUP         0002:0000b0f0   00000004
SET2___fork_child1__   DATA           DGROUP         0002:0000b0f4   00000004
SET3___fork_child1__   DATA           DGROUP         0002:0000b0f8   00000004
________DATA           DATA           DGROUP         0002:0000b100   00000000
BSS32                  BSS            DGROUP         0002:0000b100   00017140
c_common               BSS            DGROUP         0002:00022240   000022a0
________BSS            BSS            DGROUP         0002:000244e0   00000000


                        +----------------+
                        |   Memory Map   |
                        +----------------+

* = unreferenced symbol
+ = symbol only referenced locally

Address        Symbol
=======        ======

Module: U:\usr\lib\dll0.obj({standard input})
0001:00000000* __text
0002:00000000* __data
0002:00000000* ___data_start
0002:0000b100* ___bss_start
0002:0000b090+ __os2dll
0002:0000b098  ___CTOR_LIST__
0002:0000b0a0  ___DTOR_LIST__
0002:0000b0a8* ___crtinit1__
0002:0000b0b0* ___crtexit1__
0002:0000b0b8  ___eh_frame__
0002:0000b0d0  ___eh_init__
0002:0000b0dc  ___eh_term__
0002:0000b0e8+ ___fork_parent1__
0002:0000b0f0+ ___fork_child1__
Module: U:\dev\php-5.3.6\ext\date\php_date.o(php_date.o)
0002:00022240  _date_globals_id
0002:00022250  _date_ce_date
0002:00022260  _date_ce_timezone
0002:00022270  _php_date_global_timezone_db
0002:00022280  _php_date_global_timezone_db_enabled
0002:00022290  _date_ce_interval
0002:000222a0  _date_ce_period
0001:00001a40  _date_functions
0001:00004244  _zif_strtotime
0001:00004044  _zif_date
0001:000040c4  _zif_idate
0001:00004068  _zif_gmdate
0001:00004728  _zif_mktime
0001:0000474c  _zif_gmmktime
0001:00004774  _zif_checkdate
0001:000049ec  _zif_strftime
0001:00004a10  _zif_gmstrftime
0001:00004a34  _zif_time
0001:00004a9c  _zif_localtime
0001:00004ce4  _zif_getdate
0001:00006b24  _zif_date_create
0001:00006bbc  _zif_date_create_from_format
0001:000076e4  _zif_date_parse
0001:00007760  _zif_date_parse_from_format
0001:00007140  _zif_date_get_last_errors
0001:0000783c  _zif_date_format
0001:000078dc  _zif_date_modify
0001:00007bcc  _zif_date_add
0001:00007f34  _zif_date_sub
0001:00008260  _zif_date_timezone_get
0001:00008390  _zif_date_timezone_set
0001:00008494  _zif_date_offset_get
0001:00008a40  _zif_date_diff
0001:00008590  _zif_date_time_set
0001:0000868c  _zif_date_date_set
0001:0000877c  _zif_date_isodate_set
0001:000088d4  _zif_date_timestamp_set
0001:000089a0  _zif_date_timestamp_get
0001:00008bf0  _zif_timezone_open
0001:00008d64  _zif_timezone_name_get
0001:00008ebc  _zif_timezone_name_from_abbr
0001:00008f4c  _zif_timezone_offset_get
0001:0000905c  _zif_timezone_transitions_get
0001:000096c0  _zif_timezone_location_get
0001:0000ac2c  _zif_timezone_identifiers_list
0001:0000adc4  _zif_timezone_abbreviations_list
0001:0000ad6c  _zif_timezone_version_get
0001:00009f8c  _zif_date_interval_create_from_date_string
0001:0000a448  _zif_date_interval_format
0001:0000af90  _zif_date_default_timezone_set
0001:0000b070  _zif_date_default_timezone_get
0001:0000b454  _zif_date_sunrise
0001:0000b478  _zif_date_sunset
0001:0000b540  _zif_date_sun_info
0001:00001ea0  _date_funcs_date
0001:00006c68  _zim_DateTime___construct
0001:00006fc8  _zim_DateTime___wakeup
0001:00006f34  _zim_DateTime___set_state
0001:00002080  _date_funcs_timezone
0001:00008c7c  _zim_DateTimeZone___construct
0001:00002140  _date_funcs_interval
0001:00009ef8  _zim_DateInterval___construct
0001:000021a0  _date_funcs_period
0001:0000a6cc  _zim_DatePeriod___construct
0001:000023c8  _php_date_get_date_ce
0001:000023d4  _php_date_get_timezone_ce
0001:00002640  _zm_startup_date
0001:000027d8  _zm_shutdown_date
0001:00002424  _zm_activate_date
0001:00002478  _zm_deactivate_date
0001:00002888  _zm_info_date
0001:00002ce8  _get_timezone_info
0001:00002eb8  _php_date_full_day_name
0001:00002eec  _php_date_short_day_name
0001:00003b40  _php_format_date
0001:00003bb4  _php_idate
0001:00004164  _php_date_set_tzdb
0001:0000419c  _php_parse_date
0001:0000449c  _php_mktime
0001:000047e8  _php_strftime
0001:000067d4  _php_date_instantiate
0001:00005110  _date_object_period_get_iterator
0001:000098c8  _date_interval_read_property
0001:00009af4  _date_interval_write_property
0001:00006890  _php_date_initialize
0001:00007214  _php_date_do_return_parsed_time
0002:00000050  _date_module_entry
0002:00000158  _date_period_it_funcs
Module: U:\dev\php-5.3.6\ext\date\lib\astro.o(astro.o)
0001:0000bd90  _timelib_astro_rise_set_altitude
0001:0000c13c  _timelib_ts_to_juliandate
Module: U:\dev\php-5.3.6\ext\date\lib\dow.o(dow.o)
0001:0000c2d4  _timelib_day_of_week
0001:0000c2f8  _timelib_iso_day_of_week
0001:0000c31c  _timelib_day_of_year
0001:0000c3a4  _timelib_days_in_month
0001:0000c414  _timelib_isoweek_from_date
0001:0000c688  _timelib_daynr_from_weeknr
0001:0000c710  _timelib_valid_time
0001:0000c75c  _timelib_valid_date
Module: U:\dev\php-5.3.6\ext\date\lib\parse_date.o(parse_date.o)
0001:00030c34  _timelib_strtotime
0001:00031274  _timelib_parse_from_format
0001:00032038  _timelib_fill_holes
0001:000322d8  _timelib_timezone_id_from_abbr
0001:000322fc  _timelib_timezone_abbreviations_list
Module: U:\dev\php-5.3.6\ext\date\lib\parse_tz.o(parse_tz.o)
0001:00034510  _timezonedb_idx_builtin
0001:000356f0  _timelib_timezone_db_data_builtin
0001:000758c8  _timezonedb_builtin
0001:00076050  _timelib_dump_tzinfo
0001:000762e4  _timelib_builtin_db
0001:000762f0  _timelib_timezone_builtin_identifiers_list
0001:00076304  _timelib_timezone_id_is_valid
0001:0007631c  _timelib_parse_tzfile
0001:000764e8  _timelib_timestamp_is_in_dst
0001:00076514  _timelib_get_time_zone_info
0001:000765e4  _timelib_get_current_offset
Module: U:\dev\php-5.3.6\ext\date\lib\timelib.o(timelib.o)
0001:00076650  _timelib_time_ctor
0001:00076664  _timelib_rel_time_ctor
0001:00076678  _timelib_time_clone
0001:000766cc  _timelib_rel_time_clone
0001:000766e8  _timelib_time_tz_abbr_update
0001:00076788  _timelib_time_dtor
0001:000767c4  _timelib_rel_time_dtor
0001:000767e0  _timelib_time_offset_ctor
0001:000767f4  _timelib_time_offset_dtor
0001:00076830  _timelib_tzinfo_ctor
0001:00076854  _timelib_tzinfo_clone
0001:00076954  _timelib_tzinfo_dtor
0001:00076a54  _timelib_get_tz_abbr_ptr
0001:00076a80  _timelib_error_container_dtor
0001:00076b00  _timelib_date_to_int
0001:00076b50  _timelib_decimal_hour_to_hms
0001:00076ce8  _timelib_dump_date
0001:00076fcc  _timelib_dump_rel_time
Module: U:\dev\php-5.3.6\ext\date\lib\tm2unixtime.o(tm2unixtime.o)
0001:00077814  _timelib_do_rel_normalize
0001:000782d8  _timelib_update_ts
Module: U:\dev\php-5.3.6\ext\date\lib\unixtime2tm.o(unixtime2tm.o)
0001:000783b0  _timelib_unixtime2gmt
0001:000788a0  _timelib_update_from_sse
0001:00078984  _timelib_unixtime2local
0001:00078a74  _timelib_set_timezone
0001:00078af4  _timelib_apply_localtime
Module: U:\dev\php-5.3.6\ext\date\lib\parse_iso_intervals.o(parse_iso_intervals.o)
0001:00079da4  _timelib_strtointerval
Module: U:\dev\php-5.3.6\ext\date\lib\interval.o(interval.o)
0001:0007a130  _timelib_diff
Module: U:\dev\php-5.3.6\ext\ereg\ereg.o(ereg.o)
0002:000222b0  _ereg_globals_id
0001:0007a610  _ereg_functions
0001:0007aedc  _zif_ereg
0001:0007b628  _zif_ereg_replace
0001:0007af00  _zif_eregi
0001:0007b64c  _zif_eregi_replace
0001:0007b81c  _zif_split
0001:0007b840  _zif_spliti
0001:0007b864  _zif_sql_regcase
0001:0007a92c  _zm_startup_ereg
0001:0007a94c  _zm_shutdown_ereg
0001:0007a97c  _zm_info_ereg
0001:0007af24  _php_ereg_replace
0002:00000490  _ereg_module_entry
Module: U:\dev\php-5.3.6\ext\ereg\regex\regcomp.o(regcomp.o)
0001:0007c270  _php_regcomp
Module: U:\dev\php-5.3.6\ext\ereg\regex\regexec.o(regexec.o)
0001:000814d0  _php_regexec
Module: U:\dev\php-5.3.6\ext\ereg\regex\regerror.o(regerror.o)
0001:000818c4  _php_regerror
Module: U:\dev\php-5.3.6\ext\ereg\regex\regfree.o(regfree.o)
0001:00081a00  _php_regfree
Module: U:\dev\php-5.3.6\ext\libxml\libxml.o(libxml.o)
0001:000834f0  _php_libxml_decrement_node_ptr
0001:0008359c  _php_libxml_decrement_doc_ref
0001:00082468  _php_libxml_issue_error
0001:00082694  _php_libxml_ctx_error
0001:000826b0  _php_libxml_ctx_warning
0001:000826cc  _php_libxml_structured_error_handler
0001:000826e4  _php_libxml_error_handler
0001:00082700  _php_libxml_initialize
0001:00082740  _php_libxml_shutdown
0001:0008277c  _php_libxml_switch_context
0001:00083308  _php_libxml_xmlCheckUTF8
0001:000833b0  _php_libxml_register_export
0001:000833e8  _php_libxml_import_node
0001:0008345c  _php_libxml_increment_node_ptr
0001:00083540  _php_libxml_increment_doc_ref
0001:00083634  _php_libxml_node_free_resource
0001:00083728  _php_libxml_node_decrement_resource
0002:000004f0  _libxml_module_entry
Module: U:\dev\php-5.3.6\ext\pcre\pcrelib\pcre_chartables.o(pcre_chartables.o)
0001:000837c0  _php__pcre_default_tables
Module: U:\dev\php-5.3.6\ext\pcre\pcrelib\pcre_ucd.o(pcre_ucd.o)
0001:00083c00  _php__pcre_ucd_records
0001:00084c40  _php__pcre_ucd_stage1
0001:00086e40  _php__pcre_ucd_stage2
Module: U:\dev\php-5.3.6\ext\pcre\pcrelib\pcre_compile.o(pcre_compile.o)
0001:00093b5c  __pcre_find_bracket
0001:0009adfc  _php_pcre_compile
0001:0009ae6c  _php_pcre_compile2
Module: U:\dev\php-5.3.6\ext\pcre\pcrelib\pcre_config.o(pcre_config.o)
0001:0009b860  _php_pcre_config
Module: U:\dev\php-5.3.6\ext\pcre\pcrelib\pcre_exec.o(pcre_exec.o)
0001:000b15b0  _php_pcre_exec
Module: U:\dev\php-5.3.6\ext\pcre\pcrelib\pcre_fullinfo.o(pcre_fullinfo.o)
0001:000b24c0  _php_pcre_fullinfo
Module: U:\dev\php-5.3.6\ext\pcre\pcrelib\pcre_get.o(pcre_get.o)
0001:000b2650  _php_pcre_get_stringnumber
0001:000b270c  _php_pcre_get_stringtable_entries
0001:000b28d0  _php_pcre_copy_substring
0001:000b2928  _php_pcre_copy_named_substring
0001:000b2988  _php_pcre_get_substring_list
0001:000b2a38  _php_pcre_free_substring_list
0001:000b2a4c  _php_pcre_get_substring
0001:000b2abc  _php_pcre_get_named_substring
0001:000b2b10  _php_pcre_free_substring
Module: U:\dev\php-5.3.6\ext\pcre\pcrelib\pcre_globals.o(pcre_globals.o)
0002:000005f0  _php_pcre_malloc
0002:000005f4  _php_pcre_free
0002:000005f8  _php_pcre_stack_malloc
0002:000005fc  _php_pcre_stack_free
0002:0000b340  _php_pcre_callout
Module: U:\dev\php-5.3.6\ext\pcre\pcrelib\pcre_info.o(pcre_info.o)
0001:000b2b30  _php_pcre_info
Module: U:\dev\php-5.3.6\ext\pcre\pcrelib\pcre_maketables.o(pcre_maketables.o)
0001:000b2bc0  _php_pcre_maketables
Module: U:\dev\php-5.3.6\ext\pcre\pcrelib\pcre_newline.o(pcre_newline.o)
0001:000b30e0  _php__pcre_is_newline
0001:000b3268  _php__pcre_was_newline
Module: U:\dev\php-5.3.6\ext\pcre\pcrelib\pcre_ord2utf8.o(pcre_ord2utf8.o)
0001:000b3420  _php__pcre_ord2utf8
Module: U:\dev\php-5.3.6\ext\pcre\pcrelib\pcre_refcount.o(pcre_refcount.o)
0001:000b3480  _php_pcre_refcount
Module: U:\dev\php-5.3.6\ext\pcre\pcrelib\pcre_study.o(pcre_study.o)
0001:000b440c  _php_pcre_study
Module: U:\dev\php-5.3.6\ext\pcre\pcrelib\pcre_tables.o(pcre_tables.o)
0001:000b45e0  _php__pcre_OP_lengths
0001:000b4658  _php__pcre_utf8_table1
0001:000b4670  _php__pcre_utf8_table1_size
0001:000b4674  _php__pcre_utf8_table2
0001:000b468c  _php__pcre_utf8_table3
0001:000b46c0  _php__pcre_utf8_table4
0001:000b4700  _php__pcre_ucp_gentype
0001:000b4780  _php__pcre_utt_names
0001:000b4b40  _php__pcre_utt
0001:000b4e6c  _php__pcre_utt_size
Module: U:\dev\php-5.3.6\ext\pcre\pcrelib\pcre_try_flipped.o(pcre_try_flipped.o)
0001:000b4ec4  _php__pcre_try_flipped
Module: U:\dev\php-5.3.6\ext\pcre\pcrelib\pcre_valid_utf8.o(pcre_valid_utf8.o)
0001:000b5030  _php__pcre_valid_utf8
Module: U:\dev\php-5.3.6\ext\pcre\pcrelib\pcre_version.o(pcre_version.o)
0001:000b5190  _php_pcre_version
Module: U:\dev\php-5.3.6\ext\pcre\pcrelib\pcre_xclass.o(pcre_xclass.o)
0001:000b51a0  _php__pcre_xclass
Module: U:\dev\php-5.3.6\ext\pcre\php_pcre.o(php_pcre.o)
0002:000222c0  _pcre_globals_id
0001:000b5e60  _pcre_get_compiled_regex_cache
0001:000b6490  _pcre_get_compiled_regex
0001:000b64f0  _pcre_get_compiled_regex_ex
0001:000b6684  _php_pcre_match_impl
0001:000b7640  _php_pcre_replace
0001:000b76f8  _php_pcre_replace_impl
0001:000b8778  _php_pcre_split_impl
0001:000b8fe8  _php_pcre_grep_impl
0002:00000600  _pcre_module_entry
Module: U:\dev\php-5.3.6\ext\sqlite3\sqlite3.o(sqlite3.o)
0002:000222d0  _sqlite3_globals_id
0002:000222e0  _php_sqlite3_stmt_entry
0002:000222f0  _php_sqlite3_result_entry
0002:00022300  _php_sqlite3_sc_entry
0001:000b9de0  _zim_sqlite3_open
0001:000ba05c  _zim_sqlite3_close
0001:000ba130  _zim_sqlite3_exec
0001:000ba1fc  _zim_sqlite3_version
0001:000ba270  _zim_sqlite3_lastInsertRowID
0001:000ba2dc  _zim_sqlite3_lastErrorCode
0001:000ba348  _zim_sqlite3_lastErrorMsg
0001:000ba3f8  _zim_sqlite3_busyTimeout
0001:000ba56c  _zim_sqlite3_loadExtension
0001:000ba7ec  _zim_sqlite3_changes
0001:000ba85c  _zim_sqlite3_escapeString
0001:000ba920  _zim_sqlite3_prepare
0001:000baa74  _zim_sqlite3_query
0001:000badf4  _zim_sqlite3_querySingle
0001:000bb6ac  _zim_sqlite3_createFunction
0001:000bb830  _zim_sqlite3_createAggregate
0001:000bbc18  _zim_sqlite3_openBlob
0001:000bbd30  _zim_sqlite3_enableExceptions
0001:000bbd84  _zim_sqlite3stmt_paramCount
0001:000bbdd0  _zim_sqlite3stmt_close
0001:000bbe48  _zim_sqlite3stmt_reset
0001:000bbef0  _zim_sqlite3stmt_clear
0001:000bbf78  _zim_sqlite3stmt_readOnly
0001:000bc0fc  _zim_sqlite3stmt_bindParam
0001:000bc1e4  _zim_sqlite3stmt_bindValue
0001:000bc320  _zim_sqlite3stmt_execute
0001:000bc640  _zim_sqlite3stmt___construct
0001:000bc7dc  _zim_sqlite3result_numColumns
0001:000bc854  _zim_sqlite3result_columnName
0001:000bc8fc  _zim_sqlite3result_columnType
0001:000bc988  _zim_sqlite3result_fetchArray
0001:000bcaf8  _zim_sqlite3result_reset
0001:000bcb84  _zim_sqlite3result_finalize
0001:000bcc50  _zim_sqlite3result___construct
0001:000bda60  _zm_startup_sqlite3
0001:000bdef0  _zm_shutdown_sqlite3
0001:000bdf4c  _zm_info_sqlite3
0002:000009c0  _sqlite3_module_entry
Module: U:\dev\php-5.3.6\ext\sqlite3\libsqlite\sqlite3.o(sqlite3.o)
0001:000bdfe0  _sqlite3_version
0001:000be308  _sqlite3_compileoption_used
0001:000c3ff0  _sqlite3_strnicmp
0001:000be37c  _sqlite3_compileoption_get
0001:000be3f0  _sqlite3_status
0001:000be440  _sqlite3_db_status
0001:000c0e90  _sqlite3_mutex_enter
0001:000c0ec8  _sqlite3_mutex_leave
0001:000c3470  _sqlite3_snprintf
0001:000c18b0  _sqlite3_free
0001:000c1684  _sqlite3_malloc
0001:000c6d2c  _sqlite3_os_init
0001:000c0a80  _sqlite3_vfs_find
0001:000c0b4c  _sqlite3_vfs_register
0001:000c0bc0  _sqlite3_vfs_unregister
0001:000c3508  _sqlite3_log
0001:000c0e2c  _sqlite3_mutex_alloc
0001:000c0e74  _sqlite3_mutex_free
0001:000c0eac  _sqlite3_mutex_try
0001:000c11f0  _sqlite3_release_memory
0001:000c1288  _sqlite3_memory_alarm
0001:000c1294  _sqlite3_soft_heap_limit64
0001:000c14a4  _sqlite3_memory_used
0001:000c1310  _sqlite3_soft_heap_limit
0001:000c14c4  _sqlite3_memory_highwater
0001:000c1b04  _sqlite3_realloc
0001:000c33ec  _sqlite3_vmprintf
0001:000c3448  _sqlite3_mprintf
0001:000c3640  _sqlite3_randomness
0001:000c60f4  _convertCpPathToUtf8
0001:000c6bdc  _os2CurrentTime
0001:000c6d48  _sqlite3_os_end
0001:000dd6cc  _sqlite3_context_db_handle
0001:000dd008  _sqlite3_value_text
0001:000dd058  _sqlite3_value_type
0001:000dcfe0  _sqlite3_value_double
0001:000dd0bc  _sqlite3_result_double
0001:000dd160  _sqlite3_result_text
0001:000dd24c  _sqlite3_result_error_toobig
0001:000dd274  _sqlite3_result_error_nomem
0001:001147a8  _sqlite3_initialize
0001:001149f4  _sqlite3_config
0001:000cf778  _sqlite3_enable_shared_cache
0001:000d827c  _sqlite3_backup_init
0001:000d85c4  _sqlite3_backup_step
0001:000d8b48  _sqlite3_backup_finish
0001:000d8c58  _sqlite3_backup_remaining
0001:000d8c64  _sqlite3_backup_pagecount
0001:000da018  _sqlite3_sql
0001:000dcd50  _sqlite3_expired
0001:000dce18  _sqlite3_finalize
0001:000dce8c  _sqlite3_reset
0001:000dceec  _sqlite3_clear_bindings
0001:000dcf6c  _sqlite3_value_blob
0001:000dcfb8  _sqlite3_value_bytes
0001:000dcfcc  _sqlite3_value_bytes16
0001:000dcfec  _sqlite3_value_int
0001:000dcffc  _sqlite3_value_int64
0001:000dd01c  _sqlite3_value_text16
0001:000dd030  _sqlite3_value_text16be
0001:000dd044  _sqlite3_value_text16le
0001:000dd0a0  _sqlite3_result_blob
0001:000dd0d0  _sqlite3_result_error
0001:000dd0f8  _sqlite3_result_error16
0001:000dd120  _sqlite3_result_int
0001:000dd13c  _sqlite3_result_int64
0001:000dd150  _sqlite3_result_null
0001:000dd17c  _sqlite3_result_text16
0001:000dd198  _sqlite3_result_text16be
0001:000dd1b4  _sqlite3_result_text16le
0001:000dd1d0  _sqlite3_result_value
0001:000dd1e4  _sqlite3_result_zeroblob
0001:000dd1f8  _sqlite3_result_error_code
0001:000dd598  _sqlite3_step
0001:000dd6bc  _sqlite3_user_data
0001:000dd748  _sqlite3_aggregate_context
0001:000dd7c4  _sqlite3_get_auxdata
0001:000dd7e8  _sqlite3_set_auxdata
0001:000dd8a8  _sqlite3_aggregate_count
0001:000dd8b8  _sqlite3_column_count
0001:000dd8cc  _sqlite3_data_count
0001:000dd9d8  _sqlite3_column_blob
0001:000dda08  _sqlite3_column_bytes
0001:000dda38  _sqlite3_column_bytes16
0001:000dda68  _sqlite3_column_double
0001:000ddaa8  _sqlite3_column_int
0001:000ddad8  _sqlite3_column_int64
0001:000ddb10  _sqlite3_column_text
0001:000ddb40  _sqlite3_column_value
0001:000ddb80  _sqlite3_column_text16
0001:000ddbb0  _sqlite3_column_type
0001:000ddc68  _sqlite3_column_name
0001:000ddc84  _sqlite3_column_name16
0001:000ddca0  _sqlite3_column_decltype
0001:000ddcbc  _sqlite3_column_decltype16
0001:000ddcd8  _sqlite3_column_database_name
0001:000ddcf4  _sqlite3_column_database_name16
0001:000ddd10  _sqlite3_column_table_name
0001:000ddd2c  _sqlite3_column_table_name16
0001:000ddd48  _sqlite3_column_origin_name
0001:000ddd64  _sqlite3_column_origin_name16
0001:000ddf94  _sqlite3_bind_blob
0001:000ddfb4  _sqlite3_bind_double
0001:000de010  _sqlite3_bind_int
0001:000de02c  _sqlite3_bind_int64
0001:000de088  _sqlite3_bind_null
0001:000de0c4  _sqlite3_bind_text
0001:000de0e4  _sqlite3_bind_text16
0001:000de104  _sqlite3_bind_value
0001:000de19c  _sqlite3_bind_zeroblob
0001:000de1f0  _sqlite3_bind_parameter_count
0001:000de278  _sqlite3_bind_parameter_name
0001:000de334  _sqlite3_bind_parameter_index
0001:000de3c0  _sqlite3_transfer_bindings
0001:000de414  _sqlite3_db_handle
0001:000de424  _sqlite3_stmt_readonly
0001:000de43c  _sqlite3_next_stmt
0001:000de478  _sqlite3_stmt_status
0001:000de9a8  _sqlite3_value_numeric_type
0001:000fa7e8  _sqlite3_exec
0001:00115e44  _sqlite3_errmsg
0001:000e59b0  _sqlite3_blob_open
0001:000e5eb0  _sqlite3_blob_close
0001:000e6008  _sqlite3_blob_read
0001:000e6028  _sqlite3_blob_write
0001:000e6048  _sqlite3_blob_bytes
0001:000e6064  _sqlite3_blob_reopen
0001:000eec28  _sqlite3_set_authorizer
0001:00114dec  _sqlite3_last_insert_rowid
0001:00114dfc  _sqlite3_changes
0001:00114e08  _sqlite3_total_changes
0001:00114738  _sqlite3_libversion
0001:00114784  _sqlite3_sourceid
0001:000fb0c4  _sqlite3_load_extension
0001:00115ae8  _sqlite3_overload_function
0001:000fead4  _sqlite3_prepare
0001:00116020  _sqlite3_errcode
0001:00115660  _sqlite3_busy_handler
0001:00115710  _sqlite3_busy_timeout
0001:00114f14  _sqlite3_close
0001:001168f8  _sqlite3_collation_needed
0001:00116938  _sqlite3_collation_needed16
0001:00115be4  _sqlite3_commit_hook
0001:00114264  _sqlite3_complete
0001:001146c4  _sqlite3_complete16
0001:001167e8  _sqlite3_create_collation
0001:00116884  _sqlite3_create_collation16
0001:0011599c  _sqlite3_create_function
0001:00115a7c  _sqlite3_create_function16
0001:001079d0  _sqlite3_create_module
0001:001084c0  _sqlite3_declare_vtab
0001:00115f70  _sqlite3_errmsg16
0001:00104828  _sqlite3_free_table
0001:00116980  _sqlite3_get_autocommit
0001:00104684  _sqlite3_get_table
0001:00115744  _sqlite3_interrupt
0001:00114790  _sqlite3_libversion_number
0001:00116718  _sqlite3_open
0001:0011673c  _sqlite3_open16
0001:000febec  _sqlite3_prepare16
0001:00115ba4  _sqlite3_profile
0001:001156a0  _sqlite3_progress_handler
0001:00115c64  _sqlite3_rollback_hook
0001:00116a98  _sqlite3_table_column_metadata
0001:00116a74  _sqlite3_thread_cleanup
0001:00115b64  _sqlite3_trace
0001:00115c24  _sqlite3_update_hook
0001:000feaf4  _sqlite3_prepare_v2
0001:000fec0c  _sqlite3_prepare16_v2
0001:001079ec  _sqlite3_create_module_v2
0001:00116834  _sqlite3_create_collation_v2
0001:00116d80  _sqlite3_file_control
0001:00116730  _sqlite3_open_v2
0001:00116cf8  _sqlite3_sleep
0001:0011479c  _sqlite3_threadsafe
0001:00116e60  _sqlite3_test_control
0001:00116d4c  _sqlite3_extended_result_codes
0001:001162ac  _sqlite3_limit
0001:001159c4  _sqlite3_create_function_v2
0001:00114cd8  _sqlite3_db_config
0001:00114ccc  _sqlite3_db_mutex
0001:00116068  _sqlite3_extended_errcode
0001:00115cd8  _sqlite3_wal_autocheckpoint
0001:00115d58  _sqlite3_wal_checkpoint
0001:00115d04  _sqlite3_wal_hook
0001:000fb150  _sqlite3_enable_load_extension
0001:000fb194  _sqlite3_auto_extension
0001:000fb234  _sqlite3_reset_auto_extension
0001:00114970  _sqlite3_shutdown
0001:00116978  _sqlite3_global_recover
0002:0000b4a0  _sqlite3_temp_directory
Module: U:\dev\php-5.3.6\ext\zlib\zlib.o(zlib.o)
0002:00022310  _zlib_globals_id
0001:0012522c  _php_ob_gzhandler_check
0002:000014c0  _php_zlib_module_entry
Module: U:\dev\php-5.3.6\ext\zlib\zlib_fopen_wrapper.o(zlib_fopen_wrapper.o)
0001:00125c5c  _php_stream_gzopen
0002:00001588  _php_stream_gzip_wrapper
Module: U:\dev\php-5.3.6\ext\zlib\zlib_filter.o(zlib_filter.o)
0002:000015b8  _php_zlib_filter_factory
Module: U:\dev\php-5.3.6\ext\ctype\ctype.o(ctype.o)
0002:000015c0  _ctype_module_entry
Module: U:\dev\php-5.3.6\ext\dom\php_dom.o(php_dom.o)
0002:00022320  _dom_node_class_entry
0002:00022330  _dom_object_handlers
0002:000223a0  _dom_domexception_class_entry
0002:000223b0  _dom_domstringlist_class_entry
0002:000223c0  _dom_namelist_class_entry
0002:000223d0  _dom_domimplementationlist_class_entry
0002:000223e0  _dom_domimplementationsource_class_entry
0002:000223f0  _dom_domimplementation_class_entry
0002:00022400  _dom_namespace_node_class_entry
0002:00022410  _dom_documentfragment_class_entry
0002:00022420  _dom_document_class_entry
0002:00022430  _dom_nodelist_class_entry
0002:00022440  _dom_namednodemap_class_entry
0002:00022450  _dom_characterdata_class_entry
0002:00022460  _dom_attr_class_entry
0002:00022470  _dom_element_class_entry
0002:00022480  _dom_text_class_entry
0002:00022490  _dom_comment_class_entry
0002:000224a0  _dom_typeinfo_class_entry
0002:000224b0  _dom_userdatahandler_class_entry
0002:000224c0  _dom_domerror_class_entry
0002:000224d0  _dom_domerrorhandler_class_entry
0002:000224e0  _dom_domlocator_class_entry
0002:000224f0  _dom_domconfiguration_class_entry
0002:00022500  _dom_cdatasection_class_entry
0002:00022510  _dom_documenttype_class_entry
0002:00022520  _dom_notation_class_entry
0002:00022530  _dom_entity_class_entry
0002:00022540  _dom_entityreference_class_entry
0002:00022550  _dom_processinginstruction_class_entry
0002:00022560  _dom_string_extend_class_entry
0002:00022570  _dom_xpath_class_entry
0001:001283dc  _dom_node_is_read_only
0001:00128440  _dom_node_children_valid
0001:00128498  _dom_get_doc_props
0001:0012859c  _dom_set_doc_classmap
0001:00128638  _dom_get_doc_classmap
0001:00128690  _dom_get_strict_error
0001:001286c4  _dom_object_get_node
0001:001286e0  _php_dom_object_get_data
0001:001288d4  _dom_read_property
0001:00128a24  _dom_write_property
0001:00128c48  _php_dom_export_node
0001:00128cb4  _zif_dom_import_simplexml
0001:0012d1b0  _php_dom_create_object
0001:00128d90  _dom_objects_store_clone_obj
0001:00129778  _zm_startup_dom
0001:0012ca7c  _zm_shutdown_dom
0001:0012c9c8  _zm_info_dom
0001:0012cf50  _dom_objects_new
0001:0012d0dc  _dom_nnodemap_objects_new
0001:0012cfa4  _dom_xpath_objects_new
0001:0012cb80  _node_list_unlink
0001:0012cc3c  _dom_xpath_objects_free_storage
0001:0012ccc8  _dom_objects_free_storage
0001:0012cd38  _dom_namednode_iter
0001:0012ce98  _dom_objects_clone
0001:0012d0ac  _dom_nnodemap_objects_free_storage
0001:0012d168  _php_dom_create_interator
0001:0012d3ac  _php_dom_create_implementation
0001:0012d3c8  _dom_hierarchy
0001:0012d40c  _dom_has_feature
0001:0012d49c  _dom_get_elements_by_tag_name_ns_raw
0001:0012d580  _dom_normalize
0001:0012d680  _dom_set_old_ns
0001:0012d70c  _dom_check_qname
0001:0012d7b4  _dom_get_ns
0001:0012d86c  _dom_get_nsdecl
0002:00001620  _dom_module_entry
Module: U:\dev\php-5.3.6\ext\dom\attr.o(attr.o)
0001:0012d9b0  _php_dom_attr_class_functions
0001:0012de70  _zif_dom_attr_is_id
0001:0012d9f4  _zim_domattr___construct
0001:0012daf8  _dom_attr_name_read
0001:0012db74  _dom_attr_specified_read
0001:0012dba0  _dom_attr_value_read
0001:0012dc70  _dom_attr_value_write
0001:0012dd78  _dom_attr_owner_element_read
0001:0012de20  _dom_attr_schema_type_info_read
Module: U:\dev\php-5.3.6\ext\dom\document.o(document.o)
0001:0012eab0  _php_dom_document_class_functions
0001:0012fb98  _zif_dom_document_create_element
0001:0012fca8  _zif_dom_document_create_document_fragment
0001:0012fd68  _zif_dom_document_create_text_node
0001:0012fe30  _zif_dom_document_create_comment
0001:0012fef8  _zif_dom_document_create_cdatasection
0001:0012ffc4  _zif_dom_document_create_processing_instruction
0001:001300dc  _zif_dom_document_create_attribute
0001:001301dc  _zif_dom_document_create_entity_reference
0001:001302dc  _zif_dom_document_get_elements_by_tag_name
0001:001303bc  _zif_dom_document_import_node
0001:001305cc  _zif_dom_document_create_element_ns
0001:00130834  _zif_dom_document_create_attribute_ns
0001:00130a60  _zif_dom_document_get_elements_by_tag_name_ns
0001:00130b2c  _zif_dom_document_get_element_by_id
0001:00130c14  _zif_dom_document_adopt_node
0001:00130c38  _zif_dom_document_normalize_document
0001:00130cb4  _zif_dom_document_rename_node
0001:001313b0  _zim_domdocument_load
0001:0013140c  _zif_dom_document_save
0001:001313d4  _zim_domdocument_loadXML
0001:00131544  _zif_dom_document_savexml
0001:00130ce0  _zim_domdocument___construct
0001:0013198c  _zif_dom_document_validate
0001:001318a0  _zif_dom_document_xinclude
0001:001321b4  _zim_domdocument_loadHTML
0001:00132190  _zim_domdocument_loadHTMLFile
0001:001322cc  _zif_dom_document_save_html
0001:001321d8  _zif_dom_document_save_html_file
0001:00131cb4  _zif_dom_document_schema_validate_file
0001:00131cd8  _zif_dom_document_schema_validate_xml
0001:00131f54  _zif_dom_document_relaxNG_validate_file
0001:00131f78  _zif_dom_document_relaxNG_validate_xml
0001:00132598  _zim_domdocument_registerNodeClass
0001:0012ed7c  _dom_document_doctype_read
0001:0012ee1c  _dom_document_implementation_read
0001:0012ee48  _dom_document_document_element_read
0001:0012eee8  _dom_document_encoding_read
0001:0012ef8c  _dom_document_encoding_write
0001:0012f0a4  _dom_document_standalone_read
0001:0012f104  _dom_document_standalone_write
0001:0012f1bc  _dom_document_version_read
0001:0012f248  _dom_document_version_write
0001:0012f328  _dom_document_strict_error_checking_read
0001:0012f388  _dom_document_strict_error_checking_write
0001:0012f420  _dom_document_format_output_read
0001:0012f480  _dom_document_format_output_write
0001:0012f518  _dom_document_validate_on_parse_read
0001:0012f578  _dom_document_validate_on_parse_write
0001:0012f610  _dom_document_resolve_externals_read
0001:0012f670  _dom_document_resolve_externals_write
0001:0012f708  _dom_document_preserve_whitespace_read
0001:0012f768  _dom_document_preserve_whitespace_write
0001:0012f800  _dom_document_recover_read
0001:0012f860  _dom_document_recover_write
0001:0012f8f8  _dom_document_substitue_entities_read
0001:0012f958  _dom_document_substitue_entities_write
0001:0012f9f0  _dom_document_document_uri_read
0001:0012fa7c  _dom_document_document_uri_write
0001:0012fb5c  _dom_document_config_read
0001:00130e44  __dom_get_valid_file_path
Module: U:\dev\php-5.3.6\ext\dom\domerrorhandler.o(domerrorhandler.o)
0001:001327d0  _php_dom_domerrorhandler_class_functions
0001:0013280c  _zif_dom_domerrorhandler_handle_error
Module: U:\dev\php-5.3.6\ext\dom\domstringlist.o(domstringlist.o)
0001:00132890  _php_dom_domstringlist_class_functions
0001:00132928  _zif_dom_domstringlist_item
0001:001328c0  _dom_domstringlist_length_read
Module: U:\dev\php-5.3.6\ext\dom\domexception.o(domexception.o)
0001:0013295c  _php_dom_domexception_class_functions
0001:00132970  _php_dom_throw_error_with_message
0001:00132b08  _php_dom_throw_error
Module: U:\dev\php-5.3.6\ext\dom\namelist.o(namelist.o)
0001:00132cb0  _php_dom_namelist_class_functions
0001:00132d5c  _zif_dom_namelist_get_name
0001:00132d80  _zif_dom_namelist_get_namespace_uri
0001:00132cf4  _dom_namelist_length_read
Module: U:\dev\php-5.3.6\ext\dom\processinginstruction.o(processinginstruction.o)
0001:00132e30  _php_dom_processinginstruction_class_functions
0001:00132e60  _zim_domprocessinginstruction___construct
0001:00132f68  _dom_processinginstruction_target_read
0001:00132fe4  _dom_processinginstruction_data_read
0001:001330b4  _dom_processinginstruction_data_write
Module: U:\dev\php-5.3.6\ext\dom\cdatasection.o(cdatasection.o)
0001:001331f0  _php_dom_cdatasection_class_functions
0001:0013321c  _zim_domcdatasection___construct
Module: U:\dev\php-5.3.6\ext\dom\documentfragment.o(documentfragment.o)
0001:001333b0  _php_dom_documentfragment_class_functions
0001:001333f0  _zim_domdocumentfragment___construct
0001:00133558  _zim_domdocumentfragment_appendXML
Module: U:\dev\php-5.3.6\ext\dom\domimplementation.o(domimplementation.o)
0001:00133870  _php_dom_domimplementation_class_functions
0001:00133e60  _zim_domimplementation_getFeature
0001:001338d8  _zim_domimplementation_hasFeature
0001:001339a0  _zim_domimplementation_createDocumentType
0001:00133b70  _zim_domimplementation_createDocument
Module: U:\dev\php-5.3.6\ext\dom\element.o(element.o)
0001:00134650  _php_dom_element_class_functions
0001:00134c94  _zif_dom_element_get_attribute
0001:00134e10  _zif_dom_element_set_attribute
0001:00134fe8  _zif_dom_element_remove_attribute
0001:00135114  _zif_dom_element_get_attribute_node
0001:0013529c  _zif_dom_element_set_attribute_node
0001:001354b8  _zif_dom_element_remove_attribute_node
0001:001355fc  _zif_dom_element_get_elements_by_tag_name
0001:001356d0  _zif_dom_element_get_attribute_ns
0001:00135914  _zif_dom_element_set_attribute_ns
0001:00135cf4  _zif_dom_element_remove_attribute_ns
0001:00135e74  _zif_dom_element_get_attribute_node_ns
0001:00135f4c  _zif_dom_element_set_attribute_node_ns
0001:00136190  _zif_dom_element_get_elements_by_tag_name_ns
0001:0013625c  _zif_dom_element_has_attribute
0001:00136300  _zif_dom_element_has_attribute_ns
0001:00136450  _zif_dom_element_set_id_attribute
0001:00136548  _zif_dom_element_set_id_attribute_ns
0001:00136648  _zif_dom_element_set_id_attribute_node
0001:001347e8  _zim_domelement___construct
0001:00134a4c  _dom_element_tag_name_read
0001:00134b4c  _dom_element_schema_type_info_read
Module: U:\dev\php-5.3.6\ext\dom\node.o(node.o)
0001:00136ef0  _php_dom_node_class_functions
0001:001382b4  _zif_dom_node_insert_before
0001:0013884c  _zif_dom_node_replace_child
0001:00138b5c  _zif_dom_node_remove_child
0001:00138cfc  _zif_dom_node_append_child
0001:00139060  _zif_dom_node_has_child_nodes
0001:00139104  _zif_dom_node_clone_node
0001:00139298  _zif_dom_node_normalize
0001:00139318  _zif_dom_node_is_supported
0001:00139388  _zif_dom_node_has_attributes
0001:00139434  _zif_dom_node_compare_document_position
0001:00139458  _zif_dom_node_is_same_node
0001:0013950c  _zif_dom_node_lookup_prefix
0001:0013964c  _zif_dom_node_is_default_namespace
0001:0013973c  _zif_dom_node_lookup_namespace_uri
0001:00139828  _zif_dom_node_is_equal_node
0001:0013984c  _zif_dom_node_get_feature
0001:00139870  _zif_dom_node_set_user_data
0001:00139894  _zif_dom_node_get_user_data
0001:00139ea0  _zim_domnode_getNodePath
0001:00139f5c  _zim_domnode_getLineNo
0001:00139e40  _zim_domnode_C14N
0001:00139e64  _zim_domnode_C14NFile
0001:001371cc  _dom_node_node_name_read
0001:001373a4  _dom_node_node_value_read
0001:001374b4  _dom_node_node_value_write
0001:001375cc  _dom_node_node_type_read
0001:0013765c  _dom_node_parent_node_read
0001:001376f0  _dom_node_child_nodes_read
0001:00137784  _dom_node_first_child_read
0001:00137830  _dom_node_last_child_read
0001:001378dc  _dom_node_previous_sibling_read
0001:00137970  _dom_node_next_sibling_read
0001:001379fc  _dom_node_attributes_read
0001:00137a88  _dom_node_owner_document_read
0001:00137b44  _dom_node_namespace_uri_read
0001:00137bf0  _dom_node_prefix_read
0001:00137cfc  _dom_node_prefix_write
0001:00137f7c  _dom_node_local_name_read
0001:00138014  _dom_node_base_uri_read
0001:001380c8  _dom_node_text_content_read
0001:00138188  _dom_node_text_content_write
Module: U:\dev\php-5.3.6\ext\dom\string_extend.o(string_extend.o)
0001:0013a0d0  _php_dom_string_extend_class_functions
0001:0013a120  _zif_dom_string_extend_find_offset16
0001:0013a144  _zif_dom_string_extend_find_offset32
Module: U:\dev\php-5.3.6\ext\dom\characterdata.o(characterdata.o)
0001:0013a390  _php_dom_characterdata_class_functions
0001:0013a638  _zif_dom_characterdata_substring_data
0001:0013a7c4  _zif_dom_characterdata_append_data
0001:0013a85c  _zif_dom_characterdata_insert_data
0001:0013a9bc  _zif_dom_characterdata_delete_data
0001:0013ab38  _zif_dom_characterdata_replace_data
0001:0013a40c  _dom_characterdata_data_read
0001:0013a4dc  _dom_characterdata_data_write
0001:0013a5a0  _dom_characterdata_length_read
Module: U:\dev\php-5.3.6\ext\dom\documenttype.o(documenttype.o)
0001:0013acfc  _php_dom_documenttype_class_functions
0001:0013ad10  _dom_documenttype_name_read
0001:0013ad8c  _dom_documenttype_entities_read
0001:0013ae14  _dom_documenttype_notations_read
0001:0013ae9c  _dom_documenttype_public_id_read
0001:0013af34  _dom_documenttype_system_id_read
0001:0013afcc  _dom_documenttype_internal_subset_read
Module: U:\dev\php-5.3.6\ext\dom\domimplementationlist.o(domimplementationlist.o)
0001:0013b110  _php_dom_domimplementationlist_class_functions
0001:0013b1a8  _zif_dom_domimplementationlist_item
0001:0013b140  _dom_domimplementationlist_length_read
Module: U:\dev\php-5.3.6\ext\dom\entity.o(entity.o)
0001:0013b1dc  _php_dom_entity_class_functions
0001:0013b1f0  _dom_entity_public_id_read
0001:0013b280  _dom_entity_system_id_read
0001:0013b310  _dom_entity_notation_name_read
0001:0013b3b4  _dom_entity_actual_encoding_read
0001:0013b3d8  _dom_entity_actual_encoding_write
0001:0013b3e0  _dom_entity_encoding_read
0001:0013b404  _dom_entity_encoding_write
0001:0013b40c  _dom_entity_version_read
0001:0013b430  _dom_entity_version_write
Module: U:\dev\php-5.3.6\ext\dom\nodelist.o(nodelist.o)
0001:0013b4a0  _php_dom_nodelist_class_functions
0001:0013b614  _zif_dom_nodelist_item
0001:0013b4c8  _dom_nodelist_length_read
Module: U:\dev\php-5.3.6\ext\dom\text.o(text.o)
0001:0013b960  _php_dom_text_class_functions
0001:0013bbec  _zif_dom_text_split_text
0001:0013bd88  _zif_dom_text_is_whitespace_in_element_content
0001:0013be38  _zif_dom_text_replace_whole_text
0001:0013b9dc  _zim_domtext___construct
0001:0013bab8  _dom_text_whole_text_read
Module: U:\dev\php-5.3.6\ext\dom\comment.o(comment.o)
0001:0013bec0  _php_dom_comment_class_functions
0001:0013beec  _zim_domcomment___construct
Module: U:\dev\php-5.3.6\ext\dom\domconfiguration.o(domconfiguration.o)
0001:0013c120  _php_dom_domconfiguration_class_functions
0001:0013c184  _zif_dom_domconfiguration_set_parameter
0001:0013c1a8  _zif_dom_domconfiguration_get_parameter
0001:0013c1cc  _zif_dom_domconfiguration_can_set_parameter
Module: U:\dev\php-5.3.6\ext\dom\domimplementationsource.o(domimplementationsource.o)
0001:0013c2c0  _php_dom_domimplementationsource_class_functions
0001:0013c310  _zif_dom_domimplementationsource_get_domimplementation
0001:0013c334  _zif_dom_domimplementationsource_get_domimplementations
Module: U:\dev\php-5.3.6\ext\dom\entityreference.o(entityreference.o)
0001:0013c3c0  _php_dom_entityreference_class_functions
0001:0013c3ec  _zim_domentityreference___construct
Module: U:\dev\php-5.3.6\ext\dom\notation.o(notation.o)
0001:0013c4ec  _php_dom_notation_class_functions
0001:0013c504  _dom_notation_public_id_read
0001:0013c59c  _dom_notation_system_id_read
Module: U:\dev\php-5.3.6\ext\dom\xpath.o(xpath.o)
0001:0013c840  _php_dom_xpath_class_functions
0001:0013d224  _zim_domxpath___construct
0001:0013d440  _zif_dom_xpath_register_ns
0001:0013d904  _zif_dom_xpath_query
0001:0013d928  _zif_dom_xpath_evaluate
0001:0013d968  _zif_dom_xpath_register_php_functions
0001:0013d3b8  _dom_xpath_document_read
Module: U:\dev\php-5.3.6\ext\dom\dom_iterators.o(dom_iterators.o)
0001:0013dc70  _create_notation
0001:0013dd08  _php_dom_libxml_hash_iter
0001:0013dd70  _php_dom_libxml_notation_iter
0001:0013e0c8  _php_dom_get_iterator
0002:00001680  _php_dom_iterator_funcs
Module: U:\dev\php-5.3.6\ext\dom\typeinfo.o(typeinfo.o)
0001:0013e2ac  _php_dom_typeinfo_class_functions
0001:0013e2c0  _dom_typeinfo_type_name_read
0001:0013e2e4  _dom_typeinfo_type_namespace_read
Module: U:\dev\php-5.3.6\ext\dom\domerror.o(domerror.o)
0001:0013e31c  _php_dom_domerror_class_functions
0001:0013e338  _dom_domerror_severity_read
0001:0013e38c  _dom_domerror_message_read
0001:0013e3e0  _dom_domerror_type_read
0001:0013e434  _dom_domerror_related_exception_read
0001:0013e488  _dom_domerror_related_data_read
0001:0013e4dc  _dom_domerror_location_read
Module: U:\dev\php-5.3.6\ext\dom\domlocator.o(domlocator.o)
0001:0013e53c  _php_dom_domlocator_class_functions
0001:0013e558  _dom_domlocator_line_number_read
0001:0013e5ac  _dom_domlocator_column_number_read
0001:0013e600  _dom_domlocator_offset_read
0001:0013e654  _dom_domlocator_related_node_read
0001:0013e6a8  _dom_domlocator_uri_read
Module: U:\dev\php-5.3.6\ext\dom\namednodemap.o(namednodemap.o)
0001:0013e9a0  _php_dom_namednodemap_class_functions
0001:0013eb00  _zif_dom_namednodemap_get_named_item
0001:0013ec2c  _zif_dom_namednodemap_set_named_item
0001:0013ec50  _zif_dom_namednodemap_remove_named_item
0001:0013ec78  _zif_dom_namednodemap_item
0001:0013eda8  _zif_dom_namednodemap_get_named_item_ns
0001:0013eed0  _zif_dom_namednodemap_set_named_item_ns
0001:0013eef4  _zif_dom_namednodemap_remove_named_item_ns
0001:0013ea40  _dom_namednodemap_length_read
Module: U:\dev\php-5.3.6\ext\dom\userdatahandler.o(userdatahandler.o)
0001:0013ef40  _php_dom_userdatahandler_class_functions
0001:0013ef7c  _zif_dom_userdatahandler_handle
Module: U:\dev\php-5.3.6\ext\fileinfo\fileinfo.o(fileinfo.o)
0002:00022580  _finfo_class_entry
0001:0013eff8  _finfo_objects_new
0001:0013f828  _zif_finfo_open
0001:0013fab8  _zif_finfo_set_flags
0001:00140200  _zif_finfo_file
0001:00140224  _zif_finfo_buffer
0001:0013f428  _finfo_resource_destructor
0001:0013f9fc  _zif_finfo_close
0001:00140248  _zif_mime_content_type
0001:0013f554  _zm_startup_finfo
0001:0013f7ac  _zm_info_fileinfo
0002:000016a0  _finfo_class_functions
0002:00001720  _fileinfo_functions
0002:000017c0  _fileinfo_module_entry
Module: U:\dev\php-5.3.6\ext\fileinfo\libmagic\apprentice.o(apprentice.o)
0002:00022590  _file_names
0002:00022640  _file_formats
0001:001402e4  _file_nformats
0001:001402e8  _file_nnames
0001:00140340  _php_magic_database
0001:002ec2a0  _file_delmagic
0001:002ec308  _file_apprentice
0001:002ed0ec  _file_signextend
0001:002ef5d4  _file_showstr
Module: U:\dev\php-5.3.6\ext\fileinfo\libmagic\ascmagic.o(ascmagic.o)
0001:002f076c  _file_ascmagic
0001:002f08a8  _file_ascmagic_with_encoding
Module: U:\dev\php-5.3.6\ext\fileinfo\libmagic\cdf.o(cdf.o)
0001:002f103c  _cdf_tole2
0001:002f105c  _cdf_tole4
0001:002f1080  _cdf_tole8
0001:002f10cc  _cdf_swap_header
0001:002f1394  _cdf_unpack_header
0001:002f1448  _cdf_swap_dir
0001:002f163c  _cdf_swap_class
0001:002f16bc  _cdf_unpack_dir
0001:002f1844  _cdf_read_header
0001:002f18d8  _cdf_read_sector
0001:002f1904  _cdf_read_short_sector
0001:002f1938  _cdf_read_sat
0001:002f1b74  _cdf_count_chain
0001:002f1bf0  _cdf_read_long_sector_chain
0001:002f1d18  _cdf_read_short_sector_chain
0001:002f1e34  _cdf_read_sector_chain
0001:002f1ea4  _cdf_read_dir
0001:002f2098  _cdf_read_ssat
0001:002f2198  _cdf_read_short_stream
0001:002f22cc  _cdf_read_summary_info
0001:002f235c  _cdf_read_property_info
0001:002f2988  _cdf_unpack_summary_info
0001:002f2b90  _cdf_print_classid
0001:002f2da8  _cdf_print_property_name
0001:002f2dfc  _cdf_print_elapsed_time
Module: U:\dev\php-5.3.6\ext\fileinfo\libmagic\cdf_time.o(cdf_time.o)
0001:002f30f8  _cdf_timestamp_to_timespec
0001:002f3274  _cdf_timespec_to_timestamp
Module: U:\dev\php-5.3.6\ext\fileinfo\libmagic\compress.o(compress.o)
0001:002f3488  _sread
0001:002f3594  _file_pipe2file
Module: U:\dev\php-5.3.6\ext\fileinfo\libmagic\encoding.o(encoding.o)
0001:002f382c  _file_encoding
0001:002f3b30  _file_looks_utf8
Module: U:\dev\php-5.3.6\ext\fileinfo\libmagic\fsmagic.o(fsmagic.o)
0001:002f3f84  _file_fsmagic
Module: U:\dev\php-5.3.6\ext\fileinfo\libmagic\funcs.o(funcs.o)
0001:002f42a4  _file_printf
0001:002f4410  _file_error
0001:002f442c  _file_magerror
0001:002f4464  _file_oomem
0001:002f4498  _file_badseek
0001:002f44c8  _file_badread
0001:002f458c  _file_buffer
0001:002f48c4  _file_reset
0001:002f4938  _file_getbuffer
0001:002f4a30  _file_check_mem
Module: U:\dev\php-5.3.6\ext\fileinfo\libmagic\is_tar.o(is_tar.o)
0001:002f4b78  _file_is_tar
Module: U:\dev\php-5.3.6\ext\fileinfo\libmagic\magic.o(magic.o)
0001:002f4dc8  _magic_open
0001:002f5378  _magic_setflags
0001:002f4f98  _magic_close
0001:002f5008  _magic_load
0001:002f5040  _magic_compile
0001:002f50b8  _magic_descriptor
0001:002f50cc  _magic_file
0001:002f50e4  _magic_stream
0001:002f52f8  _magic_buffer
0001:002f5348  _magic_error
0001:002f5360  _magic_errno
Module: U:\dev\php-5.3.6\ext\fileinfo\libmagic\print.o(print.o)
0001:002f540c  _file_magwarn
0001:002f5468  _file_fmttime
Module: U:\dev\php-5.3.6\ext\fileinfo\libmagic\readcdf.o(readcdf.o)
0001:002f5b18  _file_trycdf
Module: U:\dev\php-5.3.6\ext\fileinfo\libmagic\softmagic.o(softmagic.o)
0001:002f5e24  _file_softmagic
Module: U:\dev\php-5.3.6\ext\filter\filter.o(filter.o)
0002:000226f0  _filter_globals_id
0001:002fbb10  _zif_filter_input
0001:002fbe38  _zif_filter_var
0001:002fbf10  _zif_filter_input_array
0001:002fc0d0  _zif_filter_var_array
0001:002fc160  _zif_filter_list
0001:002fb340  _zif_filter_has_var
0001:002fc1bc  _zif_filter_id
0001:002fa1c0  _zm_startup_filter
0001:002fa6d4  _zm_shutdown_filter
0001:002fa6ec  _zm_deactivate_filter
0001:002fa874  _zm_info_filter
0002:00001a80  _filter_module_entry
Module: U:\dev\php-5.3.6\ext\filter\sanitizing_filters.o(sanitizing_filters.o)
0001:002fc7f8  _php_filter_string
0001:002fc934  _php_filter_encoded
0001:002fc96c  _php_filter_special_chars
0001:002fca08  _php_filter_full_special_chars
0001:002fca64  _php_filter_unsafe_raw
0001:002fcb58  _php_filter_email
0001:002fcc04  _php_filter_url
0001:002fcc60  _php_filter_number_int
0001:002fccb4  _php_filter_number_float
0001:002fcd54  _php_filter_magic_quotes
Module: U:\dev\php-5.3.6\ext\filter\logical_filters.o(logical_filters.o)
0001:002fcfb4  _php_filter_int
0001:002fd318  _php_filter_boolean
0001:002fd52c  _php_filter_float
0001:002fd990  _php_filter_validate_regexp
0001:002fdb78  _php_filter_validate_url
0001:002fe1d8  _php_filter_validate_email
0001:002fe51c  _php_filter_validate_ip
Module: U:\dev\php-5.3.6\ext\filter\callback_filter.o(callback_filter.o)
0001:002fec90  _php_filter_callback
Module: U:\dev\php-5.3.6\ext\ftp\php_ftp.o(php_ftp.o)
0001:002ffdf0  _php_ftp_functions
0001:003002b4  _zif_ftp_connect
0001:0030035c  _zif_ftp_ssl_connect
0001:00300408  _zif_ftp_login
0001:003004b0  _zif_ftp_pwd
0001:00300560  _zif_ftp_cdup
0001:003005f4  _zif_ftp_chdir
0001:00300694  _zif_ftp_exec
0001:00300734  _zif_ftp_raw
0001:003007a4  _zif_ftp_mkdir
0001:00300854  _zif_ftp_rmdir
0001:003008f8  _zif_ftp_chmod
0001:003009a4  _zif_ftp_alloc
0001:00300a8c  _zif_ftp_nlist
0001:00300b48  _zif_ftp_rawlist
0001:00300c08  _zif_ftp_systype
0001:00301010  _zif_ftp_pasv
0001:003010c0  _zif_ftp_get
0001:00300cf0  _zif_ftp_fget
0001:00301970  _zif_ftp_put
0001:0030164c  _zif_ftp_fput
0001:00301ccc  _zif_ftp_size
0001:00301d44  _zif_ftp_mdtm
0001:00301dbc  _zif_ftp_rename
0001:00301e64  _zif_ftp_delete
0001:00301f04  _zif_ftp_site
0001:00301fa4  _zif_ftp_close
0001:003020b4  _zif_ftp_set_option
0001:003021a8  _zif_ftp_get_option
0001:00300e68  _zif_ftp_nb_fget
0001:003012d4  _zif_ftp_nb_get
0001:00301544  _zif_ftp_nb_continue
0001:00301b10  _zif_ftp_nb_put
0001:003017c8  _zif_ftp_nb_fput
0001:00300154  _zm_startup_ftp
0001:00300264  _zm_info_ftp
0002:00001ae0  _php_ftp_module_entry
Module: U:\dev\php-5.3.6\ext\ftp\ftp.o(ftp.o)
0001:00302278  _ftp_open
0001:00302388  _ftp_close
0001:003023f8  _ftp_gc
0001:00302458  _ftp_quit
0001:00302550  _ftp_login
0001:003027fc  _ftp_reinit
0001:0030286c  _ftp_syst
0001:00302924  _ftp_pwd
0001:003029d4  _ftp_exec
0001:00302a2c  _ftp_raw
0001:00302b34  _ftp_chdir
0001:00302bb4  _ftp_cdup
0001:00302c30  _ftp_mkdir
0001:00302cd8  _ftp_rmdir
0001:00302d40  _ftp_chmod
0001:00302dd0  _ftp_alloc
0001:00302e78  _ftp_nlist
0001:00302ea0  _ftp_list
0001:00302f80  _ftp_pasv
0001:003030c0  _ftp_get
0001:00303310  _ftp_put
0001:00303520  _ftp_size
0001:003035ac  _ftp_mdtm
0001:003036e4  _ftp_delete
0001:00303748  _ftp_rename
0001:003037d4  _ftp_site
0001:00303d90  _data_available
0001:00303de4  _data_writeable
0001:00304840  _ftp_nb_get
0001:00304968  _ftp_nb_continue_read
0001:00304b14  _ftp_nb_put
0001:00304c3c  _ftp_nb_continue_write
Module: U:\dev\php-5.3.6\ext\hash\hash.o(hash.o)
0002:00022700  _php_hash_hashtable
0001:00304d9c  _php_hash_fetch_ops
0001:00304dec  _php_hash_register_algo
0001:00304e50  _php_hash_copy
0001:003050bc  _zif_hash
0001:003050e0  _zif_hash_file
0001:00305418  _zif_hash_hmac
0001:0030543c  _zif_hash_hmac_file
0001:00305484  _zif_hash_init
0001:00305614  _zif_hash_update
0001:003056a0  _zif_hash_update_stream
0001:003057f0  _zif_hash_update_file
0001:0030594c  _zif_hash_final
0001:00305b20  _zif_hash_copy
0001:00305c0c  _zif_hash_algos
0001:00305e84  _zm_startup_hash
0001:003061a4  _zm_shutdown_hash
0001:003061e4  _zm_info_hash
0001:00306790  _hash_functions
0002:00001b40  _hash_module_entry
Module: U:\dev\php-5.3.6\ext\hash\hash_md.o(hash_md.o)
0001:003068bc  _php_hash_md5_ops
0001:003068d8  _php_hash_md4_ops
0001:00306ebc  _PHP_MD4Init
0001:00306ef0  _PHP_MD4Update
0001:00306fac  _PHP_MD4Final
0001:003068f4  _php_hash_md2_ops
0001:00307130  _PHP_MD2Init
0001:003071c4  _PHP_MD2Update
0001:00307294  _PHP_MD2Final
Module: U:\dev\php-5.3.6\ext\hash\hash_sha.o(hash_sha.o)
0001:00307444  _php_hash_sha1_ops
0001:00307460  _php_hash_sha256_ops
0001:003075b0  _PHP_SHA256Init
0001:003079b0  _PHP_SHA256Update
0001:00307a6c  _PHP_SHA256Final
0001:0030747c  _php_hash_sha224_ops
0001:00307804  _PHP_SHA224Init
0001:00307854  _PHP_SHA224Update
0001:00307910  _PHP_SHA224Final
0001:00308040  _PHP_SHA384Init
0001:0030874c  _PHP_SHA384Update
0001:00308858  _PHP_SHA384Final
0001:00308950  _php_hash_sha384_ops
0001:0030896c  _PHP_SHA512Init
0001:00308a00  _PHP_SHA512Update
0001:00308b0c  _PHP_SHA512Final
0001:00308c04  _php_hash_sha512_ops
Module: U:\dev\php-5.3.6\ext\hash\hash_ripemd.o(hash_ripemd.o)
0001:00308c5c  _php_hash_ripemd128_ops
0001:00308ccc  _PHP_RIPEMD128Init
0001:003092cc  _PHP_RIPEMD128Update
0001:0030a238  _PHP_RIPEMD128Final
0001:00308c78  _php_hash_ripemd160_ops
0001:00308d50  _PHP_RIPEMD160Init
0001:00309bfc  _PHP_RIPEMD160Update
0001:0030a378  _PHP_RIPEMD160Final
0001:00308c94  _php_hash_ripemd256_ops
0001:00308d00  _PHP_RIPEMD256Init
0001:00309680  _PHP_RIPEMD256Update
0001:0030a2d8  _PHP_RIPEMD256Final
0001:00308cb0  _php_hash_ripemd320_ops
0001:00308d88  _PHP_RIPEMD320Init
0001:0030a0dc  _PHP_RIPEMD320Update
0001:0030a418  _PHP_RIPEMD320Final
Module: U:\dev\php-5.3.6\ext\hash\hash_haval.o(hash_haval.o)
0001:0030b8b4  _php_hash_3haval128_ops
0001:0030b8d0  _PHP_3HAVAL128Init
0001:0030be54  _PHP_HAVALUpdate
0001:0030bf10  _PHP_HAVAL128Final
0001:0030b914  _php_hash_3haval160_ops
0001:0030b930  _PHP_3HAVAL160Init
0001:0030c05c  _PHP_HAVAL160Final
0001:0030b974  _php_hash_3haval192_ops
0001:0030b990  _PHP_3HAVAL192Init
0001:0030c198  _PHP_HAVAL192Final
0001:0030b9d4  _php_hash_3haval224_ops
0001:0030b9f0  _PHP_3HAVAL224Init
0001:0030c2bc  _PHP_HAVAL224Final
0001:0030ba34  _php_hash_3haval256_ops
0001:0030ba50  _PHP_3HAVAL256Init
0001:0030c3a0  _PHP_HAVAL256Final
0001:0030ba94  _php_hash_4haval128_ops
0001:0030bab0  _PHP_4HAVAL128Init
0001:0030baf4  _php_hash_4haval160_ops
0001:0030bb10  _PHP_4HAVAL160Init
0001:0030bb54  _php_hash_4haval192_ops
0001:0030bb70  _PHP_4HAVAL192Init
0001:0030bbb4  _php_hash_4haval224_ops
0001:0030bbd0  _PHP_4HAVAL224Init
0001:0030bc14  _php_hash_4haval256_ops
0001:0030bc30  _PHP_4HAVAL256Init
0001:0030bc74  _php_hash_5haval128_ops
0001:0030bc90  _PHP_5HAVAL128Init
0001:0030bcd4  _php_hash_5haval160_ops
0001:0030bcf0  _PHP_5HAVAL160Init
0001:0030bd34  _php_hash_5haval192_ops
0001:0030bd50  _PHP_5HAVAL192Init
0001:0030bd94  _php_hash_5haval224_ops
0001:0030bdb0  _PHP_5HAVAL224Init
0001:0030bdf4  _php_hash_5haval256_ops
0001:0030be10  _PHP_5HAVAL256Init
Module: U:\dev\php-5.3.6\ext\hash\hash_tiger.o(hash_tiger.o)
0001:0030e470  _PHP_3TIGERInit
0001:0030e4b4  _PHP_4TIGERInit
0001:0030e4fc  _PHP_TIGERUpdate
0001:003135d4  _PHP_TIGER128Final
0001:0031369c  _PHP_TIGER160Final
0001:0031378c  _PHP_TIGER192Final
0001:003138a8  _php_hash_3tiger128_ops
0001:003138c4  _php_hash_3tiger160_ops
0001:003138e0  _php_hash_3tiger192_ops
0001:003138fc  _php_hash_4tiger128_ops
0001:00313918  _php_hash_4tiger160_ops
0001:00313934  _php_hash_4tiger192_ops
Module: U:\dev\php-5.3.6\ext\hash\hash_gost.o(hash_gost.o)
0001:003199f0  _PHP_GOSTInit
0001:00319a0c  _PHP_GOSTUpdate
0001:00319c34  _PHP_GOSTFinal
0001:00319d50  _php_hash_gost_ops
Module: U:\dev\php-5.3.6\ext\hash\hash_snefru.o(hash_snefru.o)
0001:0031f550  _PHP_SNEFRUInit
0001:0031f56c  _PHP_SNEFRUUpdate
0001:0031f71c  _PHP_SNEFRUFinal
0001:0031f7f0  _php_hash_snefru_ops
Module: U:\dev\php-5.3.6\ext\hash\hash_whirlpool.o(hash_whirlpool.o)
0001:003254cc  _PHP_WHIRLPOOLInit
0001:003254e4  _PHP_WHIRLPOOLUpdate
0001:003256fc  _PHP_WHIRLPOOLFinal
0001:00325824  _php_hash_whirlpool_ops
Module: U:\dev\php-5.3.6\ext\hash\hash_adler32.o(hash_adler32.o)
0001:0032587c  _PHP_ADLER32Init
0001:0032588c  _PHP_ADLER32Update
0001:003258f0  _PHP_ADLER32Final
0001:0032591c  _PHP_ADLER32Copy
0001:00325930  _php_hash_adler32_ops
Module: U:\dev\php-5.3.6\ext\hash\hash_crc32.o(hash_crc32.o)
0001:00326180  _PHP_CRC32Init
0001:00326190  _PHP_CRC32Update
0001:003261c8  _PHP_CRC32BUpdate
0001:00326200  _PHP_CRC32Final
0001:00326230  _PHP_CRC32BFinal
0001:00326260  _PHP_CRC32Copy
0001:00326274  _php_hash_crc32_ops
0001:00326290  _php_hash_crc32b_ops
Module: U:\dev\php-5.3.6\ext\hash\hash_salsa.o(hash_salsa.o)
0001:00326708  _PHP_SALSA10Init
0001:0032672c  _PHP_SALSA20Init
0001:00326750  _PHP_SALSAUpdate
0001:00326970  _PHP_SALSAFinal
0001:00326a4c  _php_hash_salsa10_ops
0001:00326a68  _php_hash_salsa20_ops
Module: U:\dev\php-5.3.6\ext\json\json.o(json.o)
0002:00022730  _json_globals_id
0001:0032885c  _php_json_encode
0001:00328d44  _php_json_decode
0002:00001bb0  _json_module_entry
Module: U:\dev\php-5.3.6\ext\json\utf8_to_utf16.o(utf8_to_utf16.o)
0001:003294a0  _utf8_to_utf16
Module: U:\dev\php-5.3.6\ext\json\utf8_decode.o(utf8_decode.o)
0001:00329578  _utf8_decode_init
0001:003295a0  _utf8_decode_at_byte
0001:003295ac  _utf8_decode_at_character
0001:003295c8  _utf8_decode_next
Module: U:\dev\php-5.3.6\ext\json\JSON_parser.o(JSON_parser.o)
0001:0032a830  _new_JSON_parser
0001:0032a8a0  _free_JSON_parser
0001:0032aee4  _parse_JSON
Module: U:\dev\php-5.3.6\ext\pdo\pdo.o(pdo.o)
0002:00022740  _pdo_dbh_ce
0002:00022750  _pdo_exception_ce
0002:00022760  _pdo_driver_hash
0002:00022790  _pdo_globals_id
0002:000227a0  _pdo_dbstmt_ce
0002:000227b0  _pdo_row_ce
0001:0032bb0c  _php_pdo_list_entry
0001:0032bb18  _php_pdo_get_dbh_ce
0001:0032bb24  _php_pdo_get_exception
0001:0032bb30  _php_pdo_str_tolower_dup
0001:0032bb70  _php_pdo_get_exception_base
0001:0032bbd4  _zif_pdo_drivers
0001:0032bc80  _pdo_functions
0001:0032c250  _zm_startup_pdo
0001:0032c3d0  _zm_shutdown_pdo
0001:0032c410  _zm_info_pdo
0001:0032bd88  _php_pdo_register_driver
0001:0032be08  _php_pdo_unregister_driver
0001:0032be48  _pdo_find_driver
0001:0032be7c  _php_pdo_parse_data_source
0001:0032c0b0  _php_pdo_int64_to_str
0002:00001c10  _pdo_module_entry
Module: U:\dev\php-5.3.6\ext\pdo\pdo_dbh.o(pdo_dbh.o)
0001:0032c560  _pdo_raise_impl_error
0001:0032c728  _pdo_handle_error
0001:003309c0  _php_pdo_dbh_addref
0001:0032f660  _pdo_dbh_functions
0001:0032f7f4  _pdo_hash_methods
0001:0032ff6c  _pdo_dbh_init
0001:00330a64  _pdo_dbh_new
0001:003309cc  _php_pdo_dbh_delref
0001:00330b08  _php_pdo_pdbh_dtor
Module: U:\dev\php-5.3.6\ext\pdo\pdo_stmt.o(pdo_stmt.o)
0002:000227c0  _pdo_dbstmt_object_handlers
0001:00331584  _pdo_stmt_describe_columns
0001:003362c4  _pdo_row_free_storage
0001:00334788  _pdo_stmt_setup_fetch_mode
0001:003351c0  _pdo_dbstmt_functions
0001:00335b44  _pdo_dbstmt_free_storage
0001:00335698  _pdo_stmt_init
0001:00335ddc  _pdo_stmt_iter_get
0001:00335b4c  _pdo_dbstmt_new
0001:00335ef0  _pdo_row_functions
0001:003362f0  _pdo_row_new
0001:00335b1c  _php_pdo_stmt_addref
0001:00335b28  _php_pdo_stmt_delref
0002:00001c90  _pdo_row_object_handlers
Module: U:\dev\php-5.3.6\ext\pdo\pdo_sql_parser.o(pdo_sql_parser.o)
0001:00337020  _pdo_parse_params
Module: U:\dev\php-5.3.6\ext\pdo\pdo_sqlstate.o(pdo_sqlstate.o)
0001:0033a028  _pdo_sqlstate_fini_error_table
0001:0033a03c  _pdo_sqlstate_init_error_table
0001:0033a0a4  _pdo_sqlstate_state_to_description
Module: U:\dev\php-5.3.6\ext\phar\util.o(util.o)
0001:0033a588  _phar_get_link_source
0001:0033a648  _phar_get_efp
0001:0033bc00  _phar_open_archive_fp
0001:0033a7dc  _phar_seek_efp
0001:0033a99c  _phar_mount_entry
0001:0033abec  _phar_find_in_include_path
0001:0033c9c8  _phar_get_archive
0001:0033b190  _phar_get_entry_data
0001:0033d4a4  _phar_get_entry_info_dir
0001:0033ed0c  _phar_copy_on_write
0001:0033c5f8  _phar_create_writeable_entry
0001:0033c734  _phar_separate_entry_fp
0001:0033bfcc  _phar_open_entry_fp
0001:0033d258  _phar_get_entry_info
0001:0033b844  _phar_get_or_create_entry_data
0001:0033e910  _phar_add_virtual_dirs
0001:0033bd64  _phar_copy_entry_fp
0001:0033d20c  _phar_decompress_filter
0001:0033c880  _phar_open_jit
0001:0033c8f4  _phar_free_alias
0001:0033d1b4  _phar_compress_filter
0001:0033df7c  _phar_verify_signature
0001:0033e5c0  _phar_create_signature
Module: U:\dev\php-5.3.6\ext\phar\tar.o(tar.o)
0001:0033f428  _phar_is_tar
0001:0033f568  _phar_open_or_create_tar
0001:0033fba8  _phar_parse_tarfile
0001:003414d8  _phar_tar_setmetadata
0001:00341c9c  _phar_tar_flush
Module: U:\dev\php-5.3.6\ext\phar\zip.o(zip.o)
0001:00343988  _phar_parse_zipfile
0001:00346e50  _phar_open_or_create_zip
0001:00348784  _phar_zip_flush
Module: U:\dev\php-5.3.6\ext\phar\stream.o(stream.o)
0001:003499d0  _phar_parse_url
0001:0034a940  _phar_dostat
0002:00001d10  _phar_ops
0002:00001d50  _phar_stream_wops
0002:00001d78  _php_stream_phar_wrapper
Module: U:\dev\php-5.3.6\ext\phar\func_interceptors.o(func_interceptors.o)
0001:0034e8b8  _phar_fileperms
0001:0034e950  _phar_fileinode
0001:0034e9e8  _phar_filesize
0001:0034ea80  _phar_fileowner
0001:0034eb18  _phar_filegroup
0001:0034ebb0  _phar_fileatime
0001:0034ec48  _phar_filemtime
0001:0034ece0  _phar_filectime
0001:0034ed78  _phar_filetype
0001:0034ee10  _phar_is_writable
0001:0034eea8  _phar_is_readable
0001:0034ef40  _phar_is_executable
0001:0034efd8  _phar_file_exists
0001:0034f070  _phar_is_dir
0001:0034f5a4  _phar_lstat
0001:0034f63c  _phar_stat
0001:0034f6d4  _phar_intercept_functions
0001:0034f710  _phar_release_functions
0001:0034f800  _phar_intercept_functions_init
0001:0034ff8c  _phar_intercept_functions_shutdown
0001:0035087c  _phar_save_orig_functions
0001:00350998  _phar_restore_orig_functions
Module: U:\dev\php-5.3.6\ext\phar\dirstream.o(dirstream.o)
0001:00351534  _phar_wrapper_open_dir
0001:00351acc  _phar_wrapper_mkdir
0001:003520e4  _phar_wrapper_rmdir
0002:00001dd0  _phar_dir_ops
Module: U:\dev\php-5.3.6\ext\phar\phar.o(phar.o)
0002:00022830  _phar_globals_id
0002:00022840  _cached_phars
0002:00022870  _cached_alias
0002:000228a0  _phar_orig_compile_file
0002:000228b0  _phar_save_resolve_path
0001:003529ec  _phar_ini_modify_handler
0001:003568dc  _phar_open_from_filename
0001:00352fac  _phar_ini_cache_list
0001:00353120  _phar_destroy_phar_data
0001:00353338  _phar_archive_delref
0001:0035357c  _destroy_phar_manifest_entry
0001:003536fc  _phar_entry_delref
0001:00353794  _phar_entry_remove
0001:0035ac58  _phar_flush
0001:003538b8  _phar_open_parsed_phar
0001:003539f0  _phar_parse_metadata
0001:0035d118  _phar_request_initialize
0001:00355ff8  _phar_open_or_create_filename
0001:00357844  _phar_detect_phar_fname_ext
0001:003563b0  _phar_create_or_parse_filename
0001:00357dd4  _phar_fix_filepath
0001:003580e0  _phar_split_fname
0001:00358270  _phar_open_executed_filename
0001:0035869c  _phar_postprocess_file
0001:0035a624  _phar_create_default_stub
0001:0035c95c  _zm_globals_ctor_phar
0001:0035d010  _zm_globals_dtor_phar
0001:0035d028  _zm_startup_phar
0001:0035d0a0  _zm_shutdown_phar
0001:0035d304  _zm_deactivate_phar
0001:0035d700  _zm_info_phar
0002:00001e10  _phar_module_entry
0002:0000bf10  _phar_functions
Module: U:\dev\php-5.3.6\ext\phar\phar_object.o(phar_object.o)
0001:0035f028  _zim_Phar_running
0001:0035f200  _zim_Phar_mount
0001:0035f6e0  _zim_Phar_webPhar
0001:00360578  _zim_Phar_mungServer
0001:00360730  _zim_Phar_interceptFileFuncs
0001:00360744  _zim_Phar_createDefaultStub
0001:003607f4  _zim_Phar_mapPhar
0001:0036089c  _zim_Phar_loadPhar
0001:00360950  _zim_Phar_apiVersion
0001:0036097c  _zim_Phar_canCompress
0001:00360a2c  _zim_Phar_canWrite
0001:00360a5c  _zim_Phar_isValidPharFilename
0001:00360c00  _zim_Phar___construct
0001:00361004  _zim_Phar_getSupportedSignatures
0001:003610a4  _zim_Phar_getSupportedCompression
0001:00361288  _zim_Phar_unlinkArchive
0001:003614ec  _zim_Phar___destruct
0001:003620c4  _zim_Phar_buildFromDirectory
0001:003625e0  _zim_Phar_buildFromIterator
0001:003627a4  _zim_Phar_count
0001:00362828  _zim_Phar_isFileFormat
0001:00363d8c  _zim_Phar_convertToExecutable
0001:00364080  _zim_Phar_convertToData
0001:003642dc  _zim_Phar_isCompressed
0001:00364360  _zim_Phar_isWritable
0001:00364438  _zim_Phar_delete
0001:003645f0  _zim_Phar_getAlias
0001:00364660  _zim_Phar_getPath
0001:003647b0  _zim_Phar_setAlias
0001:00364c74  _zim_Phar_getVersion
0001:00364cec  _zim_Phar_startBuffering
0001:00364d3c  _zim_Phar_isBuffering
0001:00364da0  _zim_Phar_stopBuffering
0001:00364f30  _zim_Phar_setStub
0001:003651e4  _zim_Phar_setDefaultStub
0001:003654bc  _zim_Phar_setSignatureAlgorithm
0001:0036566c  _zim_Phar_getSignature
0001:003657d4  _zim_Phar_getModified
0001:00365980  _zim_Phar_compress
0001:00365bd0  _zim_Phar_decompress
0001:00365f24  _zim_Phar_compressFiles
0001:00366160  _zim_Phar_decompressFiles
0001:00366450  _zim_Phar_copy
0001:00366970  _zim_Phar_offsetExists
0001:00366ba0  _zim_Phar_offsetGet
0001:00367320  _zim_Phar_offsetSet
0001:003674ac  _zim_Phar_offsetUnset
0001:00367684  _zim_Phar_addEmptyDir
0001:00367820  _zim_Phar_addFile
0001:003679b0  _zim_Phar_addFromString
0001:00367a88  _zim_Phar_getStub
0001:00367d3c  _zim_Phar_hasMetadata
0001:00367da0  _zim_Phar_getMetadata
0001:00367eb4  _zim_Phar_setMetadata
0001:003680c8  _zim_Phar_delMetadata
0001:00368b68  _zim_Phar_extractTo
0001:00369078  _zim_PharFileInfo___construct
0001:003692b4  _zim_PharFileInfo___destruct
0001:00369350  _zim_PharFileInfo_getCompressedSize
0001:003693cc  _zim_PharFileInfo_isCompressed
0001:003694ec  _zim_PharFileInfo_getCRC32
0001:00369570  _zim_PharFileInfo_isCRCChecked
0001:003695d0  _zim_PharFileInfo_getPharFlags
0001:003696e4  _zim_PharFileInfo_chmod
0001:00369900  _zim_PharFileInfo_hasMetadata
0001:00369960  _zim_PharFileInfo_getMetadata
0001:00369ac4  _zim_PharFileInfo_setMetadata
0001:00369d5c  _zim_PharFileInfo_delMetadata
0001:00369f9c  _zim_PharFileInfo_getContent
0001:0036a428  _zim_PharFileInfo_compress
0001:0036a864  _zim_PharFileInfo_decompress
0001:0036b914  _phar_object_init
0002:00001e90  _php_archive_methods
0002:00002310  _php_entry_methods
0002:0000bf30  _phar_exception_methods
Module: U:\dev\php-5.3.6\ext\phar\phar_path_check.o(phar_path_check.o)
0001:0036c318  _phar_path_check
Module: U:\dev\php-5.3.6\ext\posix\posix.o(posix.o)
0002:000228c0  _posix_globals_id
0001:0036ce50  _posix_functions
0001:0036d2e4  _zif_posix_kill
0001:0036d358  _zif_posix_getpid
0001:0036d388  _zif_posix_getppid
0001:0036d3b8  _zif_posix_getuid
0001:0036d47c  _zif_posix_setuid
0001:0036d418  _zif_posix_geteuid
0001:0036d554  _zif_posix_seteuid
0001:0036d3e8  _zif_posix_getgid
0001:0036d4e8  _zif_posix_setgid
0001:0036d448  _zif_posix_getegid
0001:0036d5c0  _zif_posix_setegid
0001:0036d62c  _zif_posix_getgroups
0001:0036d6bc  _zif_posix_getlogin
0001:0036d734  _zif_posix_getpgrp
0001:0036d764  _zif_posix_setsid
0001:0036d794  _zif_posix_setpgid
0001:0036d804  _zif_posix_getpgid
0001:0036d86c  _zif_posix_getsid
0001:0036d900  _zif_posix_uname
0001:0036da00  _zif_posix_times
0001:0036dbec  _zif_posix_ttyname
0001:0036dd3c  _zif_posix_isatty
0001:0036de58  _zif_posix_getcwd
0001:0036deec  _zif_posix_mkfifo
0001:0036e04c  _zif_posix_mknod
0001:0036e274  _zif_posix_access
0001:0036e3cc  _zif_posix_getgrnam
0001:0036e4f8  _zif_posix_getgrgid
0001:0036e6ec  _zif_posix_getpwnam
0001:0036e7e8  _zif_posix_getpwuid
0001:0036ea7c  _zif_posix_getrlimit
0001:0036eb04  _zif_posix_get_last_error
0001:0036eb40  _zif_posix_strerror
0001:0036eba8  _zif_posix_initgroups
0001:0036e18c  _php_posix_group_to_array
0001:0036e600  _php_posix_passwd_to_array
0002:00002450  _posix_module_entry
0002:000024b0  _limits
Module: U:\dev\php-5.3.6\ext\reflection\php_reflection.o(php_reflection.o)
0002:000228d0  _reflection_exception_ptr
0002:000228e0  _reflection_class_ptr
0002:000228f0  _reflection_extension_ptr
0002:00022900  _reflection_parameter_ptr
0002:00022910  _reflection_function_ptr
0002:00022920  _reflection_method_ptr
0002:00022930  _reflection_property_ptr
0002:00022940  _reflection_ptr
0002:00022950  _reflector_ptr
0002:00022960  _reflection_function_abstract_ptr
0002:00022970  _reflection_object_ptr
0001:003710f8  _zend_reflection_class_factory
0001:00371ba8  _zim_reflection___clone
0001:00371c34  _zim_reflection_export
0001:00371e04  _zim_reflection_getModifierNames
0001:00371f14  _zim_reflection_function_export
0001:00371f5c  _zim_reflection_function___construct
0001:00372110  _zim_reflection_function___toString
0001:003721d8  _zim_reflection_function_getName
0001:0037222c  _zim_reflection_function_isClosure
0001:003722c8  _zim_reflection_function_isInternal
0001:00372364  _zim_reflection_function_isUserDefined
0001:00372424  _zim_reflection_function_isDisabled
0001:0037251c  _zim_reflection_function_getFileName
0001:003725e0  _zim_reflection_function_getStartLine
0001:00372688  _zim_reflection_function_getEndLine
0001:00372730  _zim_reflection_function_getDocComment
0001:003727ec  _zim_reflection_function_getStaticVariables
0001:003728ec  _zim_reflection_function_invoke
0001:00372b28  _zim_reflection_function_invokeArgs
0001:00372d5c  _zim_reflection_function_returnsReference
0001:00372e40  _zim_reflection_function_getNumberOfParameters
0001:00372f1c  _zim_reflection_function_getNumberOfRequiredParameters
0001:00372ff8  _zim_reflection_function_getParameters
0001:00373154  _zim_reflection_function_getExtension
0001:00373250  _zim_reflection_function_getExtensionName
0001:00373360  _zim_reflection_parameter_export
0001:003734dc  _zim_reflection_parameter___construct
0001:00373ba4  _zim_reflection_parameter___toString
0001:00373c6c  _zim_reflection_parameter_getName
0001:00373cc0  _zim_reflection_parameter_getDeclaringFunction
0001:00373dc8  _zim_reflection_parameter_getDeclaringClass
0001:00373f64  _zim_reflection_parameter_getClass
0001:003740dc  _zim_reflection_parameter_isArray
0001:0037417c  _zim_reflection_parameter_allowsNull
0001:0037421c  _zim_reflection_parameter_isPassedByReference
0001:003742bc  _zim_reflection_parameter_getPosition
0001:00374350  _zim_reflection_parameter_isOptional
0001:003743ec  _zim_reflection_parameter_isDefaultValueAvailable
0001:00374520  _zim_reflection_parameter_getDefaultValue
0001:00374658  _zim_reflection_method_export
0001:003746e4  _zim_reflection_method___construct
0001:00374aac  _zim_reflection_method___toString
0001:00374c64  _zim_reflection_method_invoke
0001:00374fd4  _zim_reflection_method_invokeArgs
0001:00375314  _zim_reflection_method_isFinal
0001:00375338  _zim_reflection_method_isAbstract
0001:0037535c  _zim_reflection_method_isPublic
0001:00375380  _zim_reflection_method_isPrivate
0001:003753a4  _zim_reflection_method_isProtected
0001:003753c8  _zim_reflection_method_isStatic
0001:003753ec  _zim_reflection_function_isDeprecated
0001:00375410  _zim_reflection_function_inNamespace
0001:003754b0  _zim_reflection_function_getNamespaceName
0001:00375578  _zim_reflection_function_getShortName
0001:00375674  _zim_reflection_method_isConstructor
0001:00375734  _zim_reflection_method_isDestructor
0001:003757d0  _zim_reflection_method_getModifiers
0001:00375864  _zim_reflection_method_getDeclaringClass
0001:00375998  _zim_reflection_method_getPrototype
0001:00375af0  _zim_reflection_method_setAccessible
0001:00375b3c  _zim_reflection_class_export
0001:00375df0  _zim_reflection_class___construct
0001:00375e14  _zim_reflection_class_getStaticProperties
0001:003760b8  _zim_reflection_class_getStaticPropertyValue
0001:003761f8  _zim_reflection_class_setStaticPropertyValue
0001:0037632c  _zim_reflection_class_getDefaultProperties
0001:00376564  _zim_reflection_class___toString
0001:0037662c  _zim_reflection_class_getName
0001:00376680  _zim_reflection_class_isInternal
0001:0037671c  _zim_reflection_class_isUserDefined
0001:003767b8  _zim_reflection_class_getFileName
0001:0037687c  _zim_reflection_class_getStartLine
0001:00376928  _zim_reflection_class_getEndLine
0001:003769d4  _zim_reflection_class_getDocComment
0001:00376a98  _zim_reflection_class_getConstructor
0001:00376b54  _zim_reflection_class_hasMethod
0001:00376cdc  _zim_reflection_class_getMethod
0001:00377070  _zim_reflection_class_getMethods
0001:003771fc  _zim_reflection_class_hasProperty
0001:00377410  _zim_reflection_class_getProperty
0001:00377814  _zim_reflection_class_getProperties
0001:00377984  _zim_reflection_class_hasConstant
0001:00377a98  _zim_reflection_class_getConstants
0001:00377b60  _zim_reflection_class_getConstant
0001:00377d54  _zim_reflection_class_isInstantiable
0001:00377e20  _zim_reflection_class_isInterface
0001:00377e44  _zim_reflection_class_isFinal
0001:00377e68  _zim_reflection_class_isAbstract
0001:00377e8c  _zim_reflection_class_getModifiers
0001:00377f20  _zim_reflection_class_isInstance
0001:003780e4  _zim_reflection_class_newInstance
0001:0037837c  _zim_reflection_class_newInstanceArgs
0001:00378638  _zim_reflection_class_getInterfaces
0001:00378748  _zim_reflection_class_getInterfaceNames
0001:0037881c  _zim_reflection_class_getParentClass
0001:0037895c  _zim_reflection_class_isSubclassOf
0001:00378b58  _zim_reflection_class_implementsInterface
0001:00378d28  _zim_reflection_class_isIterateable
0001:00378e28  _zim_reflection_class_getExtension
0001:00378f34  _zim_reflection_class_getExtensionName
0001:0037905c  _zim_reflection_class_inNamespace
0001:003790fc  _zim_reflection_class_getNamespaceName
0001:003791c4  _zim_reflection_class_getShortName
0001:003792c0  _zim_reflection_object_export
0001:003792e8  _zim_reflection_object___construct
0001:0037930c  _zim_reflection_property_export
0001:00379354  _zim_reflection_property___construct
0001:003796b8  _zim_reflection_property___toString
0001:00379778  _zim_reflection_property_getName
0001:0037986c  _zim_reflection_property_isPublic
0001:00379890  _zim_reflection_property_isPrivate
0001:003798b4  _zim_reflection_property_isProtected
0001:003798d8  _zim_reflection_property_isStatic
0001:003798fc  _zim_reflection_property_isDefault
0001:00379920  _zim_reflection_property_getModifiers
0001:00379a10  _zim_reflection_property_getValue
0001:00379ce0  _zim_reflection_property_setValue
0001:0037a054  _zim_reflection_property_getDeclaringClass
0001:0037a170  _zim_reflection_property_getDocComment
0001:0037a224  _zim_reflection_property_setAccessible
0001:0037a270  _zim_reflection_extension_export
0001:0037a2b4  _zim_reflection_extension___construct
0001:0037a44c  _zim_reflection_extension___toString
0001:0037a504  _zim_reflection_extension_getName
0001:0037a558  _zim_reflection_extension_getVersion
0001:0037a614  _zim_reflection_extension_getFunctions
0001:0037a7fc  _zim_reflection_extension_getConstants
0001:0037a958  _zim_reflection_extension_getINIEntries
0001:0037aadc  _zim_reflection_extension_getClasses
0001:0037aba0  _zim_reflection_extension_getClassNames
0001:0037ac70  _zim_reflection_extension_getDependencies
0001:0037add8  _zim_reflection_extension_info
0001:0037cb28  _reflection_ext_functions
0001:0037cd6c  _zm_startup_reflection
0001:0037db10  _zm_info_reflection
0002:00002510  _reflection_module_entry
Module: U:\dev\php-5.3.6\ext\session\session.o(session.o)
0002:00022980  _ps_globals_id
0001:0037dc74  _php_add_session_var
0001:0037e060  _php_set_session_var
0001:0037e27c  _php_get_session_var
0001:0037ea1c  _php_session_create_id
0001:00381f6c  __php_find_ps_module
0001:00381fc0  __php_find_ps_serializer
0001:00380424  _ps_srlzr_encode_php_binary
0001:00380718  _ps_srlzr_decode_php_binary
0001:003808bc  _ps_srlzr_encode_php
0001:00380c6c  _ps_srlzr_decode_php
0001:00380e24  _php_session_register_serializer
0001:00380e70  _php_session_register_module
0001:003824b4  _php_session_start
0001:00382c98  _session_adapt_url
0002:00002750  _session_module_entry
Module: U:\dev\php-5.3.6\ext\session\mod_files.o(mod_files.o)
0001:00385590  _ps_open_files
0001:00385728  _ps_close_files
0001:003857b8  _ps_read_files
0001:0038590c  _ps_write_files
0001:003859c0  _ps_delete_files
0001:00385a38  _ps_gc_files
0002:000027b0  _ps_mod_files
Module: U:\dev\php-5.3.6\ext\session\mod_user.o(mod_user.o)
0001:00385b3c  _ps_open_user
0001:00385c38  _ps_close_user
0001:00385c9c  _ps_read_user
0001:00385d78  _ps_write_user
0001:00385e7c  _ps_delete_user
0001:00385f3c  _ps_gc_user
0002:000027d0  _ps_mod_user
Module: U:\dev\php-5.3.6\ext\simplexml\simplexml.o(simplexml.o)
0001:00385ffc  _sxe_get_element_class_entry
0001:003885f8  _zim_simplexml_element_xpath
0001:0038881c  _zim_simplexml_element_registerXPathNamespace
0001:003888b4  _zim_simplexml_element_asXML
0001:00388c44  _zim_simplexml_element_getNamespaces
0001:00388e1c  _zim_simplexml_element_getDocNamespaces
0001:00388e8c  _zim_simplexml_element_children
0001:00388f30  _zim_simplexml_element_getName
0001:00388fc8  _zim_simplexml_element_attributes
0001:003890f4  _zim_simplexml_element_addChild
0001:0038933c  _zim_simplexml_element_addAttribute
0001:00389770  _zim_simplexml_element___toString
0001:003899f0  _zim_simplexml_element_count
0001:00389d38  _sxe_object_new
0001:00389d64  _zif_simplexml_load_file
0001:00389e70  _zif_simplexml_load_string
0001:00389fb0  _zim_simplexml_element___construct
0001:0038a324  _php_sxe_get_iterator
0001:0038a43c  _php_sxe_move_forward_iterator
0001:0038a4e4  _simplexml_export_node
0001:0038a580  _zif_simplexml_import_dom
0001:0038ab50  _simplexml_functions
0001:0038add0  _zm_startup_simplexml
0001:0038af5c  _zm_shutdown_simplexml
0001:0038afb4  _zm_info_simplexml
0002:00002854  _php_sxe_iterator_funcs
0002:00002870  _simplexml_module_entry
0002:0000c020  _sxe_class_entry
Module: U:\dev\php-5.3.6\ext\simplexml\sxe.o(sxe.o)
0002:00022990  _ce_SimpleXMLElement
0001:0038b01c  _zim_ce_SimpleXMLIterator_rewind
0001:0038b04c  _zim_ce_SimpleXMLIterator_valid
0001:0038b07c  _zim_ce_SimpleXMLIterator_current
0001:0038b0e0  _zim_ce_SimpleXMLIterator_key
0001:0038b150  _zim_ce_SimpleXMLIterator_next
0001:0038b198  _zim_ce_SimpleXMLIterator_hasChildren
0001:0038b234  _zim_ce_SimpleXMLIterator_getChildren
0001:0038b3b4  _zm_startup_sxe
0002:0000c030  _ce_SimpleXMLIterator
Module: U:\dev\php-5.3.6\ext\soap\soap.o(soap.o)
0002:000229a0  _soap_globals_id
0002:000229b0  _soap_var_class_entry
0001:00392c40  _zif_use_soap_error_handler
0001:00392ca0  _zif_is_soap_fault
0001:0038e040  _zim_SoapFault_SoapFault
0001:0038e23c  _zim_SoapFault___toString
0001:0038ec6c  _zim_SoapServer_SoapServer
0001:0038f1dc  _zim_SoapServer_setPersistence
0001:0038f340  _zim_SoapServer_setClass
0001:0038f50c  _zim_SoapServer_setObject
0001:0038f920  _zim_SoapServer_addFunction
0001:0038f67c  _zim_SoapServer_getFunctions
0001:00390058  _zim_SoapServer_handle
0001:00391b9c  _zim_SoapServer_fault
0001:00391d70  _zim_SoapServer_addSoapHeader
0001:00392f30  _zim_SoapClient_SoapClient
0001:003951e8  _zim_SoapClient___call
0001:003957cc  _zim_SoapClient___getLastRequest
0001:00395844  _zim_SoapClient___getLastResponse
0001:003958d4  _zim_SoapClient___getLastRequestHeaders
0001:00395964  _zim_SoapClient___getLastResponseHeaders
0001:00395590  _zim_SoapClient___getFunctions
0001:003956a8  _zim_SoapClient___getTypes
0001:003959e4  _zim_SoapClient___doRequest
0001:00395ad8  _zim_SoapClient___setCookie
0001:00395dc4  _zim_SoapClient___setLocation
0001:00395c60  _zim_SoapClient___setSoapHeaders
0001:0038e3dc  _zim_SoapVar_SoapVar
0001:0038de00  _zim_SoapParam_SoapParam
0001:0038dec4  _zim_SoapHeader_SoapHeader
0001:0038d018  _zm_startup_soap
0001:0038ca6c  _zm_shutdown_soap
0001:0038cb10  _zm_activate_soap
0001:0038dd88  _zm_info_soap
0001:0038c42c  _OnUpdateCacheEnabled
0001:0038c490  _OnUpdateCacheMode
0001:00395ee8  _add_soap_fault
0002:000028d0  _soap_module_entry
0002:0000c040  _le_url
Module: U:\dev\php-5.3.6\ext\soap\php_encoding.o(php_encoding.o)
0001:0039d0c8  _whiteSpace_replace
0001:0039d0f4  _whiteSpace_collapse
0001:003a6d6c  _get_conversion
0001:0039e380  _master_to_xml
0001:003a68d0  _encode_add_ns
0001:0039e8e8  _master_to_zval
0001:0039e9fc  _to_xml_user
0001:0039eb74  _to_zval_user
0001:003a6394  _sdl_guess_convert_zval
0001:003a6478  _sdl_guess_convert_xml
0001:003a6c3c  _encode_reset_ns
0001:003a6cc0  _encode_finish
0001:003a7938  _delete_encoder
0001:003a7994  _delete_encoder_persistent
0002:00002930  _defaultEncoding
0002:00003180  _numDefaultEncodings
Module: U:\dev\php-5.3.6\ext\soap\php_http.o(php_http.o)
0001:003a7ec4  _proxy_authentication
0001:003a82b0  _basic_authentication
0001:003a9680  _make_http_soap_request
Module: U:\dev\php-5.3.6\ext\soap\php_packet_soap.o(php_packet_soap.o)
0001:003afd7c  _parse_packet_soap
Module: U:\dev\php-5.3.6\ext\soap\php_schema.o(php_schema.o)
0001:003b1548  _load_schema
0001:003b8190  _delete_type
0001:003b85c8  _delete_attribute
0001:003b8760  _delete_restriction_var_char
0001:003b37d4  _schema_min_max
0001:003b80d8  _delete_model
0001:003b8540  _delete_extra_attribute
0001:003b7ed8  _schema_pass2
0001:003b8134  _delete_model_persistent
0001:003b8728  _delete_restriction_var_int
0001:003b8368  _delete_type_persistent
0001:003b8744  _delete_restriction_var_int_persistent
0001:003b8798  _delete_restriction_var_char_persistent
0001:003b8584  _delete_extra_attribute_persistent
0001:003b8678  _delete_attribute_persistent
Module: U:\dev\php-5.3.6\ext\soap\php_sdl.o(php_sdl.o)
0001:003b87ec  _get_encoder_from_prefix
0001:003b8a90  _get_encoder
0001:003b8d2c  _get_encoder_ex
0001:003b8d9c  _get_binding_from_type
0001:003b8e00  _get_binding_from_name
0001:003b9164  _sdl_set_uri_credentials
0001:003b9378  _sdl_restore_uri_credentials
0001:003c5528  _get_sdl
0001:003c640c  _delete_sdl_impl
0001:003c6538  _delete_sdl
Module: U:\dev\php-5.3.6\ext\soap\php_xml.o(php_xml.o)
0001:003c6c38  _soap_xmlParseFile
0001:003c6d28  _soap_xmlParseMemory
0001:003c6ddc  _attr_find_ns
0001:003c6e08  _node_find_ns
0001:003c6e2c  _attr_is_equal_ex
0001:003c6e90  _node_is_equal_ex
0001:003c6ef4  _get_attribute_ex
0001:003c6f34  _get_node_ex
0001:003c6f74  _get_node_recurisve_ex
0001:003c6fd0  _get_node_with_attribute_ex
0001:003c7044  _get_node_with_attribute_recursive_ex
0001:003c70e0  _parse_namespace
Module: U:\dev\php-5.3.6\ext\sockets\sockets.o(sockets.o)
0002:000229c0  _sockets_globals_id
0001:003c7e00  _sockets_functions
0001:003c977c  _zif_socket_select
0001:003ca76c  _zif_socket_create
0001:003c9b00  _zif_socket_create_listen
0001:003cbf78  _zif_socket_create_pair
0001:003c9b80  _zif_socket_accept
0001:003c9c14  _zif_socket_set_nonblock
0001:003c9c94  _zif_socket_set_block
0001:003c9d18  _zif_socket_listen
0001:003c9df4  _zif_socket_close
0001:003c9e80  _zif_socket_write
0001:003c9fbc  _zif_socket_read
0001:003ca1d0  _zif_socket_getsockname
0001:003ca450  _zif_socket_getpeername
0001:003ca918  _zif_socket_connect
0001:003caac8  _zif_socket_strerror
0001:003cab88  _zif_socket_bind
0001:003cad3c  _zif_socket_recv
0001:003caec4  _zif_socket_send
0001:003cafcc  _zif_socket_recvfrom
0001:003cb3fc  _zif_socket_sendto
0001:003cb65c  _zif_socket_get_option
0001:003cb868  _zif_socket_set_option
0001:003cc1dc  _zif_socket_shutdown
0001:003cc2bc  _zif_socket_last_error
0001:003cc344  _zif_socket_clear_error
0001:003c8bc0  _zm_startup_sockets
0001:003c94d0  _zm_deactivate_sockets
0001:003c94a8  _zm_info_sockets
0001:003c8048  _php_sockets_le_socket
0002:000031b0  _sockets_module_entry
0002:0000c170  _inet_ntoa_lock
Module: U:\dev\php-5.3.6\ext\spl\php_spl.o(php_spl.o)
0002:000229d0  _spl_globals_id
0001:003cc550  _zif_class_parents
0001:003cc614  _zif_class_implements
0001:003cc6c4  _zif_spl_classes
0001:003ccd74  _zif_spl_autoload
0001:003ccf88  _zif_spl_autoload_extensions
0001:003cd0b0  _zif_spl_autoload_call
0001:003cd3b8  _zif_spl_autoload_register
0001:003cd958  _zif_spl_autoload_unregister
0001:003cdc9c  _zif_spl_autoload_functions
0001:003cdeb8  _zif_spl_object_hash
0001:003cdf2c  _php_spl_object_hash
0001:003ce050  _spl_build_class_list_string
0001:003ce0b0  _zm_info_spl
0001:003cf120  _spl_functions
0001:003cf238  _zm_startup_spl
0001:003cf2ac  _zm_activate_spl
0001:003cf2dc  _zm_deactivate_spl
0002:00003210  _spl_module_entry
Module: U:\dev\php-5.3.6\ext\spl\spl_functions.o(spl_functions.o)
0001:003cf3ac  _spl_register_interface
0001:003cf4b0  _spl_register_std_class
0001:003cf5c8  _spl_register_sub_class
0001:003cf704  _spl_register_property
0001:003cf710  _spl_add_class_name
0001:003cf7bc  _spl_add_interfaces
0001:003cf80c  _spl_add_classes
0001:003cf888  _spl_gen_private_prop_name
Module: U:\dev\php-5.3.6\ext\spl\spl_engine.o(spl_engine.o)
0001:003cf8bc  _spl_instantiate
0001:003cf908  _spl_offset_convert_to_long
Module: U:\dev\php-5.3.6\ext\spl\spl_iterators.o(spl_iterators.o)
0002:000229e0  _spl_ce_RecursiveIterator
0002:000229f0  _spl_ce_RecursiveIteratorIterator
0002:00022a00  _spl_ce_RecursiveCachingIterator
0002:00022a10  _spl_ce_RecursiveTreeIterator
0002:00022a20  _spl_ce_FilterIterator
0002:00022a30  _spl_ce_RecursiveFilterIterator
0002:00022a40  _spl_ce_ParentIterator
0002:00022a50  _spl_ce_RegexIterator
0002:00022a60  _spl_ce_RecursiveRegexIterator
0002:00022a70  _spl_ce_LimitIterator
0002:00022a80  _spl_ce_CachingIterator
0002:00022a90  _spl_ce_IteratorIterator
0002:00022aa0  _spl_ce_NoRewindIterator
0002:00022ab0  _spl_ce_InfiniteIterator
0002:00022ac0  _spl_ce_AppendIterator
0002:00022ad0  _spl_ce_OuterIterator
0002:00022ae0  _spl_ce_Countable
0002:00022af0  _spl_ce_SeekableIterator
0002:00022b00  _spl_ce_EmptyIterator
0001:003cfa50  _spl_funcs_RecursiveIterator
0001:003d0b58  _zim_spl_RecursiveIteratorIterator___construct
0001:003d0b88  _zim_spl_RecursiveIteratorIterator_rewind
0001:003d0bdc  _zim_spl_RecursiveIteratorIterator_valid
0001:003d0c34  _zim_spl_RecursiveIteratorIterator_key
0001:003d0cc8  _zim_spl_RecursiveIteratorIterator_current
0001:003d0d64  _zim_spl_RecursiveIteratorIterator_next
0001:003d0db8  _zim_spl_RecursiveIteratorIterator_getDepth
0001:003d0e00  _zim_spl_RecursiveIteratorIterator_getSubIterator
0001:003d0e9c  _zim_spl_RecursiveIteratorIterator_getInnerIterator
0001:003d0f28  _zim_spl_RecursiveIteratorIterator_beginIteration
0001:003d0f44  _zim_spl_RecursiveIteratorIterator_endIteration
0001:003d0f60  _zim_spl_RecursiveIteratorIterator_callHasChildren
0001:003d1030  _zim_spl_RecursiveIteratorIterator_callGetChildren
0001:003d10f4  _zim_spl_RecursiveIteratorIterator_beginChildren
0001:003d1110  _zim_spl_RecursiveIteratorIterator_endChildren
0001:003d112c  _zim_spl_RecursiveIteratorIterator_nextElement
0001:003d116c  _zim_spl_RecursiveIteratorIterator_setMaxDepth
0001:003d11cc  _zim_spl_RecursiveIteratorIterator_getMaxDepth
0001:003d2090  _zim_spl_RecursiveTreeIterator___construct
0001:003d20f0  _zim_spl_RecursiveTreeIterator_setPrefixPart
0001:003d2220  _zim_spl_RecursiveTreeIterator_getPrefix
0001:003d2278  _zim_spl_RecursiveTreeIterator_getEntry
0001:003d22d0  _zim_spl_RecursiveTreeIterator_getPostfix
0001:003d2328  _zim_spl_RecursiveTreeIterator_current
0001:003d24bc  _zim_spl_RecursiveTreeIterator_key
0001:003d30e0  _zim_spl_FilterIterator___construct
0001:003d3110  _zim_spl_dual_it_getInnerIterator
0001:003d3194  _zim_spl_dual_it_rewind
0001:003d3290  _zim_spl_dual_it_valid
0001:003d32d8  _zim_spl_dual_it_key
0001:003d334c  _zim_spl_dual_it_current
0001:003d33d0  _zim_spl_dual_it_next
0001:003d34b0  _zim_spl_FilterIterator_rewind
0001:003d366c  _zim_spl_FilterIterator_next
0001:003d380c  _zim_spl_RecursiveFilterIterator___construct
0001:003d383c  _zim_spl_RecursiveFilterIterator_hasChildren
0001:003d38e8  _zim_spl_RecursiveFilterIterator_getChildren
0001:003d39d8  _zim_spl_ParentIterator___construct
0001:003d3a08  _zim_spl_RegexIterator___construct
0001:003d3a48  _zim_spl_RegexIterator_accept
0001:003d3de4  _zim_spl_RegexIterator_getMode
0001:003d3e28  _zim_spl_RegexIterator_setMode
0001:003d3e84  _zim_spl_RegexIterator_getFlags
0001:003d3ec8  _zim_spl_RegexIterator_setFlags
0001:003d3f04  _zim_spl_RegexIterator_getPregFlags
0001:003d3f50  _zim_spl_RegexIterator_setPregFlags
0001:003d3f94  _zim_spl_RecursiveRegexIterator___construct
0001:003d3fc4  _zim_spl_RecursiveRegexIterator_getChildren
0001:003d4840  _zim_spl_LimitIterator___construct
0001:003d4870  _zim_spl_LimitIterator_rewind
0001:003d48d0  _zim_spl_LimitIterator_valid
0001:003d491c  _zim_spl_LimitIterator_next
0001:003d49f8  _zim_spl_LimitIterator_seek
0001:003d4a4c  _zim_spl_LimitIterator_getPosition
0001:003d4c78  _zim_spl_CachingIterator___construct
0001:003d4ca8  _zim_spl_CachingIterator_rewind
0001:003d4d58  _zim_spl_CachingIterator_valid
0001:003d4da0  _zim_spl_CachingIterator_next
0001:003d4de8  _zim_spl_CachingIterator_hasNext
0001:003d4e94  _zim_spl_CachingIterator___toString
0001:003d4fdc  _zim_spl_CachingIterator_offsetSet
0001:003d50ac  _zim_spl_CachingIterator_offsetGet
0001:003d51c0  _zim_spl_CachingIterator_offsetUnset
0001:003d5264  _zim_spl_CachingIterator_offsetExists
0001:003d5360  _zim_spl_CachingIterator_getCache
0001:003d5418  _zim_spl_CachingIterator_getFlags
0001:003d5524  _zim_spl_CachingIterator_setFlags
0001:003d5638  _zim_spl_CachingIterator_count
0001:003d59d8  _zim_spl_RecursiveCachingIterator___construct
0001:003d5a08  _zim_spl_RecursiveCachingIterator_hasChildren
0001:003d5a50  _zim_spl_RecursiveCachingIterator_getChildren
0001:003d5ba0  _zim_spl_IteratorIterator___construct
0001:003d5cb0  _zim_spl_NoRewindIterator___construct
0001:003d5ce0  _zim_spl_NoRewindIterator_rewind
0001:003d5cfc  _zim_spl_NoRewindIterator_valid
0001:003d5d50  _zim_spl_NoRewindIterator_key
0001:003d5ddc  _zim_spl_NoRewindIterator_current
0001:003d5e70  _zim_spl_NoRewindIterator_next
0001:003d5f90  _zim_spl_InfiniteIterator___construct
0001:003d5fc0  _zim_spl_InfiniteIterator_next
0001:003d616c  _zim_spl_EmptyIterator_rewind
0001:003d6188  _zim_spl_EmptyIterator_valid
0001:003d61e0  _zim_spl_EmptyIterator_key
0001:003d6250  _zim_spl_EmptyIterator_current
0001:003d6298  _zim_spl_EmptyIterator_next
0001:003d6348  _spl_append_it_next_iterator
0001:003d6454  _spl_append_it_fetch
0001:003d6510  _spl_append_it_next
0001:003d6568  _zim_spl_AppendIterator___construct
0001:003d65cc  _zim_spl_AppendIterator_append
0001:003d66b8  _zim_spl_AppendIterator_rewind
0001:003d6720  _zim_spl_AppendIterator_valid
0001:003d6768  _zim_spl_AppendIterator_next
0001:003d67b0  _zim_spl_AppendIterator_getIteratorIndex
0001:003d6840  _zim_spl_AppendIterator_getArrayIterator
0001:003d6a4c  _spl_iterator_apply
0001:003d6ca4  _zif_iterator_to_array
0001:003d6d44  _zif_iterator_count
0001:003d6e14  _zif_iterator_apply
0001:003d7188  _zm_startup_spl_iterators
0002:00003270  _spl_recursive_it_iterator_funcs
Module: U:\dev\php-5.3.6\ext\spl\spl_array.o(spl_array.o)
0002:00022b10  _spl_ce_ArrayIterator
0002:00022b20  _spl_handler_ArrayObject
0002:00022b90  _spl_handler_ArrayIterator
0002:00022c00  _spl_ce_RecursiveArrayIterator
0002:00022c10  _spl_ce_ArrayObject
0001:003d8520  _spl_hash_verify_pos_ex
0001:003d8564  _spl_hash_verify_pos
0001:003db148  _spl_array_get_iterator
0001:003d9c50  _zim_spl_Array_offsetExists
0001:003d9ca4  _zim_spl_Array_offsetGet
0001:003d9d28  _zim_spl_Array_offsetSet
0001:003d9de8  _spl_array_iterator_append
0001:003d9f08  _zim_spl_Array_append
0001:003d9f3c  _zim_spl_Array_offsetUnset
0001:003d9f70  _zim_spl_Array_getArrayCopy
0001:003db1bc  _zim_spl_Array___construct
0001:003db26c  _zim_spl_Array_setIteratorClass
0001:003db2b0  _zim_spl_Array_getIteratorClass
0001:003db314  _zim_spl_Array_getFlags
0001:003db35c  _zim_spl_Array_setFlags
0001:003db3a4  _zim_spl_Array_exchangeArray
0001:003db4b4  _zim_spl_Array_getIterator
0001:003db5ac  _zim_spl_Array_rewind
0001:003db61c  _zim_spl_Array_seek
0001:003db860  _spl_array_object_count_elements
0001:003db97c  _zim_spl_Array_count
0001:003dbbf4  _zim_spl_Array_asort
0001:003dbc24  _zim_spl_Array_ksort
0001:003dbc54  _zim_spl_Array_uasort
0001:003dbc84  _zim_spl_Array_uksort
0001:003dbcb4  _zim_spl_Array_natsort
0001:003dbce8  _zim_spl_Array_natcasesort
0001:003dbd10  _zim_spl_Array_current
0001:003dbe58  _zim_spl_Array_key
0001:003dbe98  _spl_array_iterator_key
0001:003dbfbc  _zim_spl_Array_next
0001:003dc0ac  _zim_spl_Array_valid
0001:003dc1f8  _zim_spl_Array_hasChildren
0001:003dc354  _zim_spl_Array_getChildren
0001:003dc584  _spl_array_serialize_helper
0001:003dc850  _zim_spl_Array_serialize
0001:003dc914  _spl_array_serialize
0001:003dc9c0  _spl_array_unserialize_helper
0001:003dcc30  _zim_spl_Array_unserialize
0001:003dccf8  _spl_array_unserialize
0001:003dd5cc  _zm_startup_spl_array
0002:00003290  _spl_array_it_funcs
Module: U:\dev\php-5.3.6\ext\spl\spl_directory.o(spl_directory.o)
0002:00022c20  _spl_ce_SplFileObject
0002:00022c30  _spl_ce_SplFileInfo
0002:00022c40  _spl_ce_DirectoryIterator
0002:00022c50  _spl_ce_RecursiveDirectoryIterator
0002:00022c60  _spl_ce_FilesystemIterator
0002:00022c70  _spl_ce_GlobIterator
0002:00022c80  _spl_ce_SplTempFileObject
0001:003ddf30  _spl_filesystem_object_get_path
0001:003de4bc  _spl_filesystem_info_set_filename
0001:003df078  _spl_filesystem_object_construct
0001:003df1d4  _zim_spl_DirectoryIterator___construct
0001:003df1f8  _zim_spl_DirectoryIterator_rewind
0001:003df26c  _zim_spl_DirectoryIterator_key
0001:003df2c4  _zim_spl_DirectoryIterator_current
0001:003df334  _zim_spl_DirectoryIterator_next
0001:003df3fc  _zim_spl_DirectoryIterator_seek
0001:003df56c  _zim_spl_DirectoryIterator_valid
0001:003df5b4  _zim_spl_SplFileInfo_getPath
0001:003df610  _zim_spl_SplFileInfo_getFilename
0001:003df690  _zim_spl_DirectoryIterator_getFilename
0001:003df6f0  _zim_spl_SplFileInfo_getExtension
0001:003df81c  _zim_spl_DirectoryIterator_getExtension
0001:003df904  _zim_spl_SplFileInfo_getBasename
0001:003df9c0  _zim_spl_DirectoryIterator_getBasename
0001:003dfa48  _zim_spl_SplFileInfo_getPathname
0001:003dfab8  _zim_spl_FilesystemIterator_key
0001:003dfba4  _zim_spl_FilesystemIterator_current
0001:003dfd70  _zim_spl_DirectoryIterator_isDot
0001:003dfdf0  _zim_spl_SplFileInfo___construct
0001:003dfe5c  _zim_spl_SplFileInfo_getPerms
0001:003dff3c  _zim_spl_SplFileInfo_getInode
0001:003e001c  _zim_spl_SplFileInfo_getSize
0001:003e00fc  _zim_spl_SplFileInfo_getOwner
0001:003e01dc  _zim_spl_SplFileInfo_getGroup
0001:003e02bc  _zim_spl_SplFileInfo_getATime
0001:003e039c  _zim_spl_SplFileInfo_getMTime
0001:003e047c  _zim_spl_SplFileInfo_getCTime
0001:003e055c  _zim_spl_SplFileInfo_getType
0001:003e063c  _zim_spl_SplFileInfo_isWritable
0001:003e071c  _zim_spl_SplFileInfo_isReadable
0001:003e07fc  _zim_spl_SplFileInfo_isExecutable
0001:003e08dc  _zim_spl_SplFileInfo_isFile
0001:003e09bc  _zim_spl_SplFileInfo_isDir
0001:003e0a9c  _zim_spl_SplFileInfo_isLink
0001:003e0bbc  _zim_spl_SplFileInfo_getLinkTarget
0001:003e0d48  _zim_spl_SplFileInfo_getRealPath
0001:003e0eb8  _zim_spl_SplFileInfo_openFile
0001:003e0f00  _zim_spl_SplFileInfo_setFileClass
0001:003e0f68  _zim_spl_SplFileInfo_setInfoClass
0001:003e0fd0  _zim_spl_SplFileInfo_getFileInfo
0001:003e104c  _zim_spl_SplFileInfo_getPathInfo
0001:003e1100  _zim_spl_FilesystemIterator___construct
0001:003e1124  _zim_spl_FilesystemIterator_rewind
0001:003e11c4  _zim_spl_FilesystemIterator_getFlags
0001:003e120c  _zim_spl_FilesystemIterator_setFlags
0001:003e1260  _zim_spl_RecursiveDirectoryIterator_hasChildren
0001:003e1378  _zim_spl_RecursiveDirectoryIterator_getChildren
0001:003e15cc  _zim_spl_RecursiveDirectoryIterator_getSubPath
0001:003e163c  _zim_spl_RecursiveDirectoryIterator_getSubPathname
0001:003e16e4  _zim_spl_RecursiveDirectoryIterator___construct
0001:003e1708  _zim_spl_GlobIterator___construct
0001:003e1748  _zim_spl_GlobIterator_count
0001:003e1804  _spl_filesystem_dir_get_iterator
0001:003e1dec  _spl_filesystem_tree_get_iterator
0001:003e30c8  _zim_spl_SplFileObject___construct
0001:003e3220  _zim_spl_SplTempFileObject___construct
0001:003e3318  _zim_spl_SplFileObject_rewind
0001:003e336c  _zim_spl_SplFileObject_eof
0001:003e33c4  _zim_spl_SplFileObject_valid
0001:003e3444  _zim_spl_SplFileObject_fgets
0001:003e34b4  _zim_spl_SplFileObject_current
0001:003e3590  _zim_spl_SplFileObject_key
0001:003e35d4  _zim_spl_SplFileObject_next
0001:003e3634  _zim_spl_SplFileObject_setFlags
0001:003e366c  _zim_spl_SplFileObject_getFlags
0001:003e36ec  _zim_spl_SplFileObject_setMaxLineLen
0001:003e3740  _zim_spl_SplFileObject_getMaxLineLen
0001:003e3784  _zim_spl_SplFileObject_hasChildren
0001:003e37b4  _zim_spl_SplFileObject_getChildren
0001:003e382c  _zim_spl_SplFileObject_fgetcsv
0001:003e394c  _zim_spl_SplFileObject_setCsvControl
0001:003e3a54  _zim_spl_SplFileObject_getCsvControl
0001:003e3af0  _zim_spl_SplFileObject_flock
0001:003e3b68  _zim_spl_SplFileObject_fflush
0001:003e3ba8  _zim_spl_SplFileObject_ftell
0001:003e3bf0  _zim_spl_SplFileObject_fseek
0001:003e3c5c  _zim_spl_SplFileObject_fgetc
0001:003e3ce0  _zim_spl_SplFileObject_fgetss
0001:003e3dc4  _zim_spl_SplFileObject_fpassthru
0001:003e3dfc  _zim_spl_SplFileObject_fscanf
0001:003e3e80  _zim_spl_SplFileObject_fwrite
0001:003e3f70  _zim_spl_SplFileObject_fstat
0001:003e4000  _zim_spl_SplFileObject_ftruncate
0001:003e40c0  _zim_spl_SplFileObject_seek
0001:003e49d0  _zm_startup_spl_directory
0002:000032b0  _spl_filesystem_dir_it_funcs
0002:000032cc  _spl_filesystem_tree_it_funcs
Module: U:\dev\php-5.3.6\ext\spl\spl_exceptions.o(spl_exceptions.o)
0002:00022c90  _spl_ce_LogicException
0002:00022ca0  _spl_ce_BadFunctionCallException
0002:00022cb0  _spl_ce_BadMethodCallException
0002:00022cc0  _spl_ce_DomainException
0002:00022cd0  _spl_ce_InvalidArgumentException
0002:00022ce0  _spl_ce_LengthException
0002:00022cf0  _spl_ce_OutOfRangeException
0002:00022d00  _spl_ce_RuntimeException
0002:00022d10  _spl_ce_OutOfBoundsException
0002:00022d20  _spl_ce_OverflowException
0002:00022d30  _spl_ce_RangeException
0002:00022d40  _spl_ce_UnderflowException
0002:00022d50  _spl_ce_UnexpectedValueException
0001:003e4e3c  _zm_startup_spl_exceptions
Module: U:\dev\php-5.3.6\ext\spl\spl_observer.o(spl_observer.o)
0002:00022d60  _spl_handler_SplObjectStorage
0002:00022dd0  _spl_ce_SplObjectStorage
0002:00022de0  _spl_ce_SplObserver
0002:00022df0  _spl_ce_SplSubject
0002:00022e00  _spl_ce_MultipleIterator
0001:003e5120  _spl_SplOjectStorage_free_storage
0001:003e5190  _spl_object_storage_get
0001:003e51bc  _spl_object_storage_attach
0001:003e525c  _spl_object_storage_detach
0001:003e527c  _spl_object_storage_addall
0001:003e5800  _spl_object_storage_contains
0001:003e5820  _zim_spl_SplObjectStorage_attach
0001:003e5874  _zim_spl_SplObjectStorage_detach
0001:003e58dc  _zim_spl_SplObjectStorage_offsetGet
0001:003e5980  _zim_spl_SplObjectStorage_addAll
0001:003e59ec  _zim_spl_SplObjectStorage_removeAll
0001:003e5aa8  _zim_spl_SplObjectStorage_removeAllExcept
0001:003e5b88  _zim_spl_SplObjectStorage_contains
0001:003e5be0  _zim_spl_SplObjectStorage_count
0001:003e5c2c  _zim_spl_SplObjectStorage_rewind
0001:003e5c78  _zim_spl_SplObjectStorage_valid
0001:003e5cd4  _zim_spl_SplObjectStorage_key
0001:003e5d18  _zim_spl_SplObjectStorage_current
0001:003e5da8  _zim_spl_SplObjectStorage_getInfo
0001:003e5e38  _zim_spl_SplObjectStorage_setInfo
0001:003e5ea4  _zim_spl_SplObjectStorage_next
0001:003e5eec  _zim_spl_SplObjectStorage_serialize
0001:003e6420  _zim_spl_SplObjectStorage_unserialize
0001:003e6bb8  _zim_spl_MultipleIterator___construct
0001:003e6c20  _zim_spl_MultipleIterator_getFlags
0001:003e6c64  _zim_spl_MultipleIterator_setFlags
0001:003e6cd4  _zim_spl_MultipleIterator_attachIterator
0001:003e6dc8  _zim_spl_MultipleIterator_rewind
0001:003e6e8c  _zim_spl_MultipleIterator_next
0001:003e6f50  _zim_spl_MultipleIterator_valid
0001:003e73e4  _zim_spl_MultipleIterator_current
0001:003e7440  _zim_spl_MultipleIterator_key
0001:003e77b0  _zm_startup_spl_observer
Module: U:\dev\php-5.3.6\ext\spl\spl_dllist.o(spl_dllist.o)
0002:00022e10  _spl_ce_SplStack
0002:00022e20  _spl_ce_SplDoublyLinkedList
0002:00022e30  _spl_ce_SplQueue
0002:00022e40  _spl_handler_SplDoublyLinkedList
0001:003e84e8  _zim_spl_SplDoublyLinkedList_push
0001:003e8590  _zim_spl_SplDoublyLinkedList_unshift
0001:003e8660  _zim_spl_SplDoublyLinkedList_pop
0001:003e8738  _zim_spl_SplDoublyLinkedList_shift
0001:003e8810  _zim_spl_SplDoublyLinkedList_top
0001:003e88bc  _zim_spl_SplDoublyLinkedList_bottom
0001:003e8968  _zim_spl_SplDoublyLinkedList_count
0001:003e89b8  _zim_spl_SplDoublyLinkedList_isEmpty
0001:003e8a48  _zim_spl_SplDoublyLinkedList_setIteratorMode
0001:003e8ad0  _zim_spl_SplDoublyLinkedList_getIteratorMode
0001:003e8b0c  _zim_spl_SplDoublyLinkedList_offsetExists
0001:003e8bac  _zim_spl_SplDoublyLinkedList_offsetGet
0001:003e8c7c  _zim_spl_SplDoublyLinkedList_offsetSet
0001:003e8e04  _zim_spl_SplDoublyLinkedList_offsetUnset
0001:003e9124  _zim_spl_SplDoublyLinkedList_key
0001:003e9168  _zim_spl_SplDoublyLinkedList_prev
0001:003e91cc  _zim_spl_SplDoublyLinkedList_next
0001:003e922c  _zim_spl_SplDoublyLinkedList_valid
0001:003e9274  _zim_spl_SplDoublyLinkedList_rewind
0001:003e92d4  _zim_spl_SplDoublyLinkedList_current
0001:003e9394  _spl_dllist_get_iterator
0001:003e9850  _zm_startup_spl_dllist
0002:000032f0  _spl_dllist_it_funcs
Module: U:\dev\php-5.3.6\ext\spl\spl_heap.o(spl_heap.o)
0002:00022eb0  _spl_handler_SplHeap
0002:00022f20  _spl_ce_SplPriorityQueue
0002:00022f30  _spl_ce_SplMinHeap
0002:00022f40  _spl_ce_SplMaxHeap
0002:00022f50  _spl_ce_SplHeap
0002:00022f60  _spl_handler_SplPriorityQueue
0001:003ea780  _zim_spl_SplHeap_count
0001:003ea7d0  _zim_spl_SplHeap_isEmpty
0001:003ea864  _zim_spl_SplHeap_insert
0001:003ea958  _zim_spl_SplHeap_extract
0001:003eaa20  _zim_spl_SplPriorityQueue_insert
0001:003eabc4  _zim_spl_SplPriorityQueue_extract
0001:003eacf8  _zim_spl_SplPriorityQueue_top
0001:003eade0  _zim_spl_SplPriorityQueue_setExtractFlags
0001:003eae2c  _zim_spl_SplHeap_recoverFromCorruption
0001:003eae70  _zim_spl_SplPriorityQueue_compare
0001:003eaeb8  _zim_spl_SplHeap_top
0001:003eaf80  _zim_spl_SplMinHeap_compare
0001:003eafc8  _zim_spl_SplMaxHeap_compare
0001:003eb1b8  _zim_spl_SplHeap_key
0001:003eb200  _zim_spl_SplHeap_next
0001:003eb260  _zim_spl_SplHeap_valid
0001:003eb2b0  _zim_spl_SplHeap_rewind
0001:003eb2cc  _zim_spl_SplHeap_current
0001:003eb360  _zim_spl_SplPriorityQueue_current
0001:003eb45c  _spl_heap_get_iterator
0001:003eb4cc  _spl_pqueue_get_iterator
0001:003eba08  _zm_startup_spl_heap
0002:00003310  _spl_heap_it_funcs
0002:0000332c  _spl_pqueue_it_funcs
Module: U:\dev\php-5.3.6\ext\spl\spl_fixedarray.o(spl_fixedarray.o)
0002:00022fd0  _spl_ce_SplFixedArray
0002:00022fe0  _spl_handler_SplFixedArray
0001:003ed600  _spl_fixedarray_get_iterator
0001:003eca48  _zim_spl_SplFixedArray___construct
0001:003ecad0  _zim_spl_SplFixedArray_count
0001:003ecb28  _zim_spl_SplFixedArray_toArray
0001:003ecc88  _zim_spl_SplFixedArray_fromArray
0001:003ecf60  _zim_spl_SplFixedArray_getSize
0001:003ecfbc  _zim_spl_SplFixedArray_setSize
0001:003ed050  _zim_spl_SplFixedArray_offsetExists
0001:003ed0a8  _zim_spl_SplFixedArray_offsetGet
0001:003ed13c  _zim_spl_SplFixedArray_offsetSet
0001:003ed180  _zim_spl_SplFixedArray_offsetUnset
0001:003ed3c8  _zim_spl_SplFixedArray_key
0001:003ed40c  _zim_spl_SplFixedArray_next
0001:003ed444  _zim_spl_SplFixedArray_valid
0001:003ed4a8  _zim_spl_SplFixedArray_rewind
0001:003ed4e4  _zim_spl_SplFixedArray_current
0001:003ed84c  _zm_startup_spl_fixedarray
0002:00003350  _spl_fixedarray_it_funcs
Module: U:\dev\php-5.3.6\ext\standard\crypt_freesec.o(crypt_freesec.o)
0001:003edaf0  __crypt_extended_init
0001:003ee73c  __crypt_extended_r
Module: U:\dev\php-5.3.6\ext\standard\crypt_blowfish.o(crypt_blowfish.o)
0001:003eed20  _php_crypt_blowfish_rn
0001:003f1220  _php_crypt_gensalt_blowfish_rn
Module: U:\dev\php-5.3.6\ext\standard\crypt_sha512.o(crypt_sha512.o)
0001:003f241c  _php_sha512_crypt_r
0001:003f3050  _php_sha512_crypt
Module: U:\dev\php-5.3.6\ext\standard\crypt_sha256.o(crypt_sha256.o)
0001:003f30dc  ___php_stpncpy
0001:003f3118  ___php_mempcpy
0001:003f38bc  _php_sha256_crypt_r
0001:003f4234  _php_sha256_crypt
Module: U:\dev\php-5.3.6\ext\standard\php_crypt_r.o(php_crypt_r.o)
0002:00023050  _php_crypt_extended_init_lock
0001:003f42bc  _php_init_crypt_r
0001:003f42d0  _php_shutdown_crypt_r
0001:003f42e4  __crypt_extended_init_r
0001:003f434c  _php_md5_crypt_r
Module: U:\dev\php-5.3.6\ext\standard\array.o(array.o)
0002:00023060  _array_globals_id
0001:003f4890  _zm_startup_array
0001:003f4a34  _zm_shutdown_array
0001:003f4bc4  _zif_krsort
0001:003f4c40  _zif_ksort
0001:003f4d7c  _zif_count
0001:003f517c  _zif_natsort
0001:003f51a0  _zif_natcasesort
0001:003f51c4  _zif_asort
0001:003f5240  _zif_arsort
0001:003f52bc  _zif_sort
0001:003f5338  _zif_rsort
0001:003f5520  _zif_usort
0001:003f56b8  _zif_uasort
0001:003f5a8c  _zif_uksort
0001:003f5c24  _zif_end
0001:003f5cd0  _zif_prev
0001:003f5d7c  _zif_next
0001:003f5e28  _zif_reset
0001:003f5ed4  _zif_current
0001:003f5f64  _zif_key
0001:003f6044  _zif_min
0001:003f61dc  _zif_max
0001:003f66d4  _zif_array_walk
0001:003f67fc  _zif_array_walk_recursive
0001:003f6a54  _zif_in_array
0001:003f6a78  _zif_array_search
0001:003f6b30  _php_prefix_varname
0001:003f6c24  _zif_extract
0001:003f744c  _zif_compact
0001:003f7554  _zif_array_fill
0001:003f7614  _zif_array_fill_keys
0001:003f77a8  _zif_range
0001:003f7f04  _zif_shuffle
0001:003f7f54  _php_splice
0001:003f8208  _zif_array_push
0001:003f84ac  _zif_array_pop
0001:003f84d0  _zif_array_shift
0001:003f84f4  _zif_array_unshift
0001:003f85d4  _zif_array_splice
0001:003f87c4  _zif_array_slice
0001:003f8a48  _php_array_merge
0001:003f8f40  _php_array_replace_recursive
0001:003f936c  _zif_array_merge
0001:003f9390  _zif_array_merge_recursive
0001:003f93b4  _zif_array_replace
0001:003f93d8  _zif_array_replace_recursive
0001:003f9400  _zif_array_keys
0001:003f9590  _zif_array_values
0001:003f965c  _zif_array_count_values
0001:003f97cc  _zif_array_reverse
0001:003f9918  _zif_array_pad
0001:003f9b24  _zif_array_flip
0001:003f9c8c  _zif_array_change_key_case
0001:003f9dec  _zif_array_unique
0001:003fafa4  _zif_array_intersect_key
0001:003fafc8  _zif_array_intersect_ukey
0001:003faff0  _zif_array_intersect
0001:003fb018  _zif_array_uintersect
0001:003fb040  _zif_array_intersect_assoc
0001:003fb064  _zif_array_intersect_uassoc
0001:003fb08c  _zif_array_uintersect_assoc
0001:003fb0b0  _zif_array_uintersect_uassoc
0001:003fbdec  _zif_array_diff_key
0001:003fbe10  _zif_array_diff_ukey
0001:003fbe38  _zif_array_diff
0001:003fbe60  _zif_array_udiff
0001:003fbe88  _zif_array_diff_assoc
0001:003fbeac  _zif_array_diff_uassoc
0001:003fbed4  _zif_array_udiff_assoc
0001:003fbef8  _zif_array_udiff_uassoc
0001:003fbf20  _php_multisort_compare
0001:003fc090  _zif_array_multisort
0001:003fc6c8  _zif_array_rand
0001:003fc858  _zif_array_sum
0001:003fc9a0  _zif_array_product
0001:003fcb24  _zif_array_reduce
0001:003fcdd4  _zif_array_filter
0001:003fd038  _zif_array_map
0001:003fd5d8  _zif_array_key_exists
0001:003fd6b8  _zif_array_chunk
0001:003fd8e4  _zif_array_combine
Module: U:\dev\php-5.3.6\ext\standard\base64.o(base64.o)
0001:003fe390  _php_base64_encode
0001:003fe4cc  _php_base64_decode
0001:003fe4e4  _php_base64_decode_ex
0001:003fe6a8  _zif_base64_encode
0001:003fe70c  _zif_base64_decode
Module: U:\dev\php-5.3.6\ext\standard\basic_functions.o(basic_functions.o)
0002:00023070  _basic_globals_id
0001:0040a430  _basic_functions
0001:0040dd1c  _zif_constant
0001:0040ddb8  _php_inet_ntop
0001:0040de68  _php_inet_pton
0001:0040df10  _zif_ip2long
0001:0040df78  _zif_long2ip
0001:0040e00c  _zif_getenv
0001:0040e164  _zif_putenv
0001:0040e5cc  _zif_getopt
0001:0040d2cc  _zm_startup_basic
0001:0040d884  _zm_shutdown_basic
0001:0040d93c  _zm_activate_basic
0001:0040db0c  _zm_deactivate_basic
0001:0040dcc4  _zm_info_basic
0001:0040d0dc  _php_get_nan
0001:0040d0ec  _php_get_inf
0001:0040ed6c  _zif_sleep
0001:0040ee08  _zif_usleep
0001:0040eeb4  _zif_time_nanosleep
0001:0040efb4  _zif_time_sleep_until
0001:0040ed20  _zif_flush
0001:00411484  _zif_getservbyname
0001:004114ec  _zif_getservbyport
0001:00411570  _zif_getprotobyname
0001:004115c4  _zif_getprotobynumber
0001:004126a4  _zif_sys_getloadavg
0001:0040f0cc  _zif_get_current_user
0001:0040f1dc  _zif_get_cfg_var
0001:0040f284  _zif_set_magic_quotes_runtime
0001:0040f2ec  _zif_get_magic_quotes_gpc
0001:0040f2cc  _zif_get_magic_quotes_runtime
0001:00412424  _zif_import_request_variables
0001:0040f314  _zif_error_log
0001:0040f52c  _zif_error_get_last
0001:0040f620  _zif_call_user_func
0001:0040f714  _zif_call_user_func_array
0001:0040f84c  _zif_call_user_method
0001:0040f9d0  _zif_call_user_method_array
0001:0040fbf8  _zif_forward_static_call
0001:0040fd74  _zif_forward_static_call_array
0001:0041131c  _zif_print_r
0001:00410474  _zif_register_shutdown_function
0001:00411658  _zif_register_tick_function
0001:0041187c  _zif_unregister_tick_function
0001:004106a4  _zif_highlight_file
0001:00410968  _zif_highlight_string
0001:00410814  _zif_php_strip_whitespace
0001:00410b4c  _zif_ini_get
0001:00410d64  _zif_ini_get_all
0001:00410ee4  _zif_ini_set
0001:00411150  _zif_ini_restore
0001:0041126c  _zif_get_include_path
0001:00411194  _zif_set_include_path
0001:004112dc  _zif_restore_include_path
0001:004113b4  _zif_connection_aborted
0001:004113dc  _zif_connection_status
0001:00411404  _zif_ignore_user_abort
0001:00411f94  _zif_parse_ini_file
0001:004120ac  _zif_parse_ini_string
0001:00411918  _zif_is_uploaded_file
0001:004119d4  _zif_move_uploaded_file
0001:0040f450  __php_error_log_ex
0001:0040f3d8  __php_error_log
0001:004102f0  _php_call_shutdown_functions
0001:00410394  _php_free_shutdown_functions
0001:0041062c  _php_get_highlight_struct
0002:00004a70  _basic_functions_module
Module: U:\dev\php-5.3.6\ext\standard\browscap.o(browscap.o)
0001:004135e4  _zm_startup_browscap
0001:004136e4  _zm_shutdown_browscap
0001:00413920  _zif_get_browser
Module: U:\dev\php-5.3.6\ext\standard\crc32.o(crc32.o)
0001:00414024  _php_if_crc32
Module: U:\dev\php-5.3.6\ext\standard\crypt.o(crypt.o)
0001:0041410c  _zm_startup_crypt
0001:004141bc  _zm_shutdown_crypt
0001:00414200  _zif_crypt
Module: U:\dev\php-5.3.6\ext\standard\cyr_convert.o(cyr_convert.o)
0001:00415258  _zif_convert_cyr_string
Module: U:\dev\php-5.3.6\ext\standard\datetime.o(datetime.o)
0001:0041542c  _php_std_date
0001:0041553c  _zif_strptime
0002:00004b30  _mon_full_names
0002:00004b70  _mon_short_names
0002:00004ba0  _day_full_names
0002:00004bbc  _day_short_names
Module: U:\dev\php-5.3.6\ext\standard\dir.o(dir.o)
0002:00023080  _dir_globals_id
0001:00415c24  _zif_closedir
0001:00416060  _zif_rewinddir
0001:00416194  _php_if_readdir
0001:00415780  _zm_activate_dir
0001:00415830  _zm_startup_dir
0001:00415b90  _zif_opendir
0001:00415bb4  _zif_getdir
0001:00415d8c  _zif_chdir
0001:00415fe8  _zif_getcwd
0001:004163bc  _zif_glob
0001:004167b8  _zif_scandir
Module: U:\dev\php-5.3.6\ext\standard\dl.o(dl.o)
0001:00416a64  _zif_dl
0001:004170a0  _php_dl
0001:00416db0  _php_load_extension
0001:004170fc  _zm_info_dl
Module: U:\dev\php-5.3.6\ext\standard\dns.o(dns.o)
0001:0041714c  _zif_gethostname
0001:00417218  _zif_gethostbyaddr
0001:004172ec  _zif_gethostbyname
0001:00417344  _zif_gethostbynamel
Module: U:\dev\php-5.3.6\ext\standard\exec.o(exec.o)
0001:0041747c  _php_exec
0001:00417a50  _php_escape_shell_cmd
0001:004179e4  _zif_exec
0001:00417a08  _zif_system
0001:00417a2c  _zif_passthru
0001:00417dc4  _php_escape_shell_arg
0001:00417ed8  _zif_escapeshellcmd
0001:00417f58  _zif_escapeshellarg
0001:00418000  _zif_shell_exec
0001:0041812c  _zif_proc_nice
Module: U:\dev\php-5.3.6\ext\standard\file.o(file.o)
0002:00023090  _file_globals_id
0001:004181bc  _php_le_stream_context
0001:004188f0  _zm_startup_file
0001:00418e98  _zm_shutdown_file
0001:00418ec8  _zif_flock
0001:00419098  _zif_get_meta_tags
0001:0041dbd4  _php_next_meta_token
0001:004195c8  _zif_file_get_contents
0001:004198c0  _zif_file_put_contents
0001:00419e6c  _zif_file
0001:0041a194  _zif_tempnam
0001:0041a2dc  _php_if_tmpfile
0001:0041a330  _php_if_fopen
0001:0041a440  _zif_fclose
0001:0041a500  _zif_popen
0001:0041a78c  _zif_pclose
0001:0041a814  _zif_feof
0001:0041a8c4  _zif_fgets
0001:0041aa44  _zif_fgetc
0001:0041aae8  _zif_fgetss
0001:0041ac38  _zif_fscanf
0001:0041ad48  _zif_fwrite
0001:0041ae80  _zif_fflush
0001:0041af04  _zif_rewind
0001:0041af8c  _zif_ftell
0001:0041b014  _zif_fseek
0001:0041b0a4  _php_mkdir_ex
0001:0041b140  _php_mkdir
0001:0041b160  _zif_mkdir
0001:0041b250  _zif_rmdir
0001:0041b320  _zif_readfile
0001:0041b424  _zif_umask
0001:0041b4b0  _zif_fpassthru
0001:0041b5ac  _zif_rename
0001:0041b758  _zif_unlink
0001:0041b8b4  _php_if_ftruncate
0001:0041b9ac  _php_if_fstat
0001:0041c524  _zif_copy
0001:0041c720  _php_copy_file_ctx
0001:0041c66c  _php_copy_file
0001:0041c688  _php_copy_file_ex
0001:0041c940  _zif_fread
0001:0041cb44  _zif_fputcsv
0001:0041d294  _zif_fgetcsv
0001:0041d564  _php_fgetcsv
0001:0041dac8  _zif_realpath
0001:0041dfd0  _zif_fnmatch
0001:0041e0dc  _zif_sys_get_temp_dir
Module: U:\dev\php-5.3.6\ext\standard\filestat.o(filestat.o)
0001:0041e1fc  _zm_activate_filestat
0001:0041e228  _zm_deactivate_filestat
0001:0041e310  _zif_disk_total_space
0001:0041e3f0  _zif_disk_free_space
0001:0041e670  _zif_chgrp
0001:0041e694  _zif_lchgrp
0001:0041e86c  _zif_chown
0001:0041e898  _zif_lchown
0001:0041e8dc  _zif_chmod
0001:0041ea9c  _zif_touch
0001:0041ec30  _php_clear_stat_cache
0001:0041ecf4  _zif_clearstatcache
0001:0041ee10  _php_stat
0001:00420188  _zif_fileperms
0001:004201c8  _zif_fileinode
0001:00420208  _zif_filesize
0001:00420248  _zif_fileowner
0001:00420288  _zif_filegroup
0001:004202c8  _zif_fileatime
0001:00420308  _zif_filemtime
0001:00420348  _zif_filectime
0001:00420388  _zif_filetype
0001:004203c8  _zif_is_writable
0001:00420408  _zif_is_readable
0001:00420448  _zif_is_executable
0001:00420488  _zif_is_file
0001:004204c8  _zif_is_dir
0001:00420508  _zif_is_link
0001:00420548  _zif_file_exists
0001:00420588  _php_if_lstat
0001:004205c8  _php_if_stat
0001:00420608  _zif_realpath_cache_size
0001:0042065c  _zif_realpath_cache_get
Module: U:\dev\php-5.3.6\ext\standard\flock_compat.o(flock_compat.o)
0001:0042078c  _php_flock
Module: U:\dev\php-5.3.6\ext\standard\formatted_print.o(formatted_print.o)
0001:004218e8  _zif_user_sprintf
0001:0042192c  _zif_vsprintf
0001:00421970  _zif_user_printf
0001:004219c8  _zif_vprintf
0001:00421a2c  _zif_fprintf
0001:00421ae8  _zif_vfprintf
Module: U:\dev\php-5.3.6\ext\standard\fsock.o(fsock.o)
0001:0042252c  _zif_fsockopen
0001:00422550  _zif_pfsockopen
Module: U:\dev\php-5.3.6\ext\standard\head.o(head.o)
0001:00422590  _zif_header
0001:004225ec  _zif_header_remove
0001:00422640  _php_header
0001:004227c8  _php_setcookie
0001:00422ae0  _zif_setcookie
0001:00422bbc  _zif_setrawcookie
0001:00422c9c  _zif_headers_sent
0001:00422e30  _zif_headers_list
Module: U:\dev\php-5.3.6\ext\standard\html.o(html.o)
0001:00425704  _php_utf32_utf8
0001:00425880  _php_unescape_html_entities
0001:00425c9c  _php_escape_html_entities
0001:00425cec  _php_escape_html_entities_ex
0001:004261d8  _register_html_constants
0001:00426268  _zif_htmlspecialchars
0001:00426290  _zif_htmlspecialchars_decode
0001:00426508  _zif_html_entity_decode
0001:00426594  _zif_htmlentities
0001:004265c4  _zif_get_html_translation_table
Module: U:\dev\php-5.3.6\ext\standard\image.o(image.o)
0001:00426ebb  _php_sig_gif
0001:00426ebe  _php_sig_psd
0001:00426ec2  _php_sig_bmp
0001:00426ec4  _php_sig_swf
0001:00426ec7  _php_sig_swc
0001:00426eca  _php_sig_jpg
0001:00426ecd  _php_sig_png
0001:00426ed5  _php_sig_tif_ii
0001:00426ed9  _php_sig_tif_mm
0001:00426edd  _php_sig_jpc
0001:00426ee0  _php_sig_jp2
0001:00426eec  _php_sig_iff
0001:00426ef0  _php_sig_ico
0001:00427020  _zm_startup_imagetypes
0001:00427e90  _php_tiff_bytes_per_format
0001:00428758  _php_image_type_to_mime_type
0001:00428818  _zif_image_type_to_mime_type
0001:004288c0  _zif_image_type_to_extension
0001:00428af4  _php_getimagetype
0001:00428dd4  _zif_getimagesize
Module: U:\dev\php-5.3.6\ext\standard\info.o(info.o)
0001:00429174  _php_info_print_module
0001:0042ba84  _php_info_print_table_start
0001:0042c080  _php_info_print_table_row
0001:0042bac4  _php_info_print_table_end
0001:0042bce4  _php_info_print_table_header
0001:0042976c  _php_info_html_esc_write
0001:0042973c  _php_info_print_style
0001:004297ac  _php_info_html_esc
0001:00429820  _php_get_uname
0001:004299ac  _php_print_info_htmlhead
0001:0042a804  _php_print_info
0001:0042bb14  _php_info_print_box_start
0001:0042bb68  _php_info_print_box_end
0001:0042bbec  _php_info_print_hr
0001:0042c538  _php_logo_guid
0001:0042bc58  _php_info_print_table_colspan_header
0001:0042c09c  _php_info_print_table_row_ex
0001:0042c194  _register_phpinfo_constants
0001:0042c2fc  _zif_phpinfo
0001:0042c364  _zif_phpversion
0001:0042c49c  _zif_phpcredits
0001:0042c584  _zif_php_logo_guid
0001:0042c5d0  _zif_php_real_logo_guid
0001:0042c614  _zif_php_egg_logo_guid
0001:0042c680  _zif_zend_logo_guid
0001:0042c6c4  _zif_php_sapi_name
0001:0042c72c  _zif_php_uname
0001:0042c798  _zif_php_ini_scanned_files
0001:0042c7c8  _zif_php_ini_loaded_file
Module: U:\dev\php-5.3.6\ext\standard\iptc.o(iptc.o)
0001:0042ca40  _zif_iptcembed
0001:0042cf90  _zif_iptcparse
Module: U:\dev\php-5.3.6\ext\standard\lcg.o(lcg.o)
0002:000230a0  _lcg_globals_id
0001:0042d1b8  _php_combined_lcg
0001:0042d3cc  _zm_startup_lcg
0001:0042d3ec  _zif_lcg_value
Module: U:\dev\php-5.3.6\ext\standard\link.o(link.o)
0001:0042d420  _zif_readlink
0001:0042d53c  _zif_linkinfo
0001:0042d5f4  _zif_symlink
0001:0042d890  _zif_link
Module: U:\dev\php-5.3.6\ext\standard\mail.o(mail.o)
0001:0042da90  _zif_ezmlm_hash
0001:0042dba0  _zif_mail
0001:0042e150  _php_mail
0001:0042e46c  _zm_info_mail
Module: U:\dev\php-5.3.6\ext\standard\math.o(math.o)
0001:0042e698  __php_math_round
0001:0042ec34  _zif_abs
0001:0042ed58  _zif_ceil
0001:0042eef8  _zif_floor
0001:0042f09c  _zif_round
0001:0042f1e0  _zif_sin
0001:0042f220  _zif_cos
0001:0042f260  _zif_tan
0001:0042f2a0  _zif_asin
0001:0042f2e0  _zif_acos
0001:0042f320  _zif_atan
0001:0042f360  _zif_atan2
0001:0042f3a4  _zif_sinh
0001:0042f3e4  _zif_cosh
0001:0042f424  _zif_tanh
0001:0042f464  _zif_asinh
0001:0042f4a4  _zif_acosh
0001:0042f4e4  _zif_atanh
0001:0042f524  _zif_pi
0001:0042f540  _zif_is_finite
0001:0042f588  _zif_is_infinite
0001:0042f5d0  _zif_is_nan
0001:0042f620  _zif_pow
0001:0042f7c0  _zif_exp
0001:0042f800  _zif_expm1
0001:0042f840  _zif_log1p
0001:0042f8a0  _zif_log
0001:0042f96c  _zif_log10
0001:0042f9ac  _zif_sqrt
0001:0042fa04  _zif_hypot
0001:0042fa58  _zif_deg2rad
0001:0042faa4  _zif_rad2deg
0001:0042fb0c  __php_math_basetolong
0001:0042fbc4  __php_math_basetozval
0001:0042fcdc  __php_math_longtobase
0001:0042fd60  __php_math_zvaltobase
0001:0042fe88  _zif_bindec
0001:0042ff6c  _zif_hexdec
0001:00430050  _zif_octdec
0001:00430134  _zif_decbin
0001:00430218  _zif_decoct
0001:004302fc  _zif_dechex
0001:00430418  _zif_base_convert
0001:00430570  __php_math_number_format
0001:0043078c  _zif_number_format
0001:0043089c  _zif_fmod
Module: U:\dev\php-5.3.6\ext\standard\md5.o(md5.o)
0001:004309ec  _make_digest
0001:00430a14  _make_digest_ex
0001:00430a5c  _php_if_md5
0001:0043129c  _PHP_MD5Init
0001:004312d0  _PHP_MD5Update
0001:00431388  _PHP_MD5Final
0001:00430b44  _php_if_md5_file
Module: U:\dev\php-5.3.6\ext\standard\metaphone.o(metaphone.o)
0001:004314d0  _zif_metaphone
0002:00004d50  __codes
Module: U:\dev\php-5.3.6\ext\standard\microtime.o(microtime.o)
0001:0043304c  _zif_microtime
0001:00433070  _zif_gettimeofday
Module: U:\dev\php-5.3.6\ext\standard\pack.o(pack.o)
0002:000230b0  _machine_little_endian
0001:0043326c  _zif_pack
0001:004343ac  _zif_unpack
0001:00434f0c  _zm_startup_pack
Module: U:\dev\php-5.3.6\ext\standard\pageinfo.o(pageinfo.o)
0001:00434ffc  _php_statpage
0001:00435088  _php_getuid
0001:004350b8  _php_getgid
0001:004350e8  _zif_getmyuid
0001:00435110  _zif_getmygid
0001:00435138  _zif_getmypid
0001:00435160  _zif_getmyinode
0001:004351b8  _php_getlastmod
0001:004351e0  _zif_getlastmod
Module: U:\dev\php-5.3.6\ext\standard\quot_print.o(quot_print.o)
0001:00435270  _php_quot_print_decode
0001:004353c8  _php_quot_print_encode
0001:0043552c  _zif_quoted_printable_decode
0001:004356fc  _zif_quoted_printable_encode
Module: U:\dev\php-5.3.6\ext\standard\rand.o(rand.o)
0001:0043577c  _php_srand
0001:004357a4  _php_rand
0001:00435838  _php_mt_srand
0001:00435998  _php_mt_rand
0001:00435af4  _zif_srand
0001:00435b88  _zif_mt_srand
0001:00435c28  _zif_rand
0001:00435cf8  _zif_mt_rand
0001:00435e40  _zif_getrandmax
0001:00435e70  _zif_mt_getrandmax
Module: U:\dev\php-5.3.6\ext\standard\soundex.o(soundex.o)
0001:00435eb0  _zif_soundex
Module: U:\dev\php-5.3.6\ext\standard\string.o(string.o)
0001:0043608c  _register_string_constants
0001:00436250  _localeconv_r
0001:0043628c  _zm_startup_localeconv
0001:004362a0  _zm_shutdown_localeconv
0001:004362c4  _zif_bin2hex
0001:00438728  _php_strcspn
0001:004386f0  _php_strspn
0001:00436448  _zif_strspn
0001:0043646c  _zif_strcspn
0001:00436638  _zm_startup_nl_langinfo
0001:00436b14  _zif_nl_langinfo
0001:00436bb0  _zif_strcoll
0001:00436c04  _php_trim
0001:00436d30  _zif_trim
0001:00436d54  _zif_rtrim
0001:00436d78  _zif_ltrim
0001:00436de4  _zif_wordwrap
0001:00437248  _php_explode
0001:00437310  _php_explode_negative_limit
0001:0043742c  _zif_explode
0001:00437538  _php_implode
0001:00437b04  _zif_implode
0001:00437db4  _zif_strtok
0001:00438014  _php_strtoupper
0001:00438058  _zif_strtoupper
0001:004380b0  _php_strtolower
0001:004380f4  _zif_strtolower
0001:0043814c  _php_basename
0001:00438284  _zif_basename
0001:004382f8  _php_dirname
0001:00438304  _zif_dirname
0001:00438380  _zif_pathinfo
0001:004386a4  _php_stristr
0001:00438864  _zif_stristr
0001:004389c0  _zif_strstr
0001:00438ac8  _zif_strpos
0001:00438b9c  _zif_stripos
0001:00438d5c  _zif_strrpos
0001:00438efc  _zif_strripos
0001:004391e0  _zif_strrchr
0001:00439404  _zif_chunk_split
0001:00439518  _zif_substr
0001:00439704  _zif_substr_replace
0001:0043a4b0  _zif_quotemeta
0001:0043a658  _zif_ord
0001:0043a694  _zif_chr
0001:0043a72c  _zif_ucfirst
0001:0043a7c8  _zif_lcfirst
0001:0043a838  _zif_ucwords
0001:0043a930  _php_strtr
0001:0043ade8  _zif_strtr
0001:0043afc0  _zif_strrev
0001:0043b178  _zif_similar_text
0001:0043b2c4  _php_stripslashes
0001:0043b394  _zif_addcslashes
0001:0043b794  _php_addcslashes
0001:0043b41c  _zif_addslashes
0001:0043b924  _php_addslashes
0001:0043b4a0  _zif_stripcslashes
0001:0043b54c  _php_stripcslashes
0001:0043b4f4  _zif_stripslashes
0001:0043b944  _php_addslashes_ex
0001:0043ba7c  _php_char_to_str_ex
0001:0043bcd4  _php_char_to_str
0001:0043bcfc  _php_str_to_str_ex
0001:0043c208  _php_str_to_str
0001:0043cc24  _zif_str_replace
0001:0043cc48  _zif_str_ireplace
0001:0043d1c0  _zif_hebrev
0001:0043d1e4  _zif_hebrevc
0001:0043d20c  _zif_nl2br
0001:0043d34c  _zif_strip_tags
0001:0043dc24  _php_strip_tags_ex
0001:0043d558  _zif_setlocale
0001:0043d9e8  _zif_parse_str
0001:0043dad8  _php_tag_find
0001:0043dc00  _php_strip_tags
0001:0043e534  _zif_str_getcsv
0001:0043e644  _zif_str_repeat
0001:0043e768  _zif_count_chars
0001:0043e958  _zif_strnatcmp
0001:0043ea7c  _zif_localeconv
0001:0043ed04  _zif_strnatcasecmp
0001:0043edd4  _zif_substr_count
0001:0043ef90  _zif_str_pad
0001:0043f138  _zif_sscanf
0001:0043f1cc  _zif_str_rot13
0001:0043f2c8  _zif_str_shuffle
0001:0043f344  _zif_str_word_count
0001:0043f65c  _zif_str_split
0001:0043f764  _zif_strpbrk
0001:0043f85c  _zif_substr_compare
Module: U:\dev\php-5.3.6\ext\standard\scanf.o(scanf.o)
0001:0043ff74  _ValidateFormat
0001:004404ac  _php_sscanf_internal
Module: U:\dev\php-5.3.6\ext\standard\syslog.o(syslog.o)
0001:004416cc  _zm_startup_syslog
0001:004419dc  _zm_activate_syslog
0001:00441a3c  _zm_shutdown_syslog
0001:0044463c  _zif_define_syslog_variables
0001:00444688  _zif_openlog
0001:00444734  _zif_closelog
0001:004447ac  _zif_syslog
Module: U:\dev\php-5.3.6\ext\standard\type.o(type.o)
0001:00444854  _zif_gettype
0001:00444a58  _zif_settype
0001:00444c40  _zif_intval
0001:00444d08  _zif_floatval
0001:00444d80  _zif_strval
0001:00444ef4  _zif_is_null
0001:00444f18  _zif_is_resource
0001:00444f3c  _zif_is_bool
0001:00444f60  _zif_is_long
0001:00444f84  _zif_is_float
0001:00444fa8  _zif_is_string
0001:00444fcc  _zif_is_array
0001:00444ff0  _zif_is_object
0001:00445014  _zif_is_numeric
0001:00445088  _zif_is_scalar
0001:004450e8  _zif_is_callable
Module: U:\dev\php-5.3.6\ext\standard\uniqid.o(uniqid.o)
0001:004455a0  _zif_uniqid
Module: U:\dev\php-5.3.6\ext\standard\url.o(url.o)
0001:004456ac  _php_url_free
0001:0044576c  _php_replace_controlchars_ex
0001:004457bc  _php_replace_controlchars
0001:004457e4  _php_url_parse
0001:00445810  _php_url_parse_ex
0001:00445f1c  _zif_parse_url
0001:00446244  _php_url_encode
0001:004462f0  _zif_urlencode
0001:0044633c  _zif_urldecode
0001:00446390  _php_url_decode
0001:00446464  _php_raw_url_encode
0001:0044651c  _zif_rawurlencode
0001:00446568  _zif_rawurldecode
0001:004465bc  _php_raw_url_decode
0001:0044668c  _zif_get_headers
Module: U:\dev\php-5.3.6\ext\standard\var.o(var.o)
0001:00446c40  _php_var_dump
0001:00446fd0  _zif_var_dump
0001:00447284  _php_debug_zval_dump
0001:00447678  _zif_debug_zval_dump
0001:00448004  _php_var_export_ex
0001:00448ac8  _php_var_export
0001:00448b3c  _zif_var_export
0001:0044aab8  _php_var_serialize
0001:0044aae8  _zif_serialize
0001:0044aba4  _zif_unserialize
0001:0044ac78  _zif_memory_get_usage
0001:0044accc  _zif_memory_get_peak_usage
Module: U:\dev\php-5.3.6\ext\standard\versioning.o(versioning.o)
0001:0044b70c  _php_canonicalize_version
0001:0044b9c0  _php_version_compare
0001:0044bd08  _zif_version_compare
Module: U:\dev\php-5.3.6\ext\standard\assert.o(assert.o)
0002:000230b8  _assert_globals_id
0001:0044c38c  _zm_startup_assert
0001:0044c42c  _zm_shutdown_assert
0001:0044c474  _zm_deactivate_assert
0001:0044c4bc  _zm_info_assert
0001:0044c548  _zif_assert
0001:0044ca7c  _zif_assert_options
Module: U:\dev\php-5.3.6\ext\standard\strnatcmp.o(strnatcmp.o)
0001:0044d130  _strnatcmp_ex
Module: U:\dev\php-5.3.6\ext\standard\levenshtein.o(levenshtein.o)
0001:0044d594  _zif_levenshtein
Module: U:\dev\php-5.3.6\ext\standard\incomplete_class.o(incomplete_class.o)
0001:0044db08  _php_lookup_class_name
0001:0044d9a8  _php_create_incomplete_class
0001:0044db7c  _php_store_class_name
Module: U:\dev\php-5.3.6\ext\standard\url_scanner_ex.o(url_scanner_ex.o)
0001:0044e6c0  _php_url_scanner_adapt_single_url
0001:0044ee10  _php_url_scanner_add_var
0001:0044f530  _php_url_scanner_reset_vars
0001:0044f55c  _zm_startup_url_scanner_ex
0001:0044f5b4  _zm_shutdown_url_scanner_ex
0001:0044f5cc  _zm_activate_url_scanner_ex
0001:0044f5ec  _zm_deactivate_url_scanner_ex
Module: U:\dev\php-5.3.6\ext\standard\ftp_fopen_wrapper.o(ftp_fopen_wrapper.o)
0001:0045164c  _php_stream_url_wrap_ftp
0001:004521b0  _php_stream_ftp_opendir
0002:00005318  _php_stream_ftp_wrapper
Module: U:\dev\php-5.3.6\ext\standard\http_fopen_wrapper.o(http_fopen_wrapper.o)
0001:00453e24  _php_stream_url_wrap_http_ex
0001:00457240  _php_stream_url_wrap_http
0002:00005358  _php_stream_http_wrapper
Module: U:\dev\php-5.3.6\ext\standard\php_fopen_wrapper.o(php_fopen_wrapper.o)
0001:004576c4  _php_stream_url_wrap_php
0002:00005370  _php_stream_output_ops
0002:000053b0  _php_stream_input_ops
0002:00005418  _php_stream_php_wrapper
Module: U:\dev\php-5.3.6\ext\standard\credits.o(credits.o)
0001:004596f8  _php_print_credits
Module: U:\dev\php-5.3.6\ext\standard\css.o(css.o)
0001:0045a610  _php_info_print_css
Module: U:\dev\php-5.3.6\ext\standard\var_unserializer.o(var_unserializer.o)
0001:0045a88c  _var_push_dtor
0001:0045a924  _var_replace
0001:0045a9dc  _var_destroy
0001:0045adf4  _php_var_unserialize
Module: U:\dev\php-5.3.6\ext\standard\ftok.o(ftok.o)
0001:0045c734  _zif_ftok
Module: U:\dev\php-5.3.6\ext\standard\sha1.o(sha1.o)
0001:0045c86c  _make_sha1_digest
0001:0045c888  _zif_sha1
0001:0045cacc  _PHP_SHA1Init
0001:0045cb04  _PHP_SHA1Update
0001:0045cbc0  _PHP_SHA1Final
0001:0045c970  _zif_sha1_file
Module: U:\dev\php-5.3.6\ext\standard\user_filters.o(user_filters.o)
0001:0045df9c  _zif_user_filter_nop
0001:0045e1c8  _zm_startup_user_filters
0001:0045e42c  _zm_deactivate_user_filters
0001:0045e574  _userfilter_filter
0001:0045ed6c  _zif_stream_bucket_make_writeable
0001:0045f0a0  _zif_stream_bucket_prepend
0001:0045f0c4  _zif_stream_bucket_append
0001:0045f0e8  _zif_stream_bucket_new
0001:0045f294  _zif_stream_get_filters
0001:0045f37c  _zif_stream_filter_register
Module: U:\dev\php-5.3.6\ext\standard\uuencode.o(uuencode.o)
0001:0045f50c  _php_uuencode
0001:0045f808  _php_uudecode
0001:0045f9d4  _zif_convert_uuencode
0001:0045fa64  _zif_convert_uudecode
Module: U:\dev\php-5.3.6\ext\standard\filters.o(filters.o)
0001:00462840  _zm_startup_standard_filters
0001:00462890  _zm_shutdown_standard_filters
0002:00005ab0  _consumed_filter_factory
Module: U:\dev\php-5.3.6\ext\standard\proc_open.o(proc_open.o)
0001:00463240  _zm_startup_proc_open
0001:00463268  _zif_proc_terminate
0001:004632f0  _zif_proc_close
0001:004633ac  _zif_proc_get_status
0001:00463754  _zif_proc_open
Module: U:\dev\php-5.3.6\ext\standard\streamsfuncs.o(streamsfuncs.o)
0001:00464394  _zif_stream_socket_pair
0001:004644ec  _zif_stream_socket_client
0001:00464890  _zif_stream_socket_server
0001:00464b5c  _zif_stream_socket_accept
0001:00464d3c  _zif_stream_socket_get_name
0001:00464e1c  _zif_stream_socket_sendto
0001:00464f90  _zif_stream_socket_recvfrom
0001:00465150  _zif_stream_get_contents
0001:00465324  _zif_stream_copy_to_stream
0001:00465494  _zif_stream_get_meta_data
0001:004656a0  _zif_stream_get_transports
0001:00465730  _zif_stream_get_wrappers
0001:00465c20  _zif_stream_select
0001:00466524  _zif_stream_context_get_options
0001:00466604  _zif_stream_context_set_option
0001:004666fc  _zif_stream_context_set_params
0001:00466778  _zif_stream_context_get_params
0001:004668b8  _zif_stream_context_get_default
0001:00466958  _zif_stream_context_set_default
0001:004669e0  _zif_stream_context_create
0001:00466c6c  _zif_stream_filter_prepend
0001:00466c90  _zif_stream_filter_append
0001:00466d34  _zif_stream_filter_remove
0001:00466e38  _zif_stream_get_line
0001:00466f0c  _zif_stream_set_blocking
0001:00466fa8  _zif_stream_set_timeout
0001:004670a8  _zif_stream_set_write_buffer
0001:0046714c  _zif_stream_set_read_buffer
0001:00467234  _zif_stream_socket_enable_crypto
0001:00467368  _zif_stream_resolve_include_path
0001:004673d8  _zif_stream_is_local
0001:00467518  _zif_stream_supports_lock
0001:004675a4  _zif_stream_socket_shutdown
Module: U:\dev\php-5.3.6\ext\standard\http.o(http.o)
0001:00467690  _php_url_encode_hash_ex
0001:00468050  _zif_http_build_query
Module: U:\dev\php-5.3.6\ext\tokenizer\tokenizer.o(tokenizer.o)
0001:00468260  _tokenizer_functions
0001:00468504  _zif_token_get_all
0001:004685ec  _zif_token_name
0001:004682bc  _zm_startup_tokenizer
0001:004682f0  _zm_info_tokenizer
0002:00005ae0  _tokenizer_module_entry
Module: U:\dev\php-5.3.6\ext\tokenizer\tokenizer_data.o(tokenizer_data.o)
0001:00468bec  _tokenizer_register_constants
0001:004697a8  _get_token_type_name
Module: U:\dev\php-5.3.6\ext\xml\xml.o(xml.o)
0002:000230c8  _xml_globals_id
0001:0046a8f0  _xml_functions
0001:0046c9f4  _zif_xml_parser_create
0001:0046ca18  _zif_xml_parser_create_ns
0001:0046ca48  _zif_xml_set_object
0001:0046cb34  _zif_xml_set_element_handler
0001:0046cbdc  _zif_xml_set_character_data_handler
0001:0046cc68  _zif_xml_set_processing_instruction_handler
0001:0046ccf4  _zif_xml_set_default_handler
0001:0046cd80  _zif_xml_set_unparsed_entity_decl_handler
0001:0046ce0c  _zif_xml_set_notation_decl_handler
0001:0046ce98  _zif_xml_set_external_entity_ref_handler
0001:0046cf24  _zif_xml_set_start_namespace_decl_handler
0001:0046cfb0  _zif_xml_set_end_namespace_decl_handler
0001:0046d044  _zif_xml_parse
0001:0046d0e8  _zif_xml_parse_into_struct
0001:0046d260  _zif_xml_get_error_code
0001:0046d2d0  _zif_xml_error_string
0001:0046d338  _zif_xml_get_current_line_number
0001:0046d3a4  _zif_xml_get_current_column_number
0001:0046d410  _zif_xml_get_current_byte_index
0001:0046d4a8  _zif_xml_parser_free
0001:0046d570  _zif_xml_parser_set_option
0001:0046d8c8  _zif_xml_parser_get_option
0001:0046d978  _zif_utf8_encode
0001:0046d9dc  _zif_utf8_decode
0001:0046ae48  _zm_startup_xml
0001:0046b10c  _zm_info_xml
0001:0046b900  _xml_utf8_decode
0001:0046b7bc  _xml_utf8_encode
0001:0046ba08  __xml_zval_strdup
0001:0046bb1c  __xml_startElementHandler
0001:0046bf08  __xml_endElementHandler
0001:0046c0d8  __xml_characterDataHandler
0001:0046c414  __xml_processingInstructionHandler
0001:0046c494  __xml_defaultHandler
0001:0046c500  __xml_unparsedEntityDeclHandler
0001:0046c5c0  __xml_notationDeclHandler
0001:0046c668  __xml_externalEntityRefHandler
0001:0046c728  __xml_startNamespaceDeclHandler
0001:0046c7a8  __xml_endNamespaceDeclHandler
0002:00005b40  _xml_module_entry
0002:00005ba0  _xml_encodings
Module: U:\dev\php-5.3.6\ext\xml\compat.o(compat.o)
0001:0046e6a0  _php_XML_ParserCreate
0001:0046e6d4  _php_XML_ParserCreate_MM
0001:0046e6b4  _php_XML_ParserCreateNS
0001:0046e78c  _php_XML_SetUserData
0001:0046e79c  _XML_GetUserData
0001:0046e7a8  _php_XML_SetElementHandler
0001:0046e7bc  _php_XML_SetCharacterDataHandler
0001:0046e7cc  _php_XML_SetProcessingInstructionHandler
0001:0046e7dc  _php_XML_SetCommentHandler
0001:0046e7ec  _php_XML_SetDefaultHandler
0001:0046e7fc  _php_XML_SetUnparsedEntityDeclHandler
0001:0046e80c  _php_XML_SetNotationDeclHandler
0001:0046e81c  _php_XML_SetExternalEntityRefHandler
0001:0046e82c  _php_XML_SetStartNamespaceDeclHandler
0001:0046e83c  _php_XML_SetEndNamespaceDeclHandler
0001:0046e84c  _php_XML_Parse
0001:0046e888  _php_XML_GetErrorCode
0001:0046f4f0  _php_XML_ErrorString
0001:0046f50c  _php_XML_GetCurrentLineNumber
0001:0046f520  _php_XML_GetCurrentColumnNumber
0001:0046f534  _php_XML_GetCurrentByteIndex
0001:0046f54c  _php_XML_GetCurrentByteCount
0001:0046f568  _php_XML_ExpatVersion
0001:0046f574  _php_XML_ParserFree
Module: U:\dev\php-5.3.6\ext\xmlreader\php_xmlreader.o(php_xmlreader.o)
0002:000230d8  _xmlreader_class_entry
0001:0046f77c  _xmlreader_get_property_ptr_ptr
0001:0046f858  _xmlreader_read_property
0001:0046f988  _xmlreader_write_property
0001:0046fa8c  __xmlreader_get_valid_file_path
0001:00471a04  _zm_startup_xmlreader
0001:00471ef4  _zm_shutdown_xmlreader
0001:00471f10  _zm_info_xmlreader
0001:0046fc70  _xmlreader_objects_clone
0001:0046fce8  _xmlreader_objects_free_storage
0001:0046fd14  _xmlreader_objects_new
0001:004700e8  _zim_xmlreader_close
0001:00470114  _zim_xmlreader_getAttribute
0001:0047013c  _zim_xmlreader_getAttributeNo
0001:00470220  _zim_xmlreader_getAttributeNs
0001:00470328  _zim_xmlreader_getParserProperty
0001:004703b0  _zim_xmlreader_isValid
0001:004703d4  _zim_xmlreader_lookupNamespace
0001:00470414  _zim_xmlreader_moveToAttribute
0001:004704a8  _zim_xmlreader_moveToAttributeNo
0001:0047051c  _zim_xmlreader_moveToAttributeNs
0001:004705c8  _zim_xmlreader_moveToElement
0001:004705ec  _zim_xmlreader_moveToFirstAttribute
0001:00470610  _zim_xmlreader_moveToNextAttribute
0001:00470674  _zim_xmlreader_read
0001:004706e8  _zim_xmlreader_next
0001:0047081c  _zim_xmlreader_open
0001:0047099c  _zim_xmlreader_readInnerXml
0001:004709c0  _zim_xmlreader_readOuterXml
0001:004709e4  _zim_xmlreader_readString
0001:00470a08  _zim_xmlreader_setSchema
0001:00470ab4  _zim_xmlreader_setParserProperty
0001:00470b40  _zim_xmlreader_setRelaxNGSchema
0001:00470b64  _zim_xmlreader_setRelaxNGSchemaSource
0001:00470ba0  _zim_xmlreader_XML
0001:00470e70  _zim_xmlreader_expand
0002:00005c60  _xmlreader_module_entry
Module: U:\dev\php-5.3.6\ext\xmlrpc\xmlrpc-epi-php.o(xmlrpc-epi-php.o)
0001:00472570  _xmlrpc_functions
0001:00473504  _zif_xmlrpc_encode
0001:00473754  _zif_xmlrpc_decode
0001:00473698  _zif_xmlrpc_decode_request
0001:004733bc  _zif_xmlrpc_encode_request
0001:00474aa4  _zif_xmlrpc_get_type
0001:00474a18  _zif_xmlrpc_set_type
0001:00474b6c  _zif_xmlrpc_is_fault
0001:00473804  _zif_xmlrpc_server_create
0001:004738d4  _zif_xmlrpc_server_destroy
0001:00473d90  _zif_xmlrpc_server_register_method
0001:00473f4c  _zif_xmlrpc_server_call_method
0001:00474404  _zif_xmlrpc_parse_method_descriptions
0001:004742a4  _zif_xmlrpc_server_add_introspection_data
0001:00473e7c  _zif_xmlrpc_server_register_introspection_callback
0001:004727a4  _zm_startup_xmlrpc
0001:0047284c  _zm_info_xmlrpc
0001:004748a4  _get_zval_xmlrpc_type
0001:004746bc  _set_zval_xmlrpc_type
0001:004735a0  _decode_request_worker
0001:004745ec  _xmlrpc_type_as_str
0001:00474614  _xmlrpc_str_as_type
0001:00474658  _xmlrpc_str_as_vector_type
0002:00005cc0  _xmlrpc_module_entry
Module: U:\dev\php-5.3.6\ext\xmlwriter\php_xmlwriter.o(php_xmlwriter.o)
0002:00005d20  _xmlwriter_module_entry
Module: U:\dev\php-5.3.6\ext\zip\php_zip.o(php_zip.o)
0001:00479da0  _php_zip_glob
0001:00479fd8  _php_zip_pcre
0002:00005d80  _zip_module_entry
Module: U:\dev\php-5.3.6\ext\zip\zip_stream.o(zip_stream.o)
0001:0047f0f8  _php_stream_zip_open
0001:0047f1f0  _php_stream_zip_opener
0002:00005de0  _php_stream_zipio_ops
0002:00005e48  _php_stream_zip_wrapper
Module: U:\dev\php-5.3.6\ext\zip\lib\zip_add.o(zip_add.o)
0001:0047f3dc  _zip_add
Module: U:\dev\php-5.3.6\ext\zip\lib\zip_error.o(zip_error.o)
0001:0047f42c  __zip_error_clear
0001:0047f444  __zip_error_copy
0001:0047f45c  __zip_error_fini
0001:0047f47c  __zip_error_get
0001:0047f4bc  __zip_error_init
0001:0047f4d8  __zip_error_set
Module: U:\dev\php-5.3.6\ext\zip\lib\zip_fclose.o(zip_fclose.o)
0001:0047f4fc  _zip_fclose
Module: U:\dev\php-5.3.6\ext\zip\lib\zip_fread.o(zip_fread.o)
0001:0047f5bc  _zip_fread
Module: U:\dev\php-5.3.6\ext\zip\lib\zip_open.o(zip_open.o)
0001:0047f770  _zip_open
Module: U:\dev\php-5.3.6\ext\zip\lib\zip_source_filep.o(zip_source_filep.o)
0001:004802ec  _zip_source_filep
0001:00480350  __zip_source_file_or_p
Module: U:\dev\php-5.3.6\ext\zip\lib\zip_strerror.o(zip_strerror.o)
0001:0048067c  _zip_strerror
Module: U:\dev\php-5.3.6\ext\zip\lib\zip_close.o(zip_close.o)
0001:004806b8  _zip_close
Module: U:\dev\php-5.3.6\ext\zip\lib\zip_error_get.o(zip_error_get.o)
0001:0048183c  _zip_error_get
Module: U:\dev\php-5.3.6\ext\zip\lib\zip_file_error_get.o(zip_file_error_get.o)
0001:0048185c  _zip_file_error_get
Module: U:\dev\php-5.3.6\ext\zip\lib\zip_free.o(zip_free.o)
0001:0048187c  __zip_free
Module: U:\dev\php-5.3.6\ext\zip\lib\zip_rename.o(zip_rename.o)
0001:0048198c  _zip_rename
Module: U:\dev\php-5.3.6\ext\zip\lib\zip_source_free.o(zip_source_free.o)
0001:00481a3c  _zip_source_free
Module: U:\dev\php-5.3.6\ext\zip\lib\zip_unchange_all.o(zip_unchange_all.o)
0001:00481a7c  _zip_unchange_all
Module: U:\dev\php-5.3.6\ext\zip\lib\zip_delete.o(zip_delete.o)
0001:00481acc  _zip_delete
Module: U:\dev\php-5.3.6\ext\zip\lib\zip_error_get_sys_type.o(zip_error_get_sys_type.o)
0001:00481b3c  _zip_error_get_sys_type
Module: U:\dev\php-5.3.6\ext\zip\lib\zip_file_get_offset.o(zip_file_get_offset.o)
0001:00481b6c  __zip_file_get_offset
Module: U:\dev\php-5.3.6\ext\zip\lib\zip_get_name.o(zip_get_name.o)
0001:00481c0c  _zip_get_name
0001:00481c28  __zip_get_name
Module: U:\dev\php-5.3.6\ext\zip\lib\zip_replace.o(zip_replace.o)
0001:00481cac  _zip_replace
0001:00481cfc  __zip_replace
Module: U:\dev\php-5.3.6\ext\zip\lib\zip_source_function.o(zip_source_function.o)
0001:00481dac  _zip_source_function
Module: U:\dev\php-5.3.6\ext\zip\lib\zip_unchange.o(zip_unchange.o)
0001:00481e0c  _zip_unchange
0001:00481e24  __zip_unchange
Module: U:\dev\php-5.3.6\ext\zip\lib\zip_dirent.o(zip_dirent.o)
0001:00481f0c  __zip_cdir_free
0001:00482168  __zip_dirent_finalize
0001:00481f70  __zip_cdir_grow
0001:00481fcc  __zip_cdir_new
0001:00482058  __zip_cdir_write
0001:004826a4  __zip_dirent_write
0001:004821a8  __zip_dirent_init
0001:00482230  __zip_dirent_read
0001:004828d4  __zip_read2
0001:004828f8  __zip_read4
0001:004825b8  __zip_dirent_torrent_normalize
Module: U:\dev\php-5.3.6\ext\zip\lib\zip_error_strerror.o(zip_error_strerror.o)
0001:00482b28  __zip_error_strerror
Module: U:\dev\php-5.3.6\ext\zip\lib\zip_filerange_crc.o(zip_filerange_crc.o)
0001:00482c8c  __zip_filerange_crc
Module: U:\dev\php-5.3.6\ext\zip\lib\zip_file_strerror.o(zip_file_strerror.o)
0001:00482dbc  _zip_file_strerror
Module: U:\dev\php-5.3.6\ext\zip\lib\zip_get_num_files.o(zip_get_num_files.o)
0001:00482ddc  _zip_get_num_files
Module: U:\dev\php-5.3.6\ext\zip\lib\zip_get_archive_flag.o(zip_get_archive_flag.o)
0001:00482dfc  _zip_get_archive_flag
Module: U:\dev\php-5.3.6\ext\zip\lib\zip_set_archive_flag.o(zip_set_archive_flag.o)
0001:00482e2c  _zip_set_archive_flag
Module: U:\dev\php-5.3.6\ext\zip\lib\zip_set_name.o(zip_set_name.o)
0001:00482e5c  __zip_set_name
Module: U:\dev\php-5.3.6\ext\zip\lib\zip_source_zip.o(zip_source_zip.o)
0001:00482f2c  _zip_source_zip
Module: U:\dev\php-5.3.6\ext\zip\lib\zip_unchange_data.o(zip_unchange_data.o)
0001:0048330c  __zip_unchange_data
Module: U:\dev\php-5.3.6\ext\zip\lib\zip_entry_free.o(zip_entry_free.o)
0001:0048335c  __zip_entry_free
Module: U:\dev\php-5.3.6\ext\zip\lib\zip_error_to_str.o(zip_error_to_str.o)
0001:004833c8  _zip_error_to_str
Module: U:\dev\php-5.3.6\ext\zip\lib\zip_fopen.o(zip_fopen.o)
0001:0048348c  _zip_fopen
Module: U:\dev\php-5.3.6\ext\zip\lib\zip_name_locate.o(zip_name_locate.o)
0001:004834dc  _zip_name_locate
0001:004834f8  __zip_name_locate
Module: U:\dev\php-5.3.6\ext\zip\lib\zip_source_buffer.o(zip_source_buffer.o)
0001:004835ec  _zip_source_buffer
Module: U:\dev\php-5.3.6\ext\zip\lib\zip_stat.o(zip_stat.o)
0001:004837ac  _zip_stat
Module: U:\dev\php-5.3.6\ext\zip\lib\zip_entry_new.o(zip_entry_new.o)
0001:0048380c  __zip_entry_new
Module: U:\dev\php-5.3.6\ext\zip\lib\zip_err_str.o(zip_err_str.o)
0001:00483ab0  __zip_err_str
0001:00483b10  __zip_nerr_str
0001:00483b30  __zip_err_type
Module: U:\dev\php-5.3.6\ext\zip\lib\zip_fopen_index.o(zip_fopen_index.o)
0001:00483ba4  _zip_fopen_index
0001:00483da0  __zip_file_fillbuf
Module: U:\dev\php-5.3.6\ext\zip\lib\zip_get_archive_comment.o(zip_get_archive_comment.o)
0001:00483f7c  _zip_get_archive_comment
Module: U:\dev\php-5.3.6\ext\zip\lib\zip_get_file_comment.o(zip_get_file_comment.o)
0001:00483fdc  _zip_get_file_comment
Module: U:\dev\php-5.3.6\ext\zip\lib\zip_new.o(zip_new.o)
0001:0048406c  __zip_new
Module: U:\dev\php-5.3.6\ext\zip\lib\zip_source_file.o(zip_source_file.o)
0001:0048411c  _zip_source_file
Module: U:\dev\php-5.3.6\ext\zip\lib\zip_stat_index.o(zip_stat_index.o)
0001:0048418c  _zip_stat_index
Module: U:\dev\php-5.3.6\ext\zip\lib\zip_set_archive_comment.o(zip_set_archive_comment.o)
0001:004842ac  _zip_set_archive_comment
Module: U:\dev\php-5.3.6\ext\zip\lib\zip_set_file_comment.o(zip_set_file_comment.o)
0001:0048432c  _zip_set_file_comment
Module: U:\dev\php-5.3.6\ext\zip\lib\zip_unchange_archive.o(zip_unchange_archive.o)
0001:004843dc  _zip_unchange_archive
Module: U:\dev\php-5.3.6\ext\zip\lib\zip_memdup.o(zip_memdup.o)
0001:0048441c  __zip_memdup
Module: U:\dev\php-5.3.6\ext\zip\lib\zip_stat_init.o(zip_stat_init.o)
0001:0048446c  _zip_stat_init
Module: U:\dev\php-5.3.6\ext\zip\lib\zip_add_dir.o(zip_add_dir.o)
0001:004844cc  _zip_add_dir
Module: U:\dev\php-5.3.6\ext\zip\lib\zip_error_clear.o(zip_error_clear.o)
0001:004845cc  _zip_error_clear
Module: U:\dev\php-5.3.6\ext\zip\lib\zip_file_error_clear.o(zip_file_error_clear.o)
0001:004845ec  _zip_file_error_clear
Module: U:\dev\php-5.3.6\ext\mysqlnd\mysqlnd.o(mysqlnd.o)
0001:004847a4  _mysqlnd_old_passwd
0001:004847c4  _mysqlnd_server_gone
0001:00484800  _mysqlnd_out_of_sync
0001:00484814  _mysqlnd_out_of_memory
0001:00484818  _mysqlnd_library_end
0001:00486dc8  _mysqlnd_connect
0001:00489514  __mysqlnd_init
0001:00487184  _mysqlnd_stream_array_check_for_readiness
0001:0048743c  __mysqlnd_poll
0001:00487690  _php_mysqlnd_conn_list_fields_pub
0001:0048781c  _php_mysqlnd_conn_list_method_pub
0001:00487928  _mysqlnd_old_escape_string
0001:004883a0  _mysqlnd_get_client_info
0001:004883ac  _mysqlnd_get_client_version
0001:0048879c  _mysqlnd_field_type_name
0001:00489624  _mysqlnd_plugin_count
0001:004895b0  _mysqlnd_library_init
0001:004895f4  _mysqlnd_conn_get_methods
0001:00489600  _mysqlnd_conn_set_methods
0001:00489610  _mysqlnd_plugin_register
0001:00489630  __mysqlnd_plugin_get_plugin_connection_data
0002:0001d9e0  _mysqlnd_global_stats
Module: U:\dev\php-5.3.6\ext\mysqlnd\mysqlnd_charset.o(mysqlnd_charset.o)
0001:0048a700  _mysqlnd_charsets
0001:0048bae0  _mysqlnd_find_charset_nr
0001:0048bb0c  _mysqlnd_find_charset_name
0001:0048bb48  _mysqlnd_cset_escape_quotes
0001:0048bbfc  _mysqlnd_cset_escape_slashes
Module: U:\dev\php-5.3.6\ext\mysqlnd\mysqlnd_wireprotocol.o(mysqlnd_wireprotocol.o)
0001:0048bd54  _mysqlnd_empty_string
0001:0048bd58  _mysqlnd_read_header_name
0001:0048bd6c  _mysqlnd_read_body_name
0001:0048bec0  _mysqlnd_command_to_text
0001:0048bf38  _php_mysqlnd_net_field_length
0001:0048bfb0  _php_mysqlnd_net_field_length_ll
0001:0048c02c  _php_mysqlnd_net_store_length
0001:0048cc1c  _php_mysqlnd_scramble
0001:0048da18  _php_mysqlnd_cmd_write
0001:0048ef20  _php_mysqlnd_rowp_read_binary_protocol
0001:0048f85c  _php_mysqlnd_rowp_read_text_protocol
0001:00491b14  _mysqlnd_protocol_init
0001:00491b64  _mysqlnd_protocol_free
0001:00491b88  __mysqlnd_plugin_get_plugin_protocol_data
0001:00491bac  _mysqlnd_protocol_get_methods
Module: U:\dev\php-5.3.6\ext\mysqlnd\mysqlnd_ps.o(mysqlnd_ps.o)
0001:00491c08  _mysqlnd_not_bound_as_blob
0001:00491c24  _mysqlnd_stmt_not_prepared
0001:0049326c  _mysqlnd_fetch_stmt_row_buffered
0001:00493c4c  _mysqlnd_fetch_stmt_row_cursor
0001:00495a38  _php_mysqlnd_stmt_free_parameter_bind_pub
0001:00495a64  _php_mysqlnd_stmt_free_result_bind_pub
0001:00495a90  __mysqlnd_stmt_init
0001:00495bb8  __mysqlnd_plugin_get_plugin_stmt_data
0001:00495bdc  __mysqlnd_init_ps_subsystem
0001:00495bf0  _mysqlnd_stmt_get_methods
0001:00495bfc  _mysqlnd_stmt_set_methods
0002:00006140  _mysqlnd_mysqlnd_stmt_methods
Module: U:\dev\php-5.3.6\ext\mysqlnd\mysqlnd_loaddata.o(mysqlnd_loaddata.o)
0001:00495e20  _mysqlnd_local_infile_default
0001:00495e44  _mysqlnd_set_local_infile_handler
0001:00495f40  _mysqlnd_handle_local_infile
Module: U:\dev\php-5.3.6\ext\mysqlnd\mysqlnd_net.o(mysqlnd_net.o)
0001:004965b4  _php_mysqlnd_net_send_pub
0001:00496e1c  _php_mysqlnd_net_consume_uneaten_data_pub
0001:00497210  _mysqlnd_net_init
0001:0049728c  _mysqlnd_net_free
0001:0049731c  __mysqlnd_plugin_get_plugin_net_data
0001:00497344  _mysqlnd_net_get_methods
Module: U:\dev\php-5.3.6\ext\mysqlnd\mysqlnd_ps_codec.o(mysqlnd_ps_codec.o)
0002:000230e8  _mysqlnd_ps_fetch_functions
0001:00497368  _ps_fetch_from_1_to_8_bytes
0001:00497ac0  __mysqlnd_init_ps_fetch_subsystem
0001:00498b54  _mysqlnd_stmt_execute_generate_request
Module: U:\dev\php-5.3.6\ext\mysqlnd\mysqlnd_statistics.o(mysqlnd_statistics.o)
0001:004999f0  _mysqlnd_stats_values_names
0001:00499ef8  _mysqlnd_fill_stats_hash
0001:00499f80  __mysqlnd_get_client_stats
0001:00499fb8  _mysqlnd_stats_init
0001:0049a014  _mysqlnd_stats_end
0001:0049a048  _mysqlnd_stats_set_trigger
0001:0049a08c  _mysqlnd_stats_reset_triggers
Module: U:\dev\php-5.3.6\ext\mysqlnd\mysqlnd_result.o(mysqlnd_result.o)
0001:0049ac90  _mysqlnd_query_read_result_set_header
0001:0049b6f4  __mysqlnd_fetch_lengths
0001:0049c77c  _php_mysqlnd_res_store_result_fetch_data_pub
0001:0049d8a4  _mysqlnd_result_init
0001:0049d904  __mysqlnd_plugin_get_plugin_result_data
0001:0049d92c  _mysqlnd_result_get_methods
Module: U:\dev\php-5.3.6\ext\mysqlnd\mysqlnd_result_meta.o(mysqlnd_result_meta.o)
0001:0049e078  _mysqlnd_result_meta_init
0001:0049e114  _mysqlnd_result_metadata_get_methods
0001:0049e120  __mysqlnd_plugin_get_plugin_result_metadata_data
Module: U:\dev\php-5.3.6\ext\mysqlnd\mysqlnd_debug.o(mysqlnd_debug.o)
0001:0049fa34  _mysqlnd_debug_init
0001:0049fab8  __mysqlnd_debug
0001:0049fb64  __mysqlnd_emalloc
0001:0049fd38  __mysqlnd_pemalloc
0001:0049ff68  __mysqlnd_ecalloc
0001:004a014c  __mysqlnd_pecalloc
0001:004a036c  __mysqlnd_erealloc
0001:004a0554  __mysqlnd_perealloc
0001:004a07c4  __mysqlnd_efree
0001:004a0960  __mysqlnd_pefree
0001:004a0b1c  __mysqlnd_malloc
0001:004a0ce0  __mysqlnd_calloc
0001:004a0ea8  __mysqlnd_realloc
0001:004a10a4  __mysqlnd_free
0001:004a1240  __mysqlnd_pestrndup
0001:004a13d4  __mysqlnd_pestrdup
0001:004a1d80  _mysqlnd_get_backtrace
0002:00006310  _mysqlnd_debug_std_no_trace_funcs
0002:00006350  _mysqlnd_mysqlnd_debug_methods
0002:00006370  _mysqlnd_allocator
Module: U:\dev\php-5.3.6\ext\mysqlnd\mysqlnd_block_alloc.o(mysqlnd_block_alloc.o)
0001:004a2088  _mysqlnd_mempool_create
0001:004a20f4  _mysqlnd_mempool_destroy
Module: U:\dev\php-5.3.6\ext\mysqlnd\php_mysqlnd.o(php_mysqlnd.o)
0002:000240e8  _mysqlnd_globals_id
0001:004a212c  _mysqlnd_minfo_print_hash
0001:004a2284  _zm_info_mysqlnd
0002:000063b0  _mysqlnd_module_entry
Module: U:\dev\php-5.3.6\TSRM\TSRM.o(TSRM.o)
0001:004a2c00  _tsrm_startup
0001:004a35e4  _tsrm_error_set
0001:004a358c  _tsrm_mutex_alloc
0001:004a2ce0  _tsrm_shutdown
0001:004a3594  _tsrm_mutex_free
0001:004a2e58  _ts_allocate_id
0001:004a35a8  _tsrm_mutex_lock
0001:004a35b4  _tsrm_mutex_unlock
0001:004a30e8  _ts_resource_ex
0001:004a357c  _tsrm_thread_id
0001:004a31a0  _tsrm_free_interpreter_context
0001:004a3230  _tsrm_set_interpreter_context
0001:004a3244  _tsrm_new_interpreter_context
0001:004a3284  _ts_free_thread
0001:004a3394  _ts_free_worker_threads
0001:004a34bc  _ts_free_id
0001:004a35bc  _tsrm_set_new_thread_begin_handler
0001:004a35d0  _tsrm_set_new_thread_end_handler
Module: U:\dev\php-5.3.6\TSRM\tsrm_strtok_r.o(tsrm_strtok_r.o)
0001:004a3600  _tsrm_strtok_r
Module: U:\dev\php-5.3.6\TSRM\tsrm_virtual_cwd.o(tsrm_virtual_cwd.o)
0002:000240f8  _main_cwd_state
0002:00024108  _cwd_globals_id
0002:00024118  _cwd_mutex
0001:004a3970  _realpath_cache_clean
0001:004a379c  _virtual_cwd_startup
0001:004a381c  _virtual_cwd_shutdown
0001:004a383c  _virtual_getcwd_ex
0001:004a3910  _virtual_getcwd
0001:004a39d8  _realpath_cache_del
0001:004a3ac8  _realpath_cache_lookup
0001:004a3bb8  _realpath_cache_size
0001:004a3bd0  _realpath_cache_max_buckets
0001:004a3bdc  _realpath_cache_get_buckets
0001:004a4430  _virtual_file_ex
0001:004a4a5c  _virtual_chdir
0001:004a4a90  _virtual_chdir_file
0001:004a4ba8  _virtual_realpath
0001:004a4d54  _virtual_filepath_ex
0001:004a4db8  _virtual_filepath
0001:004a4dd4  _virtual_fopen
0001:004a4e70  _virtual_access
0001:004a4f00  _virtual_utime
0001:004a4f90  _virtual_chmod
0001:004a5020  _virtual_chown
0001:004a50cc  _virtual_open
0001:004a516c  _virtual_creat
0001:004a51fc  _virtual_rename
0001:004a5300  _virtual_stat
0001:004a5390  _virtual_lstat
0001:004a5420  _virtual_unlink
0001:004a54ac  _virtual_mkdir
0001:004a553c  _virtual_rmdir
0001:004a55c8  _virtual_opendir
0001:004a5650  _virtual_popen
0001:004a56d0  _tsrm_realpath
0001:004a5898  _realpath
Module: U:\dev\php-5.3.6\main\internal_functions.o(internal_functions.o)
0001:004a5a7c  _php_register_internal_extensions
Module: U:\dev\php-5.3.6\main\main.o(main.o)
0002:00024128  _core_globals_id
0001:004a7d5c  _php_log_err
0001:004a7e98  _php_write
0001:004a7ea4  _php_printf
0001:004a7fa8  _php_verror
0001:004a85b4  _php_error_docref0
0001:004a85d8  _php_error_docref1
0001:004a8604  _php_error_docref2
0001:004a8664  _php_html_puts
0001:004a9160  _zif_set_time_limit
0001:004a92b4  _php_stream_open_for_zend_ex
0001:004a9694  _php_on_timeout
0001:004a9850  _php_request_startup
0001:004a9ac8  _php_request_startup_for_hook
0001:004a9b08  _php_request_shutdown_for_exec
0001:004a9b28  _php_request_shutdown_for_hook
0001:004a9e2c  _php_request_shutdown
0001:004aa3fc  _php_com_initialize
0001:004aa4d8  _zm_info_php_core
0001:004aa50c  _php_register_extensions
0001:004aa898  _php_module_startup
0001:004ab080  _php_module_shutdown_for_exec
0001:004ab088  _php_module_shutdown_wrapper
0001:004ab0a4  _php_module_shutdown
0001:004ab120  _php_execute_script
0001:004ab43c  _php_execute_simple_script
0001:004ab57c  _php_handle_aborted_connection
0001:004ab5f4  _php_handle_auth_data
0001:004ab764  _php_lint_script
0002:00006490  _php_register_internal_extensions_func
Module: U:\dev\php-5.3.6\main\snprintf.o(snprintf.o)
0001:004ab994  _php_gcvt
0001:004ad0f8  _ap_php_snprintf
0001:004abbe8  _ap_php_conv_10
0001:004abc94  _php_conv_fp
0001:004abf2c  _ap_php_conv_p2
0001:004ad080  _ap_php_slprintf
0001:004ad0bc  _ap_php_vslprintf
0001:004ad11c  _ap_php_vsnprintf
0001:004ad13c  _ap_php_vasprintf
0001:004ad1b0  _ap_php_asprintf
Module: U:\dev\php-5.3.6\main\spprintf.o(spprintf.o)
0001:004ae584  _vspprintf
0001:004ae5e8  _spprintf
Module: U:\dev\php-5.3.6\main\php_sprintf.o(php_sprintf.o)
0001:004ae61c  _php_sprintf
Module: U:\dev\php-5.3.6\main\safe_mode.o(safe_mode.o)
0001:004ae758  _php_checkuid_ex
0001:004aebf8  _php_checkuid
0001:004aec14  _php_get_current_user
Module: U:\dev\php-5.3.6\main\fopen_wrappers.o(fopen_wrappers.o)
0001:004aed1c  _OnUpdateBaseDir
0001:004af178  _php_check_open_basedir_ex
0001:004aedf4  _php_check_specific_open_basedir
0001:004b01ec  _expand_filepath
0001:004af0b4  _php_check_open_basedir
0001:004af2b8  _php_check_safe_mode_include_dir
0001:004af41c  _php_fopen_primary_script
0001:004af888  _php_resolve_path
0001:004afe18  _php_fopen_with_path
0001:004b016c  _php_strip_url_passwd
0001:004b0208  _expand_filepath_ex
Module: U:\dev\php-5.3.6\main\php_scandir.o(php_scandir.o)
0001:004b042c  _php_alphasort
0001:004b044c  _php_scandir
Module: U:\dev\php-5.3.6\main\php_ini.o(php_ini.o)
0001:004b0960  _display_ini_entries
0001:004b09fc  _config_zval_dtor
0001:004b0ec4  _php_init_config
0001:004b1770  _php_shutdown_config
0001:004b17cc  _php_ini_register_extensions
0001:004b1818  _php_parse_user_ini_file
0001:004b18f8  _php_ini_activate_config
0001:004b1974  _php_ini_has_per_dir_config
0001:004b1980  _php_ini_activate_per_dir_config
0001:004b1a10  _php_ini_has_per_host_config
0001:004b1a1c  _php_ini_activate_per_host_config
0001:004b1a70  _cfg_get_entry
0001:004b1a9c  _cfg_get_long
0001:004b1b24  _cfg_get_double
0001:004b1bb8  _cfg_get_string
0001:004b1c08  _php_ini_get_configuration_hash
0002:0001db20  _php_ini_opened_path
0002:0001db24  _php_ini_scanned_path
0002:0001db28  _php_ini_scanned_files
Module: U:\dev\php-5.3.6\main\SAPI.o(SAPI.o)
0002:00024138  _sapi_module
0002:000241d8  _sapi_globals_id
0001:004b1d90  _sapi_startup
0001:004b1dd8  _sapi_shutdown
0001:004b1de4  _sapi_free_header
0001:004b1df8  _sapi_handle_post
0001:004b20bc  _sapi_read_standard_form_data
0001:004b2224  _sapi_get_default_content_type
0001:004b22f8  _sapi_get_default_content_type_header
0001:004b2390  _sapi_apply_default_charset
0001:004b24a4  _sapi_activate_headers_only
0001:004b2600  _sapi_activate
0001:004b284c  _sapi_deactivate
0001:004b2ad0  _sapi_initialize_empty_request
0001:004b2bf8  _sapi_add_header_ex
0001:004b2e14  _sapi_header_op
0001:004b367c  _sapi_send_headers
0001:004b38bc  _sapi_register_post_entries
0001:004b38f8  _sapi_register_post_entry
0001:004b3954  _sapi_unregister_post_entry
0001:004b39a4  _sapi_register_default_post_reader
0001:004b39f0  _sapi_register_treat_data
0001:004b3a3c  _sapi_register_input_filter
0001:004b3a90  _sapi_flush
0001:004b3ac0  _sapi_get_stat
0001:004b3b20  _sapi_getenv
0001:004b3b88  _sapi_get_fd
0001:004b3bac  _sapi_force_http_10
0001:004b3bcc  _sapi_get_target_uid
0001:004b3bf0  _sapi_get_target_gid
0001:004b3c14  _sapi_get_request_time
0001:004b3c78  _sapi_terminate_process
Module: U:\dev\php-5.3.6\main\rfc1867.o(rfc1867.o)
0001:004b3d4c  _php_rfc1867_register_constants
0001:004b4190  _destroy_uploaded_files_hash
0001:004b4d7c  _rfc1867_post_handler
0002:0001dbe0  _php_rfc1867_callback
Module: U:\dev\php-5.3.6\main\php_content_types.o(php_content_types.o)
0001:004b62ac  _php_default_post_reader
0001:004b64ec  _php_startup_sapi_content_types
0001:004b651c  _php_setup_sapi_content_types
Module: U:\dev\php-5.3.6\main\mergesort.o(mergesort.o)
0001:004b656c  _php_mergesort
Module: U:\dev\php-5.3.6\main\php_variables.o(php_variables.o)
0001:004b78a0  __php_import_environment_variables
0001:004b6cec  _php_register_variable
0001:004b6d1c  _php_register_variable_safe
0001:004b6dfc  _php_register_variable_ex
0001:004b7388  _php_std_post_handler
0001:004b7480  _php_default_input_filter
0001:004b749c  _php_default_treat_data
0001:004b79e8  _php_std_auto_global_callback
0001:004b7ddc  _php_handle_special_queries
0001:004b813c  _php_hash_environment
0001:004b8ce4  _php_startup_auto_globals
0002:00006540  _php_import_environment_variables
Module: U:\dev\php-5.3.6\main\php_ticks.o(php_ticks.o)
0001:004b91fc  _php_startup_ticks
0001:004b9228  _php_deactivate_ticks
0001:004b9248  _php_shutdown_ticks
0001:004b9280  _php_add_tick_function
0001:004b92b0  _php_remove_tick_function
0001:004b92f8  _php_run_ticks
Module: U:\dev\php-5.3.6\main\network.o(network.o)
0001:004b94b8  _php_network_connect_socket
0001:004b9f9c  _php_socket_strerror
0001:004b9658  _php_network_bind_socket_to_local_addr
0001:004b97a4  _php_network_parse_network_address_with_port
0001:004b9930  _php_network_populate_name_from_sockaddr
0001:004b9a30  _php_network_get_peer_name
0001:004b9a9c  _php_network_get_sock_name
0001:004b9b08  _php_network_accept_incoming
0001:004b9c68  _php_network_connect_socket_to_host
0001:004b9f34  _php_any_addr
0001:004b9f78  _php_sockaddr_size
0001:004b9fec  __php_stream_sock_open_from_socket
0001:004ba0d8  __php_stream_sock_open_host
0001:004ba12c  _php_set_sock_blocking
0001:004ba2ac  __php_emit_fd_setsize_warning
Module: U:\dev\php-5.3.6\main\php_open_temporary_file.o(php_open_temporary_file.o)
0001:004ba48c  _php_shutdown_temporary_directory
0001:004ba4c8  _php_get_temporary_directory
0001:004ba558  _php_open_temporary_fd_ex
0001:004ba60c  _php_open_temporary_fd
0001:004ba62c  _php_open_temporary_file
Module: U:\dev\php-5.3.6\main\php_logos.o(php_logos.o)
0001:004bcfd0  _php_register_info_logo
0001:004bd02c  _php_unregister_info_logo
0001:004bd0dc  _php_init_info_logos
0001:004bd154  _php_shutdown_info_logos
0001:004bd178  _php_info_logos
Module: U:\dev\php-5.3.6\main\output.o(output.o)
0002:000241e8  _output_globals_id
0001:004bd24c  _php_default_output_func
0001:004bd2ac  _php_output_startup
0001:004bd2c8  _php_output_activate
0001:004be624  _php_ub_body_write
0001:004bd368  _php_output_register_constants
0001:004bd3b8  _php_output_set_status
0001:004bd3d4  _php_body_write
0001:004bd3f4  _php_header_write
0001:004bd474  _php_start_ob_buffer
0001:004be5ac  _php_ub_body_write_no_header
0001:004bd52c  _php_start_ob_buffer_named
0001:004bd5fc  _php_end_ob_buffer
0001:004bdb94  _php_end_ob_buffers
0001:004bdbe0  _php_start_implicit_flush
0001:004bdbf8  _php_end_implicit_flush
0001:004bdc10  _php_get_output_start_filename
0001:004bdc28  _php_get_output_start_lineno
0001:004bdc58  _php_ob_set_internal_handler
0001:004bdd78  _php_ob_init_conflict
0001:004be3e0  _php_ob_handler_used
0001:004be454  _php_ob_get_buffer
0001:004be498  _php_ob_get_length
0001:004be874  _zif_ob_start
0001:004be93c  _zif_ob_flush
0001:004bea1c  _zif_ob_clean
0001:004beaf0  _zif_ob_end_flush
0001:004beb84  _zif_ob_end_clean
0001:004bec18  _zif_ob_get_flush
0001:004bece0  _zif_ob_get_clean
0001:004beda8  _zif_ob_get_contents
0001:004bedec  _zif_ob_get_level
0001:004bee28  _zif_ob_get_length
0001:004bee6c  _zif_ob_list_handlers
0001:004beefc  _zif_ob_get_status
0001:004bf058  _zif_ob_implicit_flush
0001:004bf0a4  _zif_output_reset_rewrite_vars
0001:004bf0dc  _zif_output_add_rewrite_var
Module: U:\dev\php-5.3.6\main\getopt.o(getopt.o)
0001:004bf270  _php_getopt
0002:000065c0  _php_optidx
Module: U:\dev\php-5.3.6\main\streams\streams.o(streams.o)
0001:004bf75c  _php_file_le_stream
0001:004bf768  _php_file_le_pstream
0001:004bf774  _php_file_le_stream_filter
0001:004bf780  __php_stream_get_url_stream_wrappers_hash
0001:004bf7a0  _php_stream_get_url_stream_wrappers_hash_global
0001:004bf82c  _zm_deactivate_streams
0001:004bf858  _php_stream_from_persistent_id
0001:004bf928  _php_stream_display_wrapper_errors
0001:004bfab8  _php_stream_tidy_wrapper_error_log
0001:004bfb14  _php_stream_wrapper_log_error
0001:004bfbb4  __php_stream_alloc
0001:004bfd10  __php_stream_free
0001:004c0bc0  __php_stream_flush
0001:004c2d50  _php_stream_context_del_link
0001:004c03c0  __php_stream_read
0001:004c04c8  __php_stream_eof
0001:004c0fbc  __php_stream_set_option
0001:004c0530  __php_stream_putc
0001:004c0c18  __php_stream_write
0001:004c0560  __php_stream_getc
0001:004c0590  __php_stream_puts
0001:004c05fc  __php_stream_stat
0001:004c0654  _php_stream_locate_eol
0001:004c072c  __php_stream_get_line
0001:004c0898  _php_stream_get_record
0001:004c0c78  __php_stream_printf
0001:004c0cc0  __php_stream_tell
0001:004c0cf0  __php_stream_seek
0001:004c1038  __php_stream_truncate_set_size
0001:004c1054  __php_stream_passthru
0001:004c1130  __php_stream_copy_to_mem
0001:004c1364  __php_stream_copy_to_stream_ex
0001:004c1578  __php_stream_copy_to_stream
0001:004c1618  _php_shutdown_stream_hashes
0001:004c16e8  _php_init_stream_wrappers
0001:004c1814  _php_shutdown_stream_wrappers
0001:004c1844  _php_register_url_stream_wrapper
0001:004c18d4  _php_unregister_url_stream_wrapper
0001:004c197c  _php_register_url_stream_wrapper_volatile
0001:004c1a3c  _php_unregister_url_stream_wrapper_volatile
0001:004c1c7c  _php_stream_locate_url_wrapper
0001:004c2088  __php_stream_mkdir
0001:004c20d4  __php_stream_rmdir
0001:004c211c  __php_stream_stat_path
0001:004c22fc  __php_stream_opendir
0001:004c23bc  __php_stream_readdir
0001:004c24b8  __php_stream_open_wrapper_ex
0001:004c28e0  _php_stream_context_set
0001:004c2938  _php_stream_notification_notify
0001:004c2974  _php_stream_context_free
0001:004c2a54  _php_stream_notification_free
0001:004c29e0  _php_stream_context_alloc
0001:004c2a40  _php_stream_notification_alloc
0001:004c2a7c  _php_stream_context_get_option
0001:004c2ae4  _php_stream_context_set_option
0001:004c2c30  _php_stream_context_get_link
0001:004c2c98  _php_stream_context_set_link
0001:004c2e30  _php_stream_dirent_alphasort
0001:004c2e4c  _php_stream_dirent_alphasortr
0001:004c2e68  __php_stream_scandir
Module: U:\dev\php-5.3.6\main\streams\cast.o(cast.o)
0001:004c302c  _php_stream_mode_sanitize_fdopen_fopencookie
0001:004c31a0  __php_stream_cast
0001:004c347c  __php_stream_open_wrapper_as_file
0001:004c3504  __php_stream_make_seekable
Module: U:\dev\php-5.3.6\main\streams\memory.o(memory.o)
0001:004c3934  __php_stream_memory_create
0001:004c3994  __php_stream_memory_open
0001:004c39ec  __php_stream_memory_get_buffer
0001:004c3d3c  __php_stream_temp_create
0001:004c3dac  __php_stream_temp_open
0002:000065f0  _php_stream_memory_ops
0002:00006630  _php_stream_temp_ops
0002:00006670  _php_stream_rfc2397_ops
0002:000066b0  _php_stream_rfc2397_wops
0002:000066d8  _php_stream_rfc2397_wrapper
Module: U:\dev\php-5.3.6\main\streams\filter.o(filter.o)
0001:004c432c  _php_get_stream_filters_hash_global
0001:004c4338  __php_get_stream_filters_hash
0001:004c4358  _php_stream_filter_register_factory
0001:004c438c  _php_stream_filter_unregister_factory
0001:004c43bc  _php_stream_filter_register_factory_volatile
0001:004c4488  _php_stream_bucket_new
0001:004c4568  _php_stream_bucket_make_writeable
0001:004c4988  _php_stream_bucket_unlink
0001:004c48c4  _php_stream_bucket_delref
0001:004c4660  _php_stream_bucket_split
0001:004c492c  _php_stream_bucket_prepend
0001:004c4958  _php_stream_bucket_append
0001:004c4a14  _php_stream_filter_create
0001:004c4b9c  __php_stream_filter_alloc
0001:004c4c14  _php_stream_filter_free
0001:004c4c54  _php_stream_filter_prepend_ex
0001:004c4c84  __php_stream_filter_prepend
0001:004c4cb8  _php_stream_filter_append_ex
0001:004c4f50  __php_stream_filter_append
0001:004c4f94  __php_stream_filter_flush
0001:004c51dc  _php_stream_filter_remove
Module: U:\dev\php-5.3.6\main\streams\plain_wrapper.o(plain_wrapper.o)
0001:004c525c  _php_stream_parse_fopen_modes
0001:004c5504  __php_stream_fopen_temporary_file
0001:004c5564  __php_stream_fopen_tmpfile
0001:004c55f8  __php_stream_fopen_from_fd
0001:004c56b4  __php_stream_fopen_from_file
0001:004c5744  __php_stream_fopen_from_pipe
0001:004c5f54  __php_stream_fopen
0001:004c6814  __php_stream_fopen_with_path
0002:000066f0  _php_stream_stdio_ops
0002:00006798  _php_plain_files_wrapper
Module: U:\dev\php-5.3.6\main\streams\userspace.o(userspace.o)
0001:004c6f10  _zm_startup_user_streams
0001:004c7a78  _zif_stream_wrapper_register
0001:004c7bec  _zif_stream_wrapper_unregister
0001:004c7cdc  _zif_stream_wrapper_restore
0002:000067f0  _php_stream_userspace_ops
0002:00006830  _php_stream_userspace_dir_ops
Module: U:\dev\php-5.3.6\main\streams\transports.o(transports.o)
0001:004ca48c  _php_stream_xport_get_hash
0001:004ca498  _php_stream_xport_register
0001:004ca4cc  _php_stream_xport_unregister
0001:004ca5dc  __php_stream_xport_create
0001:004caadc  _php_stream_xport_connect
0001:004caa70  _php_stream_xport_bind
0001:004cab68  _php_stream_xport_listen
0001:004cabd0  _php_stream_xport_accept
0001:004cac80  _php_stream_xport_get_name
0001:004cad48  _php_stream_xport_crypto_setup
0001:004cadb0  _php_stream_xport_crypto_enable
0001:004cae14  _php_stream_xport_recvfrom
0001:004caefc  _php_stream_xport_sendto
0001:004cafa4  _php_stream_xport_shutdown
Module: U:\dev\php-5.3.6\main\streams\xp_socket.o(xp_socket.o)
0001:004cba40  _php_stream_generic_socket_factory
0002:00006870  _php_stream_generic_socket_ops
0002:000068b0  _php_stream_socket_ops
0002:000068f0  _php_stream_udp_socket_ops
0002:00006930  _php_stream_unix_socket_ops
0002:00006970  _php_stream_unixdg_socket_ops
Module: U:\dev\php-5.3.6\main\streams\mmap.o(mmap.o)
0001:004cc32c  __php_stream_mmap_range
0001:004cc38c  __php_stream_mmap_unmap
0001:004cc3b0  __php_stream_mmap_unmap_ex
Module: U:\dev\php-5.3.6\main\streams\glob_wrapper.o(glob_wrapper.o)
0001:004cc40c  __php_glob_stream_get_path
0001:004cc460  __php_glob_stream_get_pattern
0001:004cc4b4  __php_glob_stream_get_count
0002:000069b0  _php_glob_stream_ops
0002:00006a18  _php_glob_stream_wrapper
Module: U:\dev\php-5.3.6\Zend\zend_language_parser.o(zend_language_parser.o)
0001:004d5094  _zendparse
Module: U:\dev\php-5.3.6\Zend\zend_language_scanner.o(zend_language_scanner.o)
0002:000241f8  _language_scanner_globals_id
0001:004da0c0  _startup_scanner
0001:004da110  _shutdown_scanner
0001:004da1bc  _zend_save_lexical_state
0001:004da258  _zend_restore_lexical_state
0001:004da33c  _zend_destroy_file_handle
0001:004da39c  _open_file_for_scanning
0001:004da55c  _compile_file
0001:004da6f8  _compile_filename
0001:004da858  _zend_prepare_string_for_scanning
0001:004da8e0  _zend_get_scanned_file_offset
0001:004da8fc  _compile_string
0001:004daadc  _highlight_file
0001:004dab70  _highlight_string
0001:004db834  _lex_scan
Module: U:\dev\php-5.3.6\Zend\zend_ini_parser.o(zend_ini_parser.o)
0001:004e3d24  _zend_parse_ini_file
0001:004e4838  _ini_parse
0001:004e3db0  _zend_parse_ini_string
Module: U:\dev\php-5.3.6\Zend\zend_ini_scanner.o(zend_ini_scanner.o)
0002:00024208  _ini_scanner_globals_id
0001:004e5320  _shutdown_ini_scanner
0001:004e5364  _zend_ini_scanner_get_lineno
0001:004e5384  _zend_ini_scanner_get_filename
0001:004e53a4  _zend_ini_open_file_for_scanning
0001:004e53f8  _zend_ini_prepare_string_for_scanning
0001:004e5d44  _ini_lex
Module: U:\dev\php-5.3.6\Zend\zend_alloc.o(zend_alloc.o)
0001:004eaacc  _zend_mm_startup_ex
0001:004eadd0  _zend_mm_startup
0001:004eaf5c  _zend_mm_shutdown
0001:004ebda0  __zend_mm_alloc
0001:004ebdac  __zend_mm_free
0001:004ebdb8  __zend_mm_realloc
0001:004ebdc4  __zend_mm_block_size
0001:004ebdd8  _is_zend_mm
0001:004ebdf0  __emalloc
0001:004ebe38  __efree
0001:004ebe80  __erealloc
0001:004ebedc  __zend_mem_block_size
0001:004ebf5c  __safe_emalloc
0001:004ebfac  __safe_malloc
0001:004ec010  __safe_erealloc
0001:004ec064  __safe_realloc
0001:004ec0d0  __ecalloc
0001:004ec10c  __estrdup
0001:004ec14c  __estrndup
0001:004ec184  _zend_strndup
0001:004ec1c4  _zend_set_memory_limit
0001:004ec1f8  _zend_memory_usage
0001:004ec234  _zend_memory_peak_usage
0001:004ec268  _shutdown_memory_manager
0001:004ec30c  _start_memory_manager
0001:004ec32c  _zend_mm_set_heap
0001:004ec348  _zend_mm_get_storage
0001:004ec354  _zend_mm_set_custom_handlers
Module: U:\dev\php-5.3.6\Zend\zend_compile.o(zend_compile.o)
0002:00024218  _zend_compile_file
0002:00024228  _zend_compile_string
0001:004ec6f8  _zend_auto_global_arm
0001:004ec70c  _zend_auto_global_disable_jit
0001:004ec780  _zend_init_compiler_data_structures
0001:004ec91c  _file_handle_dtor
0001:004ec938  _init_compiler
0001:004ec9c4  _shutdown_compiler
0001:004ecab4  _zend_set_compiled_filename
0001:004ecb6c  _zend_restore_compiled_filename
0001:004ecb88  _zend_get_compiled_filename
0001:004ecba4  _zend_get_compiled_lineno
0001:004ecbc0  _zend_is_compiling
0001:004eccc0  _zend_do_binary_op
0001:004ecd3c  _zend_do_unary_op
0001:004ecddc  _zend_do_binary_assign_op
0001:004ecf54  _fetch_simple_variable_ex
0001:004f88e8  _zend_is_auto_global
0001:004ed164  _fetch_simple_variable
0001:004ed180  _zend_do_fetch_static_member
0001:004f1314  _zend_do_fetch_class
0001:004ed3bc  _fetch_array_begin
0001:004ed3f4  _fetch_array_dim
0001:004ed490  _fetch_string_offset
0001:004ed49c  _zend_do_print
0001:004ed510  _zend_do_echo
0001:004ed5f0  _zend_do_abstract_method
0001:004ed780  _zend_do_assign
0001:004ee7c4  _zend_do_end_variable_parse
0001:004edc78  _zend_do_assign_ref
0001:004ede28  _zend_do_while_cond
0001:004edef8  _zend_do_while_end
0001:004edfe0  _zend_do_for_cond
0001:004ee048  _zend_do_for_before_statement
0001:004ee12c  _zend_do_for_end
0001:004ee220  _zend_do_pre_incdec
0001:004ee354  _zend_do_post_incdec
0001:004ee484  _zend_do_if_cond
0001:004ee510  _zend_do_if_after_statement
0001:004ee5f4  _zend_do_if_end
0001:004ee714  _zend_check_writable_variable
0001:004ee758  _zend_do_begin_variable_parse
0001:004eeaa4  _zend_do_add_string
0001:004eebc4  _zend_do_add_variable
0001:004eec68  _zend_do_free
0001:004eeea8  _zend_do_verify_access_types
0001:004ef2c8  _zend_do_begin_function_declaration
0001:004f8dec  _zend_do_build_namespace_name
0001:004f00a8  _zend_do_begin_lambda_function_declaration
0001:004f0194  _zend_do_handle_exception
0001:004f01f8  _zend_do_end_function_declaration
0001:004f878c  _zend_do_extended_info
0001:004f2204  _zend_do_return
0001:004f1808  _zend_release_labels
0001:004f0430  _zend_do_receive_arg
0001:004f8d3c  _zend_get_class_fetch_type
0001:004f0fec  _zend_resolve_class_name
0001:004f080c  _zend_do_begin_function_call
0001:004f0d74  _zend_resolve_non_class_name
0001:004f87d0  _zend_do_extended_fcall_begin
0001:004f0ba0  _zend_do_begin_dynamic_function_call
0001:004f0964  _zend_do_begin_method_call
0001:004f0af0  _zend_do_clone
0001:004f14b8  _zend_do_label
0001:004f15f8  _zend_resolve_goto_label
0001:004f1790  _zend_do_goto
0001:004f18d8  _zend_do_build_full_name
0001:004f19ac  _zend_do_begin_class_member_function_call
0001:004f1b2c  _zend_do_end_function_call
0001:004f1de0  _zend_do_pass_param
0001:004f243c  _zend_do_first_catch
0001:004f2464  _zend_initialize_try_catch_element
0001:004f252c  _zend_do_mark_last_catch
0001:004f2614  _zend_do_try
0001:004f2668  _zend_do_begin_catch
0001:004f276c  _zend_do_end_catch
0001:004f2818  _zend_do_throw
0001:004f285c  _function_add_ref
0001:004f2bb8  _zend_visibility_string
0001:004f58d8  _zend_mangle_property_name
0001:004f3814  _zend_do_inherit_interfaces
0001:004f3a74  _zend_do_inheritance
0001:004f3d90  _zend_do_implement_interface
0001:004f3fd0  _do_bind_function
0001:004f40fc  _do_bind_class
0001:004f41dc  _do_bind_inherited_class
0001:004f42b0  _zend_do_early_binding
0001:004f45cc  _zend_do_delayed_early_binding
0001:004f4684  _zend_do_boolean_or_begin
0001:004f4744  _zend_do_boolean_or_end
0001:004f47d4  _zend_do_boolean_and_begin
0001:004f4894  _zend_do_boolean_and_end
0001:004f4924  _zend_do_do_while_begin
0001:004f4994  _zend_do_do_while_end
0001:004f4a5c  _zend_do_brk_cont
0001:004f4ae8  _zend_do_switch_cond
0001:004f4b98  _zend_do_switch_end
0001:004f4d5c  _zend_do_case_before_statement
0001:004f4ef8  _zend_do_case_after_statement
0001:004f4fb0  _zend_do_default_before_statement
0001:004f51b4  _zend_do_begin_class_declaration
0001:004f8aa4  _zend_initialize_class_data
0001:004f5654  _zend_do_end_class_declaration
0001:004f57ec  _zend_do_implements_interface
0001:004f59e4  _zend_unmangle_property_name
0001:004f5b50  _zend_do_declare_property
0001:004f5d68  _zend_do_declare_class_constant
0001:004f5eb8  _zend_do_fetch_property
0001:004f6074  _zend_do_halt_compiler_register
0001:004f60fc  _zend_do_declare_implicit_property
0001:004f6104  _zend_do_push_object
0001:004f6128  _zend_do_pop_object
0001:004f618c  _zend_do_begin_new_object
0001:004f6244  _zend_do_end_new_object
0001:004f6514  _zend_do_fetch_constant
0001:004f67ac  _zend_do_shell_exec
0001:004f68c4  _zend_do_init_array
0001:004f6970  _zend_do_add_array_element
0001:004f6a0c  _zend_do_add_static_array_element
0001:004f6bec  _zend_do_add_list_element
0001:004f6c6c  _zend_do_new_list_begin
0001:004f6c98  _zend_do_new_list_end
0001:004f6ccc  _zend_do_list_init
0001:004f6d60  _zend_do_list_end
0001:004f6ff4  _zend_do_fetch_static_variable
0001:004f7284  _zend_do_fetch_lexical_variable
0001:004f730c  _zend_do_fetch_global_variable
0001:004f742c  _zend_do_cast
0001:004f74a8  _zend_do_include_or_eval
0001:004f8814  _zend_do_extended_fcall_end
0001:004f7550  _zend_do_indirect_references
0001:004f762c  _zend_do_unset
0001:004f76f4  _zend_do_isset_or_isempty
0001:004f7848  _zend_do_instanceof
0001:004f7930  _zend_do_foreach_begin
0001:004f7ca0  _zend_do_foreach_cont
0001:004f7f94  _zend_do_foreach_end
0001:004f80e4  _zend_do_declare_begin
0001:004f8138  _zend_do_declare_stmt
0001:004f820c  _zend_do_declare_end
0001:004f82a0  _zend_do_exit
0001:004f82f8  _zend_do_begin_silence
0001:004f8368  _zend_do_end_silence
0001:004f83ac  _zend_do_jmp_set
0001:004f846c  _zend_do_jmp_set_else
0001:004f8524  _zend_do_begin_qm_op
0001:004f85b8  _zend_do_qm_true
0001:004f86c8  _zend_do_qm_false
0001:004f8858  _zend_do_ticks
0001:004f88d4  _zend_auto_global_dtor
0001:004f894c  _zend_register_auto_global
0001:004f89a0  _zendlex
0001:004f8dbc  _zend_get_compiled_variable_name
0001:004f8fdc  _zend_do_begin_namespace
0001:004f9438  _zend_do_use
0001:004f9938  _zend_do_declare_constant
0001:004f9a7c  _zend_verify_namespace
0001:004f9ab8  _zend_do_end_namespace
0001:004f9bc0  _zend_do_end_compilation
0001:004f9be4  _zend_dirname
Module: U:\dev\php-5.3.6\Zend\zend_constants.o(zend_constants.o)
0001:004f9ecc  _free_zend_constant
0001:004f9f00  _copy_zend_constant
0001:004f9f3c  _zend_copy_constants
0001:004f9f9c  _clean_module_constants
0001:004f9fc8  _zend_startup_constants
0001:004fa160  _zend_register_standard_constants
0001:004fa48c  _zend_register_long_constant
0001:004facf4  _zend_register_constant
0001:004fa404  _zend_shutdown_constants
0001:004fa444  _clean_non_persistent_constants
0001:004fa4d4  _zend_register_double_constant
0001:004fa520  _zend_register_stringl_constant
0001:004fa56c  _zend_register_string_constant
0001:004fa5bc  _zend_get_constant
0001:004fa86c  _zend_get_constant_ex
Module: U:\dev\php-5.3.6\Zend\zend_dynamic_array.o(zend_dynamic_array.o)
0001:004fae8c  _zend_dynamic_array_init
0001:004faec4  _zend_dynamic_array_push
0001:004faf08  _zend_dynamic_array_pop
0001:004faf20  _zend_dynamic_array_get_element
Module: U:\dev\php-5.3.6\Zend\zend_execute_API.o(zend_execute_API.o)
0002:00024238  _zend_execute
0002:00024248  _zend_execute_internal
0001:004faf60  _empty_fcall_info
0001:004faf84  _empty_fcall_info_cache
0001:004fb020  _init_executor
0001:004fbc48  __zval_ptr_dtor
0001:004fb3bc  _shutdown_destructors
0001:004fb4d0  _shutdown_executor
0001:004fbab8  _get_active_class_name
0001:004fbc2c  _zend_is_executing
0001:004fbb38  _get_active_function_name
0001:004fbba4  _zend_get_executed_filename
0001:004fbbcc  _zend_get_executed_lineno
0001:004fbd08  __zval_internal_ptr_dtor
0001:004fbd4c  _zend_is_true
0001:004fbe6c  _zval_update_constant_ex
0001:004fc578  _zval_update_constant_inline_change
0001:004fc590  _zval_update_constant_no_inline_change
0001:004fc5a8  _zval_update_constant
0001:004fc5c0  _call_user_function
0001:004fc6f0  _call_user_function_ex
0001:004fc858  _zend_call_function
0001:004fd5e4  _zend_lookup_class_ex
0001:004fd9c0  _zend_lookup_class
0001:004fd9e4  _zend_eval_stringl
0001:004fe894  _zend_rebuild_symbol_table
0001:004fdcd8  _zend_eval_string
0001:004fdd08  _zend_eval_stringl_ex
0001:004fdd68  _zend_eval_string_ex
0001:004fdd9c  _execute_new_code
0001:004fe044  _zend_timeout
0001:004fe0c4  _zend_set_timeout
0001:004fe160  _zend_unset_timeout
0001:004fe2c4  _zend_fetch_class
0001:004fe58c  _zend_verify_abstract_class
0001:004fe718  _zend_reset_all_cv
0001:004fe76c  _zend_delete_global_variable
Module: U:\dev\php-5.3.6\Zend\zend_highlight.o(zend_highlight.o)
0001:004fedc4  _zend_html_putc
0001:004fef20  _zend_html_puts
0001:004fefcc  _zend_highlight
0001:004ff1c0  _zend_strip
Module: U:\dev\php-5.3.6\Zend\zend_llist.o(zend_llist.o)
0001:004ff30c  _zend_llist_init
0001:004ff34c  _zend_llist_add_element
0001:004ff3e0  _zend_llist_prepend_element
0001:004ff474  _zend_llist_del_element
0001:004ff50c  _zend_llist_destroy
0001:004ff56c  _zend_llist_clean
0001:004ff590  _zend_llist_remove_tail
0001:004ff604  _zend_llist_copy
0001:004ff64c  _zend_llist_apply_with_del
0001:004ff6e4  _zend_llist_apply
0001:004ff718  _zend_llist_sort
0001:004ff7cc  _zend_llist_apply_with_argument
0001:004ff800  _zend_llist_apply_with_arguments
0001:004ff838  _zend_llist_count
0001:004ff844  _zend_llist_get_first_ex
0001:004ff870  _zend_llist_get_last_ex
0001:004ff89c  _zend_llist_get_next_ex
0001:004ff8c8  _zend_llist_get_prev_ex
Module: U:\dev\php-5.3.6\Zend\zend_opcode.o(zend_opcode.o)
0001:004ff980  _init_op_array
0001:004ffad8  _destroy_zend_function
0001:004ffda4  _destroy_op_array
0001:004ffaf8  _zend_function_dtor
0001:004ffb30  _zend_cleanup_function_data
0001:004ffb54  _zend_cleanup_function_data_full
0001:004ffb78  _zend_cleanup_class_data
0001:004ffc4c  _destroy_zend_class
0001:004ffd94  _zend_class_add_ref
0001:004fffdc  _init_op
0001:00500098  _get_next_op
0001:00500118  _get_next_op_number
0001:00500124  _get_next_brk_cont_element
0001:005001d0  _pass_two
0001:00500384  _print_class
0001:005003c8  _get_unary_op
0001:005003e8  _get_binary_op
Module: U:\dev\php-5.3.6\Zend\zend_operators.o(zend_operators.o)
0001:0050051c  _zend_atoi
0001:00500624  _zend_atol
0001:00500730  _zend_string_to_double
0001:0050082c  _convert_scalar_to_number
0001:00500994  _convert_to_long_base
0001:005008e0  _convert_to_long
0001:00500c9c  _convert_to_double
0001:00500ef0  _convert_to_null
0001:00500fd4  _convert_to_boolean
0001:00501274  __convert_to_string
0001:0050161c  _convert_to_array
0001:00501848  _convert_to_object
0001:005018a8  _multi_convert_to_long_ex
0001:00501954  _multi_convert_to_double_ex
0001:00501a00  _multi_convert_to_string_ex
0001:00501acc  _add_function
0001:00501e10  _sub_function
0001:005020e0  _mul_function
0001:005023c0  _div_function
0001:00502734  _mod_function
0001:00502a54  _boolean_xor_function
0001:00502c7c  _boolean_not_function
0001:00502da4  _bitwise_not_function
0001:00502ebc  _bitwise_or_function
0001:00503234  _bitwise_and_function
0001:005035b4  _bitwise_xor_function
0001:00503934  _shift_left_function
0001:00503c24  _shift_right_function
0001:00503f04  _add_char_to_string
0001:00503f4c  _add_string_to_string
0001:00503fb4  _concat_function
0001:00504150  _string_compare_function
0001:005059f0  _zend_binary_zval_strcmp
0001:0050420c  _string_locale_compare_function
0001:005042cc  _numeric_compare_function
0001:005043a0  _compare_function
0001:00505844  _zend_binary_strcmp
0001:00505c40  _zend_compare_arrays
0001:00505a7c  _zendi_smart_strcmp
0001:00505198  _is_identical_function
0001:00505290  _is_not_identical_function
0001:005052c8  _is_equal_function
0001:00505304  _is_not_equal_function
0001:00505340  _is_smaller_function
0001:00505374  _is_smaller_or_equal_function
0001:005053b0  _instanceof_function_ex
0001:00505424  _instanceof_function
0001:005055a0  _increment_function
0001:00505680  _decrement_function
0001:00505778  _zval_is_true
0001:00505798  _zend_str_tolower_copy
0001:005057e8  _zend_str_tolower_dup
0001:00505808  _zend_str_tolower
0001:00505880  _zend_binary_strncmp
0001:005058d4  _zend_binary_strcasecmp
0001:00505954  _zend_binary_strncasecmp
0001:00505a10  _zend_binary_zval_strncmp
0001:00505a38  _zend_binary_zval_strcasecmp
0001:00505a58  _zend_binary_zval_strncasecmp
0001:00505bf4  _zend_compare_symbol_tables_i
0001:00505c14  _zend_compare_symbol_tables
0001:00505c58  _zend_compare_objects
0001:00505ca4  _zend_locale_sprintf_double
Module: U:\dev\php-5.3.6\Zend\zend_ptr_stack.o(zend_ptr_stack.o)
0001:0050607c  _zend_ptr_stack_init_ex
0001:005060f4  _zend_ptr_stack_init
0001:00506108  _zend_ptr_stack_n_push
0001:005061b0  _zend_ptr_stack_n_pop
0001:005061ec  _zend_ptr_stack_destroy
0001:00506218  _zend_ptr_stack_apply
0001:00506248  _zend_ptr_stack_clean
0001:005062ac  _zend_ptr_stack_num_elements
Module: U:\dev\php-5.3.6\Zend\zend_stack.o(zend_stack.o)
0001:005062cc  _zend_stack_init
0001:00506308  _zend_stack_push
0001:0050636c  _zend_stack_top
0001:00506398  _zend_stack_del_top
0001:005063c4  _zend_stack_int_top
0001:005063ec  _zend_stack_is_empty
0001:00506400  _zend_stack_destroy
0001:00506448  _zend_stack_base
0001:00506454  _zend_stack_count
0001:00506460  _zend_stack_apply
0001:005064c8  _zend_stack_apply_with_argument
Module: U:\dev\php-5.3.6\Zend\zend_variables.o(zend_variables.o)
0001:0050654c  __zval_dtor_func
0001:00506650  __zval_internal_dtor
0001:005066b8  _zval_add_ref
0001:005066c8  __zval_copy_ctor_func
0001:005067cc  _zend_print_variable
0001:005067e0  __zval_dtor_wrapper
0001:00506828  _zval_property_ctor
Module: U:\dev\php-5.3.6\Zend\zend.o(zend.o)
0002:00024258  _executor_globals_id
0002:00024268  _zend_write
0002:00024278  _zend_printf
0002:00024288  _compiler_globals_id
0002:00024298  _zend_error_cb
0002:000242a8  _zend_fopen
0002:000242b8  _zend_stream_open_function
0002:000242c8  _zend_block_interruptions
0002:000242d8  _zend_unblock_interruptions
0002:000242e8  _zend_ticks_function
0002:000242f8  _zend_on_timeout
0002:00024308  _zend_vspprintf
0002:00024318  _zend_getenv
0002:00024328  _zend_resolve_path
0002:00024338  _zval_used_for_init
0002:00024348  _zend_uv
0001:005072b4  _zend_print_zval_r_ex
0001:00507124  _zend_print_flat_zval_r
0001:00506da4  _zend_make_printable_zval
0001:005084cc  _zend_error
0001:00507058  _zend_print_zval
0001:00507074  _zend_print_zval_ex
0001:00507288  _zend_print_zval_r
0001:005079b8  _zend_startup
0001:00507cec  _zend_register_standard_ini_entries
0001:00507d04  _zend_post_startup
0001:00507e44  _zend_shutdown
0001:00507f20  _zend_set_utility_values
0001:00507f5c  _zenderror
0001:00507fa4  __zend_bailout
0001:00508ac4  _zend_output_debug_string
0001:00508068  _zend_append_version_info
0001:00508144  _get_zend_version
0001:00508150  _zend_activate
0001:00508180  _zend_activate_modules
0001:0050819c  _zend_deactivate_modules
0001:00508218  _zend_call_destructors
0001:00508280  _zend_deactivate
0001:00508444  _zend_post_deactivate_modules
0001:00508478  _zend_message_dispatcher
0001:005084a0  _zend_get_configuration_directive
0001:005084cc  _zend_error_noreturn
0001:00508acc  _zend_execute_scripts
0001:00508d98  _zend_make_compiled_string_description
0001:00508e1c  _free_estring
0002:0001dd00  _zend_standard_class_def
Module: U:\dev\php-5.3.6\Zend\zend_API.o(zend_API.o)
0002:00024358  _module_registry
0001:00508e3c  _zend_get_parameters
0001:00508f24  __zend_get_parameters_array
0001:00508ff8  _zend_get_parameters_ex
0001:00509064  __zend_get_parameters_array_ex
0001:005090c0  _zend_copy_parameters_array
0001:0050babc  _add_next_index_zval
0001:0050915c  _zend_wrong_param_count
0001:005091d8  _zend_get_type_by_const
0001:0050924c  _zend_zval_type_name
0001:00509298  _zend_get_class_entry
0001:005092cc  _zend_get_object_classname
0001:0050fa80  _zend_fcall_info_init
0001:0050a8d4  _zend_parse_parameters_ex
0001:0050a948  _zend_parse_parameters
0001:0050a9dc  _zend_parse_method_parameters
0001:0050ab28  _zend_parse_method_parameters_ex
0001:0050ac8c  __array_init
0001:0050ad50  _zend_merge_properties
0001:0050adf0  _zend_update_class_constants
0001:0050b19c  __object_and_properties_init
0001:0050b29c  __object_init_ex
0001:0050b2b4  __object_init
0001:0050b2fc  _add_assoc_function
0001:0050b318  _add_assoc_long_ex
0001:0050b360  _add_assoc_null_ex
0001:0050b3a4  _add_assoc_bool_ex
0001:0050b3f4  _add_assoc_resource_ex
0001:0050b43c  _add_assoc_double_ex
0001:0050b490  _add_assoc_string_ex
0001:0050b51c  _add_assoc_stringl_ex
0001:0050b594  _add_assoc_zval_ex
0001:0050b5b4  _add_index_long
0001:0050b5fc  _add_index_null
0001:0050b640  _add_index_bool
0001:0050b68c  _add_index_resource
0001:0050b6d4  _add_index_double
0001:0050b728  _add_index_string
0001:0050b7b4  _add_index_stringl
0001:0050b82c  _add_index_zval
0001:0050b84c  _add_next_index_long
0001:0050b894  _add_next_index_null
0001:0050b8d4  _add_next_index_bool
0001:0050b920  _add_next_index_resource
0001:0050b968  _add_next_index_double
0001:0050b9bc  _add_next_index_string
0001:0050ba44  _add_next_index_stringl
0001:0050badc  _add_get_assoc_string_ex
0001:0050bb68  _add_get_assoc_stringl_ex
0001:0050bbe4  _add_get_index_long
0001:0050bc2c  _add_get_index_double
0001:0050bc80  _add_get_index_string
0001:0050bd0c  _add_get_index_stringl
0001:0050bd84  _add_property_long_ex
0001:0050be24  _add_property_bool_ex
0001:0050bec8  _add_property_null_ex
0001:0050bf64  _add_property_resource_ex
0001:0050c004  _add_property_double_ex
0001:0050c0ac  _add_property_string_ex
0001:0050c18c  _add_property_stringl_ex
0001:0050c258  _add_property_zval_ex
0001:0050c320  _zend_startup_module_ex
0001:0050c548  _zend_startup_modules
0001:0050c618  _zend_register_module_ex
0001:0050cf04  _zend_register_functions
0001:0050c7c4  _zend_register_internal_module
0001:0050de00  _zend_next_free_module
0001:0050c94c  _zend_check_magic_method_implementation
0001:0050db8c  _zend_unregister_functions
0001:0050dc0c  _zend_startup_module
0001:0050dc54  _zend_get_module_started
0001:0050dc9c  _module_destructor
0001:0050dd7c  _module_registry_request_startup
0001:0050ddc4  _module_registry_cleanup
0001:0050ddec  _module_registry_unload_temp
0001:0050df04  _zend_register_internal_class_ex
0001:0050dfc4  _zend_register_internal_class
0001:0050df88  _zend_class_implements
0001:0050dfdc  _zend_register_internal_interface
0001:0050dff4  _zend_register_class_alias_ex
0001:0050e054  _zend_set_hash_symbol
0001:0050e0e4  _zif_display_disabled_function
0001:0050e128  _zend_disable_function
0001:0050e218  _zend_disable_class
0001:0050f424  _zend_is_callable_ex
0001:0050f998  _zend_is_callable
0001:0050f9bc  _zend_make_callable
0001:0050fb14  _zend_fcall_info_args_clear
0001:0050fb50  _zend_fcall_info_args_save
0001:0050fb78  _zend_fcall_info_args_restore
0001:0050fb9c  _zend_fcall_info_args
0001:0050fc34  _zend_fcall_info_argp
0001:0050fca8  _zend_fcall_info_argv
0001:0050fd24  _zend_fcall_info_argn
0001:0050fd44  _zend_fcall_info_call
0001:0050fde8  _zend_get_module_version
0001:0050fe80  _zend_declare_property_ex
0001:005100f0  _zend_declare_property
0001:00510114  _zend_declare_property_null
0001:0051017c  _zend_declare_property_bool
0001:00510208  _zend_declare_property_long
0001:0051028c  _zend_declare_property_double
0001:0051031c  _zend_declare_property_string
0001:005103e4  _zend_declare_property_stringl
0001:005104a0  _zend_declare_class_constant
0001:005104c8  _zend_declare_class_constant_null
0001:00510518  _zend_declare_class_constant_long
0001:00510590  _zend_declare_class_constant_bool
0001:00510610  _zend_declare_class_constant_double
0001:00510694  _zend_declare_class_constant_stringl
0001:00510744  _zend_declare_class_constant_string
0001:005107a4  _zend_update_property
0001:00510878  _zend_update_property_null
0001:005108b4  _zend_update_property_bool
0001:00510928  _zend_update_property_long
0001:00510998  _zend_update_property_double
0001:00510a14  _zend_update_property_string
0001:00510aac  _zend_update_property_stringl
0001:00510b38  _zend_update_static_property
0001:00510c7c  _zend_update_static_property_null
0001:00510cb4  _zend_update_static_property_bool
0001:00510d1c  _zend_update_static_property_long
0001:00510d80  _zend_update_static_property_double
0001:00510df0  _zend_update_static_property_string
0001:00510e7c  _zend_update_static_property_stringl
0001:00510f24  _zend_read_property
0001:00511010  _zend_read_static_property
0001:0051106c  _zend_save_error_handling
0001:005110a4  _zend_replace_error_handling
0001:0051113c  _zend_restore_error_handling
Module: U:\dev\php-5.3.6\Zend\zend_extensions.o(zend_extensions.o)
0002:00024388  _zend_extensions
0001:005118a4  _zend_load_extension
0001:00511a78  _zend_register_extension
0001:00511bc8  _zend_extension_dispatch_message
0001:00511b18  _zend_startup_extensions_mechanism
0001:00511b84  _zend_extension_dtor
0001:00511b40  _zend_startup_extensions
0001:00511b5c  _zend_shutdown_extensions
0001:00511bf4  _zend_get_resource_handle
0001:00511c1c  _zend_get_extension
0001:00511c60  _zend_os2_load_module
0001:00511c94  _zend_os2_query_symbol
0001:00511cdc  _zend_os2_module_error
Module: U:\dev\php-5.3.6\Zend\zend_hash.o(zend_hash.o)
0001:00511e3c  _zend_hash_func
0001:00511e48  __zend_hash_init
0001:00511f18  __zend_hash_init_ex
0001:00511f48  _zend_hash_set_apply_protection
0001:00511f68  __zend_hash_add_or_update
0001:005122f0  __zend_hash_quick_add_or_update
0001:005126d8  __zend_hash_index_update_or_next_insert
0001:005126b0  _zend_hash_add_empty_element
0001:00512ae0  _zend_hash_rehash
0001:00512b30  _zend_hash_del_key_or_index
0001:00512cd0  _zend_hash_destroy
0001:00512d74  _zend_hash_clean
0001:00512f48  _zend_hash_graceful_destroy
0001:00512f90  _zend_hash_graceful_reverse_destroy
0001:00513008  _zend_hash_apply
0001:0051308c  _zend_hash_apply_with_argument
0001:00513110  _zend_hash_apply_with_arguments
0001:005131b0  _zend_hash_reverse_apply
0001:00513234  _zend_hash_copy
0001:005132dc  __zend_hash_merge
0001:0051368c  _zend_hash_index_exists
0001:005133b4  _zend_hash_merge_ex
0001:00513438  _zend_get_hash_value
0001:00513444  _zend_hash_find
0001:005134bc  _zend_hash_quick_find
0001:0051364c  _zend_hash_index_find
0001:00513550  _zend_hash_exists
0001:005135c4  _zend_hash_quick_exists
0001:005136c4  _zend_hash_num_elements
0001:005136d0  _zend_hash_get_pointer
0001:00513700  _zend_hash_set_pointer
0001:00513750  _zend_hash_internal_pointer_reset_ex
0001:0051376c  _zend_hash_internal_pointer_end_ex
0001:00513788  _zend_hash_move_forward_ex
0001:005137b0  _zend_hash_move_backwards_ex
0001:005137d8  _zend_hash_get_current_key_ex
0001:00513850  _zend_hash_get_current_key_type_ex
0001:0051387c  _zend_hash_get_current_data_ex
0001:005138a8  _zend_hash_update_current_key_ex
0001:00513cfc  _zend_hash_sort
0001:00513eb8  _zend_hash_compare
0001:005140e4  _zend_hash_minmax
0001:00514174  _zend_hash_next_free_element
Module: U:\dev\php-5.3.6\Zend\zend_list.o(zend_list.o)
0002:000243a8  _le_index_ptr
0001:005142ac  _zend_list_insert
0001:00514318  __zend_list_delete
0001:0051438c  __zend_list_find
0001:005143d8  __zend_list_addref
0001:00514418  _zend_register_resource
0001:005144fc  _zend_fetch_resource
0001:0051468c  _list_entry_destructor
0001:00514750  _plist_entry_destructor
0001:005147d8  _zend_init_rsrc_list
0001:00514830  _zend_init_rsrc_plist
0001:00514860  _zend_destroy_rsrc_list
0001:005148c8  _zend_clean_module_rsrc_dtors
0001:005148e8  _zend_register_list_destructors
0001:00514950  _zend_register_list_destructors_ex
0001:005149b8  _zend_fetch_list_dtor_id
0001:00514a2c  _zend_init_rsrc_list_dtors
0001:00514a50  _zend_destroy_rsrc_list_dtors
0001:00514a64  _zend_rsrc_list_get_rsrc_type
Module: U:\dev\php-5.3.6\Zend\zend_indent.o(zend_indent.o)
0001:00514b30  _zend_indent
Module: U:\dev\php-5.3.6\Zend\zend_builtin_functions.o(zend_builtin_functions.o)
0001:00515e1c  _zm_startup_core
0001:00515f3c  _zend_startup_builtin_functions
0001:00519240  _debug_print_backtrace_args
0001:00519708  _zend_fetch_debug_backtrace
0002:00006aa0  _zend_builtin_module
Module: U:\dev\php-5.3.6\Zend\zend_sprintf.o(zend_sprintf.o)
0001:00519d4c  _zend_sprintf
Module: U:\dev\php-5.3.6\Zend\zend_ini.o(zend_ini.o)
0001:00519ec0  _zend_ini_startup
0001:00519f10  _zend_ini_shutdown
0001:00519f50  _zend_ini_global_shutdown
0001:00519f74  _zend_ini_deactivate
0001:00519ff4  _zend_copy_ini_directives
0001:0051a0dc  _zend_ini_sort_entries
0001:0051a10c  _zend_register_ini_entries
0001:0051a208  _zend_unregister_ini_entries
0001:0051a25c  _zend_ini_refresh_caches
0001:0051a288  _zend_alter_ini_entry
0001:0051a2b4  _zend_alter_ini_entry_ex
0001:0051a464  _zend_restore_ini_entry
0001:0051a51c  _zend_ini_register_displayer
0001:0051a554  _zend_ini_long
0001:0051a5dc  _zend_ini_double
0001:0051a65c  _zend_ini_string_ex
0001:0051a6d8  _zend_ini_string
0001:0051a724  _zend_ini_boolean_displayer_cb
0001:0051a844  _zend_ini_color_displayer_cb
0001:0051a8e4  _display_link_numbers
0001:0051a94c  _OnUpdateBool
0001:0051a9e4  _OnUpdateLong
0001:0051aa14  _OnUpdateLongGEZero
0001:0051aa54  _OnUpdateReal
0001:0051aa84  _OnUpdateString
0001:0051aaa4  _OnUpdateStringUnempty
Module: U:\dev\php-5.3.6\Zend\zend_qsort.o(zend_qsort.o)
0001:0051ab40  _zend_qsort
Module: U:\dev\php-5.3.6\Zend\zend_ts_hash.o(zend_ts_hash.o)
0001:0051ad84  __zend_ts_hash_init
0001:0051ade0  __zend_ts_hash_init_ex
0001:0051ae4c  _zend_ts_hash_destroy
0001:0051ae88  _zend_ts_hash_clean
0001:0051aeb8  __zend_ts_hash_add_or_update
0001:0051aef8  __zend_ts_hash_quick_add_or_update
0001:0051af38  __zend_ts_hash_index_update_or_next_insert
0001:0051af74  _zend_ts_hash_add_empty_element
0001:0051afa8  _zend_ts_hash_graceful_destroy
0001:0051afe4  _zend_ts_hash_apply
0001:0051b01c  _zend_ts_hash_apply_with_argument
0001:0051b058  _zend_ts_hash_apply_with_arguments
0001:0051b090  _zend_ts_hash_reverse_apply
0001:0051b0c8  _zend_ts_hash_del_key_or_index
0001:0051b100  _zend_ts_get_hash_value
0001:0051b134  _zend_ts_hash_find
0001:0051b168  _zend_ts_hash_quick_find
0001:0051b1a0  _zend_ts_hash_index_find
0001:0051b1d4  _zend_ts_hash_exists
0001:0051b208  _zend_ts_hash_index_exists
0001:0051b238  _zend_ts_hash_copy
0001:0051b294  _zend_ts_hash_copy_to_hash
0001:0051b2dc  _zend_ts_hash_merge
0001:0051b344  _zend_ts_hash_merge_ex
0001:0051b3ac  _zend_ts_hash_sort
0001:0051b3e4  _zend_ts_hash_compare
0001:0051b434  _zend_ts_hash_minmax
0001:0051b46c  _zend_ts_hash_num_elements
0001:0051b498  _zend_ts_hash_rehash
Module: U:\dev\php-5.3.6\Zend\zend_stream.o(zend_stream.o)
0001:0051b650  _zend_stream_open
0001:0051b760  _zend_stream_fixup
0001:0051ba00  _zend_file_handle_dtor
0001:0051bab0  _zend_compare_file_handles
Module: U:\dev\php-5.3.6\Zend\zend_iterators.o(zend_iterators.o)
0001:0051bb50  _zend_register_iterator_wrapper
0001:0051bc8c  _zend_iterator_wrap
0001:0051bcd8  _zend_iterator_unwrap
Module: U:\dev\php-5.3.6\Zend\zend_interfaces.o(zend_interfaces.o)
0002:000243b8  _zend_ce_aggregate
0002:000243c8  _zend_ce_iterator
0002:000243d8  _zend_ce_traversable
0002:000243e8  _zend_ce_serializable
0002:000243f8  _zend_ce_arrayaccess
0001:0051bde0  _zend_call_method
0001:0051c094  _zend_user_it_new_iterator
0001:0051c0c4  _zend_user_it_invalidate_current
0001:0051c128  _zend_user_it_valid
0001:0051c1a8  _zend_user_it_get_current_data
0001:0051c248  _zend_user_it_get_current_key
0001:0051c394  _zend_user_it_move_forward
0001:0051c3e4  _zend_user_it_rewind
0001:0051c520  _zend_user_it_get_new_iterator
0001:0051c8d4  _zend_user_serialize
0001:0051c9c4  _zend_user_unserialize
0001:0051ca9c  _zend_class_serialize_deny
0001:0051caf4  _zend_class_unserialize_deny
0001:0051cba0  _zend_funcs_aggregate
0001:0051cbe0  _zend_funcs_iterator
0001:0051cd60  _zend_funcs_arrayaccess
0001:0051ce20  _zend_funcs_serializable
0001:0051ce9c  _zend_register_interfaces
0002:00006b80  _zend_interface_iterator_funcs_iterator
0002:0001e4a0  _zend_funcs_traversable
Module: U:\dev\php-5.3.6\Zend\zend_exceptions.o(zend_exceptions.o)
0002:00024408  _default_exception_ce
0002:00024418  _zend_throw_exception_hook
0002:00024428  _error_exception_ce
0001:0051d5e4  _zend_exception_set_previous
0001:0051d6b0  _zend_exception_save
0001:0051d71c  _zend_exception_restore
0001:0051d7ac  _zend_throw_exception_internal
0001:0051f668  _zend_exception_error
0001:0051d89c  _zend_clear_exception
0001:0051daac  _zim_exception___clone
0001:0051f444  _zend_throw_exception
0001:0051db48  _zim_exception___construct
0001:0051dce4  _zim_error_exception___construct
0001:0051dec4  _zim_exception_getFile
0001:0051df18  _zim_exception_getLine
0001:0051df6c  _zim_exception_getMessage
0001:0051dfc0  _zim_exception_getCode
0001:0051e014  _zim_exception_getTrace
0001:0051e068  _zim_error_exception_getSeverity
0001:0051e83c  _zim_exception_getTraceAsString
0001:0051e93c  _zim_exception_getPrevious
0001:0051e9c0  _zend_spprintf
0001:0051ea78  _zim_exception___toString
0001:0051f0d8  _zend_register_default_exception
0001:0051f3f0  _zend_exception_get_default
0001:0051f3fc  _zend_get_error_exception
0001:0051f528  _zend_throw_exception_ex
0001:0051f568  _zend_throw_error_exception
0001:0051f94c  _zend_throw_exception_object
Module: U:\dev\php-5.3.6\Zend\zend_strtod.o(zend_strtod.o)
0001:0051f9cc  _zend_startup_strtod
0001:0051f9f0  _zend_shutdown_strtod
0001:00520a34  _zend_freedtoa
0001:00520aa0  _zend_dtoa
0001:00521a18  _zend_strtod
0001:005226e8  _zend_hex_strtod
0001:00522788  _zend_oct_strtod
Module: U:\dev\php-5.3.6\Zend\zend_gc.o(zend_gc.o)
0002:00024438  _gc_globals_id
0001:00522884  _gc_globals_ctor
0001:005228a4  _gc_globals_dtor
0001:005228ac  _gc_reset
0001:00522908  _gc_init
0001:00522968  _gc_zval_possible_root
0001:0052356c  _gc_collect_cycles
0001:00522ac4  _gc_zobj_possible_root
0001:00522be0  _gc_remove_zval_from_buffer
Module: U:\dev\php-5.3.6\Zend\zend_closures.o(zend_closures.o)
0002:00024448  _zend_ce_closure
0001:00523858  _zim_Closure___invoke
0001:00523a40  _zend_get_closure_invoke_method
0001:00523ab8  _zend_get_closure_method_def
0001:00523d6c  _zend_closure_get_closure
0001:00524054  _zim_Closure___construct
0001:005240b0  _zend_register_closure_ce
0001:005244c4  _zend_create_closure
Module: U:\dev\php-5.3.6\Zend\zend_float.o(zend_float.o)
0001:005246ac  _zend_init_fpu
0001:00524714  _zend_shutdown_fpu
0001:0052475c  _zend_ensure_fpu_mode
Module: U:\dev\php-5.3.6\Zend\zend_objects.o(zend_objects.o)
0001:0052478c  _zend_object_std_init
0001:005247c8  _zend_object_std_dtor
0001:005248d4  _zend_objects_destroy_object
0001:00524b10  _zend_objects_free_object_storage
0001:00524b34  _zend_objects_new
0001:00524b80  _zend_objects_get_address
0001:00524b94  _zend_objects_clone_members
0001:00524c54  _zend_objects_clone_obj
Module: U:\dev\php-5.3.6\Zend\zend_object_handlers.o(zend_object_handlers.o)
0001:00524cec  _zend_std_get_properties
0001:00524d04  _zend_std_get_debug_info
0001:00526834  _zend_check_protected
0001:00525184  _zend_get_property_info
0001:00525394  _zend_check_property_access
0001:00525570  _zend_std_read_property
0001:00525d0c  _zend_std_read_dimension
0001:005265a0  _zend_std_call_user_call
0001:0052677c  _zend_check_private
0001:00526cec  _zend_std_callstatic_user_call
0001:00526ed0  _zend_std_get_static_method
0001:00527268  _zend_std_get_static_property
0001:005273cc  _zend_std_unset_static_property
0001:005274a8  _zend_std_get_constructor
0001:005278c8  _zend_std_object_get_class
0001:005278e0  _zend_std_object_get_class_name
0001:00527a38  _zend_std_cast_object_tostring
0001:00527db0  _zend_std_get_closure
0002:00006bb0  _std_object_handlers
Module: U:\dev\php-5.3.6\Zend\zend_objects_API.o(zend_objects_API.o)
0001:00527f6c  _zend_objects_store_init
0001:00527fb0  _zend_objects_store_destroy
0001:00527fcc  _zend_objects_store_call_destructors
0001:00528040  _zend_objects_store_mark_destructed
0001:00528080  _zend_objects_store_free_object_storage
0001:0052812c  _zend_objects_store_put
0001:00528248  _zend_objects_store_get_refcount
0001:00528270  _zend_objects_store_add_ref
0001:00528298  _zend_objects_store_add_ref_by_handle
0001:005282bc  _zend_objects_store_del_ref
0001:00528348  _zend_objects_store_del_ref_by_handle_ex
0001:005285c0  _zend_objects_store_clone_obj
0001:00528698  _zend_object_store_get_object
0001:005286c0  _zend_object_store_get_object_by_handle
0001:005286e4  _zend_object_store_set_object
0001:0052870c  _zend_object_store_ctor_failed
0001:0052873c  _zend_objects_proxy_free_storage
0001:00528768  _zend_objects_proxy_clone
0001:005287a8  _zend_object_create_proxy
0001:00528860  _zend_object_proxy_set
0001:005288f8  _zend_object_proxy_get
0001:00528948  _zend_get_std_object_handlers
Module: U:\dev\php-5.3.6\Zend\zend_default_classes.o(zend_default_classes.o)
0001:0052896c  _zend_register_default_classes
Module: U:\dev\php-5.3.6\Zend\zend_execute.o(zend_execute.o)
0002:00024458  _zend_opcode_handlers
0001:005289ac  _zend_get_compiled_variable_value
0001:005299d4  _execute_internal
0001:00529a18  _execute
0001:0057cf2c  _zend_init_opcodes_handlers
0001:0057cfb8  _zend_vm_set_opcode_handler
0001:0057cfe0  _zend_do_fcall
0001:0057cfec  _zend_set_user_opcode_handler
0001:0057d014  _zend_get_user_opcode_handler
0001:0057d024  _zend_get_zval_ptr
0001:0057d164  _zend_get_zval_ptr_ptr
Module: U:\usr\lib\libc_dll.lib(dllinit.obj)
0001:0057ecc0  _DLL_InitTerm
Module: U:\usr\lib\libend.lib(src/libend/386/endlink386.asm)
0002:000244e0  _end
0002:0000b100  _edata
Module: U:\usr\lib\libend.lib(src/libend/386/end.asm)
0001:007a6440* _etext
0001:007a6440* __etext
0000:00000000* WEAK$ZERO
0002:000244e0  __end
0002:0000b100  __edata
Module: U:\extras\lib\xml2.lib(tree.obj)
0001:0057f287  _xmlBuildQName
0001:0057f361  _xmlSplitQName2
0001:0057f41a  _xmlSplitQName3
0001:0057f47a  _xmlValidateNCName
0001:0057f7e0  _xmlValidateQName
0001:0057fd9c  _xmlValidateName
0001:00580118  _xmlValidateNMToken
0001:00580539* _xmlSetBufferAllocationScheme
0001:0058055b* _xmlGetBufferAllocationScheme
0001:0058056a  _xmlSetNs
0001:0058057c  _xmlFreeNs
0001:005805d2  _xmlNewNs
0001:00580b4a  _xmlFreeNsList
0001:00580b7d  _xmlNewDtd
0001:00580c52  _xmlGetIntSubset
0001:00580c94  _xmlCreateIntSubset
0001:00580e99  _xmlNewDoc
0001:00580f6b  _xmlNodeListGetString
0001:0058110a* _xmlNodeListGetRawString
0001:0058123b  _xmlNewDocPI
0001:00581305  _xmlNewPI
0001:00581335  _xmlNewNode
0001:005813bc* _xmlNewNodeEatName
0001:0058144d  _xmlNewDocFragment
0001:005814cb  _xmlNewText
0001:00589a43  _xmlStringText
0001:0058156e  _xmlNewCharRef
0001:00581647  _xmlNewReference
0001:00581730  _xmlNewDocText
0001:00581997  _xmlNewNsPropEatName
0001:005819ca  _xmlNewNsProp
0001:005819fd  _xmlNewProp
0001:00581a26  _xmlNewTextLen
0001:00581ab3* _xmlNewDocTextLen
0001:00581ae8  _xmlNewComment
0001:00589a52  _xmlStringComment
0001:00581b7d  _xmlNewCDataBlock
0001:00581c09  _xmlNewDocComment
0001:00581c26* _xmlSetListDoc
0001:00581c57  _xmlSetTreeDoc
0001:00581cb5  _xmlGetLastChild
0001:00581cc6* _xmlChildElementCount
0001:00581d0f* _xmlFirstElementChild
0001:00581d54* _xmlLastElementChild
0001:00581d9a* _xmlPreviousElementSibling
0001:00581e1f* _xmlNextElementSibling
0001:00581ea3  _xmlUnlinkNode
0001:00582080  _xmlFreeDoc
0001:00582755  _xmlFreeDtd
0001:00582255  _xmlFreeNodeList
0001:0058252c  _xmlFreePropList
0001:00582400  _xmlFreeProp
0001:005824a8* _xmlRemoveProp
0001:00582553  _xmlFreeNode
0001:005828d4  _xmlReplaceNode
0001:005829b5* _xmlCopyNamespace
0001:005829e8  _xmlCopyNamespaceList
0001:00582a34  _xmlGetLineNo
0001:00582af7  _xmlGetNodePath
0001:005832ef  _xmlDocGetRootElement
0001:00583314  _xmlNodeSetName
0001:00583418  _xmlGetNsList
0001:005837ee  _xmlSearchNs
0001:005839af  _xmlSearchNsByHref
0001:00583d40  _xmlReconciliateNs
0001:00584087  _xmlHasProp
0001:00584140  _xmlHasNsProp
0001:0058415c  _xmlAddChild
0001:00584429  _xmlNodeAddContent
0001:005842f3  _xmlNodeAddContentLen
0001:0058445e* _xmlTextMerge
0001:005844bb  _xmlAddChildList
0001:0058465d  _xmlAddSibling
0001:00584754  _xmlDocSetRootElement
0001:005847da  _xmlAddNextSibling
0001:00584d1b  _xmlNodeSetContent
0001:005848f8  _xmlStringGetNodeList
0001:00584e4d  _xmlNewDocNodeEatName
0001:00584eef  _xmlNewDocNode
0001:00584f91  _xmlNewChild
0001:0058507b* _xmlNewDocRawNode
0001:005850fa  _xmlNewTextChild
0001:005851e4  _xmlNewDocProp
0001:0058552d* _xmlCopyProp
0001:00585541  _xmlCopyPropList
0001:00589a48  _xmlStringTextNoenc
0001:00585c4f  _xmlCopyDoc
0001:005859d4  _xmlDocCopyNode
0001:005859ee  _xmlCopyNode
0001:00585a07  _xmlCopyDtd
0001:00585d4a  _xmlCopyNodeList
0001:00585d5d  _xmlDocCopyNodeList
0001:00585d71  _xmlStringLenGetNodeList
0001:005861fa  _xmlNodeSetContentLen
0001:0058633f  _xmlAddPrevSibling
0001:00586454  _xmlGetProp
0001:0058647a  _xmlGetNoNsProp
0001:005864a2  _xmlGetNsProp
0001:005864f3  _xmlNodeGetBase
0001:00586731  _xmlNodeGetSpacePreserve
0001:005867d5  _xmlNodeGetLang
0001:00586810  _xmlUnsetProp
0001:0058684e* _xmlUnsetNsProp
0001:00586896  _xmlSetNsProp
0001:005869f3  _xmlSetProp
0001:00586aac  _xmlNodeSetBase
0001:00586bcf* _xmlNodeSetSpacePreserve
0001:00586c56* _xmlNodeSetLang
0001:00586cab  _xmlNodeIsText
0001:00586cc2  _xmlIsBlankNode
0001:00586d14  _xmlTextConcat
0001:00586dd8  _xmlBufferCreate
0001:00586e54  _xmlBufferCreateSize
0001:00586ee5  _xmlBufferCreateStatic
0001:00586f40* _xmlBufferSetAllocationScheme
0001:00586f62  _xmlBufferFree
0001:00586fb3  _xmlBufferEmpty
0001:00586ff7  _xmlBufferShrink
0001:005870cb  _xmlBufferGrow
0001:00587176* _xmlBufferDump
0001:005871bc  _xmlBufferContent
0001:005871cc  _xmlBufferLength
0001:005871dd  _xmlBufferResize
0001:00587320  _xmlBufferAdd
0001:005873d6  _xmlBufferAddHead
0001:005874d1  _xmlBufferCat
0001:00587508  _xmlNodeBufGetContent
0001:00587703  _xmlNodeGetContent
0001:0058782f  _xmlBufferCCat
0001:005878b3  _xmlBufferWriteCHAR
0001:005878ce  _xmlBufferWriteChar
0001:005878f4  _xmlBufferWriteQuotedString
0001:00587a18* _xmlGetDocCompressMode
0001:00587a2c  _xmlSetDocCompressMode
0001:00587a59  _xmlGetCompressMode
0001:00587a63* _xmlSetCompressMode
0001:00587ab3* _xmlDOMWrapNewCtxt
0001:00587afc* _xmlDOMWrapFreeCtxt
0001:00587b2b* _xmlDOMWrapRemoveNode
0001:00587cff* _xmlDOMWrapReconcileNamespaces
0001:0058822c* _xmlDOMWrapCloneNode
0001:00588c13* _xmlDOMWrapAdoptNode
0002:0001ea00  ___xmlRegisterCallbacks
Module: U:\extras\lib\xml2.lib(globals.obj)
0002:00024470+ _xmlLastError
0001:00589b00  _xmlInitGlobals
0001:00589b1d  _xmlCleanupGlobals
0001:00589b4a  _xmlInitializeGlobalState
0001:00589d0f* _xmlThrDefSetGenericErrorFunc
0001:00589d59* _xmlThrDefSetStructuredErrorFunc
0001:00589d93* _xmlRegisterNodeDefault
0001:00589db0* _xmlThrDefRegisterNodeDefault
0001:00589df1* _xmlDeregisterNodeDefault
0001:00589e0e* _xmlThrDefDeregisterNodeDefault
0001:00589e4f* _xmlThrDefParserInputBufferCreateFilenameDefault
0001:00589e91* _xmlThrDefOutputBufferCreateFilenameDefault
0001:00589ed3  ___docbDefaultSAXHandler
0001:00589ef7  ___htmlDefaultSAXHandler
0001:00589f1b  ___xmlLastError
0001:00589f41* ___oldXMLWDcompatibility
0001:00589f65  ___xmlBufferAllocScheme
0001:00589f89* _xmlThrDefBufferAllocScheme
0001:00589fc0  ___xmlDefaultBufferSize
0001:00589fe4* _xmlThrDefDefaultBufferSize
0001:0058a01b  ___xmlDefaultSAXHandler
0001:0058a041  ___xmlDefaultSAXLocator
0001:0058a063  ___xmlDoValidityCheckingDefaultValue
0001:0058a087* _xmlThrDefDoValidityCheckingDefaultValue
0001:0058a0be  ___xmlGenericError
0001:0058a0e2  ___xmlStructuredError
0001:0058a106  ___xmlGenericErrorContext
0001:0058a12a  ___xmlStructuredErrorContext
0001:0058a14e  ___xmlGetWarningsDefaultValue
0001:0058a172* _xmlThrDefGetWarningsDefaultValue
0001:0058a1a9  ___xmlIndentTreeOutput
0001:0058a1cd* _xmlThrDefIndentTreeOutput
0001:0058a204  ___xmlTreeIndentString
0001:0058a228* _xmlThrDefTreeIndentString
0001:0058a25f  ___xmlKeepBlanksDefaultValue
0001:0058a283* _xmlThrDefKeepBlanksDefaultValue
0001:0058a2ba  ___xmlLineNumbersDefaultValue
0001:0058a2de* _xmlThrDefLineNumbersDefaultValue
0001:0058a315  ___xmlLoadExtDtdDefaultValue
0001:0058a339* _xmlThrDefLoadExtDtdDefaultValue
0001:0058a370  ___xmlParserDebugEntities
0001:0058a394* _xmlThrDefParserDebugEntities
0001:0058a3cb  ___xmlParserVersion
0001:0058a3f1  ___xmlPedanticParserDefaultValue
0001:0058a415* _xmlThrDefPedanticParserDefaultValue
0001:0058a44c  ___xmlSaveNoEmptyTags
0001:0058a471* _xmlThrDefSaveNoEmptyTags
0001:0058a4a8  ___xmlSubstituteEntitiesDefaultValue
0001:0058a4cc* _xmlThrDefSubstituteEntitiesDefaultValue
0001:0058a503  ___xmlRegisterNodeDefaultValue
0001:0058a527  ___xmlDeregisterNodeDefaultValue
0001:0058a54b  ___xmlParserInputBufferCreateFilenameValue
0001:0058a571  ___xmlOutputBufferCreateFilenameValue
0002:00006ee0* _docbDefaultSAXHandler
0002:00006e70* _htmlDefaultSAXHandler
0002:00006dc8* _xmlBufferAllocScheme
0002:00006dcc* _xmlDefaultBufferSize
0002:00006df0* _xmlDefaultSAXHandler
0002:00006e60* _xmlDefaultSAXLocator
0002:00006dd8* _xmlGenericError
0002:00006dd0* _xmlGetWarningsDefaultValue
0002:00006ddc* _xmlIndentTreeOutput
0002:00006de0* _xmlTreeIndentString
0002:00006dd4* _xmlKeepBlanksDefaultValue
0002:00006dc4* _xmlParserVersion
0002:00006db0  _xmlFree
0002:00006db4  _xmlMalloc
0002:00006db8  _xmlMallocAtomic
0002:00006dbc  _xmlRealloc
0002:00006dc0  _xmlMemStrdup
0002:0001ea3c* _xmlRegisterNodeDefaultValue
0002:0001ea40* _xmlDeregisterNodeDefaultValue
0002:0001ea20* _oldXMLWDcompatibility
0002:0001ea28* _xmlDoValidityCheckingDefaultValue
0002:0001ea4c* _xmlStructuredError
0002:0001ea50* _xmlGenericErrorContext
0002:0001ea54* _xmlStructuredErrorContext
0002:0001ea34* _xmlLineNumbersDefaultValue
0002:0001ea2c* _xmlLoadExtDtdDefaultValue
0002:0001ea24* _xmlParserDebugEntities
0002:0001ea30* _xmlPedanticParserDefaultValue
0002:0001ea58* _xmlSaveNoEmptyTags
0002:0001ea38* _xmlSubstituteEntitiesDefaultValue
0002:0001ea44* _xmlParserInputBufferCreateFilenameValue
0002:0001ea48* _xmlOutputBufferCreateFilenameValue
Module: U:\extras\lib\xml2.lib(valid.obj)
0001:0058bded  _xmlNewValidCtxt
0001:0058be2a  _xmlFreeValidCtxt
0001:0058beb3  _xmlNewDocElementContent
0001:0058c045* _xmlNewElementContent
0001:0058c067* _xmlCopyDocElementContent
0001:0058c27c* _xmlCopyElementContent
0001:0058c336  _xmlFreeDocElementContent
0001:0058c49e* _xmlFreeElementContent
0001:0058c4b9* _xmlSprintfElementContent
0001:0058c4be  _xmlSnprintfElementContent
0001:0058c828* _xmlValidBuildContentModel
0001:0058d1ff  _xmlAddElementDecl
0001:0058d67b  _xmlFreeElementTable
0001:0058d696  _xmlCopyElementTable
0001:0058d705  _xmlDumpElementDecl
0001:0058d899* _xmlDumpElementTable
0001:0058d8c5  _xmlCreateEnumeration
0001:0058d916  _xmlFreeEnumeration
0001:0058da97* _xmlCopyEnumeration
0001:0058dca1  _xmlAddAttributeDecl
0001:0058e26c  _xmlFreeAttributeTable
0001:0058e287  _xmlCopyAttributeTable
0001:0058e34a  _xmlDumpAttributeDecl
0001:0058e5c2* _xmlDumpAttributeTable
0001:0058e644  _xmlAddNotationDecl
0001:0058e77e  _xmlFreeNotationTable
0001:0058e799  _xmlCopyNotationTable
0001:0058e7d6* _xmlDumpNotationDecl
0001:0058e894  _xmlDumpNotationTable
0001:0058e8f9  _xmlAddID
0001:0058ea7a  _xmlFreeIDTable
0001:0058ea95  _xmlRemoveID
0001:0058eb39  _xmlGetID
0001:0058ef3d  _xmlAddRef
0001:0058f100  _xmlFreeRefTable
0001:0058f11b* _xmlRemoveRef
0001:0058f1ed* _xmlGetRefs
0001:0058f215* _xmlGetDtdElementDesc
0001:0058f29b  _xmlGetDtdQElementDesc
0001:0058f402  _xmlGetDtdAttrDesc
0001:0058f4a9  _xmlIsRef
0001:0058f561  _xmlIsID
0001:0058f813  _xmlGetDtdQAttrDesc
0001:0058f84f* _xmlGetDtdNotationDesc
0001:0058fe8e  _xmlValidateNotationUse
0001:0058ff7b  _xmlIsMixedElement
0001:0058ffe3* _xmlValidateNameValue
0001:0058fff4* _xmlValidateNamesValue
0001:00590005* _xmlValidateNmtokenValue
0001:00590016* _xmlValidateNmtokensValue
0001:00590027  _xmlValidateNotationDecl
0001:00590031* _xmlValidateAttributeValue
0001:0059009e  _xmlValidCtxtNormalizeAttributeValue
0001:005902c4  _xmlValidNormalizeAttributeValue
0001:005905bf  _xmlValidateAttributeDecl
0001:00590910  _xmlValidateElementDecl
0001:00590e03  _xmlValidateOneAttribute
0001:00591752  _xmlValidateOneNamespace
0001:0059203c  _xmlValidatePushElement
0001:005924e2  _xmlValidatePushCData
0001:00592606  _xmlValidatePopElement
0001:005929ad  _xmlValidateOneElement
0001:0059346a  _xmlValidateRoot
0001:005935dc  _xmlValidateElement
0001:00593773  _xmlValidateDocumentFinal
0001:005937d2  _xmlValidateDtd
0001:00593880  _xmlValidateDtdFinal
0001:005939b9  _xmlValidateDocument
0001:00593b51* _xmlValidGetPotentialChildren
0001:00593c73* _xmlValidGetValidElements
Module: U:\extras\lib\xml2.lib(uri.obj)
0001:00594358  _xmlCreateURI
0001:005943ce  _xmlSaveUri
0001:005951c5* _xmlPrintURI
0001:00595204  _xmlFreeURI
0001:005952ba* _xmlNormalizeURIPath
0001:00595531  _xmlURIUnescapeString
0001:0059664e  _xmlParseURIReference
0001:00596660  _xmlParseURIRaw
0001:005966ab  _xmlParseURI
0001:00596708  _xmlURIEscapeStr
0001:0059691f  _xmlURIEscape
0001:00596c9d  _xmlBuildURI
0001:00597170  _xmlBuildRelativeURI
0001:00597584  _xmlCanonicPath
0001:0059764a  _xmlPathToURI
Module: U:\extras\lib\xml2.lib(xmlstring.obj)
0001:005976c0  _xmlStrndup
0001:0059772c  _xmlStrdup
0001:0059775a  _xmlCharStrndup
0001:005977d6  _xmlCharStrdup
0001:00597804  _xmlStrcmp
0001:00597856  _xmlStrEqual
0001:00597892  _xmlStrQEqual
0001:005978ff  _xmlStrncmp
0001:00597947  _xmlStrcasecmp
0001:005979a7  _xmlStrncasecmp
0001:00597a12  _xmlStrchr
0001:00597a34  _xmlStrstr
0001:00597a9b  _xmlStrcasestr
0001:00597b13* _xmlStrsub
0001:00597b6a  _xmlStrlen
0001:00597b86  _xmlStrncat
0001:00597c35  _xmlStrncatNew
0001:00597d2f  _xmlStrcat
0001:00597d75  _xmlStrPrintf
0001:00597dbd* _xmlStrVPrintf
0001:00597e05* _xmlUTF8Size
0001:00597e48* _xmlUTF8Charcmp
0001:00597e87  _xmlUTF8Strlen
0001:00597f2d  _xmlGetUTF8Char
0001:00598071  _xmlCheckUTF8
0001:0059814b  _xmlUTF8Strsize
0001:005981ab  _xmlUTF8Strndup
0001:0059823f  _xmlUTF8Strpos
0001:00598297  _xmlUTF8Strloc
0001:00598338  _xmlUTF8Strsub
Module: U:\extras\lib\xml2.lib(xmlIO.obj)
0001:005984d7* _xmlFileMatch
0001:0059861f* _xmlIOFTPMatch
0001:00598652* _xmlIOHTTPMatch
0001:005987bc* _xmlIOHTTPClose
0001:00598804* _xmlIOFTPClose
0001:00598810* _xmlIOFTPRead
0001:0059883d* _xmlIOFTPOpen
0001:00598849* _xmlIOHTTPRead
0001:00598876* _xmlIOHTTPOpen
0001:00598891  ___xmlIOErr
0001:00599519* _xmlFileClose
0001:00599598* _xmlFileRead
0001:005995e9  ___xmlLoaderErr
0001:005996f9* _xmlNormalizeWindowsPath
0001:00599705  _xmlCleanupInputCallbacks
0001:0059975e* _xmlPopInputCallbacks
0001:005997b0  _xmlCleanupOutputCallbacks
0001:0059980a* _xmlCheckFilename
0001:00599ba9* _xmlFileOpen
0001:00599bfa* _xmlRegisterInputCallbacks
0001:00599c4c* _xmlRegisterOutputCallbacks
0001:00599c9e  _xmlRegisterDefaultInputCallbacks
0001:00599d4c  _xmlRegisterDefaultOutputCallbacks
0001:00599db1* _xmlRegisterHTTPPostCallbacks
0001:00599e02  _xmlAllocParserInputBuffer
0001:00599ec2  ___xmlParserInputBufferCreateFilename
0001:00599fdd  _xmlAllocOutputBuffer
0001:0059a09f  _xmlAllocOutputBufferInternal
0001:0059a15e  _xmlFreeParserInputBuffer
0001:0059a1ca  _xmlParserInputBufferCreateFilename
0001:0059a200* _xmlParserInputBufferCreateFile
0001:0059a246  _xmlOutputBufferCreateFile
0001:0059a28c  _xmlParserInputBufferCreateFd
0001:0059a2c1  _xmlParserInputBufferCreateMem
0001:0059a329  _xmlParserInputBufferCreateStatic
0001:0059a3f5  _xmlOutputBufferCreateFd
0001:0059a42a  _xmlParserInputBufferCreateIO
0001:0059a45d  _xmlOutputBufferCreateIO
0001:0059a490  _xmlOutputBufferCreateBuffer
0001:0059a4c0  _xmlParserInputBufferCreateFilenameDefault
0001:0059a4eb  _xmlOutputBufferCreateFilenameDefault
0001:0059b5dc  ___xmlOutputBufferCreateFilename
0001:0059a516  _xmlParserInputBufferPush
0001:0059a5fe  _xmlParserInputBufferGrow
0001:0059a78a  _xmlParserInputBufferRead
0001:0059a7c7  _xmlOutputBufferWrite
0001:0059abf3  _xmlOutputBufferWriteEscape
0001:0059aec9  _xmlOutputBufferWriteString
0001:0059af17  _xmlOutputBufferFlush
0001:0059b010  _xmlOutputBufferClose
0001:0059b52c* _xmlIOHTTPOpenW
0001:0059b89c  _xmlOutputBufferCreateFilename
0001:0059b902  _xmlParserGetDirectory
0001:0059ba17  _xmlCheckHTTPInput
0001:0059bba6* _xmlSetExternalEntityLoader
0001:0059bbb3* _xmlGetExternalEntityLoader
0001:0059bbd6  _xmlLoadExternalEntity
0001:0059bc52* _xmlNoNetExternalEntityLoader
Module: U:\extras\lib\xml2.lib(error.obj)
0001:0059ccc0  _xmlGenericErrorDefaultFunc
0001:0059cd04  _initGenericErrorDefaultFunc
0001:0059cd32  _xmlSetGenericErrorFunc
0001:0059cd68  _xmlSetStructuredErrorFunc
0001:0059cd84* _xmlParserPrintFileInfo
0001:0059cdf6* _xmlParserPrintFileContext
0001:0059ce2b  _xmlParserValidityWarning
0001:0059cfec  _xmlParserValidityError
0001:0059d1dd  _xmlParserWarning
0001:0059d3c9  _xmlParserError
0001:0059d5a9  _xmlGetLastError
0001:0059d5c5  _xmlResetError
0001:0059d63d  _xmlResetLastError
0001:0059d661* _xmlCtxtGetLastError
0001:0059d681* _xmlCtxtResetLastError
0001:0059d6af  _xmlCopyError
0001:0059d7e0  ___xmlRaiseError
0001:0059de3d  ___xmlSimpleError
Module: U:\extras\lib\xml2.lib(parser.obj)
0001:005a05f8* _xmlHasFeature
0001:005a0611  _xmlCheckLanguageID
0001:005a08c2  _inputPush
0001:005a0a6e  _inputPop
0001:005a0af3  _nodePush
0001:005a0b96  _nodePop
0001:005a0bdd* _namePush
0001:005a0c83* _namePop
0001:005a0cee  _xmlPopInput
0001:005a0e3f  _xmlPushInput
0001:005a0f4c  _xmlSplitQName
0001:005a1428* _xmlParsePubidLiteral
0001:005a16ae* _xmlParseVersionNum
0001:005a17fb* _xmlParseEncName
0001:005a1a14* _xmlParseEncodingDecl
0001:005a7d0c* _xmlSkipBlankChars
0001:005a1f8b  _xmlParserHandlePEReference
0001:005a1cca* _xmlParseTextDecl
0001:005aadbd* _xmlParseVersionInfo
0001:005a45e3* _xmlParseName
0001:005a2546* _xmlParseCDSect
0001:005a2b0f* _xmlParseComment
0001:005a3b45* _xmlParseCharData
0001:005a3f2b* _xmlParseSystemLiteral
0001:005a42c3* _xmlParseNmtoken
0001:005a51fc* _xmlParseEntityRef
0001:005a5524* _xmlParsePITarget
0001:005a57d9  _xmlStringLenDecodeEntities
0001:005a66e3  _xmlStringDecodeEntities
0001:005a679c* _xmlParseEntityValue
0001:005a6c13* _xmlParseCharRef
0001:005a7ce3* _xmlParseAttValue
0001:005a93fd* _xmlParseAttribute
0001:005a95ac* _xmlParseStartTag
0001:005aa354* _xmlParseElementChildrenContentDecl
0001:005aa3a9* _xmlParseEnumerationType
0001:005aa5ea* _xmlParseNotationType
0001:005aadac* _xmlParseEndTag
0001:005aaf49* _xmlParseElementMixedContentDecl
0001:005ab3be* _xmlParseElementContentDecl
0001:005ab5d7* _xmlParseElementDecl
0001:005ab979* _xmlParseEnumeratedType
0001:005aba73* _xmlParseAttributeType
0001:005abe8b* _xmlParseDefaultDecl
0001:005ac222* _xmlParseAttributeListDecl
0001:005acaa4* _xmlParsePI
0001:005ad22c* _xmlParseExternalID
0001:005ad53d* _xmlParseDocTypeDecl
0001:005ad846* _xmlParseEntityDecl
0001:005ae18c* _xmlParseNotationDecl
0001:005ae43f* _xmlParsePEReference
0001:005aedd1* _xmlParseMarkupDecl
0001:005af017  _xmlParseExternalSubset
0001:005af2e9* _xmlParseSDDecl
0001:005af63c* _xmlParseXMLDecl
0001:005af9e3* _xmlParseMisc
0001:005afa84  _xmlCreatePushParserCtxt
0001:005afd43  _xmlStopParser
0001:005afd78* _xmlCreateIOParserCtxt
0001:005afea2* _xmlIOParseDTD
0001:005b0100* _xmlSAXParseDTD
0001:005b0379  _xmlParseDTD
0001:005b039b* _xmlCreateEntityParserCtxt
0001:005b03d7* _xmlCreateURLParserCtxt
0001:005b048e  _xmlCreateFileParserCtxt
0001:005b04cf* _xmlSetupParserForBuffer
0001:005b0567  _xmlCreateMemoryParserCtxt
0001:005b3212* _xmlParseContent
0001:005b0afa* _xmlParseReference
0001:005b2e48  _xmlParseChunk
0001:005b41ad* _xmlParseElement
0001:005b38ca* _xmlParseExternalEntity
0001:005b3936  _xmlParseCtxtExternalEntity
0001:005b3e60* _xmlParseExtParsedEnt
0001:005b40bb* _xmlSAXParseEntity
0001:005b413a* _xmlParseEntity
0001:005b4605* _xmlParseBalancedChunkMemoryRecover
0001:005b49db  _xmlParseBalancedChunkMemory
0001:005b4a19  _xmlParseInNodeContext
0001:005b4e75* _xmlCreateDocParserCtxt
0001:005b4e9f* _xmlSetEntityReferenceFunc
0001:005b4eac  _xmlInitParser
0001:005b4f67  _xmlParseDocument
0001:005b5496* _xmlSAXParseDoc
0001:005b5527* _xmlParseDoc
0001:005b554a* _xmlRecoverDoc
0001:005b556d* _xmlSAXUserParseFile
0001:005b5617* _xmlSAXUserParseMemory
0001:005b56cd* _xmlSAXParseMemoryWithData
0001:005b5773* _xmlSAXParseMemory
0001:005b57a3* _xmlRecoverMemory
0001:005b57cd* _xmlParseMemory
0001:005b57f7* _xmlSAXParseFileWithData
0001:005b58cf* _xmlSAXParseFile
0001:005b58f8* _xmlRecoverFile
0001:005b591b* _xmlParseFile
0001:005b593e  _xmlCleanupParser
0001:005b5996  _xmlCtxtReset
0001:005b5cc3* _xmlCtxtResetPush
0001:005b5f38  _xmlCtxtUseOptions
0001:005b5f4c* _xmlReadDoc
0001:005b5f95  _xmlReadFile
0001:005b5fd8  _xmlReadMemory
0001:005b6024* _xmlReadFd
0001:005b60e6* _xmlReadIO
0001:005b61aa* _xmlCtxtReadDoc
0001:005b6220  _xmlCtxtReadFile
0001:005b6295  _xmlCtxtReadMemory
0001:005b634d* _xmlCtxtReadFd
0001:005b63ff* _xmlCtxtReadIO
0002:00006f80* _xmlParserMaxDepth
Module: U:\extras\lib\xml2.lib(relaxng.obj)
0001:005c5e0c  _xmlRelaxNGFree
0001:005c5efd* _xmlRelaxParserSetFlag
0001:005c5f68* _xmlRelaxNGInitTypes
0001:005c6024  _xmlRelaxNGCleanupTypes
0001:005c606d  _xmlRelaxNGNewParserCtxt
0001:005c60d3  _xmlRelaxNGNewMemParserCtxt
0001:005c6148* _xmlRelaxNGNewDocParserCtxt
0001:005c61c6  _xmlRelaxNGFreeParserCtxt
0001:005c633b  _xmlRelaxNGParse
0001:005c65e8  _xmlRelaxNGSetParserErrors
0001:005c660c* _xmlRelaxNGGetParserErrors
0001:005c6646* _xmlRelaxNGSetParserStructuredErrors
0001:005c6786* _xmlRelaxNGDump
0001:005c6a01* _xmlRelaxNGDumpTree
0001:005c6a6c  _xmlRelaxNGValidatePushElement
0001:005c6ba3  _xmlRelaxNGValidatePushCData
0001:005c6c46  _xmlRelaxNGValidatePopElement
0001:005c6cdc  _xmlRelaxNGValidateFullElement
0001:005c6d72  _xmlRelaxNGNewValidCtxt
0001:005c6e0c  _xmlRelaxNGFreeValidCtxt
0001:005c6ee9  _xmlRelaxNGSetValidErrors
0001:005c6f0d  _xmlRelaxNGSetValidStructuredErrors
0001:005c6f32* _xmlRelaxNGGetValidErrors
0001:005c6f6c  _xmlRelaxNGValidateDoc
Module: U:\extras\lib\libz.lib(zutil.obj)
0001:005c7298  _zlibVersion
0001:005c72a4* _zlibCompileFlags
0001:005c72b0  _zError
0001:005c7370  _z_errmsg
0001:005c72c4  _zcfree
0001:005c72d8  _zcalloc
Module: U:\extras\lib\libz.lib(compress.obj)
0001:005c73a0* _compressBound
0001:005c73c4  _compress2
0001:005c7478  _compress
Module: U:\extras\lib\libz.lib(uncompr.obj)
0001:005c7538  _uncompress
Module: U:\extras\lib\libz.lib(deflate.obj)
0001:005c75f0* _deflateSetHeader
0001:005c761c* _deflatePrime
0001:005c7654* _deflateTune
0001:005c7694* _deflateBound
0001:005c77c4  _deflateEnd
0001:005c7894* _deflateCopy
0001:005c7aa0* _deflateSetDictionary
0001:005c7e3c  _deflateReset
0001:005c7fb4  _deflateInit2_
0001:005c8214  _deflateInit_
0001:005c932c  _deflate
0001:005ca35c  _deflateParams
0001:005ca450* _deflate_copyright
Module: U:\extras\lib\libz.lib(inflate.obj)
0001:005ca520  _inflateReset
0001:005ca5cc* _inflatePrime
0001:005ca630  _inflateEnd
0001:005ca68c* _inflateGetHeader
0001:005ca6bc* _inflateSync
0001:005ca868* _inflateSyncPoint
0001:005ca89c* _inflateUndermine
0001:005ca8c8* _inflateMark
0001:005ca914* _inflateCopy
0001:005cabc4* _inflateSetDictionary
0001:005cae80  _inflate
0001:005ccd4c* _inflateReset2
0001:005cce7c  _inflateInit2_
0001:005ccf44  _inflateInit_
Module: U:\extras\lib\libz.lib(crc32.obj)
0001:005cd8c0* _get_crc_table
0001:005cd8cc  _crc32
0001:005cde10* _crc32_combine
0001:005cde1c* _crc32_combine64
Module: U:\extras\lib\libz.lib(gzread.obj)
0001:005cfe30  _gzclose_r
0001:005d0584  _gzdirect
0001:005d0bd0* _gzgets
0001:005d0d0c* _gzungetc
0001:005d0e2c  _gzread
0001:005d0fb0* _gzgetc
Module: U:\extras\lib\libz.lib(gzlib.obj)
0001:005d1020* _gzbuffer
0001:005d105c* _gztell64
0001:005d10b0* _gztell
0001:005d1104  _gzeof
0001:005d1138* _gzerror
0001:005d1188  _gz_error
0001:005d1254* _gzoffset64
0001:005d168c  _gzdopen
0001:005d16f4* _gzopen64
0001:005d1718  _gzopen
0001:005d173c* _gzrewind
0001:005d17e4* _gzseek64
0001:005d19b0  _gzseek
0001:005d19bc* _gzclearerr
0001:005d19f0* _gzoffset
Module: U:\extras\lib\libz.lib(gzwrite.obj)
0001:005d1eb4  _gzclose_w
0001:005d1f84  _gzflush
0001:005d2000* _gzsetparams
0001:005d20b4* _gzprintf
0001:005d21d8  _gzwrite
0001:005d2378* _gzputs
0001:005d23c0* _gzputc
Module: U:\extras\lib\libz.lib(gzclose.obj)
0001:005d2470  _gzclose
Module: U:\extras\lib\xml2.lib(xpath.obj)
0001:005d2ab7* _xmlXPathNextSelf
0001:005d2ad8* _xmlXPathNextChild
0001:005d2b81* _xmlXPathNextDescendant
0001:005d2c0b* _xmlXPathNextDescendantOrSelf
0001:005d2c4e* _xmlXPathNextFollowingSibling
0001:005d2c92* _xmlXPathNextPrecedingSibling
0001:005d2ce3* _xmlXPathNextFollowing
0001:005d2df7* _xmlXPathNextAttribute
0001:005d3456* _xmlXPathNodeSetAddUnique
0001:005d372d* _xmlXPathNextAncestor
0001:005d3920* _xmlXPathNextAncestorOrSelf
0001:005d3959* _xmlXPathNextParent
0001:005d4607* _xmlXPathNextNamespace
0001:005d480c  _xmlXPathInit
0001:005d4913  _xmlXPathIsNaN
0001:005d497c* _xmlXPathIsInf
0001:005d49b8  _xmlXPathErr
0001:005d529d* _xmlXPatherror
0001:005d54ef  _xmlXPathDebugDumpObject
0001:005d6b17* _xmlXPathDebugDumpCompExpr
0001:005d6bcf* _xmlXPathContextSetCache
0001:005d6cb5  _valuePop
0001:005d6d0e  _valuePush
0001:005d6d93* _xmlXPathOrderDocElems
0001:005d6dec  _xmlXPathCmpNodes
0001:005d7078* _xmlXPathNodeSetSort
0001:005d715e* _xmlXPathNodeSetFreeNs
0001:005d7281* _xmlXPathNodeSetCreate
0001:005d771f  _xmlXPathNodeSetContains
0001:005d77c2* _xmlXPathNodeSetAddNs
0001:005d790f* _xmlXPathNodeSetAdd
0001:005d7af5* _xmlXPathNodeSetMerge
0001:005d7c9b* _xmlXPathNodeSetDel
0001:005d7d18* _xmlXPathNodeSetRemove
0001:005d7d74* _xmlXPathFreeNodeSet
0001:005d7de5  _xmlXPathFreeObject
0001:005d7e78* _xmlXPathFreeCompExpr
0001:005d820b* _xmlXPathPopExternal
0001:005d82a0* _xmlXPathPopNodeSet
0001:005d8322  _xmlXPathNewNodeSet
0001:005d87f9* _xmlXPathNewValueTree
0001:005d885a* _xmlXPathNewNodeSetList
0001:005d88f2* _xmlXPathWrapNodeSet
0001:005d898a* _xmlXPathFreeNodeSetList
0001:005d89a1* _xmlXPathDifference
0001:005d8a5c* _xmlXPathIntersection
0001:005d8b14* _xmlXPathHasSameNodes
0001:005d8b9c* _xmlXPathNodeLeadingSorted
0001:005d8c48* _xmlXPathNodeLeading
0001:005d8c6f* _xmlXPathLeadingSorted
0001:005d8cad* _xmlXPathLeading
0001:005d8d26* _xmlXPathNodeTrailingSorted
0001:005d8ddf* _xmlXPathNodeTrailing
0001:005d8e06* _xmlXPathTrailingSorted
0001:005d8e42* _xmlXPathTrailing
0001:005d8ebb  _xmlXPathRegisterFuncNS
0001:005d8f41  _xmlXPathRegisterFunc
0001:005d8f6a* _xmlXPathRegisterFuncLookup
0001:005d8f82* _xmlXPathFunctionLookupNS
0001:005d8fe1* _xmlXPathFunctionLookup
0001:005d9036* _xmlXPathRegisteredFuncsCleanup
0001:005d9064* _xmlXPathRegisterVariableNS
0001:005d90f8* _xmlXPathRegisterVariable
0001:005d9121* _xmlXPathRegisterVariableLookup
0001:005d9139* _xmlXPathRegisteredVariablesCleanup
0001:005d9167  _xmlXPathRegisterNs
0001:005d9229* _xmlXPathNsLookup
0001:005d92d6* _xmlXPathRegisteredNsCleanup
0001:005d931c* _xmlXPathNewFloat
0001:005d93d7* _xmlXPathCountFunction
0001:005d94d4* _xmlXPathPositionFunction
0001:005d953c* _xmlXPathLastFunction
0001:005d95bd  _xmlXPathNewBoolean
0001:005d967e* _xmlXPathFalseFunction
0001:005d96c4* _xmlXPathTrueFunction
0001:005d9725  _xmlXPathNewString
0001:005d9829* _xmlXPathWrapString
0001:005d98e9* _xmlXPathNewCString
0001:005d99d5* _xmlXPathLocalNameFunction
0001:005d9c77* _xmlXPathNamespaceURIFunction
0001:005d9d5c* _xmlXPathWrapCString
0001:005d9d7e* _xmlXPathWrapExternal
0001:005d9e05  _xmlXPathObjectCopy
0001:005d9fdf* _xmlXPathVariableLookupNS
0001:005da04f* _xmlXPathVariableLookup
0001:005da09f* _xmlXPathCastBooleanToString
0001:005da0eb* _xmlXPathCastNumberToString
0001:005da4ce* _xmlXPathCastNodeToString
0001:005da4f2* _xmlXPathDistinctSorted
0001:005da5f2* _xmlXPathDistinct
0001:005da62a* _xmlXPathCastNodeSetToString
0001:005da797* _xmlXPathStringFunction
0001:005da822* _xmlXPathLangFunction
0001:005da97c* _xmlXPathTranslateFunction
0001:005dab94* _xmlXPathNormalizeFunction
0001:005dad28* _xmlXPathSubstringAfterFunction
0001:005dae5b* _xmlXPathSubstringBeforeFunction
0001:005daf5e* _xmlXPathStartsWithFunction
0001:005db0a1* _xmlXPathContainsFunction
0001:005db1d5* _xmlXPathConcatFunction
0001:005db2e4* _xmlXPathStringLengthFunction
0001:005db41e  _xmlXPathIdFunction
0001:005db570  _xmlXPathCastToString
0001:005db63d* _xmlXPathPopString
0001:005db6a2* _xmlXPathConvertString
0001:005db78a* _xmlXPathCastBooleanToNumber
0001:005db79c* _xmlXPathCastNumberToBoolean
0001:005db7e3* _xmlXPathCastStringToBoolean
0001:005db804* _xmlXPathCastNodeSetToBoolean
0001:005db81a* _xmlXPathCastToBoolean
0001:005db8dc* _xmlXPathBooleanFunction
0001:005db963* _xmlXPathNotFunction
0001:005db9d8* _xmlXPathPopBoolean
0001:005dbcc2* _xmlXPathConvertBoolean
0001:005dbd0d  _xmlXPathFreeContext
0001:005dbd7e  _xmlXPathNewParserContext
0001:005dbe0f  _xmlXPathFreeParserContext
0001:005dbe60* _xmlXPathNextPreceding
0001:005dbefb  _xmlXPathRoot
0001:005dbf2c  _xmlXPathParseNCName
0001:005dc03c  _xmlXPathParseName
0001:005dc0db* _xmlXPathStringEvalNumber
0001:005dc310* _xmlXPathCastStringToNumber
0001:005dc31c* _xmlXPathCastNodeSetToNumber
0001:005dc35d* _xmlXPathCastToNumber
0001:005dc41b* _xmlXPathConvertNumber
0001:005dc462* _xmlXPathPopNumber
0001:005dc4c7* _xmlXPathNumberFunction
0001:005dc5b7* _xmlXPathRoundFunction
0001:005dc751* _xmlXPathCeilingFunction
0001:005dc89b* _xmlXPathFloorFunction
0001:005dc9a1* _xmlXPathSubstringFunction
0001:005dcc80* _xmlXPathValueFlipSign
0001:005dd26e* _xmlXPathNotEqualValues
0001:005dd43a* _xmlXPathEqualValues
0001:005dd602* _xmlXPathModValues
0001:005dd6e1* _xmlXPathDivValues
0001:005dd86b* _xmlXPathMultValues
0001:005dd8ff* _xmlXPathSubValues
0001:005dd993* _xmlXPathAddValues
0001:005dda27* _xmlXPathCastNodeToNumber
0001:005dda6c* _xmlXPathSumFunction
0001:005dddc4* _xmlXPathCompareValues
0001:005de427* _xmlXPathIsNodeType
0001:005e0d41* _xmlXPathEvalPredicate
0001:005e0e28  _xmlXPathEvaluatePredicateResult
0001:005e4e9f* _xmlXPathCtxtCompile
0001:005e4f72* _xmlXPathCompile
0001:005e4f8d* _xmlXPathCompiledEval
0001:005e4fb4* _xmlXPathCompiledEvalToBoolean
0001:005e4fcf  _xmlXPathEvalExpr
0001:005e50db  _xmlXPathEval
0001:005e52d9  _xmlXPathEvalExpression
0001:005e5552* _xmlXPathRegisterAllFunctions
0001:005e581c  _xmlXPathNewContext
0002:00006f90  _xmlXPathPINF
0002:00006f98  _xmlXPathNINF
0002:0001edc0  _xmlXPathNAN
Module: U:\extras\lib\xml2.lib(encoding.obj)
0001:005e5e93* _isolat1ToUTF8
0001:005e5f8f* _UTF8Toisolat1
0001:005e6cc3  _xmlDetectCharEncoding
0001:005e6e54* _xmlCleanupEncodingAliases
0001:005e6ee3* _xmlGetEncodingAlias
0001:005e6f95* _xmlAddEncodingAlias
0001:005e7179* _xmlDelEncodingAlias
0001:005e7338  _xmlParseCharEncoding
0001:005e7681  _xmlGetCharEncodingName
0001:005e769a  _xmlCleanupCharEncodingHandlers
0001:005e77b1* _xmlRegisterCharEncodingHandler
0001:005e79ed  _xmlInitCharEncodingHandlers
0001:005e7879* _xmlNewCharEncodingHandler
0001:005e7b88  _xmlFindCharEncodingHandler
0001:005e7e57  _xmlGetCharEncodingHandler
0001:005e8095  _xmlCharEncFirstLineInt
0001:005e81f3* _xmlCharEncFirstLine
0001:005e826e  _xmlCharEncInFunc
0001:005e845a  _xmlCharEncOutFunc
0001:005e870a  _xmlCharEncCloseFunc
0001:005e879b  _xmlByteConsumed
Module: U:\extras\lib\xml2.lib(parserInternals.obj)
0001:005e8fe0* _xmlCheckVersion
0001:005e90d9  _xmlErrMemory
0001:005e922d  ___xmlErrEncoding
0001:005e9380* _xmlIsLetter
0001:005e9421* _xmlParserInputRead
0001:005e94ac  _xmlParserInputGrow
0001:005e952e  _xmlParserInputShrink
0001:005e967a  _xmlNextChar
0001:005e9a6b  _xmlCurrentChar
0001:005e9e3a  _xmlStringCurrentChar
0001:005ea0b4  _xmlCopyCharMultiByte
0001:005ea15d  _xmlCopyChar
0001:005ea218  _xmlSwitchEncoding
0001:005ea550  _xmlSwitchInputEncoding
0001:005ea56c  _xmlSwitchToEncoding
0001:005ea583  _xmlFreeInputStream
0001:005ea62e  _xmlNewInputStream
0001:005ea6ab  _xmlNewIOInputStream
0001:005ea814  _xmlNewEntityInputStream
0001:005ea99f  _xmlNewStringInputStream
0001:005eaaa1  _xmlNewInputFromFile
0001:005eac3e* _xmlInitParserCtxt
0001:005eb0fd  _xmlFreeParserCtxt
0001:005eb37c  _xmlNewParserCtxt
0001:005eb3d9  _xmlClearParserCtxt
0001:005eb41f  _xmlInitNodeInfoSeq
0001:005eb43f* _xmlClearNodeInfoSeq
0001:005eb477* _xmlParserFindNodeInfoIndex
0001:005eb506* _xmlParserFindNodeInfo
0001:005eb56f  _xmlParserAddNodeInfo
0001:005eb6f3* _xmlPedanticParserDefault
0001:005eb713* _xmlLineNumbersDefault
0001:005eb733* _xmlSubstituteEntitiesDefault
0001:005eb753* _xmlKeepBlanksDefault
Module: U:\extras\lib\xml2.lib(xmlsave.obj)
0001:005ec188* _xmlIsXHTML
0001:005ec253  _xmlNsListDumpOutput
0001:005ec277* _xmlSaveToFd
0001:005ec2bb* _xmlSaveToFilename
0001:005ec307* _xmlSaveToBuffer
0001:005ec37d* _xmlSaveToIO
0001:005ec3cf* _xmlSaveFlush
0001:005ec3f3* _xmlSaveClose
0001:005ec421* _xmlSaveSetEscape
0001:005ec43a* _xmlSaveSetAttrEscape
0001:005ec486  _xmlAttrSerializeTxtContent
0001:005eeaae* _xmlSaveTree
0001:005eead2* _xmlSaveDoc
0001:005eeaf7  _xmlNodeDumpOutput
0001:005eebc4  _xmlElemDump
0001:005eec68  _xmlNodeDump
0001:005eed42* _xmlDocDumpFormatMemoryEnc
0001:005eeecc  _xmlDocDumpMemory
0001:005eeefd  _xmlDocDumpFormatMemory
0001:005eef2d  _xmlDocDumpMemoryEnc
0001:005eef5d* _xmlDocFormatDump
0001:005ef051  _xmlDocDump
0001:005ef073* _xmlSaveFileTo
0001:005ef0f1  _xmlSaveFormatFileTo
0001:005ef188  _xmlSaveFormatFileEnc
0001:005ef27c* _xmlSaveFileEnc
0001:005ef2a5* _xmlSaveFormatFile
0001:005ef2ce  _xmlSaveFile
Module: U:\extras\lib\xml2.lib(xinclude.obj)
0001:005f07dd  _xmlXIncludeNewContext
0001:005f0829  _xmlXIncludeFreeContext
0001:005f263b  _xmlXIncludeSetFlags
0001:005f2654* _xmlXIncludeProcessTreeFlagsData
0001:005f26cd* _xmlXIncludeProcessFlagsData
0001:005f270e  _xmlXIncludeProcessFlags
0001:005f2730* _xmlXIncludeProcess
0001:005f274b* _xmlXIncludeProcessTreeFlags
0001:005f27bf* _xmlXIncludeProcessTree
0001:005f27da  _xmlXIncludeProcessNode
Module: U:\extras\lib\xml2.lib(xmlschemas.obj)
0001:00602951  _xmlSchemaNewFacet
0001:0060297b  _xmlSchemaFreeWildcard
0001:006029da  _xmlSchemaFreeFacet
0001:00609516  _xmlSchemaFreeType
0001:0060987a  _xmlSchemaFree
0001:0060a995* _xmlSchemaDump
0001:0060aac9  _xmlSchemaNewParserCtxt
0001:0060ab16  _xmlSchemaNewMemParserCtxt
0001:0060ab54* _xmlSchemaNewDocParserCtxt
0001:0060ab8b* _xmlSchemaGetParserErrors
0001:0060abe4  _xmlSchemaNewValidCtxt
0001:0060ac43  _xmlSchemaFreeValidCtxt
0001:0060ae62  _xmlSchemaFreeParserCtxt
0001:0060b11e  _xmlSchemaCheckFacet
0001:0060b580  _xmlSchemaIsValid
0001:0060b59a  _xmlSchemaSetValidErrors
0001:0060b5d1  _xmlSchemaSetParserErrors
0001:0060b608  _xmlSchemaSetValidStructuredErrors
0001:00612fe4* _xmlSchemaSetParserStructuredErrors
0001:00617f4b  _xmlSchemaParse
0001:00618137* _xmlSchemaGetValidErrors
0001:00618172* _xmlSchemaSetValidOptions
0001:006181ac* _xmlSchemaValidCtxtGetOptions
0001:006181c0* _xmlSchemaValidateOneElement
0001:006181f9  _xmlSchemaValidateDoc
0001:0061826f  _xmlSchemaSAXPlug
0001:0061850e  _xmlSchemaSAXUnplug
0001:00618589* _xmlSchemaValidateStream
0001:006186bd* _xmlSchemaValidateFile
0001:0061871e* _xmlSchemaValidCtxtGetParserCtxt
Module: U:\extras\lib\xml2.lib(HTMLparser.obj)
0001:0061b618  _htmlInitAutoClose
0001:0061bbaf  _htmlTagLookup
0001:0061bfb4* _htmlAutoCloseTag
0001:0061c030* _htmlIsAutoClosed
0001:0061c07e* _htmlIsScriptAttribute
0001:0061c0cb* _htmlEntityLookup
0001:0061c11f* _htmlEntityValueLookup
0001:0061c165  _UTF8ToHtml
0001:0061c3e4* _htmlEncodeEntities
0001:0061c677  _htmlNewDocNoDtD
0001:0061c75e* _htmlNewDoc
0001:0061c7d3* _htmlParseEntityRef
0001:0061c978* _htmlParseCharRef
0001:0061e1d1* _htmlParseElement
0001:0061e856  ___htmlParseContent
0001:0061e8a1  _htmlParseDocument
0001:0061ebf0  _htmlFreeParserCtxt
0001:0061ec3f* _htmlNewParserCtxt
0001:0061eebe  _htmlCreateMemoryParserCtxt
0001:0061f222* _htmlParseChunk
0001:006204be* _htmlCreatePushParserCtxt
0001:006206b4* _htmlSAXParseDoc
0001:0062073a* _htmlParseDoc
0001:00620773  _htmlCreateFileParserCtxt
0001:00620882* _htmlSAXParseFile
0001:006208f2  _htmlParseFile
0001:0062091c* _htmlHandleOmittedElem
0001:0062092f* _htmlElementAllowedHere
0001:00620984* _htmlElementStatusHere
0001:006209cf* _htmlAttrAllowed
0001:00620a90* _htmlNodeStatus
0001:00620b55* _htmlCtxtReset
0001:00620e55* _htmlCtxtUseOptions
0001:00621060* _htmlReadDoc
0001:006210b3* _htmlReadFile
0001:006210fe* _htmlReadMemory
0001:0062117e* _htmlReadFd
0001:00621245* _htmlReadIO
0001:0062131a* _htmlCtxtReadDoc
0001:00621390* _htmlCtxtReadFile
0001:00621405* _htmlCtxtReadMemory
0001:006214bd* _htmlCtxtReadFd
0001:00621568* _htmlCtxtReadIO
Module: U:\extras\lib\xml2.lib(HTMLtree.obj)
0001:00628a08  _htmlGetMetaEncoding
0001:00628ccb  _htmlSetMetaEncoding
0001:0062905a  _htmlIsBooleanAttr
0001:00629287* _htmlDocContentDumpOutput
0001:006298df  _htmlDocContentDumpFormatOutput
0001:006292df  _htmlNodeDumpFormatOutput
0001:00629a29  _htmlDocDumpMemoryFormat
0001:00629b59* _htmlDocDumpMemory
0001:00629b82  _htmlNodeDumpOutput
0001:00629bb2* _htmlNodeDumpFileFormat
0001:00629c60  _htmlNodeDumpFile
0001:00629caf  _htmlNodeDump
0001:00629d95  _htmlDocDump
0001:00629e4d  _htmlSaveFile
0001:00629f14  _htmlSaveFileFormat
0001:0062a01b* _htmlSaveFileEnc
Module: U:\extras\lib\xml2.lib(c14n.obj)
0001:0062c977* _xmlC14NExecute
0001:0062cb6e  _xmlC14NDocSaveTo
0001:0062cc13* _xmlC14NDocDumpMemory
0001:0062cd4b* _xmlC14NDocSave
Module: U:\extras\lib\xml2.lib(hash.obj)
0001:0062ceda  _xmlHashCreate
0001:0062cf56  _xmlHashCreateDict
0001:0062cf86  _xmlHashFree
0001:0062d0cd  _xmlHashAddEntry3
0001:0062d5a4  _xmlHashAddEntry2
0001:0062d5d4  _xmlHashAddEntry
0001:0062d605* _xmlHashUpdateEntry3
0001:0062d967  _xmlHashUpdateEntry2
0001:0062d99e  _xmlHashUpdateEntry
0001:0062d9d6  _xmlHashLookup3
0001:0062da9a  _xmlHashLookup2
0001:0062dac3  _xmlHashLookup
0001:0062daed* _xmlHashQLookup3
0001:0062dd1e  _xmlHashQLookup2
0001:0062dd5d* _xmlHashQLookup
0001:0062dd9e  _xmlHashScanFull
0001:0062de62  _xmlHashScan
0001:0062de90* _xmlHashScanFull3
0001:0062df92  _xmlHashScan3
0001:0062df9e  _xmlHashCopy
0001:0062e060  _xmlHashSize
0001:0062e074* _xmlHashRemoveEntry3
0001:0062e1fd  _xmlHashRemoveEntry2
0001:0062e22d  _xmlHashRemoveEntry
Module: U:\usr\lib\libc_dll.lib(getsockname.obj)
0001:0062e260  _getsockname
Module: U:\extras\lib\libssl.lib(ssl_lib.obj)
0001:0062e370  _ssl_undefined_function
0001:0062e6c0  _SSL_clear
0001:0062e940* _SSL_CTX_set_ssl_version
0001:0062e9e0* _SSL_CTX_set_session_id_context
0001:0062eaa0* _SSL_set_session_id_context
0001:0062eb60* _SSL_CTX_set_generate_session_id
0001:0062ebd0* _SSL_set_generate_session_id
0001:0062ec40  _SSL_has_matching_session_id
0001:0062edd0* _SSL_CTX_set_purpose
0001:0062edf0* _SSL_set_purpose
0001:0062ee10* _SSL_CTX_set_trust
0001:0062ee30* _SSL_set_trust
0001:0062ee50* _SSL_CTX_set1_param
0001:0062ee70* _SSL_set1_param
0001:0062ee90* _SSL_set_bio
0001:0062ef00  _SSL_get_rbio
0001:0062ef10* _SSL_get_wbio
0001:0062ef20* _SSL_get_fd
0001:0062ef70* _SSL_get_rfd
0001:0062efc0* _SSL_get_wfd
0001:0062f010  _SSL_set_fd
0001:0062f0f0* _SSL_set_wfd
0001:0062f270* _SSL_set_rfd
0001:0062f410* _SSL_get_finished
0001:0062f500* _SSL_get_peer_finished
0001:0062f5f0* _SSL_get_verify_mode
0001:0062f600* _SSL_get_verify_depth
0001:0062f620* _SSL_get_verify_callback
0001:0062f630* _SSL_CTX_get_verify_mode
0001:0062f640* _SSL_CTX_get_verify_depth
0001:0062f660* _SSL_CTX_get_verify_callback
0001:0062f670* _SSL_set_verify
0001:0062f690* _SSL_set_verify_depth
0001:0062f6b0* _SSL_set_read_ahead
0001:0062f6c0* _SSL_get_read_ahead
0001:0062f6d0* _SSL_pending
0001:0062f6f0* _SSL_get_peer_certificate
0001:0062f760* _SSL_get_peer_cert_chain
0001:0062f7a0  _SSL_copy_session_id
0001:0062f900* _SSL_CTX_check_private_key
0001:0062f9b0* _SSL_check_private_key
0001:0062faa0* _SSL_accept
0001:0062fbc0  _SSL_connect
0001:0062fce0  _SSL_get_default_timeout
0001:0062fd00  _SSL_read
0001:0062fd80  _SSL_peek
0001:0062fe00  _SSL_write
0001:0062feb0  _SSL_shutdown
0001:0062ff20* _SSL_renegotiate
0001:0062ff50* _SSL_renegotiate_pending
0001:0062ff70  _SSL_ctrl
0001:00630200* _SSL_callback_ctrl
0001:00630240* _SSL_CTX_sessions
0001:00630250  _SSL_CTX_ctrl
0001:006305c0* _SSL_CTX_callback_ctrl
0001:00630600* _ssl_cipher_id_cmp
0001:00630630  _ssl_cipher_ptr_id_cmp
0001:00630670  _SSL_get_ciphers
0001:006306b0  _ssl_get_ciphers_by_id
0001:006306e0* _SSL_get_cipher_list
0001:00630750* _SSL_CTX_set_cipher_list
0001:006307e0* _SSL_set_cipher_list
0001:00630880* _SSL_get_shared_ciphers
0001:00630940  _ssl_cipher_list_to_bytes
0001:00630a90  _ssl_bytes_to_cipher_list
0001:00630d50* _SSL_get_servername
0001:00630db0* _SSL_get_servername_type
0001:00630de0  _SSL_CTX_free
0001:00630fd0  _SSL_CTX_new
0001:00631540* _SSL_free
0001:00631850  _SSL_new
0001:00631be0* _SSL_CTX_set_default_passwd_cb
0001:00631bf0* _SSL_CTX_set_default_passwd_cb_userdata
0001:00631c00* _SSL_CTX_set_cert_verify_callback
0001:00631c20* _SSL_CTX_set_verify
0001:00631c40* _SSL_CTX_set_verify_depth
0001:00631c70  _ssl_set_cert_masks
0001:00632330  _ssl_check_srvr_ecc_cert_and_alg
0001:00632520* _ssl_get_server_send_cert
0001:00632650* _ssl_get_sign_pkey
0001:006326e0  _ssl_update_cache
0001:00632820* _SSL_get_ssl_method
0001:00632830  _SSL_set_ssl_method
0001:006328d0* _SSL_get_error
0001:00632a60* _SSL_do_handshake
0001:00632ad0* _SSL_set_accept_state
0001:00632bc0* _SSL_set_connect_state
0001:00632cb0  _ssl_undefined_void_function
0001:00632cf0  _ssl_undefined_const_function
0001:00632d30* _ssl_bad_method
0001:00632d80* _SSL_get_version
0001:00632dd0* _SSL_dup
0001:00633160* _ssl_clear_cipher_ctx
0001:00633200* _SSL_get_certificate
0001:00633230* _SSL_get_privatekey
0001:00633260* _SSL_get_current_cipher
0001:00633290* _SSL_get_current_compression
0001:006332c0* _SSL_get_current_expansion
0001:006332f0  _ssl_init_wbio_buffer
0001:00633430  _ssl_free_wbio_buffer
0001:00633470* _SSL_CTX_set_quiet_shutdown
0001:00633480* _SSL_CTX_get_quiet_shutdown
0001:00633490* _SSL_set_quiet_shutdown
0001:006334a0* _SSL_get_quiet_shutdown
0001:006334b0* _SSL_set_shutdown
0001:006334c0* _SSL_get_shutdown
0001:006334d0  _SSL_version
0001:006334e0* _SSL_get_SSL_CTX
0001:006334f0* _SSL_set_SSL_CTX
0001:00633590* _SSL_CTX_set_default_verify_paths
0001:006335b0* _SSL_CTX_load_verify_locations
0001:006335d0* _SSL_set_info_callback
0001:006335e0* _SSL_get_info_callback
0001:006335f0  _SSL_state
0001:00633600* _SSL_set_verify_result
0001:00633610* _SSL_get_verify_result
0001:00633620* _SSL_get_ex_new_index
0001:00633660* _SSL_set_ex_data
0001:00633680* _SSL_get_ex_data
0001:006336a0* _SSL_CTX_get_ex_new_index
0001:006336e0* _SSL_CTX_set_ex_data
0001:00633700* _SSL_CTX_get_ex_data
0001:00633720  _ssl_ok
0001:00633730* _SSL_CTX_get_cert_store
0001:00633740* _SSL_CTX_set_cert_store
0001:00633770* _SSL_want
0001:00633780* _SSL_CTX_set_tmp_rsa_callback
0001:006337b0* _SSL_set_tmp_rsa_callback
0001:006337e0* _SSL_CTX_set_tmp_dh_callback
0001:00633810* _SSL_set_tmp_dh_callback
0001:00633840* _SSL_CTX_set_tmp_ecdh_callback
0001:00633870* _SSL_set_tmp_ecdh_callback
0001:006338a0* _SSL_CTX_use_psk_identity_hint
0001:00633960* _SSL_use_psk_identity_hint
0001:00633a60* _SSL_get_psk_identity_hint
0001:00633aa0* _SSL_get_psk_identity
0001:00633ae0* _SSL_set_psk_client_callback
0001:00633af0* _SSL_CTX_set_psk_client_callback
0001:00633b00* _SSL_set_psk_server_callback
0001:00633b10* _SSL_CTX_set_psk_server_callback
0001:00633b20* _SSL_CTX_set_msg_callback
0001:00633b30* _SSL_set_msg_callback
0001:00633b40  _ssl_replace_hash
0001:00633b90* _ssl_clear_hash_ctx
0001:00633bc0  _OBJ_bsearch_ssl_cipher_id
0002:00006fe0* _SSL_version_str
0002:00006ff0  _ssl3_undef_enc_method
Module: U:\extras\lib\libssl.lib(s23_clnt.obj)
0001:00633c70* _ssl23_connect
0001:00634c10  _SSLv23_client_method
Module: U:\extras\lib\poll.lib(poll.obj)
0001:00634ca0  _poll
Module: U:\usr\lib\libc_dll.lib(send.obj)
0001:006350b0  _send
Module: U:\usr\lib\libc_dll.lib(recv.obj)
0001:00635160  _recv
Module: U:\usr\lib\libc_dll.lib(accept.obj)
0001:00635210  _accept
Module: U:\usr\lib\libc_dll.lib(socket.obj)
0001:006352f0  _socket
Module: U:\usr\lib\libc_dll.lib(bind.obj)
0001:00635370  _bind
Module: U:\usr\lib\libc_dll.lib(listen.obj)
0001:00635410  _listen
Module: U:\extras\lib\xml2.lib(entities.obj)
0001:00635b82  _xmlGetPredefinedEntity
0001:00635cba  _xmlAddDtdEntity
0001:00635d9a  _xmlAddDocEntity
0001:00635e24* _xmlNewEntity
0001:00635e8d  _xmlGetParameterEntity
0001:00635eee* _xmlGetDtdEntity
0001:00635f16  _xmlGetDocEntity
0001:0063604f  _xmlEncodeEntitiesReentrant
0001:00636491  _xmlEncodeSpecialChars
0001:006365f1* _xmlCreateEntitiesTable
0001:00636605  _xmlFreeEntitiesTable
0001:00636620  _xmlCopyEntitiesTable
0001:006366a8  _xmlDumpEntityDecl
0001:0063691b* _xmlDumpEntitiesTable
Module: U:\usr\lib\libc_dll.lib(getpeername.obj)
0001:00636950  _getpeername
Module: U:\usr\lib\libc_dll.lib(connect.obj)
0001:006369f0  _connect
Module: U:\usr\lib\libc_dll.lib(recvfrom.obj)
0001:00636a90  _recvfrom
Module: U:\usr\lib\libc_dll.lib(sendto.obj)
0001:00636b60  _sendto
Module: U:\usr\lib\libc_dll.lib(getsockopt.obj)
0001:00636c10  _getsockopt
Module: U:\usr\lib\libc_dll.lib(setsockopt.obj)
0001:00636cf0  _setsockopt
Module: U:\usr\lib\libc_dll.lib(socketpair.obj)
0001:00636df0  _socketpair
Module: U:\usr\lib\libc_dll.lib(shutdown.obj)
0001:00636eb0  _shutdown
Module: U:\usr\lib\libc_dll.lib(syslog.obj)
0001:00636f9c  _syslog
0001:00637004* _vsyslog
0001:00637461  _openlog
0001:006374b0  _closelog
0001:006374e4* _setlogmask
Module: U:\extras\lib\xml2.lib(xmlreader.obj)
0001:0063895a* _xmlTextReaderReadState
0001:0063896d  _xmlTextReaderExpand
0001:00638b11  _xmlTextReaderReadInnerXml
0001:00638c00  _xmlTextReaderReadOuterXml
0001:00638cda  _xmlTextReaderReadString
0001:00638d8e  _xmlNewTextReader
0001:00639048* _xmlNewTextReaderFilename
0001:006390e9  _xmlFreeTextReader
0001:006392f9* _xmlTextReaderClose
0001:00639381  _xmlTextReaderGetAttributeNo
0001:0063943a  _xmlTextReaderGetAttribute
0001:006395c7  _xmlTextReaderGetAttributeNs
0001:0063968b* _xmlTextReaderGetRemainder
0001:0063973f  _xmlTextReaderLookupNamespace
0001:0063977d  _xmlTextReaderMoveToAttributeNo
0001:00639809  _xmlTextReaderMoveToAttribute
0001:006399c2  _xmlTextReaderMoveToAttributeNs
0001:00639ae2  _xmlTextReaderMoveToFirstAttribute
0001:00639b23  _xmlTextReaderMoveToNextAttribute
0001:00639b8d  _xmlTextReaderMoveToElement
0001:00639bbf* _xmlTextReaderReadAttributeValue
0001:00639c6b* _xmlTextReaderConstEncoding
0001:00639cb5  _xmlTextReaderAttributeCount
0001:00639d1a  _xmlTextReaderNodeType
0001:00639e6c  _xmlTextReaderIsEmptyElement
0001:00639ef3* _xmlTextReaderName
0001:0063a069* _xmlTextReaderLocalName
0001:0063a0c5  _xmlTextReaderConstName
0001:0063a270  _xmlTextReaderConstLocalName
0001:0063a2d5* _xmlTextReaderPrefix
0001:0063a333  _xmlTextReaderConstPrefix
0001:0063a3ba* _xmlTextReaderNamespaceUri
0001:0063a40d  _xmlTextReaderConstNamespaceUri
0001:0063a48b* _xmlTextReaderBaseUri
0001:0063a4b5  _xmlTextReaderConstBaseUri
0001:0063a512  _xmlTextReaderDepth
0001:0063a553  _xmlTextReaderHasAttributes
0001:0063a594  _xmlTextReaderHasValue
0001:0063a5cd* _xmlTextReaderValue
0001:0063a6d8  _xmlTextReaderConstValue
0001:0063a7ed  _xmlTextReaderIsDefault
0001:0063a7f8* _xmlTextReaderQuoteChar
0001:0063a806* _xmlTextReaderXmlLang
0001:0063a827  _xmlTextReaderConstXmlLang
0001:0063a87c* _xmlTextReaderConstString
0001:0063a8a7* _xmlTextReaderNormalization
0001:0063a8b5  _xmlTextReaderSetParserProp
0001:0063a99d  _xmlTextReaderGetParserProp
0001:0063aa0a* _xmlTextReaderGetParserLineNumber
0001:0063aa29* _xmlTextReaderGetParserColumnNumber
0001:0063aa48* _xmlTextReaderCurrentNode
0001:0063aa62* _xmlTextReaderPreserve
0001:0063aaf8  _xmlTextReaderRead
0001:0063b567* _xmlTextReaderNextSibling
0001:0063b5b2  _xmlTextReaderNext
0001:0063b62d* _xmlTextReaderPreservePattern
0001:0063b755* _xmlTextReaderCurrentDoc
0001:0063b781  _xmlTextReaderRelaxNGSetSchema
0001:0063b87e* _xmlTextReaderSetSchema
0001:0063ba83* _xmlTextReaderRelaxNGValidate
0001:0063bbf4* _xmlTextReaderSchemaValidateCtxt
0001:0063bc08  _xmlTextReaderSchemaValidate
0001:0063bc1c* _xmlTextReaderIsNamespaceDecl
0001:0063bc4b* _xmlTextReaderConstXmlVersion
0001:0063bc95* _xmlTextReaderStandalone
0001:0063bcc2* _xmlTextReaderLocatorLineNumber
0001:0063bd0f* _xmlTextReaderLocatorBaseURI
0001:0063bd64* _xmlTextReaderSetErrorHandler
0001:0063bed4* _xmlTextReaderSetStructuredErrorHandler
0001:0063c05d  _xmlTextReaderIsValid
0001:0063c0aa* _xmlTextReaderGetErrorHandler
0001:0063c0d4  _xmlTextReaderSetup
0001:0063c5f1* _xmlTextReaderByteConsumed
0001:0063c615* _xmlReaderWalker
0001:0063c67e  _xmlReaderForFile
0001:0063c6c4* _xmlReaderForMemory
0001:0063c73e* _xmlReaderForDoc
0001:0063c77d* _xmlReaderForFd
0001:0063c802* _xmlReaderForIO
0001:0063c891* _xmlReaderNewWalker
0001:0063c943* _xmlReaderNewFile
0001:0063c99f* _xmlReaderNewMemory
0001:0063ca08* _xmlReaderNewDoc
0001:0063ca5e* _xmlReaderNewFd
0001:0063cac7* _xmlReaderNewIO
Module: U:\extras\lib\xmlrpc.lib(xmlrpc.obj)
0001:0063cb90  _XMLRPC_RequestGetMethodName
0001:0063cba1  _XMLRPC_RequestSetRequestType
0001:0063cbb7  _XMLRPC_RequestGetRequestType
0001:0063cbc8  _XMLRPC_RequestGetData
0001:0063cbd8  _XMLRPC_RequestGetError
0001:0063cbe9  _XMLRPC_RequestGetOutputOptions
0001:0063cbfa  _XMLRPC_SetValueInt
0001:0063cc12  _XMLRPC_SetValueBoolean
0001:0063cc30  _XMLRPC_CopyValue
0001:0063cc40  _XMLRPC_SetValueDouble
0001:0063cc5c  _XMLRPC_GetValueString
0001:0063cc74  _XMLRPC_GetValueStringLen
0001:0063cc85  _XMLRPC_GetValueInt
0001:0063cca1  _XMLRPC_GetValueBoolean
0001:0063ccb9  _XMLRPC_GetValueDouble
0001:0063ccd1  _XMLRPC_GetValueBase64
0001:0063cce9  _XMLRPC_GetValueDateTime
0001:0063cd01  _XMLRPC_GetValueDateTime_ISO8601
0001:0063cd19  _XMLRPC_GetValueID
0001:0063cd33  _XMLRPC_GetValueType
0001:0063cd46  _XMLRPC_GetVectorType
0001:0063cd61  _XMLRPC_GetValueTypeEasy
0001:0063cdf2  _type_to_str
0001:0063ce93  _XMLRPC_GetDefaultIdCase
0001:0063ce9d* _XMLRPC_SetDefaultIdCase
0001:0063ceaa  _XMLRPC_GetDefaultIdCaseComparison
0001:0063ceb4* _XMLRPC_SetDefaultIdCaseComparison
0001:0063ced4  _XMLRPC_GetVersionString
0001:0063cede* _XMLRPC_Free
0001:0063cef3* _XMLRPC_ServerFindMethod
0001:0063cf40  _find_method
0001:0063cf8c  _XMLRPC_ServerRegisterMethod
0001:0063cff2  _XMLRPC_VectorRewind
0001:0063d01e  _XMLRPC_VectorNext
0001:0063d047  _XMLRPC_CreateValueEmpty
0001:0063d08c  _XMLRPC_RequestNew
0001:0063d0bd  _XMLRPC_ServerCreate
0001:0063d101* _XMLRPC_GetGlobalServer
0001:0063d11e  _XMLRPC_VectorSize
0001:0063d147  _XMLRPC_SetIsVector
0001:0063d1e4  _XMLRPC_RequestSetMethodName
0001:0063d219  _XMLRPC_SetValueBase64
0001:0063d27c  _XMLRPC_SetValueString
0001:0063d2e4  _XMLRPC_SetValueID_Case
0001:0063d3c3  _XMLRPC_CreateValueDouble
0001:0063d415  _XMLRPC_CreateValueBase64
0001:0063d46b  _XMLRPC_CreateValueBoolean
0001:0063d4bd  _XMLRPC_CreateValueInt
0001:0063d509  _XMLRPC_CreateValueString
0001:0063d567  _XMLRPC_CreateVector
0001:0063d5c2  _XMLRPC_SetValueDateTime_ISO8601
0001:0063d755  _XMLRPC_CreateValueDateTime_ISO8601
0001:0063d7b5* _XMLRPC_SetValueDateTime
0001:0063d823* _XMLRPC_CreateValueDateTime
0001:0063d8a5  _XMLRPC_CleanupValue
0001:0063d9b3  _XMLRPC_ServerDestroy
0001:0063da74  _XMLRPC_RequestSetError
0001:0063dab3  _XMLRPC_RequestSetData
0001:0063daf0  _XMLRPC_RequestFree
0001:0063dbc6  _XMLRPC_AddValueToVector
0001:0063dddb* _XMLRPC_UtilityCreateFault
0001:0063df7d  _XMLRPC_ServerCallMethod
0001:0063e016  _XMLRPC_DupValueNew
0001:0063e15f  _XMLRPC_VectorRemoveValue
0001:0063e1d3  _XMLRPC_VectorGetValueWithID_Case
0001:0063e24d* _XMLRPC_GetValueFaultString
0001:0063e281* _XMLRPC_GetResponseFaultString
0001:0063e298* _XMLRPC_GetValueFaultCode
0001:0063e2cc* _XMLRPC_GetResponseFaultCode
0001:0063e2e3* _XMLRPC_ValueIsFault
0001:0063e333* _XMLRPC_ResponseIsFault
0001:0063e34a  _XMLRPC_AddValuesToVector
0001:0063e45f  _XMLRPC_REQUEST_FromXML
0001:0063e575* _XMLRPC_VALUE_FromXML
0001:0063e5b5  _XMLRPC_REQUEST_ToXML
0001:0063e633  _XMLRPC_VALUE_ToXML
0001:0063e678  _XMLRPC_RequestSetOutputOptions
Module: U:\extras\lib\xmlrpc.lib(xmlrpc_introspection.obj)
0001:0063e744* _XMLRPC_ServerSetValidationLevel
0001:0063e762* _find_named_value
0001:0063e7d6* _validate_scalar
0001:0063e933* _validate_value
0001:0063eb34* _validate_vector
0001:0063ea27* _validate_method
0001:0063eab2  _XMLRPC_ServerValidateRequest
0001:0063ec49  _XMLRPC_ServerRegisterIntrospectionCallback
0001:0063ecb2* _describe_method
0001:0063edd4* _xml_element_to_method_description
0001:0063f3c1  _XMLRPC_IntrospectionCreateDescription
0001:0063f470  _xi_register_system_methods
0001:0063f8cb  _XMLRPC_ServerAddIntrospectionData
Module: U:\extras\lib\xml2.lib(xmlwriter.obj)
0001:00640171* _xmlNewTextWriter
0001:006402f7  _xmlNewTextWriterFilename
0001:0064039d  _xmlNewTextWriterMemory
0001:006404b1* _xmlNewTextWriterPushParser
0001:006405f0* _xmlNewTextWriterDoc
0001:0064074b* _xmlNewTextWriterTree
0001:00640856  _xmlFreeTextWriter
0001:006409c0  _xmlTextWriterStartDocument
0001:00640d62  _xmlTextWriterEndComment
0001:00640e2a  _xmlTextWriterEndAttribute
0001:00640e95  _xmlTextWriterStartAttribute
0001:00640fdc  _xmlTextWriterStartAttributeNS
0001:00641197  _xmlTextWriterWriteAttribute
0001:0064186b  _xmlTextWriterWriteString
0001:006413f4* _xmlTextWriterWriteBinHex
0001:0064152d* _xmlTextWriterWriteBase64
0001:00641779* _xmlTextWriterWriteRawLen
0001:00641840  _xmlTextWriterWriteRaw
0001:00641924* _xmlTextWriterWriteVFormatString
0001:00641976* _xmlTextWriterWriteFormatString
0001:006419a6* _xmlTextWriterWriteVFormatRaw
0001:006419ef* _xmlTextWriterWriteFormatRaw
0001:00641a15  _xmlTextWriterFullEndElement
0001:00641b90  _xmlTextWriterEndElement
0001:00641d52  _xmlTextWriterStartElement
0001:00641f76  _xmlTextWriterStartElementNS
0001:006420e6  _xmlTextWriterStartComment
0001:00642255  _xmlTextWriterWriteComment
0001:006422e0* _xmlTextWriterWriteVFormatComment
0001:00642344* _xmlTextWriterWriteFormatComment
0001:00642365* _xmlTextWriterWriteVFormatAttribute
0001:006423b5* _xmlTextWriterWriteFormatAttribute
0001:006423dd  _xmlTextWriterWriteAttributeNS
0001:00642457* _xmlTextWriterWriteVFormatAttributeNS
0001:006424b5* _xmlTextWriterWriteFormatAttributeNS
0001:006424eb  _xmlTextWriterWriteElement
0001:0064254a* _xmlTextWriterWriteVFormatElement
0001:0064259a* _xmlTextWriterWriteFormatElement
0001:006425c2  _xmlTextWriterWriteElementNS
0001:0064263e* _xmlTextWriterWriteVFormatElementNS
0001:0064269c* _xmlTextWriterWriteFormatElementNS
0001:0064277e  _xmlTextWriterStartPI
0001:006429b3  _xmlTextWriterEndPI
0001:00642a4b  _xmlTextWriterWritePI
0001:00642abe* _xmlTextWriterWriteVFormatPI
0001:00642b0e* _xmlTextWriterWriteFormatPI
0001:00642bac  _xmlTextWriterStartCDATA
0001:00642d1b  _xmlTextWriterEndCDATA
0001:00642d84  _xmlTextWriterWriteCDATA
0001:00642df0* _xmlTextWriterWriteVFormatCDATA
0001:00642e39* _xmlTextWriterWriteFormatCDATA
0001:00642f14  _xmlTextWriterStartDTD
0001:006432a2  _xmlTextWriterStartDTDElement
0001:0064344b  _xmlTextWriterEndDTDElement
0001:006434db  _xmlTextWriterWriteDTDElement
0001:0064353f* _xmlTextWriterWriteVFormatDTDElement
0001:0064358f* _xmlTextWriterWriteFormatDTDElement
0001:006435f2  _xmlTextWriterStartDTDAttlist
0001:0064379b  _xmlTextWriterEndDTDAttlist
0001:0064382b  _xmlTextWriterWriteDTDAttlist
0001:0064388f* _xmlTextWriterWriteVFormatDTDAttlist
0001:006438df* _xmlTextWriterWriteFormatDTDAttlist
0001:00643914  _xmlTextWriterStartDTDEntity
0001:00643af7  _xmlTextWriterEndDTDEntity
0001:00643bbd  _xmlTextWriterEndDTD
0001:00643cd2  _xmlTextWriterWriteDTD
0001:00643d53* _xmlTextWriterWriteVFormatDTD
0001:00643db1* _xmlTextWriterWriteFormatDTD
0001:00643de7* _xmlTextWriterWriteDTDInternalEntity
0001:00643e6a* _xmlTextWriterWriteVFormatDTDInternalEntity
0001:00643ec1* _xmlTextWriterWriteFormatDTDInternalEntity
0001:00644071* _xmlTextWriterWriteDTDExternalEntityContents
0001:00644312* _xmlTextWriterWriteDTDExternalEntity
0001:006443b0  _xmlTextWriterWriteDTDEntity
0001:00644450* _xmlTextWriterWriteDTDNotation
0001:00644700  _xmlTextWriterFlush
0001:00644754  _xmlTextWriterEndDocument
0001:0064488f  _xmlTextWriterSetIndent
0001:006448b8  _xmlTextWriterSetIndentString
Module: U:\usr\lib\libos2.lib(code2.obj)
0001:00644954  DosGetMessage
0001:00644940* __msgseg32
Module: U:\usr\lib\gcc-lib\i386-pc-os2-emx\3.3.5\libgcc_so_d.lib(emx-ctordtor.obj)
0001:00644970  ___ctordtorInit
0001:0064497a* ___POST$__ctordtorInit
0001:0064499e  ___ctordtorTerm
0001:006449a8* ___POST$__ctordtorTerm
Module: U:\extras\lib\xml2.lib(chvalid.obj)
0001:00644a30  _xmlCharInRange
0001:00644ace* _xmlIsBaseChar
0001:00644da0  _xmlIsBaseCharGroup
0001:00644b34* _xmlIsBlank
0001:00644b62* _xmlIsChar
0001:00644bbc* _xmlIsCombining
0001:00644dc0  _xmlIsCombiningGroup
0001:00644be3* _xmlIsDigit
0001:00644dd0  _xmlIsDigitGroup
0001:00644c13* _xmlIsExtender
0001:00644de0  _xmlIsExtenderGroup
0001:00644c42* _xmlIsIdeographic
0001:00644c7e* _xmlIsPubidChar
0001:00644ca0  _xmlIsPubidChar_tab
0001:00644db0* _xmlIsCharGroup
0001:00644df0* _xmlIsIdeographicGroup
Module: U:\extras\lib\xml2.lib(dict.obj)
0001:00645995  _xmlDictCleanup
0001:006459c0  _xmlDictCreate
0001:00645a52  _xmlDictReference
0001:00645aa9* _xmlDictCreateSub
0001:00645ae0  _xmlDictFree
0001:00645bfa  _xmlDictLookup
0001:00645f19  _xmlDictExists
0001:00646110  _xmlDictQLookup
0001:006465cd  _xmlDictOwns
0001:00646620* _xmlDictSize
Module: U:\extras\lib\xml2.lib(threads.obj)
0001:0064669b  _xmlNewMutex
0001:006466d5  _xmlFreeMutex
0001:00646715  _xmlMutexLock
0001:00646734  _xmlMutexUnlock
0001:00646752  _xmlNewRMutex
0001:006467ae  _xmlFreeRMutex
0001:006467f9  _xmlRMutexLock
0001:00646892  _xmlRMutexUnlock
0001:006468ed  ___xmlGlobalInitMutexLock
0001:00646901  ___xmlGlobalInitMutexUnlock
0001:00646915  ___xmlGlobalInitMutexDestroy
0001:0064693e  _xmlGetGlobalState
0001:006469e8  _xmlGetThreadId
0001:00646a01* _xmlLockLibrary
0001:00646a15* _xmlUnlockLibrary
0001:00646a29  _xmlInitThreads
0001:00646a43  _xmlIsMainThread
0001:00646a98  _xmlCleanupThreads
Module: U:\extras\lib\xml2.lib(SAX.obj)
0001:00646ac0  _initxmlDefaultSAXHandler
0001:00646b9e  _inithtmlDefaultSAXHandler
0001:00646c73  _initdocbDefaultSAXHandler
Module: U:\extras\lib\xml2.lib(SAX2.obj)
0001:00646d50  _xmlSAX2IsStandalone
0001:00646d6e  _xmlSAX2HasInternalSubset
0001:00646d8c  _xmlSAX2HasExternalSubset
0001:00646daa  _xmlSAX2SetDocumentLocator
0001:00646daf  _xmlSAX2IgnorableWhitespace
0001:00646db4  _xmlSAX2CDataBlock
0001:00646e24  _xmlSAX2Comment
0001:00646eed  _xmlSAX2ProcessingInstruction
0001:00647281  _xmlSAX2Characters
0001:0064759a  _xmlSAX2Reference
0001:006475fd* _xmlSAX2EndElementNs
0001:00647692  _xmlSAX2EndElement
0001:00647aae* _xmlSAX2StartElementNs
0001:00649128  _xmlSAX2StartElement
0001:0064997b  _xmlSAX2EndDocument
0001:00649a53  _xmlSAX2StartDocument
0001:00649b98  _xmlSAX2GetParameterEntity
0001:00649bb5  _xmlSAX2ResolveEntity
0001:00649c30  _xmlSAX2ExternalSubset
0001:00649e7d  _xmlSAX2InternalSubset
0001:0064a106  _xmlSAX2GetEntity
0001:0064a2e5  _xmlSAX2AttributeDecl
0001:0064a4e3  _xmlSAX2ElementDecl
0001:0064a634  _xmlSAX2NotationDecl
0001:0064a7c6  _xmlSAX2EntityDecl
0001:0064a9de  _xmlSAX2UnparsedEntityDecl
0001:0064ab1f  _xmlSAX2GetPublicId
0001:0064ab26  _xmlSAX2GetSystemId
0001:0064ab41  _xmlSAX2GetLineNumber
0001:0064ab59  _xmlSAX2GetColumnNumber
0001:0064ab71* _xmlSAXDefaultVersion
0001:0064ab93  _xmlSAXVersion
0001:0064acad  _xmlSAX2InitDefaultSAXHandler
0001:0064ade2  _xmlDefaultSAXHandlerInit
0001:0064aeba* _xmlSAX2InitHtmlDefaultSAXHandler
0001:0064af98  _htmlDefaultSAXHandlerInit
0001:0064b07b* _xmlSAX2InitDocbDefaultSAXHandler
0001:0064b159* _docbDefaultSAXHandlerInit
Module: U:\extras\lib\xml2.lib(list.obj)
0001:0064b376  _xmlListCreate
0001:0064b439  _xmlListSearch
0001:0064b468* _xmlListReverseSearch
0001:0064b4be  _xmlListInsert
0001:0064b548  _xmlListAppend
0001:0064b5d1  _xmlListRemoveFirst
0001:0064b623* _xmlListRemoveLast
0001:0064b675* _xmlListRemoveAll
0001:0064b6a9* _xmlListClear
0001:0064b6f2  _xmlListDelete
0001:0064b728  _xmlListEmpty
0001:0064b743  _xmlListFront
0001:0064b755* _xmlListEnd
0001:0064b768  _xmlListSize
0001:0064b78c  _xmlListPopFront
0001:0064b7cf* _xmlListPopBack
0001:0064b813  _xmlListPushFront
0001:0064b876* _xmlListPushBack
0001:0064b8dc  _xmlLinkGetData
0001:0064b8ed* _xmlListReverse
0001:0064b925  _xmlListWalk
0001:0064b967* _xmlListReverseWalk
0001:0064b9ab* _xmlListCopy
0001:0064ba13* _xmlListDup
0001:0064ba60* _xmlListMerge
0001:0064ba86* _xmlListSort
Module: U:\extras\lib\xml2.lib(xmlregexp.obj)
0001:00651dc2  _xmlRegNewExecCtxt
0001:00651efc  _xmlRegFreeExecCtxt
0001:00651fc3  _xmlRegExecPushString
0001:00651fdf  _xmlRegExecPushString2
0001:0065216b  _xmlRegExecNextValues
0001:00652196  _xmlRegExecErrInfo
0001:00652389* _xmlRegexpPrint
0001:00652bb5  _xmlRegexpExec
0001:00653159  _xmlRegFreeRegexp
0001:0065326b  _xmlFreeAutomata
0001:00653280  _xmlNewAutomata
0001:006532e0  _xmlRegexpIsDeterminist
0001:00653aef  _xmlRegexpCompile
0001:00653b97  _xmlAutomataSetFlags
0001:00653ba9  _xmlAutomataGetInitState
0001:00653bba  _xmlAutomataSetFinalState
0001:00653bdc  _xmlAutomataNewTransition
0001:00653c5f  _xmlAutomataNewTransition2
0001:00653d9d  _xmlAutomataNewNegTrans
0001:00653f58  _xmlAutomataNewCountTrans2
0001:0065416f* _xmlAutomataNewCountTrans
0001:006542ba  _xmlAutomataNewOnceTrans2
0001:00654475* _xmlAutomataNewOnceTrans
0001:00654564  _xmlAutomataNewState
0001:0065458a  _xmlAutomataNewEpsilon
0001:006545ba  _xmlAutomataNewAllTrans
0001:00654650  _xmlAutomataNewCounter
0001:00654692  _xmlAutomataNewCountedTrans
0001:006546d2  _xmlAutomataNewCounterTrans
0001:00654712  _xmlAutomataCompile
0001:00654742* _xmlAutomataIsDeterminist
0001:0065475c* _xmlExpNewCtxt
0001:0065480b* _xmlExpFreeCtxt
0001:00654848* _xmlExpFree
0001:00656040* _xmlExpRef
0001:00656050* _xmlExpNewAtom
0001:006560b5* _xmlExpNewOr
0001:0065611e* _xmlExpNewSeq
0001:00656187* _xmlExpNewRange
0001:006561f3* _xmlExpGetLanguage
0001:00656236* _xmlExpGetStart
0001:00656278* _xmlExpIsNillable
0001:00656290* _xmlExpStringDerive
0001:006562e7* _xmlExpExpDerive
0001:0065633c* _xmlExpSubsume
0001:006563eb* _xmlExpParse
0001:00656441* _xmlExpDump
0001:00656465* _xmlExpMaxToken
0001:00656479* _xmlExpCtxtNbNodes
0001:0065648d* _xmlExpCtxtNbCons
0002:00007260* _forbiddenExp
0002:00007264* _emptyExp
Module: U:\extras\lib\xml2.lib(nanohttp.obj)
0001:0065717a* _xmlNanoHTTPCleanup
0001:006571bb* _xmlNanoHTTPScanProxy
0001:006572bd* _xmlNanoHTTPInit
0001:00657335  _xmlNanoHTTPRead
0001:00657431  _xmlNanoHTTPClose
0001:006575c9* _xmlNanoHTTPMethodRedir
0001:0065829b* _xmlNanoHTTPOpenRedir
0001:006582f0  _xmlNanoHTTPMethod
0001:0065832e  _xmlNanoHTTPOpen
0001:00658374* _xmlNanoHTTPFetch
0001:00658464* _xmlNanoHTTPSave
0001:00658526  _xmlNanoHTTPReturnCode
0001:0065853a* _xmlNanoHTTPAuthHeader
0001:0065854b* _xmlNanoHTTPContentLength
0001:0065855f  _xmlNanoHTTPRedir
0001:00658570  _xmlNanoHTTPEncoding
0001:00658581  _xmlNanoHTTPMimeType
Module: U:\extras\lib\xml2.lib(nanoftp.obj)
0001:0065892d* _xmlNanoFTPCleanup
0001:00658993* _xmlNanoFTPProxy
0001:00658a47* _xmlNanoFTPUpdateURL
0001:00658b3e* _xmlNanoFTPScanProxy
0001:00658c60* _xmlNanoFTPInit
0001:00658d21* _xmlNanoFTPNewCtxt
0001:00658de3* _xmlNanoFTPFreeCtxt
0001:00658e67* _xmlNanoFTPGetResponse
0001:00658e7d* _xmlNanoFTPCheckResponse
0001:00658f65* _xmlNanoFTPQuit
0001:006590fe* _xmlNanoFTPConnect
0001:00659782* _xmlNanoFTPConnectTo
0001:006597f9* _xmlNanoFTPCwd
0001:006598e1* _xmlNanoFTPDele
0001:00659a62* _xmlNanoFTPGetConnection
0001:00659e61* _xmlNanoFTPCloseConnection
0001:00659fce* _xmlNanoFTPList
0001:0065a790* _xmlNanoFTPGetSocket
0001:0065a951* _xmlNanoFTPGet
0001:0065ab07  _xmlNanoFTPRead
0001:0065ab97  _xmlNanoFTPOpen
0001:0065ac08  _xmlNanoFTPClose
Module: U:\extras\lib\xml2.lib(catalog.obj)
0001:0065ceae* _xmlFreeCatalog
0001:0065cf14* _xmlConvertSGMLCatalog
0001:0065cf89* _xmlParseCatalogFile
0001:0065e3e2* _xmlLoadSGMLSuperCatalog
0001:0065e453* _xmlLoadACatalog
0001:0065e554* _xmlACatalogResolveSystem
0001:0065e5f7* _xmlACatalogResolvePublic
0001:0065e6ca* _xmlACatalogResolve
0001:0065e7d5* _xmlACatalogResolveURI
0001:0065e8e1* _xmlACatalogDump
0001:0065ea92* _xmlACatalogAdd
0001:0065efde* _xmlACatalogRemove
0001:0065f0ed* _xmlNewCatalog
0001:0065f146* _xmlCatalogIsEmpty
0001:0065f1d7* _xmlInitializeCatalog
0001:0065f314* _xmlLoadCatalog
0001:0065f3a0* _xmlLoadCatalogs
0001:0065f44c  _xmlCatalogCleanup
0001:0065f50c* _xmlCatalogResolveSystem
0001:0065f536* _xmlCatalogResolvePublic
0001:0065f561  _xmlCatalogResolve
0001:0065f593  _xmlCatalogResolveURI
0001:0065f5bd* _xmlCatalogDump
0001:0065f5f3* _xmlCatalogAdd
0001:0065f6c6* _xmlCatalogRemove
0001:0065f711* _xmlCatalogConvert
0001:0065f756  _xmlCatalogGetDefaults
0001:0065f7dd* _xmlCatalogSetDefaults
0001:0065f8fa* _xmlCatalogSetDefaultPrefer
0001:0065f96e* _xmlCatalogSetDebug
0001:0065f991  _xmlCatalogFreeLocal
0001:0065f9db  _xmlCatalogAddLocal
0001:0065facc  _xmlCatalogLocalResolve
0001:0065fbab  _xmlCatalogLocalResolveURI
0001:0065fc55* _xmlCatalogGetSystem
0001:0065fd56* _xmlCatalogGetPublic
Module: U:\extras\lib\xml2.lib(xmlmemory.obj)
0001:0065fead* _xmlMallocBreakpoint
0001:0065ff31* _xmlMemFree
0001:0066005f* _xmlMemUsed
0001:00660069* _xmlMemBlocks
0001:006600b7* _xmlMemDisplayLast
0001:00660139* _xmlMemDisplay
0001:006601df  _xmlMemShow
0001:00660212* _xmlMemoryDump
0001:0066023f  _xmlInitMemory
0001:006602dd* _xmlMemStrdupLoc
0001:0066040c* _xmlMemoryStrdup
0001:00660467* _xmlMallocAtomicLoc
0001:00660590* _xmlMallocLoc
0001:006606ad* _xmlMemMalloc
0001:006606ef* _xmlReallocLoc
0001:00660887* _xmlMemRealloc
0001:006608b1  _xmlCleanupMemory
0001:006608e5* _xmlMemSetup
0001:00660934* _xmlMemGet
0001:0066097b* _xmlGcMemSetup
0001:006609d4* _xmlGcMemGet
Module: U:\extras\lib\xml2.lib(xmlschemastypes.obj)
0001:00661f67  _xmlSchemaInitTypes
0001:0066253b  _xmlSchemaCleanupTypes
0001:006625ca  _xmlSchemaIsBuiltInTypeFacet
0001:00662758  _xmlSchemaGetBuiltInType
0001:00662a17  _xmlSchemaValueAppend
0001:00662a36  _xmlSchemaValueGetNext
0001:00662a47  _xmlSchemaValueGetAsString
0001:00662b2d  _xmlSchemaValueGetAsBoolean
0001:00662b45* _xmlSchemaNewStringValue
0001:00662b85  _xmlSchemaNewNOTATIONValue
0001:00662bb0  _xmlSchemaNewQNameValue
0001:00662bd2  _xmlSchemaFreeValue
0001:006645df  _xmlSchemaGetPredefinedType
0001:0066461d* _xmlSchemaGetBuiltInListSimpleTypeItemType
0001:00664657  _xmlSchemaWhiteSpaceReplace
0001:006646dc  _xmlSchemaCollapseString
0001:00664881  _xmlSchemaValPredefTypeNode
0001:006670d5  _xmlSchemaValPredefTypeNodeNoNorm
0001:0066710a  _xmlSchemaValidatePredefinedType
0001:00667133  _xmlSchemaCopyValue
0001:006672bc  _xmlSchemaCompareValues
0001:006677b0  _xmlSchemaCompareValuesWhtsp
0001:006677f7  _xmlSchemaGetFacetValueAsULong
0001:0066780b* _xmlSchemaValidateLengthFacet
0001:00667844  _xmlSchemaValidateLengthFacetWhtsp
0001:00667870  _xmlSchemaValidateFacet
0001:006678c7  _xmlSchemaValidateListSimpleTypeFacet
0001:00667969  _xmlSchemaValidateFacetWhtsp
0001:00667ae2  _xmlSchemaGetCanonValue
0001:00668938* _xmlSchemaGetCanonValueWhtsp
0001:00668a34  _xmlSchemaGetValType
Module: U:\extras\lib\libz.lib(adler32.obj)
0001:00668be0  _adler32
0001:00668e50* _adler32_combine
0001:00668ef8* _adler32_combine64
Module: U:\extras\lib\libz.lib(trees.obj)
0001:00668fa0  __tr_init
0001:0066965c  __tr_stored_block
0001:006697c0  __tr_align
0001:00669b3c* __tr_tally
0001:0066b6d0  __length_code
0001:0066b4d0  __dist_code
0001:0066a9ec  __tr_flush_block
Module: U:\extras\lib\libz.lib(inftrees.obj)
0001:0066bf40  _inflate_table
0001:0066c8f0* _inflate_copyright
Module: U:\extras\lib\libz.lib(inffast.obj)
0001:0066ca70  _inflate_fast
Module: U:\extras\lib\xml2.lib(pattern.obj)
0001:0066e9f5  _xmlFreePattern
0001:0066ead6  _xmlFreePatternList
0001:0066eb04  _xmlFreeStreamCtxt
0001:0066eb3d  _xmlStreamPush
0001:0066eb59  _xmlStreamPushNode
0001:0066eb74  _xmlStreamPushAttr
0001:0066eb90  _xmlStreamPop
0001:0066ebf3  _xmlStreamWantsAnyNode
0001:0066ec2c  _xmlPatterncompile
0001:0066f8bd  _xmlPatternMatch
0001:0066fe42  _xmlPatternGetStreamCtxt
0001:0066ff1b  _xmlPatternStreamable
0001:0066ff4e  _xmlPatternMaxDepth
0001:0066ffb8  _xmlPatternMinDepth
0001:00670009  _xmlPatternFromRoot
Module: U:\extras\lib\xml2.lib(debugXML.obj)
0001:00672efa  _xmlDebugDumpString
0001:00672fd7  _xmlDebugDumpAttr
0001:006730c4* _xmlDebugDumpEntities
0001:00673258* _xmlDebugDumpAttrList
0001:0067334c  _xmlDebugDumpOneNode
0001:006733bc* _xmlDebugDumpNode
0001:00673434* _xmlDebugDumpNodeList
0001:006734ac* _xmlDebugDumpDocumentHead
0001:00673525* _xmlDebugDumpDocument
0001:006735bd* _xmlDebugDumpDTD
0001:006736b3* _xmlDebugCheckDocument
0001:0067372f* _xmlLsCountNode
0001:006737fb* _xmlLsOneNode
0001:00673b47* _xmlBoolToText
0001:00673bf5* _xmlShellPrintXPathError
0001:00673d7a* _xmlShellPrintNode
0001:00673d89* _xmlShellPrintXPathResult
0001:00673d8e* _xmlShellList
0001:00673e2d* _xmlShellBase
0001:00673ecb* _xmlShellDir
0001:00673f5f* _xmlShellCat
0001:00674013* _xmlShellLoad
0001:006740e3* _xmlShellWrite
0001:006741ff* _xmlShellSave
0001:006742b9* _xmlShellValidate
0001:0067435e* _xmlShellDu
0001:006744e0* _xmlShellPwd
0001:00674d05* _xmlShell
Module: U:\extras\lib\xml2.lib(xpointer.obj)
0001:00676e13  _xmlXPtrNewRange
0001:00676e9b* _xmlXPtrNewRangePoints
0001:00676f22* _xmlXPtrNewRangePointNode
0001:00676fa2* _xmlXPtrNewRangeNodePoint
0001:00677027* _xmlXPtrNewRangeNodes
0001:0067709d* _xmlXPtrNewCollapsedRange
0001:00677129  _xmlXPtrNewRangeNodeObject
0001:00677261  _xmlXPtrLocationSetCreate
0001:00677313  _xmlXPtrLocationSetAdd
0001:00677438  _xmlXPtrLocationSetMerge
0001:00677483* _xmlXPtrLocationSetDel
0001:006774db* _xmlXPtrLocationSetRemove
0001:00677518  _xmlXPtrFreeLocationSet
0001:00677578* _xmlXPtrNewLocationSetNodes
0001:006776cb* _xmlXPtrNewLocationSetNodeSet
0001:0067776d  _xmlXPtrWrapLocationSet
0001:006777b8* _xmlXPtrRangeToFunction
0001:006782c5  _xmlXPtrNewContext
0001:00678483  _xmlXPtrEval
0001:00678b04  _xmlXPtrAdvanceNode
0001:00678bac* _xmlXPtrBuildNodeList
0001:0067996e* _xmlXPtrEvalRangePredicate
Module: U:\extras\lib\libcrypto.lib(err.obj)
0001:0067acf0* _ERR_get_implementation
0001:0067ad70* _ERR_set_implementation
0001:0067ade0* _ERR_load_ERR_strings
0001:0067af30* _ERR_load_strings
0001:0067b0c0* _ERR_unload_strings
0001:0067b120* _ERR_free_strings
0001:0067b1e0  _ERR_error_string_n
0001:0067b6a0* _ERR_error_string
0001:0067bb50* _ERR_get_string_table
0001:0067bbf0* _ERR_get_err_state_table
0001:0067bc90* _ERR_release_err_state_table
0001:0067bd30* _ERR_lib_error_string
0001:0067bdf0* _ERR_func_error_string
0001:0067beb0* _ERR_reason_error_string
0001:0067bf90* _ERR_remove_thread_state
0001:0067c060* _ERR_remove_state
0001:0067c070* _ERR_get_state
0001:0067cc80* _ERR_peek_last_error_line_data
0001:0067ccb0* _ERR_peek_last_error_line
0001:0067cce0  _ERR_peek_last_error
0001:0067cd10* _ERR_peek_error_line_data
0001:0067cd40* _ERR_peek_error_line
0001:0067cd70  _ERR_peek_error
0001:0067cda0  _ERR_get_error_line_data
0001:0067cdd0* _ERR_get_error_line
0001:0067ce00* _ERR_get_error
0001:0067ce30  _ERR_clear_error
0001:0067d490  _ERR_put_error
0001:0067d590* _ERR_get_next_error_library
0001:0067d620* _ERR_set_error_data
0001:0067d690  _ERR_add_error_data
0001:0067d7e0  _ERR_set_mark
0001:0067d820  _ERR_pop_to_mark
Module: U:\extras\lib\libssl.lib(ssl_sess.obj)
0001:0067dfb0  _SSL_get_session
0001:0067dfd0* _SSL_get1_session
0001:0067e040* _SSL_SESSION_get_ex_new_index
0001:0067e080* _SSL_SESSION_set_ex_data
0001:0067e0a0* _SSL_SESSION_get_ex_data
0001:0067e0c0  _SSL_SESSION_new
0001:0067e1e0* _SSL_SESSION_get_id
0001:0067e200  _SSL_SESSION_free
0001:0067e670  _SSL_CTX_remove_session
0001:0067e690  _SSL_CTX_add_session
0001:0067e960* _ssl_get_prev_session
0001:0067edd0  _ssl_get_new_session
0001:0067f4c0  _SSL_set_session
0001:0067f660* _SSL_SESSION_set_timeout
0001:0067f690* _SSL_SESSION_get_timeout
0001:0067f6b0* _SSL_SESSION_get_time
0001:0067f6d0* _SSL_SESSION_set_time
0001:0067f700* _SSL_CTX_set_timeout
0001:0067f730* _SSL_CTX_get_timeout
0001:0067f750* _SSL_set_session_secret_cb
0001:0067f790* _SSL_set_session_ticket_ext_cb
0001:0067f7d0* _SSL_set_session_ticket_ext
0001:0067f940  _SSL_CTX_flush_sessions
0001:0067f9e0  _ssl_clear_bad_session
0001:0067fa40* _SSL_CTX_sess_set_new_cb
0001:0067fa50* _SSL_CTX_sess_get_new_cb
0001:0067fa60* _SSL_CTX_sess_set_remove_cb
0001:0067fa70* _SSL_CTX_sess_get_remove_cb
0001:0067fa80* _SSL_CTX_sess_set_get_cb
0001:0067fa90* _SSL_CTX_sess_get_get_cb
0001:0067faa0* _SSL_CTX_set_info_callback
0001:0067fab0* _SSL_CTX_get_info_callback
0001:0067fac0* _SSL_CTX_set_client_cert_cb
0001:0067fad0* _SSL_CTX_get_client_cert_cb
0001:0067fae0* _SSL_CTX_set_client_cert_engine
0001:0067fba0* _SSL_CTX_set_cookie_generate_cb
0001:0067fbb0* _SSL_CTX_set_cookie_verify_cb
0001:0067fbe0* _PEM_read_bio_SSL_SESSION
0001:0067fc20* _PEM_read_SSL_SESSION
0001:0067fc60* _PEM_write_bio_SSL_SESSION
0001:0067fcc0* _PEM_write_SSL_SESSION
Module: U:\extras\lib\libcrypto.lib(buffer.obj)
0001:0067fd40  _BUF_MEM_new
0001:0067fdc0  _BUF_MEM_free
0001:0067fe70  _BUF_MEM_grow
0001:0067ffa0  _BUF_MEM_grow_clean
0001:00680170  _BUF_strdup
0001:00680240  _BUF_strndup
0001:00680310  _BUF_memdup
0001:00680430  _BUF_strlcpy
0001:006804a0  _BUF_strlcat
0001:00680540* _BUF_reverse
Module: U:\extras\lib\libcrypto.lib(evp_enc.obj)
0001:006805b0  _EVP_CIPHER_CTX_init
0001:006805e0* _EVP_CIPHER_CTX_new
0001:006806b0  _EVP_CipherInit_ex
0001:00680bc0* _EVP_CipherInit
0001:00680c10* _EVP_EncryptInit
0001:00680c60  _EVP_EncryptInit_ex
0001:00680ca0* _EVP_DecryptInit
0001:00680cf0  _EVP_DecryptInit_ex
0001:00680d50  _EVP_EncryptUpdate
0001:006810c0* _EVP_EncryptFinal
0001:006812c0  _EVP_EncryptFinal_ex
0001:006814d0  _EVP_DecryptUpdate
0001:00681740  _EVP_CipherUpdate
0001:00681790  _EVP_DecryptFinal_ex
0001:006819f0  _EVP_DecryptFinal
0001:00681a00* _EVP_CipherFinal
0001:00681c10  _EVP_CipherFinal_ex
0001:00681e20* _EVP_CIPHER_CTX_free
0001:00681eb0  _EVP_CIPHER_CTX_cleanup
0001:00681f30  _EVP_CIPHER_CTX_set_key_length
0001:00682050* _EVP_CIPHER_CTX_set_padding
0001:00682080  _EVP_CIPHER_CTX_ctrl
0001:00682170  _EVP_CIPHER_CTX_rand_key
0001:00682240  _EVP_CIPHER_CTX_copy
0001:00682490* _EVP_version
Module: U:\extras\lib\libcrypto.lib(mem.obj)
0001:006824f0* _CRYPTO_set_mem_functions
0001:00682580* _CRYPTO_set_mem_ex_functions
0001:00682610* _CRYPTO_set_locked_mem_functions
0001:00682670* _CRYPTO_set_locked_mem_ex_functions
0001:006826d0* _CRYPTO_set_mem_debug_functions
0001:00682720* _CRYPTO_get_mem_functions
0001:00682790* _CRYPTO_get_mem_ex_functions
0001:00682800* _CRYPTO_get_locked_mem_functions
0001:00682840* _CRYPTO_get_locked_mem_ex_functions
0001:00682880* _CRYPTO_get_mem_debug_functions
0001:006828e0  _CRYPTO_malloc_locked
0001:00682990  _CRYPTO_free_locked
0001:006829e0  _CRYPTO_malloc
0001:00682a90* _CRYPTO_strdup
0001:00682b60  _CRYPTO_realloc
0001:00682ca0  _CRYPTO_realloc_clean
0001:00682ee0  _CRYPTO_free
0001:00682f40* _CRYPTO_remalloc
0001:00683040* _CRYPTO_set_mem_debug_options
0001:00683070* _CRYPTO_get_mem_debug_options
Module: U:\extras\lib\libcrypto.lib(comp_lib.obj)
0001:006830c0  _COMP_CTX_new
0001:00683140  _COMP_CTX_free
0001:00683180  _COMP_compress_block
0001:006831e0  _COMP_expand_block
Module: U:\extras\lib\libcrypto.lib(digest.obj)
0001:00683240  _EVP_MD_CTX_init
0001:00683270  _EVP_MD_CTX_create
0001:006832b0  _EVP_DigestInit_ex
0001:00683540  _EVP_DigestInit
0001:00683570  _EVP_DigestUpdate
0001:006835b0  _EVP_DigestFinal_ex
0001:006836b0  _EVP_MD_CTX_cleanup
0001:00683770  _EVP_MD_CTX_destroy
0001:00683790  _EVP_Digest
0001:00683900  _EVP_MD_CTX_copy_ex
0001:00683b90  _EVP_MD_CTX_copy
0001:00683bb0  _EVP_DigestFinal
Module: U:\extras\lib\libssl.lib(ssl_ciph.obj)
0001:006848b0* _ssl_load_ciphers
0001:00684b10  _ssl_cipher_get_evp
0001:00684dd0  _ssl_get_handshake_digest
0001:00684e50  _ssl_create_cipher_list
0001:00685a10* _SSL_CIPHER_description
0001:00686010* _SSL_CIPHER_get_version
0001:00686060* _SSL_CIPHER_get_name
0001:00686080* _SSL_CIPHER_get_bits
0001:006860b0  _ssl3_comp_find
0001:00686110  _SSL_COMP_get_compression_methods
0001:00686130* _SSL_COMP_add_compression_method
0001:006862e0* _SSL_COMP_get_name
Module: U:\extras\lib\libcrypto.lib(stack.obj)
0001:00687130  _sk_set_cmp_func
0001:00687170  _sk_dup
0001:00687280  _sk_new_null
0001:00687320  _sk_new
0001:006873c0  _sk_insert
0001:00687490  _sk_delete_ptr
0001:00687500  _sk_delete
0001:00687550  _sk_find
0001:00687620* _sk_find_ex
0001:006876f0  _sk_push
0001:00687720* _sk_unshift
0001:00687750* _sk_shift
0001:006877b0  _sk_pop
0001:006877f0  _sk_zero
0001:00687830  _sk_pop_free
0001:006878a0  _sk_free
0001:006878e0  _sk_num
0001:00687900  _sk_value
0001:00687930  _sk_set
0001:00687970  _sk_sort
0001:006879b0  _sk_is_sorted
0001:006879d0* _STACK_version
Module: U:\extras\lib\libcrypto.lib(cryptlib.obj)
0001:00687a20* _CRYPTO_get_new_lockid
0001:00687ae0* _CRYPTO_num_locks
0001:00687af0* _CRYPTO_get_dynlock_create_callback
0001:00687b00* _CRYPTO_get_dynlock_lock_callback
0001:00687b10* _CRYPTO_get_dynlock_destroy_callback
0001:00687b20* _CRYPTO_set_dynlock_create_callback
0001:00687b30* _CRYPTO_set_dynlock_lock_callback
0001:00687b40* _CRYPTO_set_dynlock_destroy_callback
0001:00687b50* _CRYPTO_get_locking_callback
0001:00687b60* _CRYPTO_get_add_lock_callback
0001:00687b70* _CRYPTO_set_locking_callback
0001:00687b80* _CRYPTO_set_add_lock_callback
0001:00687b90* _CRYPTO_THREADID_set_numeric
0001:00687bb0* _CRYPTO_THREADID_set_pointer
0001:00687bc0* _CRYPTO_THREADID_set_callback
0001:00687be0* _CRYPTO_THREADID_get_callback
0001:00687bf0  _CRYPTO_THREADID_current
0001:00687c40  _CRYPTO_THREADID_cmp
0001:00687c60  _CRYPTO_THREADID_cpy
0001:00687c80  _CRYPTO_THREADID_hash
0001:00687c90* _CRYPTO_get_id_callback
0001:00687ca0* _CRYPTO_set_id_callback
0001:00687cb0* _CRYPTO_thread_id
0001:00687cf0* _CRYPTO_get_lock_name
0001:00687d60* _OPENSSL_ia32cap_loc
0001:00687d80  _OPENSSL_cpuid_setup
0001:00687df0* _OPENSSL_showfatal
0001:00687e20* _CRYPTO_destroy_dynlockid
0001:00687f50* _CRYPTO_get_dynlock_value
0001:00688050  _CRYPTO_lock
0001:00688110  _CRYPTO_add_lock
0001:00688290* _CRYPTO_get_new_dynlockid
0001:00688530* _OPENSSL_isservice
0001:00688540  _OpenSSLDie
0001:00688570* _OPENSSL_stderr
0002:00021510  _OPENSSL_ia32cap_P
0002:00021514* _OPENSSL_NONPIC_relocated
Module: U:\extras\lib\libcrypto.lib(lhash.obj)
0001:00688770  _lh_strhash
0001:006887f0  _lh_new
0001:006889a0  _lh_free
0001:00688a10  _lh_insert
0001:00688c20  _lh_delete
0001:00688db0  _lh_retrieve
0001:00688e50  _lh_doall
0001:00688eb0  _lh_doall_arg
0001:00688f20  _lh_num_items
0001:00688f40* _lh_version
Module: U:\extras\lib\libcrypto.lib(x509_vpm.obj)
0001:00688fc0  _X509_VERIFY_PARAM_free
0001:00689040  _X509_VERIFY_PARAM_new
0001:006890d0  _X509_VERIFY_PARAM_inherit
0001:006892e0  _X509_VERIFY_PARAM_set1
0001:00689310* _X509_VERIFY_PARAM_set1_name
0001:00689350  _X509_VERIFY_PARAM_set_flags
0001:00689380* _X509_VERIFY_PARAM_clear_flags
0001:006893a0* _X509_VERIFY_PARAM_get_flags
0001:006893b0  _X509_VERIFY_PARAM_set_purpose
0001:006893d0  _X509_VERIFY_PARAM_set_trust
0001:006893f0  _X509_VERIFY_PARAM_set_depth
0001:00689400  _X509_VERIFY_PARAM_set_time
0001:00689410* _X509_VERIFY_PARAM_add0_policy
0001:00689450* _X509_VERIFY_PARAM_set1_policies
0001:00689540  _X509_VERIFY_PARAM_get_depth
0001:00689550* _X509_VERIFY_PARAM_add0_table
0001:00689640  _X509_VERIFY_PARAM_lookup
0001:006896d0* _X509_VERIFY_PARAM_table_cleanup
Module: U:\extras\lib\libcrypto.lib(bio_lib.obj)
0001:006897f0  _BIO_new
0001:00689910  _BIO_set
0001:006899d0  _BIO_free
0001:00689ab0  _BIO_vfree
0001:00689b60  _BIO_clear_flags
0001:00689b70  _BIO_test_flags
0001:00689b80  _BIO_set_flags
0001:00689b90* _BIO_get_callback
0001:00689ba0* _BIO_set_callback
0001:00689bb0* _BIO_set_callback_arg
0001:00689bc0* _BIO_get_callback_arg
0001:00689bd0* _BIO_method_name
0001:00689be0  _BIO_method_type
0001:00689bf0  _BIO_read
0001:00689d20  _BIO_write
0001:00689e50  _BIO_puts
0001:00689f80  _BIO_gets
0001:0068a0b0  _BIO_indent
0001:0068a240  _BIO_int_ctrl
0001:0068a360* _BIO_ptr_ctrl
0001:0068a480  _BIO_ctrl
0001:0068a590  _BIO_callback_ctrl
0001:0068a690* _BIO_ctrl_pending
0001:0068a7c0* _BIO_ctrl_wpending
0001:0068a8f0  _BIO_push
0001:0068aa30  _BIO_pop
0001:0068ab70* _BIO_get_retry_BIO
0001:0068aba0  _BIO_get_retry_reason
0001:0068abb0  _BIO_find_type
0001:0068ac00  _BIO_next
0001:0068ac20  _BIO_free_all
0001:0068ad10* _BIO_dup_chain
0001:0068b260  _BIO_copy_next_retry
0001:0068b280* _BIO_get_ex_new_index
0001:0068b2c0* _BIO_set_ex_data
0001:0068b2e0* _BIO_get_ex_data
0001:0068b300* _BIO_number_read
0001:0068b320* _BIO_number_written
Module: U:\extras\lib\libcrypto.lib(bss_sock.obj)
0001:0068b700  _BIO_s_socket
0001:0068b710* _BIO_new_socket
0001:0068b750* _BIO_sock_should_retry
0001:0068b7b0* _BIO_sock_non_fatal_error
Module: U:\extras\lib\libssl.lib(ssl_cert.obj)
0001:0068b840  _SSL_get_ex_data_X509_STORE_CTX_idx
0001:0068b960  _ssl_cert_new
0001:0068b9e0  _ssl_cert_dup
0001:0068c0a0  _ssl_cert_free
0001:0068c210  _ssl_cert_inst
0001:0068c320  _ssl_sess_cert_new
0001:0068c3a0  _ssl_sess_cert_free
0001:0068c4b0  _ssl_set_peer_cert_type
0001:0068c4e0  _ssl_verify_cert_chain
0001:0068c760* _SSL_dup_CA_list
0001:0068c7e0* _SSL_set_client_CA_list
0001:0068c820* _SSL_CTX_set_client_CA_list
0001:0068c860* _SSL_CTX_get_client_CA_list
0001:0068c870  _SSL_get_client_CA_list
0001:0068c8c0* _SSL_add_client_CA
0001:0068c950* _SSL_CTX_add_client_CA
0001:0068c9e0* _SSL_load_client_CA_file
0001:0068cb90* _SSL_add_file_cert_subjects_to_stack
0001:0068cd40* _SSL_add_dir_cert_subjects_to_stack
Module: U:\extras\lib\libcrypto.lib(x509_cmp.obj)
0001:0068cf20* _X509_issuer_and_serial_cmp
0001:0068cfe0* _X509_issuer_and_serial_hash
0001:0068d0c0* _X509_issuer_name_cmp
0001:0068d160  _X509_subject_name_cmp
0001:0068d200  _X509_CRL_cmp
0001:0068d2a0  _X509_CRL_match
0001:0068d2d0  _X509_get_issuer_name
0001:0068d2e0* _X509_issuer_name_hash
0001:0068d360* _X509_issuer_name_hash_old
0001:0068d3e0  _X509_get_subject_name
0001:0068d3f0  _X509_get_serialNumber
0001:0068d400* _X509_subject_name_hash
0001:0068d480* _X509_subject_name_hash_old
0001:0068d500  _X509_cmp
0001:0068d560  _X509_NAME_cmp
0001:0068d5f0  _X509_NAME_hash
0001:0068d670* _X509_NAME_hash_old
0001:0068d6f0  _X509_find_by_issuer_and_serial
0001:0068d7f0* _X509_find_by_subject
0001:0068d8c0  _X509_get_pubkey
0001:0068d900  _X509_get0_pubkey_bitstr
0001:0068d940  _X509_check_private_key
Module: U:\extras\lib\libssl.lib(s3_pkt.obj)
0001:0068da70* _ssl3_read_n
0001:0068de10* _ssl3_do_uncompress
0001:0068de80* _ssl3_do_compress
0001:0068def0* _ssl3_write_pending
0001:0068e5a0  _ssl3_write_bytes
0001:0068e6f0* _ssl3_do_change_cipher_spec
0001:0068e820  _ssl3_read_bytes
0001:0068fae0  _ssl3_send_alert
0001:0068fbb0  _ssl3_dispatch_alert
Module: U:\extras\lib\libcrypto.lib(ex_data.obj)
0001:006909a0* _CRYPTO_get_ex_data_implementation
0001:00690a20* _CRYPTO_set_ex_data_implementation
0001:00690a90* _CRYPTO_ex_data_new_class
0001:00690b20* _CRYPTO_cleanup_all_ex_data
0001:00690bb0  _CRYPTO_get_ex_new_index
0001:00690c90  _CRYPTO_new_ex_data
0001:00690d40  _CRYPTO_dup_ex_data
0001:00690df0  _CRYPTO_free_ex_data
0001:00690ea0  _CRYPTO_set_ex_data
0001:00690f70  _CRYPTO_get_ex_data
Module: U:\extras\lib\libcrypto.lib(x509_lu.obj)
0001:006911d0* _X509_LOOKUP_new
0001:00691250* _X509_LOOKUP_free
0001:00691290* _X509_LOOKUP_init
0001:006912d0* _X509_LOOKUP_shutdown
0001:00691310  _X509_LOOKUP_ctrl
0001:00691350* _X509_LOOKUP_by_subject
0001:00691390* _X509_LOOKUP_by_issuer_serial
0001:006913c0* _X509_LOOKUP_by_fingerprint
0001:006913f0* _X509_LOOKUP_by_alias
0001:00691420  _X509_STORE_new
0001:00691520  _X509_STORE_free
0001:006915f0  _X509_STORE_add_lookup
0001:006916d0* _X509_STORE_get_by_subject
0001:00691900* _X509_OBJECT_up_ref_count
0001:00691990* _X509_OBJECT_free_contents
0001:006919d0* _X509_OBJECT_idx_by_subject
0001:006919f0* _X509_OBJECT_retrieve_by_subject
0001:00691a40  _X509_STORE_get1_certs
0001:00691c80  _X509_STORE_get1_crls
0001:00691f00* _X509_OBJECT_retrieve_match
0001:00692020  _X509_STORE_add_crl
0001:00692230  _X509_STORE_add_cert
0001:00692440  _X509_STORE_CTX_get1_issuer
0001:00692750* _X509_STORE_set_flags
0001:00692770* _X509_STORE_set_depth
0001:006927a0* _X509_STORE_set_purpose
0001:006927c0* _X509_STORE_set_trust
0001:006927e0* _X509_STORE_set1_param
0001:00692800* _X509_STORE_set_verify_cb
Module: U:\extras\lib\libcrypto.lib(x_name.obj)
0001:006929f0  _X509_NAME_ENTRY_free
0001:006935d0  _X509_NAME_ENTRY_it
0001:00693600* _X509_NAME_ENTRIES_it
0001:00693630* _X509_NAME_INTERNAL_it
0001:006933e0* _d2i_X509_NAME_ENTRY
0001:00693410* _i2d_X509_NAME_ENTRY
0001:00693440  _X509_NAME_ENTRY_new
0001:00693460  _X509_NAME_ENTRY_dup
0001:00693480  _d2i_X509_NAME
0001:00693680  _X509_NAME_it
0001:006934b0  _i2d_X509_NAME
0001:006934e0  _X509_NAME_new
0001:00693500  _X509_NAME_free
0001:00693520  _X509_NAME_dup
0001:00693540  _X509_NAME_set
0001:00693650* _x509_name_ff
Module: U:\extras\lib\libcrypto.lib(x_x509.obj)
0001:006938a0* _d2i_X509_CINF
0001:00693b50  _X509_CINF_it
0001:006938d0* _i2d_X509_CINF
0001:00693900* _X509_CINF_new
0001:00693920* _X509_CINF_free
0001:00693940  _d2i_X509
0001:00693b80  _X509_it
0001:00693970  _i2d_X509
0001:006939a0* _X509_new
0001:006939c0  _X509_free
0001:006939e0* _X509_dup
0001:00693a00* _X509_get_ex_new_index
0001:00693a40* _X509_set_ex_data
0001:00693a60* _X509_get_ex_data
0001:00693a80  _d2i_X509_AUX
0001:00693b00  _i2d_X509_AUX
Module: U:\extras\lib\libcrypto.lib(eng_init.obj)
0001:00693d60  _engine_unlocked_init
0001:00693dc0  _engine_unlocked_finish
0001:00693eb0  _ENGINE_init
0001:00693f80  _ENGINE_finish
Module: U:\extras\lib\libcrypto.lib(names.obj)
0001:00694230* _EVP_add_cipher
0001:00694290* _EVP_add_digest
0001:00694360  _EVP_get_cipherbyname
0001:00694380  _EVP_get_digestbyname
0001:006943a0* _EVP_cleanup
0001:00694400* _EVP_CIPHER_do_all
0001:00694440* _EVP_CIPHER_do_all_sorted
0001:00694480* _EVP_MD_do_all
0001:006944c0* _EVP_MD_do_all_sorted
Module: U:\extras\lib\libcrypto.lib(rand_lib.obj)
0001:00694500  _RAND_set_rand_method
0001:00694530* _RAND_get_rand_method
0001:00694590* _RAND_set_rand_engine
0001:00694620* _RAND_cleanup
0001:006946a0  _RAND_seed
0001:00694730  _RAND_add
0001:006947d0  _RAND_bytes
0001:00694860  _RAND_pseudo_bytes
0001:006948f0  _RAND_status
Module: U:\extras\lib\libcrypto.lib(x_exten.obj)
0001:00694970* _d2i_X509_EXTENSION
0001:00694aa0  _X509_EXTENSION_it
0001:006949a0* _i2d_X509_EXTENSION
0001:006949d0  _X509_EXTENSION_new
0001:006949f0  _X509_EXTENSION_free
0001:00694a10  _d2i_X509_EXTENSIONS
0001:00694ad0  _X509_EXTENSIONS_it
0001:00694a40  _i2d_X509_EXTENSIONS
0001:00694a70  _X509_EXTENSION_dup
Module: U:\extras\lib\libcrypto.lib(ocsp_asn.obj)
0001:00694b80* _d2i_OCSP_SIGNATURE
0001:006954f0* _OCSP_SIGNATURE_it
0001:00694bb0* _i2d_OCSP_SIGNATURE
0001:00694be0* _OCSP_SIGNATURE_new
0001:00694c00* _OCSP_SIGNATURE_free
0001:00694c20* _d2i_OCSP_CERTID
0001:00695520* _OCSP_CERTID_it
0001:00694c50* _i2d_OCSP_CERTID
0001:00694c80* _OCSP_CERTID_new
0001:00694ca0* _OCSP_CERTID_free
0001:00694cc0* _d2i_OCSP_ONEREQ
0001:00695550* _OCSP_ONEREQ_it
0001:00694cf0* _i2d_OCSP_ONEREQ
0001:00694d20* _OCSP_ONEREQ_new
0001:00694d40* _OCSP_ONEREQ_free
0001:00694d60* _d2i_OCSP_REQINFO
0001:00695580* _OCSP_REQINFO_it
0001:00694d90* _i2d_OCSP_REQINFO
0001:00694dc0* _OCSP_REQINFO_new
0001:00694de0* _OCSP_REQINFO_free
0001:00694e00* _d2i_OCSP_REQUEST
0001:006955b0* _OCSP_REQUEST_it
0001:00694e30* _i2d_OCSP_REQUEST
0001:00694e60* _OCSP_REQUEST_new
0001:00694e80* _OCSP_REQUEST_free
0001:00694ea0* _d2i_OCSP_RESPBYTES
0001:006955e0* _OCSP_RESPBYTES_it
0001:00694ed0* _i2d_OCSP_RESPBYTES
0001:00694f00* _OCSP_RESPBYTES_new
0001:00694f20* _OCSP_RESPBYTES_free
0001:00694f40* _d2i_OCSP_RESPONSE
0001:00695610* _OCSP_RESPONSE_it
0001:00694f70* _i2d_OCSP_RESPONSE
0001:00694fa0* _OCSP_RESPONSE_new
0001:00694fc0* _OCSP_RESPONSE_free
0001:00694fe0  _d2i_OCSP_RESPID
0001:00695640* _OCSP_RESPID_it
0001:00695010  _i2d_OCSP_RESPID
0001:00695040* _OCSP_RESPID_new
0001:00695060  _OCSP_RESPID_free
0001:00695080* _d2i_OCSP_REVOKEDINFO
0001:00695670* _OCSP_REVOKEDINFO_it
0001:006950b0* _i2d_OCSP_REVOKEDINFO
0001:006950e0* _OCSP_REVOKEDINFO_new
0001:00695100* _OCSP_REVOKEDINFO_free
0001:00695120* _d2i_OCSP_CERTSTATUS
0001:006956a0* _OCSP_CERTSTATUS_it
0001:00695150* _i2d_OCSP_CERTSTATUS
0001:00695180* _OCSP_CERTSTATUS_new
0001:006951a0* _OCSP_CERTSTATUS_free
0001:006951c0* _d2i_OCSP_SINGLERESP
0001:006956d0* _OCSP_SINGLERESP_it
0001:006951f0* _i2d_OCSP_SINGLERESP
0001:00695220* _OCSP_SINGLERESP_new
0001:00695240* _OCSP_SINGLERESP_free
0001:00695260* _d2i_OCSP_RESPDATA
0001:00695700* _OCSP_RESPDATA_it
0001:00695290* _i2d_OCSP_RESPDATA
0001:006952c0* _OCSP_RESPDATA_new
0001:006952e0* _OCSP_RESPDATA_free
0001:00695300* _d2i_OCSP_BASICRESP
0001:00695730* _OCSP_BASICRESP_it
0001:00695330* _i2d_OCSP_BASICRESP
0001:00695360* _OCSP_BASICRESP_new
0001:00695380* _OCSP_BASICRESP_free
0001:006953a0* _d2i_OCSP_CRLID
0001:00695760  _OCSP_CRLID_it
0001:006953d0* _i2d_OCSP_CRLID
0001:00695400* _OCSP_CRLID_new
0001:00695420* _OCSP_CRLID_free
0001:00695440* _d2i_OCSP_SERVICELOC
0001:00695790  _OCSP_SERVICELOC_it
0001:00695470* _i2d_OCSP_SERVICELOC
0001:006954a0* _OCSP_SERVICELOC_new
0001:006954c0* _OCSP_SERVICELOC_free
Module: U:\extras\lib\libcrypto.lib(p_lib.obj)
0001:00695f20  _EVP_PKEY_bits
0001:00695f50  _EVP_PKEY_size
0001:00695f80* _EVP_PKEY_save_parameters
0001:00695fb0  _EVP_PKEY_copy_parameters
0001:00696080  _EVP_PKEY_missing_parameters
0001:006960b0  _EVP_PKEY_cmp_parameters
0001:006960f0  _EVP_PKEY_cmp
0001:00696150  _EVP_PKEY_new
0001:006961f0  _EVP_PKEY_set_type
0001:00696210  _EVP_PKEY_set_type_str
0001:00696230  _EVP_PKEY_assign
0001:00696280* _EVP_PKEY_get0
0001:00696290  _EVP_PKEY_set1_RSA
0001:006962e0  _EVP_PKEY_get1_RSA
0001:00696340  _EVP_PKEY_set1_DSA
0001:00696390  _EVP_PKEY_get1_DSA
0001:006963f0  _EVP_PKEY_set1_EC_KEY
0001:00696440  _EVP_PKEY_get1_EC_KEY
0001:006964b0* _EVP_PKEY_set1_DH
0001:00696500* _EVP_PKEY_get1_DH
0001:00696560  _EVP_PKEY_type
0001:006965b0  _EVP_PKEY_id
0001:006965c0* _EVP_PKEY_base_id
0001:00696610  _EVP_PKEY_free
0001:006966d0  _EVP_PKEY_print_public
0001:00696760  _EVP_PKEY_print_private
0001:006967e0  _EVP_PKEY_print_params
0001:00696860  _EVP_PKEY_get_default_digest_nid
Module: U:\extras\lib\libcrypto.lib(v3_purp.obj)
0001:006976e0  _X509_check_purpose
0001:00697810  _X509_PURPOSE_set
0001:00697890* _X509_PURPOSE_get_count
0001:006978c0  _X509_PURPOSE_get0
0001:00697920* _X509_PURPOSE_get_by_sname
0001:006979b0  _X509_PURPOSE_get_by_id
0001:00697a00* _X509_PURPOSE_add
0001:00697be0* _X509_PURPOSE_cleanup
0001:00697e30* _X509_PURPOSE_get_id
0001:00697e40* _X509_PURPOSE_get0_name
0001:00697e50* _X509_PURPOSE_get0_sname
0001:00697e60* _X509_PURPOSE_get_trust
0001:00697e70* _X509_supported_extension
0001:00697ee0  _X509_check_ca
0001:00697fc0  _X509_check_akid
0001:006980a0  _X509_check_issued
Module: U:\extras\lib\libcrypto.lib(obj_dat.obj)
0001:00698530  _check_defer
0001:00698550  _OBJ_cleanup
0001:006985e0* _OBJ_new_nid
0001:00698610* _OBJ_add_object
0001:00698890  _OBJ_nid2obj
0001:00698940  _OBJ_nid2sn
0001:006989f0  _OBJ_nid2ln
0001:00698aa0  _OBJ_obj2nid
0001:00698ba0  _OBJ_txt2obj
0001:00698f30  _OBJ_obj2txt
0001:00699560* _OBJ_txt2nid
0001:006999f0  _OBJ_ln2nid
0001:00699ae0  _OBJ_sn2nid
0001:00699bd0  _OBJ_bsearch_
0001:00699c50  _OBJ_bsearch_ex_
0001:00699d40* _OBJ_create_objects
0001:00699fb0* _OBJ_create
0002:00021620  _obj_cleanup_defer
Module: U:\extras\lib\libcrypto.lib(rsa_lib.obj)
0001:006a7fd0  _RSA_new
0001:006a81c0* _RSA_set_default_method
0001:006a81d0* _RSA_get_default_method
0001:006a81f0* _RSA_get_method
0001:006a8200* _RSA_set_method
0001:006a8250* _RSA_new_method
0001:006a84b0  _RSA_free
0001:006a85e0  _RSA_up_ref
0001:006a8620* _RSA_get_ex_new_index
0001:006a8660* _RSA_set_ex_data
0001:006a8680* _RSA_get_ex_data
0001:006a86a0  _RSA_size
0001:006a86e0  _RSA_public_encrypt
0001:006a8700  _RSA_private_encrypt
0001:006a8720  _RSA_private_decrypt
0001:006a8740  _RSA_public_decrypt
0001:006a8760  _RSA_flags
0001:006a8780* _RSA_blinding_off
0001:006a87b0  _RSA_setup_blinding
0001:006a8af0* _RSA_blinding_on
0001:006a8b60* _RSA_memory_lock
0001:006a8e20* _RSA_version
Module: U:\extras\lib\libcrypto.lib(dh_lib.obj)
0001:006a8e50* _DH_set_default_method
0001:006a8e60* _DH_get_default_method
0001:006a8e80* _DH_set_method
0001:006a8ef0  _DH_new
0001:006a90b0* _DH_new_method
0001:006a92e0  _DH_free
0001:006a93e0  _DH_up_ref
0001:006a9420* _DH_get_ex_new_index
0001:006a9460* _DH_set_ex_data
0001:006a9480* _DH_get_ex_data
0001:006a94a0  _DH_size
0001:006a94e0* _DH_version
Module: U:\extras\lib\libcrypto.lib(bf_buff.obj)
0001:006aa1d0  _BIO_f_buffer
Module: U:\extras\lib\libcrypto.lib(x509_d2.obj)
0001:006aa1e0  _X509_STORE_set_default_paths
0001:006aa290  _X509_STORE_load_locations
Module: U:\extras\lib\libssl.lib(s3_clnt.obj)
0001:006aa390  _SSLv3_client_method
0001:006aa3b0* _ssl3_client_hello
0001:006aa870* _ssl3_get_server_hello
0001:006ab030* _ssl3_get_server_certificate
0001:006ab690* _ssl3_get_key_exchange
0001:006aca80* _ssl3_get_certificate_request
0001:006acf60* _ssl3_get_new_session_ticket
0001:006ad290* _ssl3_get_cert_status
0001:006ad4b0* _ssl3_get_server_done
0001:006ad550* _ssl3_send_client_key_exchange
0001:006ae6c0* _ssl3_send_client_verify
0001:006aeac0* _ssl3_send_client_certificate
0001:006aed40* _ssl3_check_cert_and_algorithm
0001:006af1c0  _ssl3_connect
0001:006afd20* _ssl3_check_finished
0001:006afdc0* _ssl_do_client_cert_cb
Module: U:\extras\lib\libssl.lib(s2_clnt.obj)
0001:006aff00  _SSLv2_client_method
0001:006aff20* _ssl2_set_certificate
0001:006b0130* _ssl2_connect
Module: U:\extras\lib\libssl.lib(t1_clnt.obj)
0001:006b1fc0  _TLSv1_client_method
Module: U:\extras\lib\libssl.lib(s3_both.obj)
0001:006b2050  _ssl3_do_write
0001:006b2170  _ssl3_send_finished
0001:006b24a0  _ssl3_get_finished
0001:006b2770  _ssl3_send_change_cipher_spec
0001:006b27c0  _ssl3_output_cert_chain
0001:006b2c30  _ssl3_get_message
0001:006b3040  _ssl_cert_type
0001:006b3120  _ssl_verify_alarm_type
0001:006b3150  _ssl3_setup_read_buffer
0001:006b3310  _ssl3_setup_write_buffer
0001:006b34d0  _ssl3_setup_buffers
0001:006b3510  _ssl3_release_write_buffer
0001:006b3610  _ssl3_release_read_buffer
Module: U:\extras\lib\libssl.lib(s3_enc.obj)
0001:006b3800  _ssl3_change_cipher_state
0001:006b3f60  _ssl3_setup_key_block
0001:006b4510  _ssl3_cleanup_key_block
0001:006b4570  _ssl3_enc
0001:006b4770  _ssl3_init_finished_mac
0001:006b4860  _ssl3_free_digest_list
0001:006b48f0  _ssl3_finish_mac
0001:006b49c0  _ssl3_digest_cached_records
0001:006b4e10  _ssl3_cert_verify_mac
0001:006b4e40  _ssl3_final_finish_mac
0001:006b4e90  _n_ssl3_mac
0001:006b50f0* _ssl3_record_sequence_update
0001:006b5150  _ssl3_generate_master_secret
0001:006b54f0  _ssl3_alert_code
Module: U:\extras\lib\libssl.lib(s23_pkt.obj)
0001:006b56f0  _ssl23_write_bytes
0001:006b5760  _ssl23_read_bytes
Module: U:\extras\lib\libssl.lib(s2_lib.obj)
0001:006b57d0  _ssl2_default_timeout
0001:006b57e0  _ssl2_num_ciphers
0001:006b57f0  _ssl2_get_cipher
0001:006b6000* _ssl2_ciphers
0001:006b5820  _ssl2_pending
0001:006b5860  _ssl2_new
0001:006b5960  _ssl2_free
0001:006b59c0  _ssl2_clear
0001:006b5a00  _ssl2_ctrl
0001:006b5a20  _ssl2_callback_ctrl
0001:006b5a30  _ssl2_ctx_ctrl
0001:006b5a40  _ssl2_ctx_callback_ctrl
0001:006b5a50  _ssl2_get_cipher_by_char
0001:006b5ab0  _ssl2_put_cipher_by_char
0001:006b5b80  _ssl2_generate_key_material
0001:006b5d90  _ssl2_return_error
0001:006b5e80  _ssl2_write_error
0001:006b5f60  _ssl2_shutdown
0001:006b5f80* _ssl2_version_str
Module: U:\extras\lib\libssl.lib(s3_lib.obj)
0001:006b6150  _ssl3_default_timeout
0001:006b6160  _ssl3_num_ciphers
0001:006b6170  _ssl3_get_cipher
0001:006b61a0  _ssl3_pending
0001:006b61f0  _ssl3_new
0001:006b6250  _ssl3_free
0001:006b6350  _ssl3_clear
0001:006b64a0  _ssl3_ctrl
0001:006b6b80  _ssl3_callback_ctrl
0001:006b6c80  _ssl3_ctx_ctrl
0001:006b7300  _ssl3_ctx_callback_ctrl
0001:006b73a0  _ssl3_get_cipher_by_char
0001:006b7400  _ssl3_put_cipher_by_char
0001:006b7450* _ssl3_choose_cipher
0001:006b7af0* _ssl3_get_req_cert_type
0001:006b7bf0  _ssl3_shutdown
0001:006b7cf0  _ssl3_write
0001:006b7e40  _ssl3_read
0001:006b7f60  _ssl3_peek
0001:006b8080  _ssl3_renegotiate
0001:006b80d0  _ssl3_renegotiate_check
0001:006b8140* _ssl3_version_str
0002:000077f0* _ssl3_ciphers
0002:000088d0  _SSLv3_enc_data
Module: U:\extras\lib\libssl.lib(t1_lib.obj)
0001:006b8b90  _tls1_default_timeout
0001:006b8ba0  _tls1_new
0001:006b8be0  _tls1_free
0001:006b8c10  _tls1_clear
0001:006b8c30  _tls1_ec_curve_id2nid
0001:006b8c60  _tls1_ec_nid2curve_id
0001:006b8f00  _ssl_add_clienthello_tlsext
0001:006b9810* _ssl_add_serverhello_tlsext
0001:006b9c30* _ssl_parse_clienthello_tlsext
0001:006ba6f0  _ssl_parse_serverhello_tlsext
0001:006bac20  _ssl_prepare_clienthello_tlsext
0001:006bad90* _ssl_prepare_serverhello_tlsext
0001:006bae70* _ssl_check_clienthello_tlsext
0001:006bb020  _ssl_check_serverhello_tlsext
0001:006bb290  _tls1_process_ticket
0001:006bb450* _tls1_version_str
0002:00008910  _TLSv1_enc_data
Module: U:\extras\lib\libssl.lib(s23_lib.obj)
0001:006bb540  _ssl23_default_timeout
0001:006bb550  _ssl23_num_ciphers
0001:006bb570  _ssl23_get_cipher
0001:006bb5a0  _ssl23_get_cipher_by_char
0001:006bb5d0  _ssl23_put_cipher_by_char
0001:006bb610  _ssl23_read
0001:006bb6d0  _ssl23_peek
0001:006bb790  _ssl23_write
Module: U:\extras\lib\xmlrpc.lib(queue.obj)
0001:006bb850  _Q_Init
0001:006bb883* _Q_AtHead
0001:006bb89c* _Q_AtTail
0001:006bb8b6* _Q_IsEmpty
0001:006bb8d0  _Q_Size
0001:006bb8e1  _Q_Head
0001:006bb8ff* _Q_Tail
0001:006bb91e  _Q_Next
0001:006bb941* _Q_Previous
0001:006bb960* _Q_Get
0001:006bb979* _Q_Put
0001:006bb99e* _Q_Find
0001:006bbb16* _Q_Iter_Head
0001:006bbb26* _Q_Iter_Tail
0001:006bbb37* _Q_Iter_Next
0001:006bbb48* _Q_Iter_Prev
0001:006bbb59* _Q_Iter_Get
0001:006bbb69* _Q_Iter_Put
0001:006bbb81* _Q_PopTail
0001:006bbbfb* _Q_PopHead
0001:006bbc73  _Q_Destroy
0001:006bbc98  _Q_Iter_Del
0001:006bbd2d* _Q_DelCur
0001:006bbd4d* _Q_Sort
0001:006bbe95* _Q_Seek
0001:006bbf46  _Q_PushTail
0001:006bbfbc* _Q_PushHead
0001:006bc02d* _Q_Insert
Module: U:\extras\lib\xmlrpc.lib(simplestring.obj)
0001:006bc070  _simplestring_clear
0001:006bc088  _simplestring_addn
0001:006bc17a  _simplestring_add
0001:006bc1be  _simplestring_free
0001:006bc1ed  _simplestring_init
Module: U:\extras\lib\xmlrpc.lib(system_methods.obj)
0001:006bc238  _xsm_register
Module: U:\extras\lib\xmlrpc.lib(xml_element.obj)
0001:006beb52* _xml_elem_serialize_to_stream
0001:006beb93  _xml_elem_serialize_to_string
0001:006bebda  _xml_elem_new
0001:006becc6  _xml_elem_free_non_recurse
0001:006bee11  _xml_elem_parse_buf
0001:006bf085  _xml_elem_free
Module: U:\extras\lib\xmlrpc.lib(xml_to_xmlrpc.obj)
0001:006bf159* _XMLRPC_to_xml_element_worker
0001:006bf6b8  _XMLRPC_REQUEST_to_xml_element
0001:006bf7df  _XMLRPC_VALUE_to_xml_element
0001:006bf80d* _xml_element_to_XMLRPC_REQUEST_worker
0001:006bfd45  _xml_element_to_XMLRPC_REQUEST
0001:006bfd8a* _xml_element_to_XMLRPC_VALUE
Module: U:\extras\lib\xmlrpc.lib(xml_to_soap.obj)
0001:006bff14* _SOAP_to_xml_element_worker
0001:006c06a6  _SOAP_REQUEST_to_xml_element
0001:006c0987* _SOAP_VALUE_to_xml_element
0001:006c0a64* _xml_element_to_SOAP_REQUEST_worker
0001:006c1241  _xml_element_to_SOAP_REQUEST
0001:006c1296* _xml_element_to_SOAP_VALUE
Module: U:\extras\lib\xmlrpc.lib(xml_to_dandarpc.obj)
0001:006c1371* _DANDARPC_to_xml_element_worker
0001:006c1851  _DANDARPC_REQUEST_to_xml_element
0001:006c1983* _DANDARPC_VALUE_to_xml_element
0001:006c199e* _xml_element_to_DANDARPC_REQUEST_worker
0001:006c1dca  _xml_element_to_DANDARPC_REQUEST
0001:006c1e07* _xml_element_to_DANDARPC_VALUE
Module: U:\extras\lib\pthread.lib(my_os2key.obj)
0001:006c1e30  _pthread_setspecific
0001:006c1e52  _pthread_getspecific
0001:006c1e5e  _pthread_key_delete
0001:006c1e6a  _pthread_key_create
Module: U:\extras\lib\pthread.lib(my_os2thread.obj)
0001:006c1e90  _pthread_equal
0001:006c1ea1* _pthread_dummy
0001:006c1ea9* _pthread_cleanup_push
0001:006c1eae* _pthread_cleanup_pop
0001:006c1eb3* _pthread_setcancelstate
0001:006c1eba* _pthread_setcanceltype
0001:006c1ec1* _pthread_testcancel
0001:006c1ec6* _pthread_atfork
0001:006c1ecd* _pthread_kill
0001:006c1f1c* _pthread_detach
0001:006c1f7c  _pthread_once
0001:006c1fed* _pthread_yield
0001:006c2001  _pthread_self
0001:006c205e* _pthread_setprio
0001:006c2088* _pthread_exit
0001:006c20e0* _pthread_create
0001:006c22fe* _pthread_join
Module: U:\extras\lib\pthread.lib(my_os2mutex.obj)
0001:006c23c0* _pthread_mutexattr_settype
0001:006c23e8* _pthread_mutexattr_gettype
0001:006c240f* _pthread_mutexattr_destroy
0001:006c243b* _pthread_mutexattr_init
0001:006c2476  _pthread_mutex_destroy
0001:006c24ab  _pthread_mutex_init
0001:006c24d8* _pthread_mutex_trylock
0001:006c254b  _pthread_mutex_lock
0001:006c25a4  _pthread_mutex_unlock
Module: U:\extras\lib\pthread.lib(my_os2cond.obj)
0001:006c2610  _pthread_cond_destroy
0001:006c2649  _pthread_cond_init
0001:006c269c  _pthread_cond_wait
0001:006c273e* _pthread_cond_broadcast
0001:006c27aa  _pthread_cond_signal
0001:006c280f* _pthread_cond_timedwait
Module: U:\extras\lib\xml2.lib(xmlunicode.obj)
0001:006c2920* _xmlUCSIsAegeanNumbers
0001:006c2936* _xmlUCSIsAlphabeticPresentationForms
0001:006c294c* _xmlUCSIsArabic
0001:006c2964* _xmlUCSIsArabicPresentationFormsA
0001:006c297c* _xmlUCSIsArabicPresentationFormsB
0001:006c2994* _xmlUCSIsArmenian
0001:006c29aa* _xmlUCSIsArrows
0001:006c29c0* _xmlUCSIsBasicLatin
0001:006c29ce* _xmlUCSIsBengali
0001:006c29e4* _xmlUCSIsBlockElements
0001:006c29fa* _xmlUCSIsBopomofo
0001:006c2a10* _xmlUCSIsBopomofoExtended
0001:006c2a26* _xmlUCSIsBoxDrawing
0001:006c2a3c* _xmlUCSIsBraillePatterns
0001:006c2a54* _xmlUCSIsBuhid
0001:006c2a6a* _xmlUCSIsByzantineMusicalSymbols
0001:006c2a82* _xmlUCSIsCJKCompatibility
0001:006c2a9a* _xmlUCSIsCJKCompatibilityForms
0001:006c2ab0* _xmlUCSIsCJKCompatibilityIdeographs
0001:006c2ac8* _xmlUCSIsCJKCompatibilityIdeographsSupplement
0001:006c2ae0* _xmlUCSIsCJKRadicalsSupplement
0001:006c2af6* _xmlUCSIsCJKSymbolsandPunctuation
0001:006c2b0c* _xmlUCSIsCJKUnifiedIdeographs
0001:006c2b24* _xmlUCSIsCJKUnifiedIdeographsExtensionA
0001:006c2b3c* _xmlUCSIsCJKUnifiedIdeographsExtensionB
0001:006c2b54* _xmlUCSIsCherokee
0001:006c2b6a* _xmlUCSIsCombiningDiacriticalMarks
0001:006c2b80* _xmlUCSIsCombiningDiacriticalMarksforSymbols
0001:006c2b96* _xmlUCSIsCombiningHalfMarks
0001:006c2bac* _xmlUCSIsCombiningMarksforSymbols
0001:006c2bc2* _xmlUCSIsControlPictures
0001:006c2bd8* _xmlUCSIsCurrencySymbols
0001:006c2bee* _xmlUCSIsCypriotSyllabary
0001:006c2c04* _xmlUCSIsCyrillic
0001:006c2c1c* _xmlUCSIsCyrillicSupplement
0001:006c2c32* _xmlUCSIsDeseret
0001:006c2c48* _xmlUCSIsDevanagari
0001:006c2c5e* _xmlUCSIsDingbats
0001:006c2c76* _xmlUCSIsEnclosedAlphanumerics
0001:006c2c8e* _xmlUCSIsEnclosedCJKLettersandMonths
0001:006c2ca6* _xmlUCSIsEthiopic
0001:006c2cbe* _xmlUCSIsGeneralPunctuation
0001:006c2cd4* _xmlUCSIsGeometricShapes
0001:006c2cea* _xmlUCSIsGeorgian
0001:006c2d00* _xmlUCSIsGothic
0001:006c2d16* _xmlUCSIsGreek
0001:006c2d2e* _xmlUCSIsGreekExtended
0001:006c2d46* _xmlUCSIsGreekandCoptic
0001:006c2d5e* _xmlUCSIsGujarati
0001:006c2d74* _xmlUCSIsGurmukhi
0001:006c2d8a* _xmlUCSIsHalfwidthandFullwidthForms
0001:006c2da2* _xmlUCSIsHangulCompatibilityJamo
0001:006c2db8* _xmlUCSIsHangulJamo
0001:006c2dd0* _xmlUCSIsHangulSyllables
0001:006c2de8* _xmlUCSIsHanunoo
0001:006c2dfe* _xmlUCSIsHebrew
0001:006c2e14* _xmlUCSIsHighPrivateUseSurrogates
0001:006c2e2a* _xmlUCSIsHighSurrogates
0001:006c2e42* _xmlUCSIsHiragana
0001:006c2e58* _xmlUCSIsIPAExtensions
0001:006c2e6e* _xmlUCSIsIdeographicDescriptionCharacters
0001:006c2e84* _xmlUCSIsKanbun
0001:006c2e9a* _xmlUCSIsKangxiRadicals
0001:006c2eb2* _xmlUCSIsKannada
0001:006c2ec8* _xmlUCSIsKatakana
0001:006c2ede* _xmlUCSIsKatakanaPhoneticExtensions
0001:006c2ef4* _xmlUCSIsKhmer
0001:006c2f0a* _xmlUCSIsKhmerSymbols
0001:006c2f20* _xmlUCSIsLao
0001:006c2f36* _xmlUCSIsLatin1Supplement
0001:006c2f4a* _xmlUCSIsLatinExtendedA
0001:006c2f60* _xmlUCSIsLatinExtendedB
0001:006c2f78* _xmlUCSIsLatinExtendedAdditional
0001:006c2f90* _xmlUCSIsLetterlikeSymbols
0001:006c2fa6* _xmlUCSIsLimbu
0001:006c2fbc* _xmlUCSIsLinearBIdeograms
0001:006c2fd2* _xmlUCSIsLinearBSyllabary
0001:006c2fe8* _xmlUCSIsLowSurrogates
0001:006c3000* _xmlUCSIsMalayalam
0001:006c3016* _xmlUCSIsMathematicalAlphanumericSymbols
0001:006c302e* _xmlUCSIsMathematicalOperators
0001:006c3046* _xmlUCSIsMiscellaneousMathematicalSymbolsA
0001:006c305c* _xmlUCSIsMiscellaneousMathematicalSymbolsB
0001:006c3072* _xmlUCSIsMiscellaneousSymbols
0001:006c308a* _xmlUCSIsMiscellaneousSymbolsandArrows
0001:006c30a2* _xmlUCSIsMiscellaneousTechnical
0001:006c30ba* _xmlUCSIsMongolian
0001:006c30d2* _xmlUCSIsMusicalSymbols
0001:006c30ea* _xmlUCSIsMyanmar
0001:006c3102* _xmlUCSIsNumberForms
0001:006c3118* _xmlUCSIsOgham
0001:006c312e* _xmlUCSIsOldItalic
0001:006c3144* _xmlUCSIsOpticalCharacterRecognition
0001:006c315a* _xmlUCSIsOriya
0001:006c3170* _xmlUCSIsOsmanya
0001:006c3186* _xmlUCSIsPhoneticExtensions
0001:006c319c* _xmlUCSIsPrivateUse
0001:006c31d7* _xmlUCSIsPrivateUseArea
0001:006c31ef* _xmlUCSIsRunic
0001:006c3205* _xmlUCSIsShavian
0001:006c321b* _xmlUCSIsSinhala
0001:006c3231* _xmlUCSIsSmallFormVariants
0001:006c3247* _xmlUCSIsSpacingModifierLetters
0001:006c325d* _xmlUCSIsSpecials
0001:006c3273* _xmlUCSIsSuperscriptsandSubscripts
0001:006c3289* _xmlUCSIsSupplementalArrowsA
0001:006c329f* _xmlUCSIsSupplementalArrowsB
0001:006c32b5* _xmlUCSIsSupplementalMathematicalOperators
0001:006c32cd* _xmlUCSIsSupplementaryPrivateUseAreaA
0001:006c32e5* _xmlUCSIsSupplementaryPrivateUseAreaB
0001:006c32fd* _xmlUCSIsSyriac
0001:006c3313* _xmlUCSIsTagalog
0001:006c3329* _xmlUCSIsTagbanwa
0001:006c333f* _xmlUCSIsTags
0001:006c3355* _xmlUCSIsTaiLe
0001:006c336b* _xmlUCSIsTaiXuanJingSymbols
0001:006c3381* _xmlUCSIsTamil
0001:006c3397* _xmlUCSIsTelugu
0001:006c33ad* _xmlUCSIsThaana
0001:006c33c3* _xmlUCSIsThai
0001:006c33d9* _xmlUCSIsTibetan
0001:006c33f1* _xmlUCSIsUgaritic
0001:006c3407* _xmlUCSIsUnifiedCanadianAboriginalSyllabics
0001:006c341f* _xmlUCSIsVariationSelectors
0001:006c3435* _xmlUCSIsVariationSelectorsSupplement
0001:006c344d* _xmlUCSIsYiRadicals
0001:006c3463* _xmlUCSIsYiSyllables
0001:006c347b* _xmlUCSIsYijingHexagramSymbols
0001:006c3491  _xmlUCSIsCatCc
0001:006c34b0  _xmlUCSIsCatCo
0001:006c34f6* _xmlUCSIsCatCs
0001:006c3532  _xmlUCSIsCatMe
0001:006c3572  _xmlUCSIsCatNl
0001:006c35c9  _xmlUCSIsCatPc
0001:006c3626  _xmlUCSIsCatPf
0001:006c365c  _xmlUCSIsCatPi
0001:006c3696  _xmlUCSIsCatZl
0001:006c36a7  _xmlUCSIsCatZp
0001:006c36b8  _xmlUCSIsCatZs
0001:006c3782  _xmlUCSIsCatZ
0001:006c379d  _xmlUCSIsCatSo
0001:006c37b8  _xmlUCSIsCatSm
0001:006c37d3  _xmlUCSIsCatSk
0001:006c37ee  _xmlUCSIsCatSc
0001:006c3809  _xmlUCSIsCatS
0001:006c3824  _xmlUCSIsCatPs
0001:006c383f  _xmlUCSIsCatPo
0001:006c385a  _xmlUCSIsCatPe
0001:006c3875  _xmlUCSIsCatPd
0001:006c3890  _xmlUCSIsCatP
0001:006c38ab  _xmlUCSIsCatNo
0001:006c38c6  _xmlUCSIsCatNd
0001:006c38e1  _xmlUCSIsCatN
0001:006c38fc  _xmlUCSIsCatMn
0001:006c3917  _xmlUCSIsCatMc
0001:006c3932  _xmlUCSIsCatM
0001:006c394d  _xmlUCSIsCatLu
0001:006c3968  _xmlUCSIsCatLt
0001:006c3983  _xmlUCSIsCatLo
0001:006c399e  _xmlUCSIsCatLm
0001:006c39b9  _xmlUCSIsCatLl
0001:006c39d4  _xmlUCSIsCatL
0001:006c39ef  _xmlUCSIsCatCf
0001:006c3a0a  _xmlUCSIsCatC
0001:006c3a25  _xmlUCSIsBlock
0001:006c3a55* _xmlUCSIsCat
Module: U:\extras\lib\libcrypto.lib(mem_dbg.obj)
0001:006c7540  _CRYPTO_mem_ctrl
0001:006c7740* _CRYPTO_is_mem_check_on
0001:006c77f0* _CRYPTO_dbg_set_options
0001:006c7800* _CRYPTO_dbg_get_options
0001:006c7810  _CRYPTO_push_info_
0001:006c79b0  _CRYPTO_pop_info
0001:006c7b40* _CRYPTO_remove_all_info
0001:006c7cc0* _CRYPTO_dbg_malloc
0001:006c7f40* _CRYPTO_dbg_free
0001:006c8080* _CRYPTO_dbg_realloc
0001:006c8220* _CRYPTO_mem_leaks
0001:006c8390* _CRYPTO_mem_leaks_fp
0001:006c8410* _CRYPTO_mem_leaks_cb
Module: U:\extras\lib\libcrypto.lib(b_print.obj)
0001:006c9a80* _BIO_vprintf
0001:006c9b80  _BIO_printf
0001:006c9bb0  _BIO_snprintf
0001:006c9c20* _BIO_vsnprintf
Module: U:\extras\lib\libcrypto.lib(x86cpuid.obj)
0001:006c9c90  _OPENSSL_ia32_cpuid
0001:006c9db0* _OPENSSL_rdtsc
0001:006c9dd0* _OPENSSL_instrument_halt
0001:006c9e10* _OPENSSL_far_spin
0001:006c9e40* _OPENSSL_wipe_cpu
0001:006c9ea0* _OPENSSL_atomic_add
0001:006c9ec0* _OPENSSL_indirect_call
0001:006c9f00  _OPENSSL_cleanse
0001:006c9f48* __GLOBAL_$I$_OPENSSL_cpuid_setup
Module: U:\extras\lib\libcrypto.lib(eng_pkey.obj)
0001:006c9f50* _ENGINE_set_load_privkey_function
0001:006c9f70* _ENGINE_set_load_pubkey_function
0001:006c9f90* _ENGINE_set_load_ssl_client_cert_function
0001:006c9fb0* _ENGINE_get_load_privkey_function
0001:006c9fc0* _ENGINE_get_load_pubkey_function
0001:006c9fd0  _ENGINE_get_ssl_client_cert_function
0001:006ca000* _ENGINE_load_private_key
0001:006ca1b0* _ENGINE_load_public_key
0001:006ca360  _ENGINE_load_ssl_client_cert
Module: U:\extras\lib\libssl.lib(ssl_asn1.obj)
0001:006ca510  _i2d_SSL_SESSION
0001:006cb150  _d2i_SSL_SESSION
Module: U:\extras\lib\libcrypto.lib(pem_oth.obj)
0001:006cc8b0  _PEM_ASN1_read_bio
Module: U:\extras\lib\libcrypto.lib(pem_lib.obj)
0001:006cca00  _PEM_def_callback
0001:006ccc20  _PEM_proc_type
0001:006cccd0  _PEM_dek_info
0001:006ccdb0  _PEM_ASN1_read
0001:006cce60  _PEM_do_header
0001:006cd200  _PEM_get_EVP_CIPHER_INFO
0001:006cd540  _PEM_write_bio
0001:006cd890* _PEM_write
0001:006cd9a0  _PEM_ASN1_write_bio
0001:006ce120  _PEM_ASN1_write
0001:006ce200  _PEM_read_bio
0001:006ce9e0* _PEM_read
0001:006ceb60  _PEM_bytes_read_bio
0001:006cefe0  _pem_check_suffix
0001:006cf040* _PEM_version
Module: U:\extras\lib\libcrypto.lib(tb_cipher.obj)
0001:006cf0b0* _ENGINE_unregister_ciphers
0001:006cf0d0* _ENGINE_register_ciphers
0001:006cf150* _ENGINE_register_all_ciphers
0001:006cf1e0* _ENGINE_set_default_ciphers
0001:006cf260  _ENGINE_get_cipher_engine
0001:006cf2a0  _ENGINE_get_cipher
0001:006cf320* _ENGINE_get_ciphers
0001:006cf330* _ENGINE_set_ciphers
Module: U:\extras\lib\libcrypto.lib(evp_lib.obj)
0001:006cf350  _EVP_CIPHER_param_to_asn1
0001:006cf380  _EVP_CIPHER_asn1_to_param
0001:006cf3e0  _EVP_CIPHER_get_asn1_iv
0001:006cf4b0  _EVP_CIPHER_set_asn1_iv
0001:006cf520  _EVP_CIPHER_type
0001:006cf6e0  _EVP_CIPHER_block_size
0001:006cf6f0  _EVP_CIPHER_CTX_block_size
0001:006cf700  _EVP_Cipher
0001:006cf720  _EVP_CIPHER_CTX_cipher
0001:006cf730* _EVP_CIPHER_flags
0001:006cf740  _EVP_CIPHER_CTX_flags
0001:006cf750* _EVP_CIPHER_CTX_get_app_data
0001:006cf760* _EVP_CIPHER_CTX_set_app_data
0001:006cf770  _EVP_CIPHER_iv_length
0001:006cf780  _EVP_CIPHER_CTX_iv_length
0001:006cf790  _EVP_CIPHER_key_length
0001:006cf7a0  _EVP_CIPHER_CTX_key_length
0001:006cf7b0  _EVP_CIPHER_nid
0001:006cf7c0* _EVP_CIPHER_CTX_nid
0001:006cf7d0  _EVP_MD_block_size
0001:006cf7e0  _EVP_MD_type
0001:006cf7f0  _EVP_MD_pkey_type
0001:006cf800  _EVP_MD_size
0001:006cf850* _EVP_MD_flags
0001:006cf860  _EVP_MD_CTX_md
0001:006cf880  _EVP_MD_CTX_set_flags
0001:006cf890  _EVP_MD_CTX_clear_flags
0001:006cf8a0  _EVP_MD_CTX_test_flags
0001:006cf8b0* _EVP_CIPHER_CTX_set_flags
0001:006cf8c0* _EVP_CIPHER_CTX_clear_flags
0001:006cf8d0* _EVP_CIPHER_CTX_test_flags
Module: U:\extras\lib\libcrypto.lib(tb_digest.obj)
0001:006cf900* _ENGINE_unregister_digests
0001:006cf920* _ENGINE_register_digests
0001:006cf9a0* _ENGINE_register_all_digests
0001:006cfa30* _ENGINE_set_default_digests
0001:006cfab0  _ENGINE_get_digest_engine
0001:006cfaf0  _ENGINE_get_digest
0001:006cfb70* _ENGINE_get_digests
0001:006cfb80* _ENGINE_set_digests
Module: U:\extras\lib\libcrypto.lib(pmeth_lib.obj)
0001:006cfec0* _EVP_PKEY_meth_find
0001:006cff60* _EVP_PKEY_meth_new
0001:006d0050  _EVP_PKEY_meth_free
0001:006d0080  _EVP_PKEY_CTX_new
0001:006d00a0  _EVP_PKEY_CTX_new_id
0001:006d00c0  _EVP_PKEY_CTX_dup
0001:006d0280* _EVP_PKEY_meth_add0
0001:006d02f0  _EVP_PKEY_CTX_free
0001:006d0360  _EVP_PKEY_CTX_ctrl
0001:006d04f0* _EVP_PKEY_CTX_ctrl_str
0001:006d0730* _EVP_PKEY_CTX_get_operation
0001:006d0740* _EVP_PKEY_CTX_set0_keygen_info
0001:006d0760* _EVP_PKEY_CTX_set_data
0001:006d0770* _EVP_PKEY_CTX_get_data
0001:006d0780* _EVP_PKEY_CTX_get0_pkey
0001:006d0790* _EVP_PKEY_CTX_get0_peerkey
0001:006d07a0* _EVP_PKEY_CTX_set_app_data
0001:006d07b0* _EVP_PKEY_CTX_get_app_data
0001:006d07c0* _EVP_PKEY_meth_set_init
0001:006d07d0* _EVP_PKEY_meth_set_copy
0001:006d07e0* _EVP_PKEY_meth_set_cleanup
0001:006d07f0* _EVP_PKEY_meth_set_paramgen
0001:006d0810* _EVP_PKEY_meth_set_keygen
0001:006d0830* _EVP_PKEY_meth_set_sign
0001:006d0850* _EVP_PKEY_meth_set_verify
0001:006d0870* _EVP_PKEY_meth_set_verify_recover
0001:006d0890* _EVP_PKEY_meth_set_signctx
0001:006d08b0* _EVP_PKEY_meth_set_verifyctx
0001:006d08d0* _EVP_PKEY_meth_set_encrypt
0001:006d08f0* _EVP_PKEY_meth_set_decrypt
0001:006d0910* _EVP_PKEY_meth_set_derive
0001:006d0930* _EVP_PKEY_meth_set_ctrl
0002:00021710* _app_pkey_methods
Module: U:\extras\lib\libcrypto.lib(c_zlib.obj)
0001:006d1590  _COMP_zlib
0001:006d1660* _COMP_zlib_cleanup
0001:006d1670  _BIO_f_zlib
Module: U:\extras\lib\libcrypto.lib(ameth_lib.obj)
0001:006d16e0* _EVP_PKEY_asn1_get_count
0001:006d1710* _EVP_PKEY_asn1_get0
0001:006d1760  _EVP_PKEY_asn1_find
0001:006d1870  _EVP_PKEY_asn1_find_str
0001:006d19b0* _EVP_PKEY_asn1_add0
0001:006d1a40* _EVP_PKEY_asn1_add_alias
0001:006d1b80  _EVP_PKEY_asn1_get0_info
0001:006d1c00* _EVP_PKEY_get0_asn1
0001:006d1c10* _EVP_PKEY_asn1_new
0001:006d1d80* _EVP_PKEY_asn1_copy
0001:006d1e00  _EVP_PKEY_asn1_free
0001:006d1e50* _EVP_PKEY_asn1_set_public
0001:006d1e80* _EVP_PKEY_asn1_set_private
0001:006d1ea0* _EVP_PKEY_asn1_set_param
0001:006d1ed0* _EVP_PKEY_asn1_set_free
0001:006d1ee0* _EVP_PKEY_asn1_set_ctrl
Module: U:\extras\lib\libcrypto.lib(e_null.obj)
0001:006d1fb0  _EVP_enc_null
Module: U:\extras\lib\libcrypto.lib(a_object.obj)
0001:006d2000* _i2d_ASN1_OBJECT
0001:006d2160  _a2d_ASN1_OBJECT
0001:006d26c0  _i2t_ASN1_OBJECT
0001:006d2700  _i2a_ASN1_OBJECT
0001:006d2850  _ASN1_OBJECT_new
0001:006d28e0  _ASN1_OBJECT_free
0001:006d2960  _c2i_ASN1_OBJECT
0001:006d2c40  _d2i_ASN1_OBJECT
0001:006d2d00  _ASN1_OBJECT_create
Module: U:\extras\lib\libcrypto.lib(obj_lib.obj)
0001:006d2d70  _OBJ_dup
0001:006d3180  _OBJ_cmp
Module: U:\extras\lib\libcrypto.lib(x509_trs.obj)
0001:006d3520* _X509_TRUST_set_default
0001:006d3530  _X509_check_trust
0001:006d3610* _X509_TRUST_get_count
0001:006d3640* _X509_TRUST_get0
0001:006d3690  _X509_TRUST_get_by_id
0001:006d3700  _X509_TRUST_set
0001:006d3780* _X509_TRUST_add
0001:006d3930* _X509_TRUST_cleanup
0001:006d3b30* _X509_TRUST_get_flags
0001:006d3b40* _X509_TRUST_get0_name
0001:006d3b50* _X509_TRUST_get_trust
Module: U:\extras\lib\libcrypto.lib(x509_vfy.obj)
0001:006d4280* _X509_cmp_time
0001:006d5520  _X509_verify_cert
0001:006d5f80* _X509_cmp_current_time
0001:006d5fa0  _X509_gmtime_adj
0001:006d6040* _X509_time_adj
0001:006d60f0* _X509_time_adj_ex
0001:006d61b0* _X509_get_pubkey_parameters
0001:006d6310  _X509_STORE_CTX_get_ex_new_index
0001:006d6350  _X509_STORE_CTX_set_ex_data
0001:006d6370* _X509_STORE_CTX_get_ex_data
0001:006d6390* _X509_STORE_CTX_get_error
0001:006d63a0* _X509_STORE_CTX_set_error
0001:006d63b0* _X509_STORE_CTX_get_error_depth
0001:006d63c0* _X509_STORE_CTX_get_current_cert
0001:006d63d0* _X509_STORE_CTX_get_chain
0001:006d63e0* _X509_STORE_CTX_get1_chain
0001:006d6470* _X509_STORE_CTX_get0_current_issuer
0001:006d6480* _X509_STORE_CTX_get0_current_crl
0001:006d6490* _X509_STORE_CTX_get0_parent_ctx
0001:006d64a0* _X509_STORE_CTX_set_cert
0001:006d64b0* _X509_STORE_CTX_set_chain
0001:006d64c0* _X509_STORE_CTX_set0_crls
0001:006d64d0  _X509_STORE_CTX_set_purpose
0001:006d64f0* _X509_STORE_CTX_set_trust
0001:006d6510* _X509_STORE_CTX_purpose_inherit
0001:006d6650* _X509_STORE_CTX_new
0001:006d66c0* _X509_STORE_CTX_free
0001:006d6780  _X509_STORE_CTX_init
0001:006d6ad0* _X509_STORE_CTX_trusted_stack
0001:006d6af0  _X509_STORE_CTX_cleanup
0001:006d6b90* _X509_STORE_CTX_set_depth
0001:006d6bb0* _X509_STORE_CTX_set_flags
0001:006d6bd0* _X509_STORE_CTX_set_time
0001:006d6bf0  _X509_STORE_CTX_set_verify_cb
0001:006d6c00* _X509_STORE_CTX_get0_policy_tree
0001:006d6c10* _X509_STORE_CTX_get_explicit_policy
0001:006d6c20  _X509_STORE_CTX_set_default
0001:006d6c60  _X509_STORE_CTX_get0_param
0001:006d6c70* _X509_STORE_CTX_set0_param
0001:006d6fc0* _X509_version
Module: U:\extras\lib\libcrypto.lib(dh_asn1.obj)
0001:006d7050  _d2i_DHparams
0001:006d70d0* _DHparams_it
0001:006d7080  _i2d_DHparams
0001:006d70b0  _DHparams_dup
Module: U:\extras\lib\libcrypto.lib(bn_lib.obj)
0001:006d7310* _BN_set_params
0001:006d73e0* _BN_get_params
0001:006d7440  _BN_value_one
0001:006d7450* _BN_options
0001:006d74a0  _BN_num_bits_word
0001:006d7530  _BN_num_bits
0001:006d75d0  _BN_clear_free
0001:006d7640  _BN_free
0001:006d7690  _BN_init
0001:006d76b0  _BN_new
0001:006d7730  _bn_expand2
0001:006d7780  _BN_copy
0001:006d78a0  _BN_dup
0001:006d7960* _bn_dup_expand
0001:006d7ac0* _BN_swap
0001:006d7b40  _BN_clear
0001:006d7b80* _BN_get_word
0001:006d7bb0  _BN_set_word
0001:006d7c30  _BN_bin2bn
0001:006d7e20  _BN_bn2bin
0001:006d7f40  _BN_ucmp
0001:006d7fa0  _BN_cmp
0001:006d8050  _BN_set_bit
0001:006d8120* _BN_clear_bit
0001:006d81a0  _BN_is_bit_set
0001:006d81f0  _BN_mask_bits
0001:006d8280  _BN_set_negative
0001:006d82b0  _bn_cmp_words
0001:006d8330  _bn_cmp_part_words
0001:006d8410* _BN_version
Module: U:\extras\lib\libcrypto.lib(ec_key.obj)
0001:006d8580  _EC_KEY_new
0001:006d8620* _EC_KEY_new_by_curve_name
0001:006d8750  _EC_KEY_free
0001:006d87f0* _EC_KEY_copy
0001:006d89c0  _EC_KEY_dup
0001:006d8af0  _EC_KEY_up_ref
0001:006d8b30  _EC_KEY_generate_key
0001:006d8d40* _EC_KEY_check_key
0001:006d9060  _EC_KEY_get0_group
0001:006d9070  _EC_KEY_set_group
0001:006d90b0  _EC_KEY_get0_private_key
0001:006d90c0* _EC_KEY_set_private_key
0001:006d9100  _EC_KEY_get0_public_key
0001:006d9110  _EC_KEY_set_public_key
0001:006d9150  _EC_KEY_get_enc_flags
0001:006d9160  _EC_KEY_set_enc_flags
0001:006d9170  _EC_KEY_get_conv_form
0001:006d9180* _EC_KEY_set_conv_form
0001:006d91c0  _EC_KEY_get_key_method_data
0001:006d91e0  _EC_KEY_insert_key_method_data
0001:006d92a0* _EC_KEY_set_asn1_flag
0001:006d92d0* _EC_KEY_precompute_mult
Module: U:\extras\lib\libcrypto.lib(bss_file.obj)
0001:006d9a40  _BIO_new_file
0001:006d9ba0  _BIO_new_fp
0001:006d9bf0  _BIO_s_file
Module: U:\extras\lib\libcrypto.lib(pem_x509.obj)
0001:006d9c20  _PEM_read_bio_X509
0001:006d9c60* _PEM_read_X509
0001:006d9ca0  _PEM_write_bio_X509
0001:006d9d00* _PEM_write_X509
Module: U:\extras\lib\libcrypto.lib(o_dir.obj)
0001:006d9d60  _OPENSSL_DIR_read
0001:006d9d80  _OPENSSL_DIR_end
Module: U:\extras\lib\libcrypto.lib(asn1_lib.obj)
0001:006d9da0* _ASN1_check_infinite_end
0001:006d9e00  _ASN1_const_check_infinite_end
0001:006d9e70  _ASN1_get_object
0001:006da080  _ASN1_put_object
0001:006da1b0  _ASN1_put_eoc
0001:006da1d0  _ASN1_object_size
0001:006da220* _asn1_Finish
0001:006da2a0  _asn1_const_Finish
0001:006da320  _asn1_GetSequence
0001:006da3d0  _ASN1_STRING_set
0001:006da570  _ASN1_STRING_copy
0001:006da5d0  _ASN1_STRING_dup
0001:006da6c0  _ASN1_STRING_set0
0001:006da6f0  _ASN1_STRING_new
0001:006da770  _ASN1_STRING_type_new
0001:006da7f0  _ASN1_STRING_free
0001:006da850  _ASN1_STRING_cmp
0001:006da8a0  _asn1_add_error
0001:006da920* _ASN1_STRING_length
0001:006da930* _ASN1_STRING_length_set
0001:006da940* _ASN1_STRING_type
0001:006da950  _ASN1_STRING_data
0001:006da960* _ASN1_version
Module: U:\extras\lib\libcrypto.lib(x509_obj.obj)
0001:006da9c0  _X509_NAME_oneline
Module: U:\extras\lib\libcrypto.lib(m_md5.obj)
0001:006daf90  _EVP_md5
Module: U:\extras\lib\libcrypto.lib(m_sha1.obj)
0001:006db150  _EVP_sha1
0001:006db160* _EVP_sha224
0001:006db170  _EVP_sha256
0001:006db180* _EVP_sha384
0001:006db190* _EVP_sha512
Module: U:\extras\lib\libcrypto.lib(x_pubkey.obj)
0001:006db370* _d2i_X509_PUBKEY
0001:006dbde0  _X509_PUBKEY_it
0001:006db3a0* _i2d_X509_PUBKEY
0001:006db3d0* _X509_PUBKEY_new
0001:006db3f0* _X509_PUBKEY_free
0001:006db430  _X509_PUBKEY_set
0001:006db570  _X509_PUBKEY_get
0001:006db730  _d2i_PUBKEY
0001:006db7b0  _i2d_PUBKEY
0001:006db820  _d2i_RSA_PUBKEY
0001:006db8d0  _i2d_RSA_PUBKEY
0001:006db9c0  _d2i_DSA_PUBKEY
0001:006dba70  _i2d_DSA_PUBKEY
0001:006dbb60  _d2i_EC_PUBKEY
0001:006dbc10  _i2d_EC_PUBKEY
0001:006dbd00  _X509_PUBKEY_set0_param
0001:006dbd90  _X509_PUBKEY_get0_param
Module: U:\extras\lib\libcrypto.lib(x_crl.obj)
0001:006dca30  _X509_CRL_INFO_it
0001:006dc5c0* _d2i_X509_REVOKED
0001:006dca00* _X509_REVOKED_it
0001:006dc5f0* _i2d_X509_REVOKED
0001:006dc620* _X509_REVOKED_new
0001:006dc640* _X509_REVOKED_free
0001:006dc660* _d2i_X509_CRL_INFO
0001:006dc690* _i2d_X509_CRL_INFO
0001:006dc6c0* _X509_CRL_INFO_new
0001:006dc6e0* _X509_CRL_INFO_free
0001:006dc700  _d2i_X509_CRL
0001:006dca60  _X509_CRL_it
0001:006dc730  _i2d_X509_CRL
0001:006dc760* _X509_CRL_new
0001:006dc780  _X509_CRL_free
0001:006dc7a0* _X509_CRL_dup
0001:006dc7c0* _X509_CRL_add0_revoked
0001:006dc860  _X509_CRL_verify
0001:006dc890* _X509_CRL_get0_by_serial
0001:006dc8e0  _X509_CRL_get0_by_cert
0001:006dc940* _X509_CRL_set_default_method
0001:006dc960* _X509_CRL_METHOD_new
0001:006dc9b0* _X509_CRL_METHOD_free
0001:006dc9d0* _X509_CRL_set_meth_data
0001:006dc9e0* _X509_CRL_get_meth_data
Module: U:\extras\lib\libcrypto.lib(a_strex.obj)
0001:006ddab0  _X509_NAME_print_ex
0001:006ddaf0* _X509_NAME_print_ex_fp
0001:006ddb70  _ASN1_STRING_print_ex
0001:006ddb90* _ASN1_STRING_print_ex_fp
0001:006ddbb0  _ASN1_STRING_to_UTF8
Module: U:\extras\lib\libcrypto.lib(tasn_fre.obj)
0001:006ddcd0  _ASN1_primitive_free
0001:006de280  _ASN1_template_free
0001:006de310  _ASN1_item_ex_free
0001:006de330  _ASN1_item_free
Module: U:\extras\lib\libcrypto.lib(tasn_new.obj)
0001:006de420* _ASN1_primitive_new
0001:006dea40* _ASN1_template_new
0001:006deb10  _ASN1_item_ex_new
0001:006deb30  _ASN1_item_new
Module: U:\extras\lib\libcrypto.lib(tasn_dec.obj)
0001:006df1e0  _ASN1_tag2bit
0001:006df210* _asn1_ex_c2i
0001:006dfc50  _ASN1_item_ex_d2i
0001:006e0e90* _ASN1_template_d2i
0001:006e0ed0  _ASN1_item_d2i
Module: U:\extras\lib\libcrypto.lib(tasn_enc.obj)
0001:006e1020* _asn1_ex_i2c
0001:006e1470  _ASN1_item_ex_i2d
0001:006e2020* _ASN1_template_i2d
0001:006e2050  _ASN1_item_i2d
0001:006e2140  _ASN1_item_ndef_i2d
Module: U:\extras\lib\libcrypto.lib(a_dup.obj)
0001:006e2250  _ASN1_dup
0001:006e2320  _ASN1_item_dup
Module: U:\extras\lib\libcrypto.lib(tasn_typ.obj)
0001:006e23d0  _d2i_ASN1_INTEGER
0001:006e3070  _ASN1_INTEGER_it
0001:006e2400  _i2d_ASN1_INTEGER
0001:006e2430  _ASN1_INTEGER_new
0001:006e2450  _ASN1_INTEGER_free
0001:006e2470  _d2i_ASN1_ENUMERATED
0001:006e30a0  _ASN1_ENUMERATED_it
0001:006e24a0* _i2d_ASN1_ENUMERATED
0001:006e24d0* _ASN1_ENUMERATED_new
0001:006e24f0  _ASN1_ENUMERATED_free
0001:006e2510  _d2i_ASN1_BIT_STRING
0001:006e30d0  _ASN1_BIT_STRING_it
0001:006e2540  _i2d_ASN1_BIT_STRING
0001:006e2570  _ASN1_BIT_STRING_new
0001:006e2590  _ASN1_BIT_STRING_free
0001:006e25b0  _d2i_ASN1_OCTET_STRING
0001:006e3100  _ASN1_OCTET_STRING_it
0001:006e25e0  _i2d_ASN1_OCTET_STRING
0001:006e2610  _ASN1_OCTET_STRING_new
0001:006e2630  _ASN1_OCTET_STRING_free
0001:006e2650* _d2i_ASN1_NULL
0001:006e3130  _ASN1_NULL_it
0001:006e2680* _i2d_ASN1_NULL
0001:006e26b0  _ASN1_NULL_new
0001:006e26d0* _ASN1_NULL_free
0001:006e26f0* _d2i_ASN1_UTF8STRING
0001:006e3190  _ASN1_UTF8STRING_it
0001:006e2720* _i2d_ASN1_UTF8STRING
0001:006e2750  _ASN1_UTF8STRING_new
0001:006e2770  _ASN1_UTF8STRING_free
0001:006e2790* _d2i_ASN1_PRINTABLESTRING
0001:006e31d0* _ASN1_PRINTABLESTRING_it
0001:006e27c0* _i2d_ASN1_PRINTABLESTRING
0001:006e27f0* _ASN1_PRINTABLESTRING_new
0001:006e2810* _ASN1_PRINTABLESTRING_free
0001:006e2830* _d2i_ASN1_T61STRING
0001:006e3200* _ASN1_T61STRING_it
0001:006e2860* _i2d_ASN1_T61STRING
0001:006e2890* _ASN1_T61STRING_new
0001:006e28b0* _ASN1_T61STRING_free
0001:006e28d0* _d2i_ASN1_IA5STRING
0001:006e3230  _ASN1_IA5STRING_it
0001:006e2900* _i2d_ASN1_IA5STRING
0001:006e2930* _ASN1_IA5STRING_new
0001:006e2950* _ASN1_IA5STRING_free
0001:006e2970* _d2i_ASN1_GENERALSTRING
0001:006e3260* _ASN1_GENERALSTRING_it
0001:006e29a0* _i2d_ASN1_GENERALSTRING
0001:006e29d0* _ASN1_GENERALSTRING_new
0001:006e29f0* _ASN1_GENERALSTRING_free
0001:006e2a10* _d2i_ASN1_UTCTIME
0001:006e3290* _ASN1_UTCTIME_it
0001:006e2a40* _i2d_ASN1_UTCTIME
0001:006e2a70* _ASN1_UTCTIME_new
0001:006e2a90* _ASN1_UTCTIME_free
0001:006e2ab0* _d2i_ASN1_GENERALIZEDTIME
0001:006e32d0  _ASN1_GENERALIZEDTIME_it
0001:006e2ae0* _i2d_ASN1_GENERALIZEDTIME
0001:006e2b10  _ASN1_GENERALIZEDTIME_new
0001:006e2b30* _ASN1_GENERALIZEDTIME_free
0001:006e2b50* _d2i_ASN1_VISIBLESTRING
0001:006e3300* _ASN1_VISIBLESTRING_it
0001:006e2b80* _i2d_ASN1_VISIBLESTRING
0001:006e2bb0* _ASN1_VISIBLESTRING_new
0001:006e2bd0* _ASN1_VISIBLESTRING_free
0001:006e2bf0* _d2i_ASN1_UNIVERSALSTRING
0001:006e3340* _ASN1_UNIVERSALSTRING_it
0001:006e2c20* _i2d_ASN1_UNIVERSALSTRING
0001:006e2c50* _ASN1_UNIVERSALSTRING_new
0001:006e2c70* _ASN1_UNIVERSALSTRING_free
0001:006e2c90* _d2i_ASN1_BMPSTRING
0001:006e3370* _ASN1_BMPSTRING_it
0001:006e2cc0* _i2d_ASN1_BMPSTRING
0001:006e2cf0* _ASN1_BMPSTRING_new
0001:006e2d10* _ASN1_BMPSTRING_free
0001:006e2d30  _d2i_ASN1_TYPE
0001:006e33a0  _ASN1_ANY_it
0001:006e2d60  _i2d_ASN1_TYPE
0001:006e2d90  _ASN1_TYPE_new
0001:006e2db0  _ASN1_TYPE_free
0001:006e2dd0* _d2i_ASN1_PRINTABLE
0001:006e3400  _ASN1_PRINTABLE_it
0001:006e2e00* _i2d_ASN1_PRINTABLE
0001:006e2e30* _ASN1_PRINTABLE_new
0001:006e2e50* _ASN1_PRINTABLE_free
0001:006e2e70* _d2i_DISPLAYTEXT
0001:006e3430  _DISPLAYTEXT_it
0001:006e2ea0* _i2d_DISPLAYTEXT
0001:006e2ed0* _DISPLAYTEXT_new
0001:006e2ef0* _DISPLAYTEXT_free
0001:006e2f10* _d2i_DIRECTORYSTRING
0001:006e3460  _DIRECTORYSTRING_it
0001:006e2f40* _i2d_DIRECTORYSTRING
0001:006e2f70* _DIRECTORYSTRING_new
0001:006e2f90* _DIRECTORYSTRING_free
0001:006e2fb0  _d2i_ASN1_SEQUENCE_ANY
0001:006e3560* _ASN1_SEQUENCE_ANY_it
0001:006e2fe0  _i2d_ASN1_SEQUENCE_ANY
0001:006e3010* _d2i_ASN1_SET_ANY
0001:006e3590* _ASN1_SET_ANY_it
0001:006e3040  _i2d_ASN1_SET_ANY
0001:006e3160  _ASN1_OBJECT_it
0001:006e33d0  _ASN1_SEQUENCE_it
0001:006e3490  _ASN1_BOOLEAN_it
0001:006e34c0* _ASN1_TBOOLEAN_it
0001:006e34f0  _ASN1_FBOOLEAN_it
0001:006e3530  _ASN1_OCTET_STRING_NDEF_it
Module: U:\extras\lib\libcrypto.lib(x_x509a.obj)
0001:006e35f0  _d2i_X509_CERT_AUX
0001:006e3b10* _X509_CERT_AUX_it
0001:006e3620  _i2d_X509_CERT_AUX
0001:006e3650* _X509_CERT_AUX_new
0001:006e3670  _X509_CERT_AUX_free
0001:006e3690* _X509_alias_set1
0001:006e3770* _X509_keyid_set1
0001:006e3850* _X509_alias_get0
0001:006e38a0* _X509_keyid_get0
0001:006e38f0* _X509_add1_trust_object
0001:006e3960* _X509_add1_reject_object
0001:006e39e0* _X509_trust_clear
0001:006e3a20* _X509_reject_clear
0001:006e3a60  _d2i_X509_CERT_PAIR
0001:006e3b40* _X509_CERT_PAIR_it
0001:006e3a90  _i2d_X509_CERT_PAIR
0001:006e3ac0* _X509_CERT_PAIR_new
0001:006e3ae0* _X509_CERT_PAIR_free
Module: U:\extras\lib\libcrypto.lib(v3_akeya.obj)
0001:006e3c30* _d2i_AUTHORITY_KEYID
0001:006e3ce0  _AUTHORITY_KEYID_it
0001:006e3c60* _i2d_AUTHORITY_KEYID
0001:006e3c90  _AUTHORITY_KEYID_new
0001:006e3cb0  _AUTHORITY_KEYID_free
Module: U:\extras\lib\libcrypto.lib(v3_crld.obj)
0001:006e3ea0* _DIST_POINT_free
0001:006e53a0* _DIST_POINT_it
0001:006e5370* _DIST_POINT_NAME_it
0001:006e5400* _ISSUING_DIST_POINT_it
0001:006e4fc0* _d2i_DIST_POINT_NAME
0001:006e4ff0* _i2d_DIST_POINT_NAME
0001:006e5020* _DIST_POINT_NAME_new
0001:006e5040* _DIST_POINT_NAME_free
0001:006e5060* _d2i_DIST_POINT
0001:006e5090* _i2d_DIST_POINT
0001:006e50c0* _DIST_POINT_new
0001:006e50e0* _d2i_CRL_DIST_POINTS
0001:006e53d0* _CRL_DIST_POINTS_it
0001:006e5110* _i2d_CRL_DIST_POINTS
0001:006e5140* _CRL_DIST_POINTS_new
0001:006e5160  _CRL_DIST_POINTS_free
0001:006e5180* _d2i_ISSUING_DIST_POINT
0001:006e51b0* _i2d_ISSUING_DIST_POINT
0001:006e51e0* _ISSUING_DIST_POINT_new
0001:006e5200  _ISSUING_DIST_POINT_free
0001:006e5220  _DIST_POINT_set_dpname
0001:006e52e0  _v3_crld
0001:006e5320  _v3_freshest_crl
0001:006e5420  _v3_idp
Module: U:\extras\lib\libcrypto.lib(pcy_cache.obj)
0001:006e57a0  _policy_cache_free
0001:006e5810  _policy_cache_set
0001:006e5bf0  _policy_cache_find_data
Module: U:\extras\lib\libcrypto.lib(v3_genn.obj)
0001:006e5c40* _i2d_GENERAL_NAME
0001:006e6230  _GENERAL_NAME_it
0001:006e5c70* _d2i_GENERAL_NAME
0001:006e5ca0* _d2i_OTHERNAME
0001:006e61d0* _OTHERNAME_it
0001:006e5cd0* _i2d_OTHERNAME
0001:006e5d00  _OTHERNAME_new
0001:006e5d20* _OTHERNAME_free
0001:006e5d40* _d2i_EDIPARTYNAME
0001:006e6200* _EDIPARTYNAME_it
0001:006e5d70* _i2d_EDIPARTYNAME
0001:006e5da0* _EDIPARTYNAME_new
0001:006e5dc0* _EDIPARTYNAME_free
0001:006e5de0  _GENERAL_NAME_new
0001:006e5e00  _GENERAL_NAME_free
0001:006e5e20* _d2i_GENERAL_NAMES
0001:006e6260  _GENERAL_NAMES_it
0001:006e5e50* _i2d_GENERAL_NAMES
0001:006e5e80  _GENERAL_NAMES_new
0001:006e5ea0  _GENERAL_NAMES_free
0001:006e5ec0* _GENERAL_NAME_dup
0001:006e5ef0  _GENERAL_NAME_cmp
0001:006e6010* _OTHERNAME_cmp
0001:006e6060* _GENERAL_NAME_set0_value
0001:006e60b0* _GENERAL_NAME_get0_value
0001:006e6110* _GENERAL_NAME_set0_othername
0001:006e6160* _GENERAL_NAME_get0_otherName
Module: U:\extras\lib\libcrypto.lib(v3_ncons.obj)
0001:006e7030* _NAME_CONSTRAINTS_it
0001:006e7000* _GENERAL_SUBTREE_it
0001:006e6e40* _GENERAL_SUBTREE_new
0001:006e6e60* _GENERAL_SUBTREE_free
0001:006e6e80* _NAME_CONSTRAINTS_new
0001:006e6ea0  _NAME_CONSTRAINTS_free
0001:006e6ec0  _NAME_CONSTRAINTS_check
0001:006e6fb0  _v3_name_constraints
Module: U:\extras\lib\libcrypto.lib(v3_addr.obj)
0001:006e7900  _IPAddressFamily_free
0001:006ea5d0* _IPAddressFamily_it
0001:006ea570* _IPAddressOrRange_it
0001:006ea540* _IPAddressRange_it
0001:006ea5a0* _IPAddressChoice_it
0001:006e8610* _d2i_IPAddressRange
0001:006e8640* _i2d_IPAddressRange
0001:006e8670* _IPAddressRange_new
0001:006e8690* _IPAddressRange_free
0001:006e86b0* _d2i_IPAddressOrRange
0001:006e86e0* _i2d_IPAddressOrRange
0001:006e8710* _IPAddressOrRange_new
0001:006e8730* _IPAddressOrRange_free
0001:006e8750* _d2i_IPAddressChoice
0001:006e8780* _i2d_IPAddressChoice
0001:006e87b0* _IPAddressChoice_new
0001:006e87d0* _IPAddressChoice_free
0001:006e87f0* _d2i_IPAddressFamily
0001:006e8820* _i2d_IPAddressFamily
0001:006e8850* _IPAddressFamily_new
0001:006e8870* _v3_addr_get_afi
0001:006e88c0* _v3_addr_add_inherit
0001:006e8960* _v3_addr_add_prefix
0001:006e8a70* _v3_addr_add_range
0001:006e8bc0* _v3_addr_get_range
0001:006e8c80* _v3_addr_is_canonical
0001:006e9760* _v3_addr_canonize
0001:006ea2d0* _v3_addr_inherits
0001:006ea330* _v3_addr_subset
0001:006ea480  _v3_addr_validate_path
0001:006ea4a0* _v3_addr_validate_resource_set
0001:006ea600* _IPAddrBlocks_it
0001:006ea620  _v3_addr
Module: U:\extras\lib\libcrypto.lib(v3_asid.obj)
0001:006ec940* _ASIdOrRange_it
0001:006ebd50* _d2i_ASRange
0001:006ec910* _ASRange_it
0001:006ebd80* _i2d_ASRange
0001:006ebdb0* _ASRange_new
0001:006ebdd0* _ASRange_free
0001:006ebdf0* _d2i_ASIdOrRange
0001:006ebe20* _i2d_ASIdOrRange
0001:006ebe50* _ASIdOrRange_new
0001:006ebe70* _ASIdOrRange_free
0001:006ebe90* _d2i_ASIdentifierChoice
0001:006ec970* _ASIdentifierChoice_it
0001:006ebec0* _i2d_ASIdentifierChoice
0001:006ebef0* _ASIdentifierChoice_new
0001:006ebf10* _ASIdentifierChoice_free
0001:006ebf30* _d2i_ASIdentifiers
0001:006ec9a0* _ASIdentifiers_it
0001:006ebf60* _i2d_ASIdentifiers
0001:006ebf90* _ASIdentifiers_new
0001:006ebfb0  _ASIdentifiers_free
0001:006ebff0* _v3_asid_add_inherit
0001:006ec0d0* _v3_asid_add_id_or_range
0001:006ec6c0* _v3_asid_is_canonical
0001:006ec710* _v3_asid_canonize
0001:006ec760* _v3_asid_inherits
0001:006ec7c0* _v3_asid_subset
0001:006ec860  _v3_asid_validate_path
0001:006ec880* _v3_asid_validate_resource_set
0001:006ec9c0  _v3_asid
Module: U:\extras\lib\libcrypto.lib(x_algor.obj)
0001:006ecb00  _d2i_X509_ALGOR
0001:006ecd40  _X509_ALGOR_it
0001:006ecb30* _i2d_X509_ALGOR
0001:006ecb60  _X509_ALGOR_new
0001:006ecb80  _X509_ALGOR_free
0001:006ecba0* _d2i_X509_ALGORS
0001:006ecd70  _X509_ALGORS_it
0001:006ecbd0  _i2d_X509_ALGORS
0001:006ecc00* _X509_ALGOR_dup
0001:006ecc20  _X509_ALGOR_set0
0001:006ecce0  _X509_ALGOR_get0
Module: U:\extras\lib\libcrypto.lib(x_val.obj)
0001:006ece00* _d2i_X509_VAL
0001:006eceb0  _X509_VAL_it
0001:006ece30* _i2d_X509_VAL
0001:006ece60* _X509_VAL_new
0001:006ece80* _X509_VAL_free
Module: U:\extras\lib\libcrypto.lib(eng_lib.obj)
0001:006ecf50  _ENGINE_new
0001:006ecfe0* _engine_set_all_null
0001:006ed060  _engine_free_util
0001:006ed150  _ENGINE_free
0001:006ed230  _engine_cleanup_add_first
0001:006ed2a0  _engine_cleanup_add_last
0001:006ed310* _ENGINE_cleanup
0001:006ed350* _ENGINE_get_ex_new_index
0001:006ed390* _ENGINE_set_ex_data
0001:006ed3b0* _ENGINE_get_ex_data
0001:006ed3d0* _ENGINE_set_id
0001:006ed420* _ENGINE_set_name
0001:006ed470* _ENGINE_set_destroy_function
0001:006ed490* _ENGINE_set_init_function
0001:006ed4b0* _ENGINE_set_finish_function
0001:006ed4d0* _ENGINE_set_ctrl_function
0001:006ed4f0* _ENGINE_set_flags
0001:006ed510* _ENGINE_set_cmd_defns
0001:006ed530* _ENGINE_get_id
0001:006ed540* _ENGINE_get_name
0001:006ed550* _ENGINE_get_destroy_function
0001:006ed560* _ENGINE_get_init_function
0001:006ed570* _ENGINE_get_finish_function
0001:006ed580* _ENGINE_get_ctrl_function
0001:006ed590* _ENGINE_get_flags
0001:006ed5a0* _ENGINE_get_cmd_defns
0001:006ed5b0* _ENGINE_get_static_state
Module: U:\extras\lib\libcrypto.lib(o_names.obj)
0001:006ed810* _OBJ_NAME_init
0001:006ed890* _OBJ_NAME_new_index
0001:006eda10  _OBJ_NAME_get
0001:006edc70  _OBJ_NAME_add
0001:006eddb0* _OBJ_NAME_remove
0001:006ede50  _OBJ_NAME_do_all
0001:006ede90  _OBJ_NAME_do_all_sorted
0001:006edf70  _OBJ_NAME_cleanup
Module: U:\extras\lib\libcrypto.lib(evp_pbe.obj)
0001:006ee070  _EVP_PBE_CipherInit
0001:006ee390* _EVP_PBE_alg_add_type
0001:006ee460* _EVP_PBE_alg_add
0001:006ee560  _EVP_PBE_find
0001:006ee660  _EVP_PBE_cleanup
Module: U:\extras\lib\libcrypto.lib(obj_xref.obj)
0002:000244b0+ _sig_app
0002:000244c0+ _sigx_app
0001:006ee8a0  _OBJ_find_sigid_algs
0001:006ee940  _OBJ_find_sigid_by_algs
0001:006eea00* _OBJ_add_sigid
0001:006eeb10  _OBJ_sigid_free
Module: U:\extras\lib\libcrypto.lib(tb_rand.obj)
0001:006eed60* _ENGINE_unregister_RAND
0001:006eed80* _ENGINE_register_RAND
0001:006eede0* _ENGINE_register_all_RAND
0001:006eee40* _ENGINE_set_default_RAND
0001:006eeea0  _ENGINE_get_default_RAND
0001:006eeec0  _ENGINE_get_RAND
0001:006eeed0* _ENGINE_set_RAND
Module: U:\extras\lib\libcrypto.lib(md_rand.obj)
0001:006efd50  _RAND_SSLeay
0001:006efd60* _RAND_version
0002:00009390* _rand_ssleay_meth
Module: U:\extras\lib\libcrypto.lib(v3_info.obj)
0001:006eff60* _ACCESS_DESCRIPTION_free
0001:006f0400  _ACCESS_DESCRIPTION_it
0001:006f0220* _d2i_ACCESS_DESCRIPTION
0001:006f0250* _i2d_ACCESS_DESCRIPTION
0001:006f0280* _ACCESS_DESCRIPTION_new
0001:006f02a0* _d2i_AUTHORITY_INFO_ACCESS
0001:006f0440* _AUTHORITY_INFO_ACCESS_it
0001:006f02d0* _i2d_AUTHORITY_INFO_ACCESS
0001:006f0300* _AUTHORITY_INFO_ACCESS_new
0001:006f0320  _AUTHORITY_INFO_ACCESS_free
0001:006f0340* _i2a_ACCESS_DESCRIPTION
0001:006f0370  _v3_info
0001:006f03b0  _v3_sinfo
Module: U:\extras\lib\libcrypto.lib(dsa_lib.obj)
0001:006f04d0* _DSA_set_default_method
0001:006f04e0* _DSA_get_default_method
0001:006f0520  _DSA_new
0001:006f06d0* _DSA_set_method
0001:006f0720* _DSA_new_method
0001:006f0940  _DSA_free
0001:006f0a30  _DSA_up_ref
0001:006f0a70  _DSA_size
0001:006f0af0* _DSA_get_ex_new_index
0001:006f0b30* _DSA_set_ex_data
0001:006f0b50* _DSA_get_ex_data
0001:006f0b70* _DSA_dup_DH
0001:006f0c20* _DSA_version
Module: U:\extras\lib\libcrypto.lib(x_attrib.obj)
0001:006f0c50* _d2i_X509_ATTRIBUTE
0001:006f0e10  _X509_ATTRIBUTE_it
0001:006f0c80* _i2d_X509_ATTRIBUTE
0001:006f0cb0  _X509_ATTRIBUTE_new
0001:006f0cd0  _X509_ATTRIBUTE_free
0001:006f0cf0  _X509_ATTRIBUTE_dup
0001:006f0d10  _X509_ATTRIBUTE_create
0001:006f0df0* _X509_ATTRIBUTE_SET_it
Module: U:\extras\lib\libcrypto.lib(x_all.obj)
0001:006f0eb0  _X509_verify
0001:006f0ef0* _X509_REQ_verify
0001:006f0f30* _NETSCAPE_SPKI_verify
0001:006f0f70* _X509_sign
0001:006f0fc0  _X509_REQ_sign
0001:006f1010* _X509_CRL_sign
0001:006f1060* _NETSCAPE_SPKI_sign
0001:006f10b0* _d2i_X509_fp
0001:006f10e0* _i2d_X509_fp
0001:006f1110  _d2i_X509_bio
0001:006f1140* _i2d_X509_bio
0001:006f1170* _d2i_X509_CRL_fp
0001:006f11a0* _i2d_X509_CRL_fp
0001:006f11d0  _d2i_X509_CRL_bio
0001:006f1200* _i2d_X509_CRL_bio
0001:006f1230* _d2i_PKCS7_fp
0001:006f1260* _i2d_PKCS7_fp
0001:006f1290* _d2i_PKCS7_bio
0001:006f12c0* _i2d_PKCS7_bio
0001:006f12f0* _d2i_X509_REQ_fp
0001:006f1320* _i2d_X509_REQ_fp
0001:006f1350* _d2i_X509_REQ_bio
0001:006f1380* _i2d_X509_REQ_bio
0001:006f13b0* _d2i_RSAPrivateKey_fp
0001:006f13e0* _i2d_RSAPrivateKey_fp
0001:006f1410* _d2i_RSAPublicKey_fp
0001:006f1440* _d2i_RSA_PUBKEY_fp
0001:006f1470* _i2d_RSAPublicKey_fp
0001:006f14a0* _i2d_RSA_PUBKEY_fp
0001:006f14d0  _d2i_RSAPrivateKey_bio
0001:006f1500* _i2d_RSAPrivateKey_bio
0001:006f1530* _d2i_RSAPublicKey_bio
0001:006f1560* _d2i_RSA_PUBKEY_bio
0001:006f1590* _i2d_RSAPublicKey_bio
0001:006f15c0* _i2d_RSA_PUBKEY_bio
0001:006f15f0* _d2i_DSAPrivateKey_fp
0001:006f1620* _i2d_DSAPrivateKey_fp
0001:006f1650* _d2i_DSA_PUBKEY_fp
0001:006f1680* _i2d_DSA_PUBKEY_fp
0001:006f16b0* _d2i_DSAPrivateKey_bio
0001:006f16e0* _i2d_DSAPrivateKey_bio
0001:006f1710* _d2i_DSA_PUBKEY_bio
0001:006f1740* _i2d_DSA_PUBKEY_bio
0001:006f1770* _d2i_EC_PUBKEY_fp
0001:006f17a0* _i2d_EC_PUBKEY_fp
0001:006f17d0* _d2i_ECPrivateKey_fp
0001:006f1800* _i2d_ECPrivateKey_fp
0001:006f1830* _d2i_EC_PUBKEY_bio
0001:006f1860* _i2d_EC_PUBKEY_bio
0001:006f1890* _d2i_ECPrivateKey_bio
0001:006f18c0* _i2d_ECPrivateKey_bio
0001:006f18f0* _X509_pubkey_digest
0001:006f1950  _X509_digest
0001:006f1990  _X509_CRL_digest
0001:006f19d0* _X509_REQ_digest
0001:006f1a10* _X509_NAME_digest
0001:006f1a50* _PKCS7_ISSUER_AND_SERIAL_digest
0001:006f1a90* _d2i_PKCS8_fp
0001:006f1ac0* _i2d_PKCS8_fp
0001:006f1af0  _d2i_PKCS8_bio
0001:006f1b20  _i2d_PKCS8_bio
0001:006f1b50* _d2i_PKCS8_PRIV_KEY_INFO_fp
0001:006f1b80* _i2d_PKCS8_PRIV_KEY_INFO_fp
0001:006f1bb0* _i2d_PKCS8PrivateKeyInfo_fp
0001:006f1c10* _i2d_PrivateKey_fp
0001:006f1c40* _d2i_PrivateKey_fp
0001:006f1c70* _i2d_PUBKEY_fp
0001:006f1ca0* _d2i_PUBKEY_fp
0001:006f1cd0* _d2i_PKCS8_PRIV_KEY_INFO_bio
0001:006f1d00  _i2d_PKCS8_PRIV_KEY_INFO_bio
0001:006f1d30* _i2d_PKCS8PrivateKeyInfo_bio
0001:006f1d90* _i2d_PrivateKey_bio
0001:006f1dc0  _d2i_PrivateKey_bio
0001:006f1df0* _i2d_PUBKEY_bio
0001:006f1e20* _d2i_PUBKEY_bio
Module: U:\extras\lib\libcrypto.lib(a_int.obj)
0001:006f1e50* _ASN1_INTEGER_dup
0001:006f1e60  _ASN1_INTEGER_cmp
0001:006f1eb0  _i2c_ASN1_INTEGER
0001:006f20f0  _c2i_ASN1_INTEGER
0001:006f2420  _d2i_ASN1_UINTEGER
0001:006f26b0  _ASN1_INTEGER_set
0001:006f27e0  _ASN1_INTEGER_get
0001:006f2860  _BN_to_ASN1_INTEGER
0001:006f29b0  _ASN1_INTEGER_to_BN
Module: U:\extras\lib\libcrypto.lib(x509_ext.obj)
0001:006f2a50* _X509_CRL_get_ext_count
0001:006f2a70  _X509_CRL_get_ext_by_NID
0001:006f2a90* _X509_CRL_get_ext_by_OBJ
0001:006f2ab0* _X509_CRL_get_ext_by_critical
0001:006f2ad0  _X509_CRL_get_ext
0001:006f2af0* _X509_CRL_delete_ext
0001:006f2b10  _X509_CRL_get_ext_d2i
0001:006f2b30* _X509_CRL_add1_ext_i2d
0001:006f2b50* _X509_CRL_add_ext
0001:006f2b90  _X509_get_ext_count
0001:006f2bb0  _X509_get_ext_by_NID
0001:006f2bd0* _X509_get_ext_by_OBJ
0001:006f2bf0* _X509_get_ext_by_critical
0001:006f2c10  _X509_get_ext
0001:006f2c30* _X509_delete_ext
0001:006f2c50* _X509_add_ext
0001:006f2c90  _X509_get_ext_d2i
0001:006f2cb0* _X509_add1_ext_i2d
0001:006f2cd0* _X509_REVOKED_get_ext_count
0001:006f2cf0* _X509_REVOKED_get_ext_by_NID
0001:006f2d10* _X509_REVOKED_get_ext_by_OBJ
0001:006f2d30* _X509_REVOKED_get_ext_by_critical
0001:006f2d50* _X509_REVOKED_get_ext
0001:006f2d70* _X509_REVOKED_delete_ext
0001:006f2d90* _X509_REVOKED_add_ext
0001:006f2dc0  _X509_REVOKED_get_ext_d2i
0001:006f2de0* _X509_REVOKED_add1_ext_i2d
Module: U:\extras\lib\libcrypto.lib(v3_bcons.obj)
0001:006f3110* _BASIC_CONSTRAINTS_it
0001:006f3020* _d2i_BASIC_CONSTRAINTS
0001:006f3050* _i2d_BASIC_CONSTRAINTS
0001:006f3080* _BASIC_CONSTRAINTS_new
0001:006f30a0  _BASIC_CONSTRAINTS_free
0001:006f30c0  _v3_bcons
Module: U:\extras\lib\libcrypto.lib(v3_pcia.obj)
0001:006f3160* _d2i_PROXY_POLICY
0001:006f32b0* _PROXY_POLICY_it
0001:006f3190* _i2d_PROXY_POLICY
0001:006f31c0* _PROXY_POLICY_new
0001:006f31e0* _PROXY_POLICY_free
0001:006f3200* _d2i_PROXY_CERT_INFO_EXTENSION
0001:006f32f0  _PROXY_CERT_INFO_EXTENSION_it
0001:006f3230* _i2d_PROXY_CERT_INFO_EXTENSION
0001:006f3260  _PROXY_CERT_INFO_EXTENSION_new
0001:006f3280  _PROXY_CERT_INFO_EXTENSION_free
Module: U:\extras\lib\libcrypto.lib(x509_v3.obj)
0001:006f33b0  _X509v3_get_ext_count
0001:006f33e0  _X509v3_get_ext_by_NID
0001:006f3490  _X509v3_get_ext_by_OBJ
0001:006f3520  _X509v3_get_ext_by_critical
0001:006f35b0  _X509v3_get_ext
0001:006f3600  _X509v3_delete_ext
0001:006f3660  _X509v3_add_ext
0001:006f37a0  _X509_EXTENSION_create_by_OBJ
0001:006f38a0  _X509_EXTENSION_create_by_NID
0001:006f3930* _X509_EXTENSION_set_object
0001:006f3980* _X509_EXTENSION_set_critical
0001:006f39b0* _X509_EXTENSION_set_data
0001:006f3a00  _X509_EXTENSION_get_object
0001:006f3a20  _X509_EXTENSION_get_data
0001:006f3a40  _X509_EXTENSION_get_critical
Module: U:\extras\lib\libcrypto.lib(a_octet.obj)
0001:006f3a70  _ASN1_OCTET_STRING_dup
0001:006f3a80  _ASN1_OCTET_STRING_cmp
0001:006f3a90  _ASN1_OCTET_STRING_set
Module: U:\extras\lib\libcrypto.lib(bn_shift.obj)
0001:006f3aa0  _BN_lshift1
0001:006f3b90  _BN_rshift1
0001:006f3c80  _BN_lshift
0001:006f3e30  _BN_rshift
Module: U:\extras\lib\libcrypto.lib(bn_word.obj)
0001:006f4000  _BN_mod_word
0001:006f4080  _BN_div_word
0001:006f4180  _BN_sub_word
0001:006f4290  _BN_add_word
0001:006f43b0  _BN_mul_word
Module: U:\extras\lib\libcrypto.lib(bn_print.obj)
0001:006f4470* _BN_bn2hex
0001:006f4650  _BN_bn2dec
0001:006f4900  _BN_hex2bn
0001:006f4b20  _BN_dec2bn
0001:006f4ce0  _BN_asc2bn
0001:006f4d80* _BN_print_fp
0001:006f5060* _BN_print
Module: U:\extras\lib\libcrypto.lib(tb_rsa.obj)
0001:006f5320* _ENGINE_unregister_RSA
0001:006f5340* _ENGINE_register_RSA
0001:006f53a0* _ENGINE_register_all_RSA
0001:006f5400* _ENGINE_set_default_RSA
0001:006f5460  _ENGINE_get_default_RSA
0001:006f5480  _ENGINE_get_RSA
0001:006f5490* _ENGINE_set_RSA
Module: U:\extras\lib\libcrypto.lib(rsa_eay.obj)
0001:006f74c0  _RSA_PKCS1_SSLeay
Module: U:\extras\lib\libcrypto.lib(bn_blind.obj)
0001:006f7500* _BN_BLINDING_new
0001:006f7640  _BN_BLINDING_free
0001:006f76b0* _BN_BLINDING_update
0001:006f78c0* _BN_BLINDING_convert
0001:006f7950  _BN_BLINDING_convert_ex
0001:006f7a20* _BN_BLINDING_invert
0001:006f7ad0  _BN_BLINDING_invert_ex
0001:006f7bc0* _BN_BLINDING_get_thread_id
0001:006f7bd0* _BN_BLINDING_set_thread_id
0001:006f7be0  _BN_BLINDING_thread_id
0001:006f7bf0* _BN_BLINDING_get_flags
0001:006f7c00* _BN_BLINDING_set_flags
0001:006f7c10  _BN_BLINDING_create_param
Module: U:\extras\lib\libcrypto.lib(bn_ctx.obj)
0001:006f7e60* _BN_CTX_init
0001:006f8030  _BN_CTX_new
0001:006f80e0  _BN_CTX_free
0001:006f82b0  _BN_CTX_start
0001:006f83e0  _BN_CTX_end
0001:006f8470  _BN_CTX_get
Module: U:\extras\lib\libcrypto.lib(bn_add.obj)
0001:006f8660  _BN_uadd
0001:006f8790  _BN_usub
0001:006f89b0  _BN_add
0001:006f8a90  _BN_sub
Module: U:\extras\lib\libcrypto.lib(bn_mul.obj)
0001:006f8ba0* _bn_add_part_words
0001:006f8e60* _bn_mul_normal
0001:006f8fd0* _bn_mul_recursive
0001:006f96c0* _bn_mul_high
0001:006f9c60* _bn_mul_part_recursive
0001:006fa3e0  _BN_mul
0001:006fa800* _bn_mul_low_normal
0001:006fa8d0* _bn_mul_low_recursive
Module: U:\extras\lib\libcrypto.lib(bn_gcd.obj)
0001:006faa50  _BN_gcd
0001:006fac30  _BN_mod_inverse
Module: U:\extras\lib\libcrypto.lib(dh_key.obj)
0001:006fbd20  _DH_generate_key
0001:006fbd40  _DH_compute_key
0001:006fbd60  _DH_OpenSSL
Module: U:\extras\lib\libcrypto.lib(tb_dh.obj)
0001:006fbda0* _ENGINE_unregister_DH
0001:006fbdc0* _ENGINE_register_DH
0001:006fbe20* _ENGINE_register_all_DH
0001:006fbe80* _ENGINE_set_default_DH
0001:006fbee0  _ENGINE_get_default_DH
0001:006fbf00  _ENGINE_get_DH
0001:006fbf10* _ENGINE_set_DH
Module: U:\extras\lib\libcrypto.lib(by_file.obj)
0001:006fbf30  _X509_LOOKUP_file
0001:006fbf50  _X509_load_cert_file
0001:006fc3c0  _X509_load_crl_file
0001:006fc5f0* _X509_load_cert_crl_file
0002:00009420* _x509_file_lookup
Module: U:\extras\lib\libcrypto.lib(by_dir.obj)
0001:006fd260  _X509_LOOKUP_hash_dir
0002:00009450* _x509_dir_lookup
Module: U:\extras\lib\libcrypto.lib(ec_lib.obj)
0001:006fd2b0  _EC_GROUP_new
0001:006fd400  _EC_GROUP_free
0001:006fd4c0  _EC_GROUP_clear_free
0001:006fd5d0  _EC_GROUP_copy
0001:006fdac0  _EC_GROUP_dup
0001:006fdb10  _EC_GROUP_method_of
0001:006fdb20  _EC_METHOD_get_field_type
0001:006fdb30  _EC_GROUP_set_generator
0001:006fdda0  _EC_GROUP_get0_generator
0001:006fddb0  _EC_GROUP_get_order
0001:006fde00  _EC_GROUP_get_cofactor
0001:006fde50  _EC_GROUP_set_curve_name
0001:006fde60  _EC_GROUP_get_curve_name
0001:006fde70  _EC_GROUP_set_asn1_flag
0001:006fde80  _EC_GROUP_get_asn1_flag
0001:006fde90  _EC_GROUP_set_point_conversion_form
0001:006fdea0  _EC_GROUP_get_point_conversion_form
0001:006fdeb0  _EC_GROUP_set_seed
0001:006fdfd0  _EC_GROUP_get0_seed
0001:006fdfe0  _EC_GROUP_get_seed_len
0001:006fdff0  _EC_GROUP_set_curve_GFp
0001:006fe070  _EC_GROUP_get_curve_GFp
0001:006fe0f0  _EC_GROUP_set_curve_GF2m
0001:006fe170  _EC_GROUP_get_curve_GF2m
0001:006fe1f0  _EC_GROUP_get_degree
0001:006fe250* _EC_GROUP_check_discriminant
0001:006fe2c0  _EC_GROUP_cmp
0001:006fe640  _EC_EX_DATA_set_data
0001:006fe730  _EC_EX_DATA_get_data
0001:006fe780  _EC_EX_DATA_free_data
0001:006fe7f0* _EC_EX_DATA_clear_free_data
0001:006fe860  _EC_EX_DATA_free_all_data
0001:006fe8b0* _EC_EX_DATA_clear_free_all_data
0001:006fe900  _EC_POINT_new
0001:006fea10  _EC_POINT_free
0001:006fea50  _EC_POINT_clear_free
0001:006feab0  _EC_POINT_copy
0001:006feb60  _EC_POINT_dup
0001:006fed20* _EC_POINT_method_of
0001:006fed30  _EC_POINT_set_to_infinity
0001:006fedc0  _EC_POINT_set_Jprojective_coordinates_GFp
0001:006fee90* _EC_POINT_get_Jprojective_coordinates_GFp
0001:006fef60  _EC_POINT_set_affine_coordinates_GFp
0001:006ff010  _EC_POINT_set_affine_coordinates_GF2m
0001:006ff0c0  _EC_POINT_get_affine_coordinates_GFp
0001:006ff170  _EC_POINT_get_affine_coordinates_GF2m
0001:006ff220  _EC_POINT_set_compressed_coordinates_GFp
0001:006ff2d0  _EC_POINT_set_compressed_coordinates_GF2m
0001:006ff380  _EC_POINT_point2oct
0001:006ff450  _EC_POINT_oct2point
0001:006ff500  _EC_POINT_add
0001:006ff5c0  _EC_POINT_dbl
0001:006ff670  _EC_POINT_invert
0001:006ff710  _EC_POINT_is_at_infinity
0001:006ff7a0  _EC_POINT_is_on_curve
0001:006ff850  _EC_POINT_cmp
0001:006ff900  _EC_POINT_make_affine
0001:006ff9b0  _EC_POINTs_make_affine
0001:006ffa90* _EC_POINTs_mul
0001:006ffb00  _EC_POINT_mul
0001:006ffbb0  _EC_GROUP_precompute_mult
0001:006ffc00  _EC_GROUP_have_precompute_mult
Module: U:\extras\lib\libcrypto.lib(m_ecdsa.obj)
0001:006ffca0  _EVP_ecdsa
Module: U:\extras\lib\libcrypto.lib(p_verify.obj)
0001:006ffd20  _EVP_VerifyFinal
Module: U:\extras\lib\libcrypto.lib(rsa_sign.obj)
0001:006fff50  _RSA_sign
0001:007002c0  _int_rsa_verify
0001:007007b0  _RSA_verify
Module: U:\extras\lib\libcrypto.lib(ec_curve.obj)
0001:00700b80  _EC_GROUP_new_by_curve_name
0001:007010b0* _EC_get_builtin_curves
Module: U:\extras\lib\libcrypto.lib(m_dss1.obj)
0001:00704da0  _EVP_dss1
Module: U:\extras\lib\libcrypto.lib(ech_key.obj)
0001:00704e00  _ECDH_compute_key
Module: U:\extras\lib\libcrypto.lib(pmeth_fn.obj)
0001:00704e90  _EVP_PKEY_sign_init
0001:00704f30  _EVP_PKEY_sign
0001:00705090  _EVP_PKEY_verify_init
0001:00705130  _EVP_PKEY_verify
0001:00705200* _EVP_PKEY_verify_recover_init
0001:007052a0* _EVP_PKEY_verify_recover
0001:00705400  _EVP_PKEY_encrypt_init
0001:007054a0  _EVP_PKEY_encrypt
0001:00705600  _EVP_PKEY_decrypt_init
0001:007056a0  _EVP_PKEY_decrypt
0001:00705800* _EVP_PKEY_derive_init
0001:007058a0  _EVP_PKEY_derive_set_peer
0001:00705b30* _EVP_PKEY_derive
Module: U:\extras\lib\libcrypto.lib(dsa_sign.obj)
0001:00705c70* _DSA_do_sign
0001:00705c90  _DSA_sign
0001:00705d10  _DSA_sign_setup
Module: U:\extras\lib\libcrypto.lib(ecs_sign.obj)
0001:00705d30* _ECDSA_do_sign
0001:00705d90* _ECDSA_do_sign_ex
0001:00705e00  _ECDSA_sign
0001:00705eb0* _ECDSA_sign_ex
0001:00705f50  _ECDSA_sign_setup
Module: U:\extras\lib\libssl.lib(ssl_rsa.obj)
0001:00706280  _SSL_use_certificate
0001:00706340* _SSL_use_certificate_file
0001:00706560* _SSL_use_certificate_ASN1
0001:00706630* _SSL_use_RSAPrivateKey
0001:00706770* _SSL_use_RSAPrivateKey_file
0001:00706a00* _SSL_use_RSAPrivateKey_ASN1
0001:00706b50  _SSL_use_PrivateKey
0001:00706c10* _SSL_use_PrivateKey_file
0001:00706e20* _SSL_use_PrivateKey_ASN1
0001:00706f00* _SSL_CTX_use_certificate
0001:00706fc0* _SSL_CTX_use_certificate_file
0001:007071d0* _SSL_CTX_use_certificate_ASN1
0001:007072a0* _SSL_CTX_use_RSAPrivateKey
0001:007073e0* _SSL_CTX_use_RSAPrivateKey_file
0001:00707670* _SSL_CTX_use_RSAPrivateKey_ASN1
0001:007077c0* _SSL_CTX_use_PrivateKey
0001:00707880* _SSL_CTX_use_PrivateKey_file
0001:00707a90* _SSL_CTX_use_PrivateKey_ASN1
0001:00707b70* _SSL_CTX_use_certificate_chain_file
Module: U:\extras\lib\libcrypto.lib(x509type.obj)
0001:00707e10  _X509_certificate_type
Module: U:\extras\lib\libssl.lib(s2_pkt.obj)
0001:00708a10  _ssl2_read
0001:00708a30  _ssl2_peek
0001:00708a50  _ssl2_write
0001:00708fe0  _ssl2_part_read
0001:007090a0  _ssl2_do_write
Module: U:\extras\lib\libssl.lib(s2_enc.obj)
0001:007091e0  _ssl2_enc_init
0001:00709510  _ssl2_enc
0001:00709580  _ssl2_mac
Module: U:\extras\lib\libcrypto.lib(p_sign.obj)
0001:007096a0  _EVP_SignFinal
Module: U:\extras\lib\libcrypto.lib(bss_mem.obj)
0001:0070a180  _BIO_s_mem
0001:0070a190  _BIO_new_mem_buf
Module: U:\extras\lib\libcrypto.lib(rsa_asn1.obj)
0001:0070a290  _d2i_RSAPrivateKey
0001:0070a390  _RSAPrivateKey_it
0001:0070a2c0  _i2d_RSAPrivateKey
0001:0070a2f0  _d2i_RSAPublicKey
0001:0070a3b0  _RSAPublicKey_it
0001:0070a320  _i2d_RSAPublicKey
0001:0070a350* _RSAPublicKey_dup
0001:0070a370  _RSAPrivateKey_dup
Module: U:\extras\lib\libcrypto.lib(hmac.obj)
0001:0070a8f0  _HMAC_Init_ex
0001:0070ac90* _HMAC_Init
0001:0070acf0  _HMAC_Update
0001:0070ad10  _HMAC_Final
0001:0070ada0  _HMAC_CTX_init
0001:0070add0  _HMAC_CTX_copy
0001:0070ae50  _HMAC_CTX_cleanup
0001:0070ae90  _HMAC
0001:0070afa0* _HMAC_CTX_set_flags
Module: U:\extras\lib\libcrypto.lib(e_aes.obj)
0001:0070bdb0  _EVP_aes_128_cbc
0001:0070bdc0* _EVP_aes_128_cfb128
0001:0070bdd0* _EVP_aes_128_ofb
0001:0070bde0* _EVP_aes_128_ecb
0001:0070bdf0* _EVP_aes_192_cbc
0001:0070be00* _EVP_aes_192_cfb128
0001:0070be10* _EVP_aes_192_ofb
0001:0070be20* _EVP_aes_192_ecb
0001:0070be30* _EVP_aes_256_cbc
0001:0070be40* _EVP_aes_256_cfb128
0001:0070be50* _EVP_aes_256_ofb
0001:0070be60* _EVP_aes_256_ecb
0001:0070be70* _EVP_aes_128_cfb1
0001:0070be80* _EVP_aes_192_cfb1
0001:0070be90* _EVP_aes_256_cfb1
0001:0070bea0* _EVP_aes_128_cfb8
0001:0070beb0* _EVP_aes_192_cfb8
0001:0070bec0* _EVP_aes_256_cfb8
Module: U:\extras\lib\libssl.lib(t1_reneg.obj)
0001:0070c370  _ssl_add_clienthello_renegotiate_ext
0001:0070c4d0  _ssl_parse_clienthello_renegotiate_ext
0001:0070c5d0  _ssl_add_serverhello_renegotiate_ext
0001:0070c8b0  _ssl_parse_serverhello_renegotiate_ext
Module: U:\extras\lib\libssl.lib(t1_enc.obj)
0001:0070d1d0  _tls1_change_cipher_state
0001:0070da00  _tls1_setup_key_block
0001:0070dcc0  _tls1_enc
0001:0070e050  _tls1_cert_verify_mac
0001:0070e1f0  _tls1_final_finish_mac
0001:0070e430  _tls1_mac
0001:0070e6f0  _tls1_generate_master_secret
0001:0070e780  _tls1_alert_code
Module: U:\extras\lib\xmlrpc.lib(encodings.obj)
0001:0070eabc  _utf8_decode
0001:0070eade* _utf8_encode
Module: U:\extras\lib\expat.lib(xmlparse.obj)
0001:0070eb33* _XML_UseParserAsHandlerArg
0001:0070eb3e* _XML_UseForeignDTD
0001:0070eb68* _XML_SetReturnNSTriplet
0001:0070eb8c  _XML_SetUserData
0001:0070eba7* _XML_GetBase
0001:0070ebb5* _XML_GetSpecifiedAttributeCount
0001:0070ebc3* _XML_GetIdAttributeIndex
0001:0070ebd1  _XML_SetElementHandler
0001:0070ebe5* _XML_SetStartElementHandler
0001:0070ebf3* _XML_SetEndElementHandler
0001:0070ec01  _XML_SetCharacterDataHandler
0001:0070ec0f* _XML_SetProcessingInstructionHandler
0001:0070ec1d* _XML_SetCommentHandler
0001:0070ec2b* _XML_SetCdataSectionHandler
0001:0070ec3f* _XML_SetStartCdataSectionHandler
0001:0070ec4d* _XML_SetEndCdataSectionHandler
0001:0070ec5b* _XML_SetDefaultHandler
0001:0070ec70* _XML_SetDefaultHandlerExpand
0001:0070ec85* _XML_SetDoctypeDeclHandler
0001:0070ec99* _XML_SetStartDoctypeDeclHandler
0001:0070eca7* _XML_SetEndDoctypeDeclHandler
0001:0070ecb5* _XML_SetUnparsedEntityDeclHandler
0001:0070ecc3* _XML_SetNotationDeclHandler
0001:0070ecd1* _XML_SetNamespaceDeclHandler
0001:0070ece5* _XML_SetStartNamespaceDeclHandler
0001:0070ecf3* _XML_SetEndNamespaceDeclHandler
0001:0070ed01* _XML_SetNotStandaloneHandler
0001:0070ed0f* _XML_SetExternalEntityRefHandler
0001:0070ed1d* _XML_SetExternalEntityRefHandlerArg
0001:0070ed34* _XML_SetSkippedEntityHandler
0001:0070ed42* _XML_SetUnknownEncodingHandler
0001:0070ed59* _XML_SetElementDeclHandler
0001:0070ed6a* _XML_SetAttlistDeclHandler
0001:0070ed7b* _XML_SetEntityDeclHandler
0001:0070ed8c* _XML_SetXmlDeclHandler
0001:0070ed9d* _XML_SetParamEntityParsing
0001:0070edc7* _XML_ParseBuffer
0001:0070eef8* _XML_StopParser
0001:0070ef6f* _XML_ResumeParser
0001:0070f058  _XML_GetErrorCode
0001:0070f066  _XML_GetCurrentByteIndex
0001:0070f085  _XML_GetCurrentByteCount
0001:0070f0a7* _XML_GetInputContext
0001:0070f0d8  _XML_GetCurrentLineNumber
0001:0070f131  _XML_GetCurrentColumnNumber
0001:0070f187* _XML_FreeContentModel
0001:0070f19c* _XML_MemMalloc
0001:0070f1b1* _XML_MemRealloc
0001:0070f1cc* _XML_MemFree
0001:0070f1e1  _XML_ErrorString
0001:0070f206* _XML_ExpatVersion
0001:0070f210* _XML_ExpatVersionInfo
0001:0070f22e* _XML_GetFeatureList
0001:0070f326* _XML_DefaultCurrent
0001:0070fae9  _XML_ParserFree
0001:0070ff3a* _XML_GetParsingStatus
0001:0070ff80* _XML_GetBuffer
0001:00710102  _XML_Parse
0001:00710455* _XML_SetBase
0001:0071049f* _XML_SetEncoding
0001:00711f0a* _XML_ExternalEntityParserCreate
0001:0071252d* _XML_ParserReset
0001:00712881* _XML_ParserCreate_MM
0001:007128ce* _XML_ParserCreateNS
0001:007128f6  _XML_ParserCreate
Module: U:\extras\lib\xmlrpc.lib(base64.obj)
0001:007180b0  _buffer_delete
0001:007180e5* _buffer_add
0001:00718136* _buffer_new
0001:00718168  _base64_decode
0001:007182f2  _base64_encode
Module: U:\extras\lib\pthread.lib(my_os2tls.obj)
0002:000244d0+ _tls_bits
0001:007184e6* _TlsFreeThreadLocalMemory
0001:00718620* _TlsAllocThreadLocalMemory
0001:007186d1  _TlsSetValue
0001:00718731  _TlsGetValue
0001:00718789  _TlsFree
0001:00718862  _TlsAlloc
0002:00021d40* _tls_storage
0002:00021d44* _tls_mutex
Module: U:\extras\lib\libcrypto.lib(evp_key.obj)
0001:00718a70* _EVP_set_pw_prompt
0001:00718ab0  _EVP_get_pw_prompt
0001:00718ad0* _EVP_read_pw_string
0001:00718af0  _EVP_read_pw_string_min
0001:00718c50  _EVP_BytesToKey
Module: U:\extras\lib\libcrypto.lib(encode.obj)
0001:00718f20  _EVP_EncodeInit
0001:00718f40  _EVP_EncodeBlock
0001:00719080  _EVP_EncodeFinal
0001:00719120  _EVP_EncodeUpdate
0001:007193d0  _EVP_DecodeInit
0001:007193f0  _EVP_DecodeBlock
0001:007195a0  _EVP_DecodeUpdate
0001:00719910  _EVP_DecodeFinal
Module: U:\extras\lib\libcrypto.lib(eng_table.obj)
0001:00719b50* _ENGINE_get_table_flags
0001:00719b60* _ENGINE_set_table_flags
0001:00719b90  _engine_table_register
0001:00719da0  _engine_table_unregister
0001:00719e20  _engine_table_cleanup
0001:00719ea0  _engine_table_select
0001:0071a010  _engine_table_doall
Module: U:\extras\lib\libcrypto.lib(eng_list.obj)
0001:0071a240  _ENGINE_get_first
0001:0071a2a0* _ENGINE_get_last
0001:0071a300  _ENGINE_get_next
0001:0071a3a0* _ENGINE_get_prev
0001:0071a440* _ENGINE_add
0001:0071a680* _ENGINE_remove
0001:0071a890* _ENGINE_by_id
0001:0071ab60* _ENGINE_up_ref
Module: U:\extras\lib\libcrypto.lib(evp_asn1.obj)
0001:0071abe0  _ASN1_TYPE_set_octetstring
0001:0071ac60  _ASN1_TYPE_get_octetstring
0001:0071ad80* _ASN1_TYPE_set_int_octetstring
0001:0071af10* _ASN1_TYPE_get_int_octetstring
Module: U:\extras\lib\libcrypto.lib(tb_pkmeth.obj)
0001:0071b1f0* _ENGINE_unregister_pkey_meths
0001:0071b210* _ENGINE_register_pkey_meths
0001:0071b290* _ENGINE_register_all_pkey_meths
0001:0071b320* _ENGINE_set_default_pkey_meths
0001:0071b3a0  _ENGINE_get_pkey_meth_engine
0001:0071b3e0  _ENGINE_get_pkey_meth
0001:0071b460* _ENGINE_get_pkey_meths
0001:0071b470* _ENGINE_set_pkey_meths
0001:0071b490  _engine_pkey_meths_free
Module: U:\extras\lib\libcrypto.lib(rsa_pmeth.obj)
0001:0071c730  _rsa_pkey_meth
Module: U:\extras\lib\libcrypto.lib(dh_pmeth.obj)
0001:0071cc20  _dh_pkey_meth
Module: U:\extras\lib\libcrypto.lib(dsa_pmeth.obj)
0001:0071d3c0  _dsa_pkey_meth
Module: U:\extras\lib\libcrypto.lib(ec_pmeth.obj)
0001:0071db80  _ec_pkey_meth
Module: U:\extras\lib\libcrypto.lib(hm_pmeth.obj)
0001:0071e0d0  _hmac_pkey_meth
Module: U:\extras\lib\libcrypto.lib(tb_asnmth.obj)
0001:0071e220* _ENGINE_unregister_pkey_asn1_meths
0001:0071e240* _ENGINE_register_pkey_asn1_meths
0001:0071e2c0* _ENGINE_register_all_pkey_asn1_meths
0001:0071e350* _ENGINE_set_default_pkey_asn1_meths
0001:0071e3d0  _ENGINE_get_pkey_asn1_meth_engine
0001:0071e410  _ENGINE_get_pkey_asn1_meth
0001:0071e490* _ENGINE_get_pkey_asn1_meths
0001:0071e4a0* _ENGINE_set_pkey_asn1_meths
0001:0071e4c0  _engine_pkey_asn1_meths_free
0001:0071e540* _ENGINE_get_pkey_asn1_meth_str
0001:0071e620  _ENGINE_pkey_asn1_find_str
Module: U:\extras\lib\libcrypto.lib(rsa_ameth.obj)
0001:0071f280  _rsa_asn1_meths
Module: U:\extras\lib\libcrypto.lib(dh_ameth.obj)
0001:00720180* _DHparams_print
0001:007201c0  _dh_asn1_meth
Module: U:\extras\lib\libcrypto.lib(dsa_ameth.obj)
0001:00721560  _dsa_asn1_meths
Module: U:\extras\lib\libcrypto.lib(ec_ameth.obj)
0001:00722b20  _eckey_asn1_meth
Module: U:\extras\lib\libcrypto.lib(hm_ameth.obj)
0001:00722e10  _hmac_asn1_meth
Module: U:\extras\lib\libcrypto.lib(pcy_tree.obj)
0001:00722ea0  _X509_policy_tree_free
0001:00722f80  _X509_policy_check
Module: U:\extras\lib\libcrypto.lib(a_time.obj)
0001:00723c50* _d2i_ASN1_TIME
0001:007240c0  _ASN1_TIME_it
0001:00723c80* _i2d_ASN1_TIME
0001:00723cb0* _ASN1_TIME_new
0001:00723cd0  _ASN1_TIME_free
0001:00723d10* _ASN1_TIME_set
0001:00723dd0  _ASN1_TIME_adj
0001:00723ea0  _ASN1_TIME_check
0001:00723ee0* _ASN1_TIME_to_generalizedtime
0001:00724020* _ASN1_TIME_set_string
Module: U:\extras\lib\libcrypto.lib(a_utctm.obj)
0001:007240e0  _ASN1_UTCTIME_check
0001:007243b0* _ASN1_UTCTIME_set_string
0001:00724470* _ASN1_UTCTIME_set
0001:007245e0  _ASN1_UTCTIME_adj
0001:00724770* _ASN1_UTCTIME_cmp_time_t
Module: U:\extras\lib\libcrypto.lib(a_gentm.obj)
0001:00724960  _ASN1_GENERALIZEDTIME_check
0001:00724ca0* _ASN1_GENERALIZEDTIME_set_string
0001:00724d60* _ASN1_GENERALIZEDTIME_set
0001:00724ea0  _ASN1_GENERALIZEDTIME_adj
Module: U:\extras\lib\libcrypto.lib(x_bignum.obj)
0001:007251a0  _BIGNUM_it
0001:007251c0  _CBIGNUM_it
Module: U:\extras\lib\libcrypto.lib(x_long.obj)
0001:00725450  _LONG_it
0001:00725480  _ZLONG_it
Module: U:\extras\lib\libcrypto.lib(bn_rand.obj)
0001:00725980  _BN_pseudo_rand
0001:007259b0  _BN_rand
0001:007259e0* _BN_bntest_rand
0001:00725a10  _BN_rand_range
0001:00725a30  _BN_pseudo_rand_range
Module: U:\extras\lib\libcrypto.lib(md5_dgst.obj)
0001:00725a50  _MD5_Update
0001:00725df0* _MD5_Transform
0001:00725e20  _MD5_Final
0001:00726020  _MD5_Init
0001:00726050* _MD5_version
Module: U:\extras\lib\libcrypto.lib(sha512.obj)
0001:00726080  _SHA384_Init
0001:00726130  _SHA512_Init
0001:007261e0  _SHA512_Final
0001:00726920* _SHA384_Final
0001:00726930  _SHA512_Update
0001:00726bc0* _SHA384_Update
0001:00726bd0* _SHA512_Transform
0001:00726c00* _SHA384
0001:00726d30* _SHA512
0001:00726e60* _SHA512_version
Module: U:\extras\lib\libcrypto.lib(sha256.obj)
0001:00726e90  _SHA224_Init
0001:00726ef0  _SHA256_Init
0001:00726f50  _SHA256_Update
0001:007272f0* _SHA224_Update
0001:00727300* _SHA256_Transform
0001:00727330  _SHA256_Final
0001:00727610* _SHA224_Final
0001:00727620* _SHA256
0001:007276e0* _SHA224
0001:007277a0* _SHA256_version
Module: U:\extras\lib\libcrypto.lib(sha1dgst.obj)
0001:007277d0  _SHA1_Update
0001:00727b70* _SHA1_Transform
0001:00727ba0  _SHA1_Final
0001:00727db0  _SHA1_Init
0001:00727df0* _SHA1_version
Module: U:\extras\lib\libcrypto.lib(a_verify.obj)
0001:00727e40* _ASN1_verify
0001:00727fe0  _ASN1_item_verify
Module: U:\extras\lib\libcrypto.lib(a_enum.obj)
0001:00728260* _ASN1_ENUMERATED_set
0001:00728390  _ASN1_ENUMERATED_get
0001:00728410* _BN_to_ASN1_ENUMERATED
0001:00728560  _ASN1_ENUMERATED_to_BN
Module: U:\extras\lib\libcrypto.lib(a_utf8.obj)
0001:00728600  _UTF8_getc
0001:007289f0  _UTF8_putc
Module: U:\extras\lib\libcrypto.lib(asn1_par.obj)
0001:007299b0* _ASN1_parse
0001:007299f0  _ASN1_parse_dump
0001:00729a30  _ASN1_tag2str
Module: U:\extras\lib\libcrypto.lib(x509name.obj)
0001:00729c40* _X509_NAME_get_text_by_OBJ
0001:00729d90* _X509_NAME_get_text_by_NID
0001:00729de0  _X509_NAME_entry_count
0001:00729e10  _X509_NAME_get_index_by_NID
0001:00729ec0* _X509_NAME_get_index_by_OBJ
0001:00729f50  _X509_NAME_get_entry
0001:00729fa0  _X509_NAME_delete_entry
0001:0072a070  _X509_NAME_add_entry
0001:0072a240* _X509_NAME_add_entry_by_NID
0001:0072a430  _X509_NAME_add_entry_by_txt
0001:0072a630* _X509_NAME_add_entry_by_OBJ
0001:0072a800* _X509_NAME_ENTRY_create_by_txt
0001:0072aa10* _X509_NAME_ENTRY_create_by_NID
0001:0072ac00* _X509_NAME_ENTRY_create_by_OBJ
0001:0072ae00* _X509_NAME_ENTRY_set_object
0001:0072ae80* _X509_NAME_ENTRY_set_data
0001:0072af90  _X509_NAME_ENTRY_get_object
0001:0072afb0  _X509_NAME_ENTRY_get_data
Module: U:\extras\lib\libcrypto.lib(t_x509.obj)
0001:0072b030* _X509_ocspid_print
0001:0072b1f0* _X509_signature_print
0001:0072b310  _ASN1_STRING_print
0001:0072b410  _ASN1_GENERALIZEDTIME_print
0001:0072b7b0  _ASN1_UTCTIME_print
0001:0072b9f0* _ASN1_TIME_print
0001:0072bbc0* _X509_print_ex
0001:0072c350* _X509_print_ex_fp
0001:0072ca20* _X509_print_fp
0001:0072cac0* _X509_print
0001:0072cae0  _X509_NAME_print
Module: U:\extras\lib\libcrypto.lib(a_mbstr.obj)
0001:0072cf80  _ASN1_mbstring_copy
0001:0072d490  _ASN1_mbstring_ncopy
Module: U:\extras\lib\libcrypto.lib(tasn_utl.obj)
0001:0072daa0  _asn1_get_choice_selector
0001:0072dac0  _asn1_set_choice_selector
0001:0072daf0  _asn1_do_lock
0001:0072db70  _asn1_enc_init
0001:0072dbb0  _asn1_enc_free
0001:0072dc00  _asn1_enc_save
0001:0072dd20  _asn1_enc_restore
0001:0072de30  _asn1_get_field_ptr
0001:0072de50  _asn1_do_adb
Module: U:\extras\lib\libcrypto.lib(a_type.obj)
0001:0072df20  _ASN1_TYPE_get
0001:0072df40  _ASN1_TYPE_set
0001:0072dfa0  _ASN1_TYPE_set1
0001:0072e0d0  _ASN1_TYPE_cmp
Module: U:\extras\lib\libcrypto.lib(a_bitstr.obj)
0001:0072e140  _ASN1_BIT_STRING_set
0001:0072e150  _i2c_ASN1_BIT_STRING
0001:0072e350  _c2i_ASN1_BIT_STRING
0001:0072e5c0  _ASN1_BIT_STRING_set_bit
0001:0072e790  _ASN1_BIT_STRING_get_bit
0001:0072e800* _ASN1_BIT_STRING_check
Module: U:\extras\lib\libcrypto.lib(v3_utl.obj)
0001:0072eb50  _X509V3_conf_free
0001:0072ef30  _X509V3_add_value
0001:0072f0c0  _X509V3_add_value_uchar
0001:0072f0e0  _X509V3_add_value_bool
0001:0072f120* _X509V3_add_value_bool_nf
0001:0072f150  _i2s_ASN1_ENUMERATED
0001:0072f1e0  _i2s_ASN1_INTEGER
0001:0072f270  _s2i_ASN1_INTEGER
0001:0072f420  _X509V3_add_value_int
0001:0072f520  _X509V3_get_value_bool
0001:0072f740  _X509V3_get_value_int
0001:0072f7b0  _X509V3_parse_list
0001:0072fcb0  _hex_to_string
0001:0072fd80  _string_to_hex
0001:0072ffc0  _name_cmp
0001:00730010* _X509_get1_email
0001:00730070* _X509_get1_ocsp
0001:00730190* _X509_REQ_get1_email
0001:00730210* _X509_email_free
0001:00730230  _a2i_IPADDRESS
0001:00730350  _a2i_IPADDRESS_NC
0001:007305e0  _a2i_ipadd
0001:007306c0  _X509V3_NAME_from_section
Module: U:\extras\lib\libcrypto.lib(v3_alt.obj)
0001:007314e0  _i2v_GENERAL_NAME
0001:007319f0  _i2v_GENERAL_NAMES
0001:00731b00  _GENERAL_NAME_print
0001:00731e60  _v2i_GENERAL_NAMES
0001:00731f10  _v2i_GENERAL_NAME
0001:00731f30* _a2i_GENERAL_NAME
0001:00732320  _v2i_GENERAL_NAME_ex
0001:007324e0  _v3_alt
Module: U:\extras\lib\libcrypto.lib(v3_conf.obj)
0001:00732c20* _X509V3_EXT_nconf
0001:00732dc0* _X509V3_EXT_nconf_nid
0001:00732f10  _X509V3_EXT_i2d
0001:00732f90* _X509V3_EXT_add_nconf_sk
0001:007331d0* _X509V3_EXT_add_nconf
0001:00733220* _X509V3_EXT_CRL_add_nconf
0001:00733270* _X509V3_EXT_REQ_add_nconf
0001:00733300* _X509V3_get_string
0001:00733380  _X509V3_get_section
0001:007333f0* _X509V3_string_free
0001:00733430  _X509V3_section_free
0001:00733470  _X509V3_set_nconf
0001:00733490* _X509V3_set_ctx
0001:007334c0* _X509V3_EXT_conf
0001:00733650* _X509V3_EXT_conf_nid
0001:007337b0* _X509V3_set_conf_lhash
0001:007337d0* _X509V3_EXT_add_conf
0001:00733830* _X509V3_EXT_CRL_add_conf
0001:00733890* _X509V3_EXT_REQ_add_conf
Module: U:\extras\lib\libcrypto.lib(pcy_data.obj)
0001:00733930  _policy_data_free
0001:007339a0  _policy_data_new
Module: U:\extras\lib\libcrypto.lib(v3_cpols.obj)
0001:00733e30  _POLICYINFO_free
0001:00734da0* _POLICYINFO_it
0001:00734dd0* _POLICYQUALINFO_it
0001:00734e00* _USERNOTICE_it
0001:00734e30* _NOTICEREF_it
0001:00734910* _d2i_CERTIFICATEPOLICIES
0001:00734d70* _CERTIFICATEPOLICIES_it
0001:00734940* _i2d_CERTIFICATEPOLICIES
0001:00734970* _CERTIFICATEPOLICIES_new
0001:00734990* _CERTIFICATEPOLICIES_free
0001:007349b0* _d2i_POLICYINFO
0001:007349e0* _i2d_POLICYINFO
0001:00734a10* _POLICYINFO_new
0001:00734a30* _d2i_POLICYQUALINFO
0001:00734a60* _i2d_POLICYQUALINFO
0001:00734a90* _POLICYQUALINFO_new
0001:00734ab0  _POLICYQUALINFO_free
0001:00734ad0* _d2i_USERNOTICE
0001:00734b00* _i2d_USERNOTICE
0001:00734b30* _USERNOTICE_new
0001:00734b50* _USERNOTICE_free
0001:00734b70* _d2i_NOTICEREF
0001:00734ba0* _i2d_NOTICEREF
0001:00734bd0* _NOTICEREF_new
0001:00734bf0* _NOTICEREF_free
0001:00734c40* _X509_POLICY_NODE_print
0001:00734d20  _v3_cpols
Module: U:\extras\lib\libcrypto.lib(pcy_map.obj)
0001:00735000  _policy_cache_set_mapping
Module: U:\extras\lib\libcrypto.lib(v3_pcons.obj)
0001:007354b0* _POLICY_CONSTRAINTS_it
0001:00735420* _POLICY_CONSTRAINTS_new
0001:00735440  _POLICY_CONSTRAINTS_free
0001:00735460  _v3_policy_constraints
Module: U:\extras\lib\libcrypto.lib(p5_crpt.obj)
0001:00735500* _PKCS5_PBE_add
0001:00735580  _PKCS5_PBE_keyivgen
Module: U:\extras\lib\libcrypto.lib(p12_crpt.obj)
0001:00735970* _PKCS12_PBE_add
0001:00735990  _PKCS12_PBE_keyivgen
Module: U:\extras\lib\libcrypto.lib(p5_crpt2.obj)
0001:00735c10* _PKCS5_PBKDF2_HMAC
0001:00735f40* _PKCS5_PBKDF2_HMAC_SHA1
0001:00735fc0  _PKCS5_v2_PBE_keyivgen
Module: U:\extras\lib\libcrypto.lib(rand_os2.obj)
0001:007364e0  _RAND_poll
Module: U:\extras\lib\libcrypto.lib(dsa_ossl.obj)
0001:007372f0  _DSA_OpenSSL
Module: U:\extras\lib\libcrypto.lib(tb_dsa.obj)
0001:00737330* _ENGINE_unregister_DSA
0001:00737350* _ENGINE_register_DSA
0001:007373b0* _ENGINE_register_all_DSA
0001:00737410* _ENGINE_set_default_DSA
0001:00737470  _ENGINE_get_default_DSA
0001:00737490  _ENGINE_get_DSA
0001:007374a0* _ENGINE_set_DSA
Module: U:\extras\lib\libcrypto.lib(x_req.obj)
0001:00737500* _d2i_X509_REQ_INFO
0001:00737670  _X509_REQ_INFO_it
0001:00737530* _i2d_X509_REQ_INFO
0001:00737560* _X509_REQ_INFO_new
0001:00737580* _X509_REQ_INFO_free
0001:007375a0  _d2i_X509_REQ
0001:007376a0  _X509_REQ_it
0001:007375d0  _i2d_X509_REQ
0001:00737600  _X509_REQ_new
0001:00737620  _X509_REQ_free
0001:00737640* _X509_REQ_dup
Module: U:\extras\lib\libcrypto.lib(x_spki.obj)
0001:007377d0* _d2i_NETSCAPE_SPKAC
0001:00737920  _NETSCAPE_SPKAC_it
0001:00737800* _i2d_NETSCAPE_SPKAC
0001:00737830* _NETSCAPE_SPKAC_new
0001:00737850* _NETSCAPE_SPKAC_free
0001:00737870* _d2i_NETSCAPE_SPKI
0001:00737950* _NETSCAPE_SPKI_it
0001:007378a0* _i2d_NETSCAPE_SPKI
0001:007378d0* _NETSCAPE_SPKI_new
0001:007378f0* _NETSCAPE_SPKI_free
Module: U:\extras\lib\libcrypto.lib(a_sign.obj)
0001:00737a30* _ASN1_sign
0001:00737dc0  _ASN1_item_sign
Module: U:\extras\lib\libcrypto.lib(a_d2i_fp.obj)
0001:007383f0  _ASN1_d2i_fp
0001:007384d0  _ASN1_d2i_bio
0001:00738540  _ASN1_item_d2i_bio
0001:007385c0  _ASN1_item_d2i_fp
Module: U:\extras\lib\libcrypto.lib(a_i2d_fp.obj)
0001:007386c0  _ASN1_i2d_fp
0001:00738810  _ASN1_i2d_bio
0001:007388f0  _ASN1_item_i2d_fp
0001:00738a40  _ASN1_item_i2d_bio
Module: U:\extras\lib\libcrypto.lib(pk7_asn1.obj)
0001:00738c30  _d2i_PKCS7
0001:00739300  _PKCS7_it
0001:00738c60  _i2d_PKCS7
0001:00738c90  _PKCS7_new
0001:00738cb0  _PKCS7_free
0001:00738cd0* _i2d_PKCS7_NDEF
0001:00738d00* _PKCS7_dup
0001:00738d20* _d2i_PKCS7_SIGNED
0001:00739330* _PKCS7_SIGNED_it
0001:00738d50* _i2d_PKCS7_SIGNED
0001:00738d80  _PKCS7_SIGNED_new
0001:00738da0  _PKCS7_SIGNED_free
0001:00738dc0* _d2i_PKCS7_SIGNER_INFO
0001:00739360* _PKCS7_SIGNER_INFO_it
0001:00738df0* _i2d_PKCS7_SIGNER_INFO
0001:00738e20  _PKCS7_SIGNER_INFO_new
0001:00738e40  _PKCS7_SIGNER_INFO_free
0001:00738e60* _d2i_PKCS7_ISSUER_AND_SERIAL
0001:007393a0  _PKCS7_ISSUER_AND_SERIAL_it
0001:00738e90* _i2d_PKCS7_ISSUER_AND_SERIAL
0001:00738ec0* _PKCS7_ISSUER_AND_SERIAL_new
0001:00738ee0* _PKCS7_ISSUER_AND_SERIAL_free
0001:00738f00* _d2i_PKCS7_ENVELOPE
0001:007393d0* _PKCS7_ENVELOPE_it
0001:00738f30* _i2d_PKCS7_ENVELOPE
0001:00738f60  _PKCS7_ENVELOPE_new
0001:00738f80* _PKCS7_ENVELOPE_free
0001:00738fa0* _d2i_PKCS7_RECIP_INFO
0001:00739400* _PKCS7_RECIP_INFO_it
0001:00738fd0* _i2d_PKCS7_RECIP_INFO
0001:00739000  _PKCS7_RECIP_INFO_new
0001:00739020  _PKCS7_RECIP_INFO_free
0001:00739040* _d2i_PKCS7_ENC_CONTENT
0001:00739430* _PKCS7_ENC_CONTENT_it
0001:00739070* _i2d_PKCS7_ENC_CONTENT
0001:007390a0* _PKCS7_ENC_CONTENT_new
0001:007390c0* _PKCS7_ENC_CONTENT_free
0001:007390e0* _d2i_PKCS7_SIGN_ENVELOPE
0001:00739460* _PKCS7_SIGN_ENVELOPE_it
0001:00739110* _i2d_PKCS7_SIGN_ENVELOPE
0001:00739140  _PKCS7_SIGN_ENVELOPE_new
0001:00739160* _PKCS7_SIGN_ENVELOPE_free
0001:00739180* _d2i_PKCS7_ENCRYPT
0001:00739490* _PKCS7_ENCRYPT_it
0001:007391b0* _i2d_PKCS7_ENCRYPT
0001:007391e0  _PKCS7_ENCRYPT_new
0001:00739200* _PKCS7_ENCRYPT_free
0001:00739220* _d2i_PKCS7_DIGEST
0001:007394c0* _PKCS7_DIGEST_it
0001:00739250* _i2d_PKCS7_DIGEST
0001:00739280  _PKCS7_DIGEST_new
0001:007392a0* _PKCS7_DIGEST_free
0001:007392c0* _PKCS7_print_ctx
0001:007394f0  _PKCS7_ATTR_SIGN_it
0001:00739520  _PKCS7_ATTR_VERIFY_it
Module: U:\extras\lib\libcrypto.lib(dsa_asn1.obj)
0001:00739c80  _d2i_DSA_SIG
0001:00739e70* _DSA_SIG_it
0001:00739cb0  _i2d_DSA_SIG
0001:00739ce0  _DSA_SIG_new
0001:00739d00  _DSA_SIG_free
0001:00739d20  _d2i_DSAPrivateKey
0001:00739e90* _DSAPrivateKey_it
0001:00739d50  _i2d_DSAPrivateKey
0001:00739d80  _d2i_DSAparams
0001:00739eb0* _DSAparams_it
0001:00739db0  _i2d_DSAparams
0001:00739de0* _d2i_DSAPublicKey
0001:00739ef0* _DSAPublicKey_it
0001:00739e10  _i2d_DSAPublicKey
0001:00739e40* _DSAparams_dup
0001:00739ed0* _dsa_pub_internal_it
Module: U:\extras\lib\libcrypto.lib(ec_asn1.obj)
0001:0073acc0  _EC_GROUP_get_basis_type
0001:0073ad30* _EC_GROUP_get_trinomial_basis
0001:0073add0* _EC_GROUP_get_pentanomial_basis
0001:0073aeb0* _X9_62_PENTANOMIAL_new
0001:0073cea0* _X9_62_PENTANOMIAL_it
0001:0073aed0* _X9_62_PENTANOMIAL_free
0001:0073aef0* _X9_62_CHARACTERISTIC_TWO_new
0001:0073cee0* _X9_62_CHARACTERISTIC_TWO_it
0001:0073af10* _X9_62_CHARACTERISTIC_TWO_free
0001:0073af30* _ECPARAMETERS_new
0001:0073cf70* _ECPARAMETERS_it
0001:0073af50* _ECPARAMETERS_free
0001:0073cfa0* _ECPKPARAMETERS_it
0001:0073be00* _d2i_UC_ECPKPARAMETERS
0001:0073be30* _i2d_UC_ECPKPARAMETERS
0001:0073be60* _ECPKPARAMETERS_new
0001:0073be80* _ECPKPARAMETERS_free
0001:0073bea0* _d2i_EC_PRIVATEKEY
0001:0073cfd0* _EC_PRIVATEKEY_it
0001:0073bed0* _i2d_EC_PRIVATEKEY
0001:0073bf00* _EC_PRIVATEKEY_new
0001:0073bf20* _EC_PRIVATEKEY_free
0001:0073bf40  _d2i_ECPKParameters
0001:0073c030  _i2d_ECPKParameters
0001:0073c120  _d2i_ECPrivateKey
0001:0073c450  _i2d_ECPrivateKey
0001:0073c8b0  _i2d_ECParameters
0001:0073c9e0  _d2i_ECParameters
0001:0073cbc0  _o2i_ECPublicKey
0001:0073ccf0  _i2o_ECPublicKey
0001:0073cf10* _X9_62_FIELDID_it
0001:0073cf40* _X9_62_CURVE_it
Module: U:\extras\lib\libcrypto.lib(a_digest.obj)
0001:0073d400* _ASN1_digest
0001:0073d4d0  _ASN1_item_digest
Module: U:\extras\lib\libcrypto.lib(x_sig.obj)
0001:0073d550  _d2i_X509_SIG
0001:0073d600  _X509_SIG_it
0001:0073d580  _i2d_X509_SIG
0001:0073d5b0  _X509_SIG_new
0001:0073d5d0  _X509_SIG_free
Module: U:\extras\lib\libcrypto.lib(p8_pkey.obj)
0001:0073d6b0  _d2i_PKCS8_PRIV_KEY_INFO
0001:0073d8d0  _PKCS8_PRIV_KEY_INFO_it
0001:0073d6e0  _i2d_PKCS8_PRIV_KEY_INFO
0001:0073d710  _PKCS8_PRIV_KEY_INFO_new
0001:0073d730  _PKCS8_PRIV_KEY_INFO_free
0001:0073d750  _PKCS8_pkey_set0
0001:0073d830  _PKCS8_pkey_get0
Module: U:\extras\lib\libcrypto.lib(evp_pkey.obj)
0001:0073d9a0  _EVP_PKCS82PKEY
0001:0073db50  _EVP_PKEY2PKCS8
0001:0073dc90* _EVP_PKEY2PKCS8_broken
0001:0073ddd0* _PKCS8_set_broken
0001:0073de50* _EVP_PKEY_get_attr_count
0001:0073de70* _EVP_PKEY_get_attr_by_NID
0001:0073de90* _EVP_PKEY_get_attr_by_OBJ
0001:0073deb0* _EVP_PKEY_get_attr
0001:0073ded0* _EVP_PKEY_delete_attr
0001:0073def0* _EVP_PKEY_add1_attr
0001:0073df20* _EVP_PKEY_add1_attr_by_OBJ
0001:0073df60* _EVP_PKEY_add1_attr_by_NID
0001:0073dfa0* _EVP_PKEY_add1_attr_by_txt
Module: U:\extras\lib\libcrypto.lib(i2d_pr.obj)
0001:0073e000  _i2d_PrivateKey
Module: U:\extras\lib\libcrypto.lib(d2i_pr.obj)
0001:0073e0d0  _d2i_PrivateKey
0001:0073e260  _d2i_AutoPrivateKey
Module: U:\extras\lib\libcrypto.lib(v3_lib.obj)
0001:0073e430* _X509V3_EXT_add
0001:0073e4c0  _X509V3_EXT_get_nid
0001:0073e550  _X509V3_EXT_get
0001:0073e5f0* _X509V3_EXT_add_list
0001:0073e690* _X509V3_EXT_add_alias
0001:0073e870* _X509V3_EXT_cleanup
0001:0073e8a0* _X509V3_add_standard_extensions
0001:0073e8b0  _X509V3_EXT_d2i
0001:0073e9b0  _X509V3_get_d2i
0001:0073ec20  _X509V3_add1_i2d
Module: U:\extras\lib\libcrypto.lib(bn-586.obj)
0001:0073ee20  _bn_mul_add_words
0001:0073f0f0  _bn_mul_words
0001:0073f270  _bn_sqr_words
0001:0073f3a0  _bn_div_words
0001:0073f3b0  _bn_add_words
0001:0073f560  _bn_sub_words
0001:0073f710  _bn_sub_part_words
Module: U:\extras\lib\libcrypto.lib(bn_mont.obj)
0001:00740020  _BN_mod_mul_montgomery
0001:00740190  _BN_from_montgomery
0001:00740210  _BN_MONT_CTX_new
0001:00740280* _BN_MONT_CTX_init
0001:007402d0  _BN_MONT_CTX_free
0001:00740320  _BN_MONT_CTX_set
0001:007405f0  _BN_MONT_CTX_copy
0001:00740670  _BN_MONT_CTX_set_locked
Module: U:\extras\lib\libcrypto.lib(bn_div.obj)
0001:007407f0  _BN_div
Module: U:\extras\lib\libcrypto.lib(rsa_none.obj)
0001:00741450  _RSA_padding_add_none
0001:00741570  _RSA_padding_check_none
Module: U:\extras\lib\libcrypto.lib(rsa_pk1.obj)
0001:00741730  _RSA_padding_add_PKCS1_type_1
0001:00741900  _RSA_padding_check_PKCS1_type_1
0001:00741b20  _RSA_padding_add_PKCS1_type_2
0001:00741c50  _RSA_padding_check_PKCS1_type_2
Module: U:\extras\lib\libcrypto.lib(rsa_x931.obj)
0001:00741e60  _RSA_padding_add_X931
0001:00742010  _RSA_padding_check_X931
0001:00742230  _RSA_X931_hash_id
Module: U:\extras\lib\libcrypto.lib(rsa_oaep.obj)
0001:007422a0  _PKCS1_MGF1
0001:00742490  _RSA_padding_check_PKCS1_OAEP
0001:00742a50  _RSA_padding_add_PKCS1_OAEP
Module: U:\extras\lib\libcrypto.lib(rsa_ssl.obj)
0001:00742e90  _RSA_padding_add_SSLv23
0001:00742fd0  _RSA_padding_check_SSLv23
Module: U:\extras\lib\libcrypto.lib(bn_exp.obj)
0001:007432f0* _BN_exp
0001:007434b0* _BN_mod_exp_recp
0001:00743970  _BN_mod_exp
0001:00744aa0* _BN_mod_exp_mont_consttime
0001:007452c0  _BN_mod_exp_mont
0001:007458a0  _BN_mod_exp_mont_word
0001:00745dd0* _BN_mod_exp_simple
Module: U:\extras\lib\libcrypto.lib(bn_mod.obj)
0001:00746230  _BN_nnmod
0001:007462c0  _BN_mod_add
0001:00746370  _BN_mod_add_quick
0001:007463f0* _BN_mod_sub
0001:007464a0  _BN_mod_sub_quick
0001:00746510  _BN_mod_mul
0001:00746610  _BN_mod_sqr
0001:00746670* _BN_mod_lshift1
0001:00746710  _BN_mod_lshift1_quick
0001:00746790  _BN_mod_lshift_quick
0001:007468a0* _BN_mod_lshift
Module: U:\extras\lib\libcrypto.lib(co-586.obj)
0001:00746980  _bn_mul_comba8
0001:00746dd0* _bn_mul_comba4
0001:00746f10  _bn_sqr_comba8
0001:00747240  _bn_sqr_comba4
Module: U:\extras\lib\libcrypto.lib(dh_check.obj)
0001:00747330* _DH_check
0001:007474a0  _DH_check_pub_key
Module: U:\extras\lib\libcrypto.lib(pem_xaux.obj)
0001:00747570  _PEM_read_bio_X509_AUX
0001:007475b0* _PEM_read_X509_AUX
0001:007475f0* _PEM_write_bio_X509_AUX
0001:00747650* _PEM_write_X509_AUX
0001:007476c0* _PEM_read_bio_X509_CERT_PAIR
0001:00747700* _PEM_read_X509_CERT_PAIR
0001:00747740* _PEM_write_bio_X509_CERT_PAIR
0001:007477a0* _PEM_write_X509_CERT_PAIR
Module: U:\extras\lib\libcrypto.lib(pem_info.obj)
0001:00747890  _PEM_X509_INFO_read_bio
0001:00747e20* _PEM_X509_INFO_read
0001:00747f00* _PEM_X509_INFO_write_bio
Module: U:\extras\lib\libcrypto.lib(x_info.obj)
0001:007481c0  _X509_INFO_new
0001:00748250  _X509_INFO_free
Module: U:\extras\lib\libcrypto.lib(x509_def.obj)
0001:00748300* _X509_get_default_private_dir
0001:00748320  _X509_get_default_cert_area
0001:00748340  _X509_get_default_cert_dir
0001:00748360  _X509_get_default_cert_file
0001:00748380  _X509_get_default_cert_dir_env
0001:007483a0  _X509_get_default_cert_file_env
Module: U:\extras\lib\libcrypto.lib(pem_all.obj)
0001:007483d0* _PEM_read_bio_X509_REQ
0001:00748410* _PEM_read_X509_REQ
0001:00748450* _PEM_write_bio_X509_REQ
0001:007484b0* _PEM_write_X509_REQ
0001:00748520* _PEM_write_bio_X509_REQ_NEW
0001:00748580* _PEM_write_X509_REQ_NEW
0001:007485e0  _PEM_read_bio_X509_CRL
0001:00748620* _PEM_read_X509_CRL
0001:00748660* _PEM_write_bio_X509_CRL
0001:007486c0* _PEM_write_X509_CRL
0001:00748720* _PEM_read_bio_PKCS7
0001:00748760* _PEM_read_PKCS7
0001:007487a0* _PEM_write_bio_PKCS7
0001:00748800* _PEM_write_PKCS7
0001:00748860* _PEM_read_bio_NETSCAPE_CERT_SEQUENCE
0001:007488a0* _PEM_read_NETSCAPE_CERT_SEQUENCE
0001:007488e0* _PEM_write_bio_NETSCAPE_CERT_SEQUENCE
0001:00748940* _PEM_write_NETSCAPE_CERT_SEQUENCE
0001:007489a0  _PEM_read_bio_RSAPrivateKey
0001:00748a20* _PEM_read_RSAPrivateKey
0001:00748ab0  _PEM_write_bio_RSAPrivateKey
0001:00748b10* _PEM_write_RSAPrivateKey
0001:00748b80* _PEM_read_bio_RSAPublicKey
0001:00748bc0* _PEM_read_RSAPublicKey
0001:00748c00* _PEM_write_bio_RSAPublicKey
0001:00748c60* _PEM_write_RSAPublicKey
0001:00748cc0* _PEM_read_bio_RSA_PUBKEY
0001:00748d00* _PEM_read_RSA_PUBKEY
0001:00748d40* _PEM_write_bio_RSA_PUBKEY
0001:00748da0* _PEM_write_RSA_PUBKEY
0001:00748e00* _PEM_read_bio_DSAPrivateKey
0001:00748e90* _PEM_write_bio_DSAPrivateKey
0001:00748ef0* _PEM_write_DSAPrivateKey
0001:00748f50* _PEM_read_bio_DSA_PUBKEY
0001:00748f90* _PEM_read_DSA_PUBKEY
0001:00748fd0* _PEM_write_bio_DSA_PUBKEY
0001:00749030* _PEM_write_DSA_PUBKEY
0001:00749090* _PEM_read_DSAPrivateKey
0001:00749120* _PEM_read_bio_DSAparams
0001:00749160* _PEM_read_DSAparams
0001:007491a0* _PEM_write_bio_DSAparams
0001:00749200* _PEM_write_DSAparams
0001:00749260* _PEM_read_bio_ECPrivateKey
0001:007492f0* _PEM_read_bio_ECPKParameters
0001:00749330* _PEM_read_ECPKParameters
0001:00749370* _PEM_write_bio_ECPKParameters
0001:007493d0* _PEM_write_ECPKParameters
0001:00749440* _PEM_write_bio_ECPrivateKey
0001:007494a0* _PEM_write_ECPrivateKey
0001:00749500* _PEM_read_bio_EC_PUBKEY
0001:00749540* _PEM_read_EC_PUBKEY
0001:00749580* _PEM_write_bio_EC_PUBKEY
0001:007495e0* _PEM_write_EC_PUBKEY
0001:00749640* _PEM_read_ECPrivateKey
0001:007496d0* _PEM_read_bio_DHparams
0001:00749710* _PEM_read_DHparams
0001:00749750* _PEM_write_bio_DHparams
0001:007497b0* _PEM_write_DHparams
0001:00749810* _PEM_read_bio_PUBKEY
0001:00749850* _PEM_read_PUBKEY
0001:00749890* _PEM_write_bio_PUBKEY
0001:007498f0* _PEM_write_PUBKEY
Module: U:\extras\lib\libcrypto.lib(ec_mult.obj)
0001:00749e40  _ec_wNAF_mul
0001:0074acf0  _ec_wNAF_precompute_mult
0001:0074b450  _ec_wNAF_have_precompute_mult
Module: U:\extras\lib\libcrypto.lib(ecs_vrf.obj)
0001:0074b490* _ECDSA_do_verify
0001:0074b4f0  _ECDSA_verify
Module: U:\extras\lib\libcrypto.lib(ec_cvt.obj)
0001:0074b5a0  _EC_GROUP_new_curve_GFp
0001:0074b680  _EC_GROUP_new_curve_GF2m
Module: U:\extras\lib\libcrypto.lib(dsa_vrf.obj)
0001:0074b6e0* _DSA_do_verify
0001:0074b700  _DSA_verify
Module: U:\extras\lib\libcrypto.lib(ech_lib.obj)
0001:0074b950* _ECDH_set_default_method
0001:0074b960* _ECDH_get_default_method
0001:0074b980* _ECDH_set_method
0001:0074ba10  _ecdh_check
0001:0074ba80* _ECDH_get_ex_new_index
0001:0074bac0* _ECDH_set_ex_data
0001:0074bb60* _ECDH_get_ex_data
0001:0074bbf0* _ECDH_version
Module: U:\extras\lib\libcrypto.lib(ecs_lib.obj)
0001:0074bde0* _ECDSA_set_default_method
0001:0074bdf0* _ECDSA_get_default_method
0001:0074be10* _ECDSA_set_method
0001:0074bea0  _ecdsa_check
0001:0074bf10  _ECDSA_size
0001:0074c010* _ECDSA_get_ex_new_index
0001:0074c050* _ECDSA_set_ex_data
0001:0074c0f0* _ECDSA_get_ex_data
0001:0074c180* _ECDSA_version
Module: U:\extras\lib\libcrypto.lib(ecs_asn1.obj)
0001:0074c1b0  _d2i_ECDSA_SIG
0001:0074c260* _ECDSA_SIG_it
0001:0074c1e0  _i2d_ECDSA_SIG
0001:0074c210  _ECDSA_SIG_new
0001:0074c230  _ECDSA_SIG_free
Module: U:\extras\lib\libcrypto.lib(pem_pkey.obj)
0001:0074c300  _PEM_read_bio_PrivateKey
0001:0074c650* _PEM_write_bio_PrivateKey
0001:0074c750* _PEM_read_bio_Parameters
0001:0074c8b0* _PEM_write_bio_Parameters
0001:0074c960  _PEM_read_PrivateKey
0001:0074ca00* _PEM_write_PrivateKey
Module: U:\extras\lib\libcrypto.lib(aes_cfb.obj)
0001:0074cb60  _AES_cfb128_encrypt
0001:0074cbb0  _AES_cfb1_encrypt
0001:0074cc00  _AES_cfb8_encrypt
Module: U:\extras\lib\libcrypto.lib(aes-586.obj)
0001:0074e050  _AES_encrypt
0001:0074f690  _AES_decrypt
0001:0074f740  _AES_cbc_encrypt
0001:00750030  _AES_set_encrypt_key
0001:00750040  _AES_set_decrypt_key
Module: U:\extras\lib\libcrypto.lib(aes_ecb.obj)
0001:00750350  _AES_ecb_encrypt
Module: U:\extras\lib\libcrypto.lib(aes_ofb.obj)
0001:00750390  _AES_ofb128_encrypt
Module: U:\extras\lib\libcrypto.lib(pmeth_gn.obj)
0001:00750420* _EVP_PKEY_paramgen_init
0001:007504c0* _EVP_PKEY_paramgen
0001:007505d0* _EVP_PKEY_keygen_init
0001:00750670* _EVP_PKEY_keygen
0001:00750780* _EVP_PKEY_CTX_set_cb
0001:00750790* _EVP_PKEY_CTX_get_cb
0001:007507a0  _evp_pkey_set_cb_translate
0001:007507c0* _EVP_PKEY_CTX_get_keygen_info
0001:00750810  _EVP_PKEY_new_mac_key
Module: U:\extras\lib\libcrypto.lib(m_sigver.obj)
0001:00750bb0  _EVP_DigestSignInit
0001:00750bf0  _EVP_DigestVerifyInit
0001:00750c30  _EVP_DigestSignFinal
0001:00750de0  _EVP_DigestVerifyFinal
Module: U:\extras\lib\expat.lib(xmlrole.obj)
0001:00752860  _XmlPrologStateInit
0001:00752883  _XmlPrologStateInitExternalEntity
Module: U:\extras\lib\expat.lib(xmltok.obj)
0001:0076187f  _XmlUtf8Encode
0001:0076191f* _XmlUtf16Encode
0001:00761967  _XmlSizeOfUnknownEncoding
0001:00761b9c  _XmlInitUnknownEncoding
0001:007620c2  _XmlGetUtf8InternalEncoding
0001:007620cc* _XmlGetUtf16InternalEncoding
0001:00762133  _XmlInitEncoding
0001:00762225  _XmlParseXmlDecl
0001:00762275  _XmlGetUtf8InternalEncodingNS
0001:0076227f* _XmlGetUtf16InternalEncodingNS
0001:007622e6  _XmlInitEncodingNS
0001:007623d8  _XmlParseXmlDeclNS
0001:00762428  _XmlInitUnknownEncodingNS
Module: U:\usr\lib\gcc-lib\i386-pc-os2-emx\3.3.5\libgcc_so_d.lib(emx-eh.obj)
0001:00764330  ___ehInit
0001:00764359* ___POST$__ehInit
0001:00764362* ___ehTerm
0001:0076438a* ___POST$__ehTerm
Module: U:\extras\lib\libcrypto.lib(ui_lib.obj)
0001:00764850  _UI_new
0001:00764900* _UI_new_method
0001:007649c0  _UI_free
0001:00764a20  _UI_add_input_string
0001:00764a70* _UI_dup_input_string
0001:00764b30  _UI_add_verify_string
0001:00764b80* _UI_dup_verify_string
0001:00764c40* _UI_add_input_boolean
0001:00764c90* _UI_dup_input_boolean
0001:00764e30* _UI_add_info_string
0001:00764e80* _UI_dup_info_string
0001:00764f20* _UI_add_error_string
0001:00764f70* _UI_dup_error_string
0001:00765010* _UI_construct_prompt
0001:007651e0* _UI_add_user_data
0001:007651f0* _UI_get0_user_data
0001:00765200* _UI_get0_result
0001:007652d0  _UI_process
0001:00765420* _UI_ctrl
0001:007654e0* _UI_get_ex_new_index
0001:00765520* _UI_set_ex_data
0001:00765540* _UI_get_ex_data
0001:00765560* _UI_set_default_method
0001:00765570* _UI_get_default_method
0001:00765590* _UI_get_method
0001:007655a0* _UI_set_method
0001:007655b0* _UI_create_method
0001:00765600* _UI_destroy_method
0001:00765630* _UI_method_set_opener
0001:00765660* _UI_method_set_writer
0001:00765690* _UI_method_set_flusher
0001:007656c0* _UI_method_set_reader
0001:007656f0* _UI_method_set_closer
0001:00765720* _UI_method_set_prompt_constructor
0001:00765750* _UI_method_get_opener
0001:00765770* _UI_method_get_writer
0001:00765790* _UI_method_get_flusher
0001:007657b0* _UI_method_get_reader
0001:007657d0* _UI_method_get_closer
0001:007657f0* _UI_method_get_prompt_constructor
0001:00765810  _UI_get_string_type
0001:00765830  _UI_get_input_flags
0001:00765850  _UI_get0_output_string
0001:00765870  _UI_get0_action_string
0001:007658a0  _UI_get0_result_string
0001:007658d0  _UI_get0_test_string
0001:00765900* _UI_get_result_minsize
0001:00765930* _UI_get_result_maxsize
0001:00765980  _UI_set_result
Module: U:\extras\lib\libcrypto.lib(eng_ctrl.obj)
0001:00765bd0* _ENGINE_ctrl
0001:00766080* _ENGINE_cmd_is_executable
0001:00766100* _ENGINE_ctrl_cmd
0001:00766220  _ENGINE_ctrl_cmd_string
Module: U:\extras\lib\libcrypto.lib(a_bytes.obj)
0001:007665c0* _d2i_ASN1_type_bytes
0001:00766850  _i2d_ASN1_bytes
0001:007669b0* _d2i_ASN1_bytes
Module: U:\extras\lib\libcrypto.lib(rsa_gen.obj)
0001:00766ee0  _RSA_generate_key_ex
Module: U:\extras\lib\libcrypto.lib(rsa_pss.obj)
0001:007676b0  _RSA_verify_PKCS1_PSS
0001:00767ba0  _RSA_padding_add_PKCS1_PSS
Module: U:\extras\lib\libcrypto.lib(dh_gen.obj)
0001:00768010  _DH_generate_parameters_ex
Module: U:\extras\lib\libcrypto.lib(dsa_key.obj)
0001:007682f0  _DSA_generate_key
Module: U:\extras\lib\libcrypto.lib(dsa_gen.obj)
0001:007684b0  _dsa_builtin_paramgen
0001:00768f10* _DSA_generate_parameters_ex
Module: U:\extras\lib\libcrypto.lib(pk7_lib.obj)
0001:00768ff0  _PKCS7_ctrl
0001:00769140* _PKCS7_set_content
0001:00769200  _PKCS7_set_type
0001:00769450* _PKCS7_content_new
0001:00769550* _PKCS7_set0_type_other
0001:00769580* _PKCS7_add_signer
0001:007696e0* _PKCS7_add_certificate
0001:00769800* _PKCS7_add_crl
0001:00769920* _PKCS7_SIGNER_INFO_set
0001:00769ac0* _PKCS7_add_signature
0001:00769bc0* _PKCS7_set_digest
0001:00769ca0* _PKCS7_get_signer_info
0001:00769cf0  _PKCS7_SIGNER_INFO_get0_algs
0001:00769d20  _PKCS7_RECIP_INFO_get0_alg
0001:00769d40* _PKCS7_add_recipient_info
0001:00769dd0* _PKCS7_RECIP_INFO_set
0001:00769f80* _PKCS7_add_recipient
0001:0076a030* _PKCS7_cert_from_signer_info
0001:0076a080* _PKCS7_set_cipher
0001:0076a150  _PKCS7_stream
Module: U:\extras\lib\libcrypto.lib(cms_sd.obj)
0001:0076a340* _CMS_SignedData_init
0001:0076a460  _cms_set1_SignerIdentifier
0001:0076a5c0  _cms_SignerIdentifier_get0_signer_id
0001:0076a640  _cms_SignerIdentifier_cert_cmp
0001:0076a6e0* _CMS_get0_SignerInfos
0001:0076a750* _CMS_get0_signers
0001:0076a840* _CMS_SignerInfo_set1_signer_cert
0001:0076a8b0* _CMS_SignerInfo_get0_signer_id
0001:0076a930* _CMS_SignerInfo_cert_cmp
0001:0076a9d0* _CMS_set1_signers_certs
0001:0076ad70  _CMS_SignerInfo_get0_algs
0001:0076adb0* _CMS_SignerInfo_sign
0001:0076b0a0  _cms_SignedData_final
0001:0076b3b0* _CMS_SignerInfo_verify
0001:0076b530  _cms_SignedData_init_bio
0001:0076b7f0* _CMS_SignerInfo_verify_content
0001:0076ba00* _CMS_add_smimecap
0001:0076ba80* _CMS_add_simple_smimecap
0001:0076bb70* _CMS_add_standard_smimecap
0001:0076bdf0* _CMS_add1_signer
Module: U:\extras\lib\libcrypto.lib(cms_env.obj)
0001:0076c650* _CMS_get0_RecipientInfos
0001:0076c6c0* _CMS_RecipientInfo_type
0001:0076c6d0* _CMS_EnvelopedData_create
0001:0076c840* _CMS_add1_recipient_cert
0001:0076cae0  _CMS_RecipientInfo_ktri_get0_algs
0001:0076cb80* _CMS_RecipientInfo_ktri_get0_signer_id
0001:0076cc00* _CMS_RecipientInfo_ktri_cert_cmp
0001:0076cc70* _CMS_RecipientInfo_set0_pkey
0001:0076ccd0* _CMS_RecipientInfo_kekri_id_cmp
0001:0076cd60* _CMS_add0_recipient_key
0001:0076d060* _CMS_RecipientInfo_kekri_get0_id
0001:0076d160* _CMS_RecipientInfo_set0_key
0001:0076d1d0* _CMS_RecipientInfo_decrypt
0001:0076d6b0  _cms_EnvelopedData_init_bio
Module: U:\extras\lib\libcrypto.lib(t_pkey.obj)
0001:0076dc40  _ASN1_bn_print
Module: U:\extras\lib\libcrypto.lib(ec_print.obj)
0001:0076dec0  _EC_POINT_point2bn
0001:0076dfa0* _EC_POINT_bn2point
0001:0076e0b0* _EC_POINT_point2hex
0001:0076e1f0* _EC_POINT_hex2point
Module: U:\extras\lib\libcrypto.lib(eck_prn.obj)
0001:0076e350* _EC_KEY_print_fp
0001:0076e430* _ECParameters_print_fp
0001:0076e510* _EC_KEY_print
0001:0076e580* _ECParameters_print
0001:0076e6a0  _ECPKParameters_print
0001:0076f220* _ECPKParameters_print_fp
Module: U:\extras\lib\libcrypto.lib(pcy_node.obj)
0001:0076f300  _policy_node_cmp_new
0001:0076f320  _tree_find_sk
0001:0076f370  _level_find_node
0001:0076f410  _level_add_node
0001:0076f520  _policy_node_free
0001:0076f530  _policy_node_match
Module: U:\extras\lib\libcrypto.lib(pcy_lib.obj)
0001:0076f5d0* _X509_policy_tree_level_count
0001:0076f5f0* _X509_policy_tree_get0_level
0001:0076f620* _X509_policy_tree_get0_policies
0001:0076f640  _X509_policy_tree_get0_user_policies
0001:0076f680* _X509_policy_level_node_count
0001:0076f6d0* _X509_policy_level_get0_node
0001:0076f710* _X509_policy_node_get0_policy
0001:0076f730* _X509_policy_node_get0_qualifiers
0001:0076f750* _X509_policy_node_get0_parent
Module: U:\extras\lib\libcrypto.lib(o_time.obj)
0001:0076f770  _OPENSSL_gmtime
0001:0076f7a0  _OPENSSL_gmtime_adj
Module: U:\extras\lib\libcrypto.lib(md5-586.obj)
0001:0076faf0  _md5_block_asm_data_order
Module: U:\extras\lib\libcrypto.lib(sha512-586.obj)
0001:007701a0  _sha512_block_data_order
Module: U:\extras\lib\libcrypto.lib(sha256-586.obj)
0001:00770de0  _sha256_block_data_order
Module: U:\extras\lib\libcrypto.lib(sha1-586.obj)
0001:00771220  _sha1_block_data_order
Module: U:\extras\lib\libcrypto.lib(b_dump.obj)
0001:00772280* _BIO_dump_indent_cb
0001:007726f0* _BIO_dump_cb
0001:00772730* _BIO_dump_fp
0001:00772770* _BIO_dump_indent_fp
0001:007727b0* _BIO_dump
0001:007727f0  _BIO_dump_indent
Module: U:\extras\lib\libcrypto.lib(a_bool.obj)
0001:00772830* _i2d_ASN1_BOOLEAN
0001:007728c0  _d2i_ASN1_BOOLEAN
Module: U:\extras\lib\libcrypto.lib(a_strnid.obj)
0001:007729f0* _ASN1_STRING_set_default_mask
0001:00772a00* _ASN1_STRING_get_default_mask
0001:00772a30* _ASN1_STRING_set_default_mask_asc
0001:00772b20  _ASN1_STRING_set_by_NID
0001:00772c50* _ASN1_STRING_TABLE_get
0001:00772cf0* _ASN1_STRING_TABLE_add
0001:00772e80* _ASN1_STRING_TABLE_cleanup
Module: U:\extras\lib\libcrypto.lib(a_print.obj)
0001:00773030  _ASN1_PRINTABLE_type
0001:00773130* _ASN1_UNIVERSALSTRING_to_string
Module: U:\extras\lib\libcrypto.lib(t_x509a.obj)
0001:00773280  _X509_CERT_AUX_print
Module: U:\extras\lib\libcrypto.lib(v3_prn.obj)
0001:007735b0* _X509V3_EXT_val_prn
0001:007737b0* _X509V3_EXT_print
0001:00773a90  _X509V3_extensions_print
0001:00773c30* _X509V3_EXT_print_fp
Module: U:\extras\lib\libcrypto.lib(err_prn.obj)
0001:00773d40  _ERR_print_errors_cb
0001:00773e90* _ERR_print_errors_fp
0001:00773eb0  _ERR_print_errors
Module: U:\extras\lib\libcrypto.lib(conf_mod.obj)
0001:00773f40* _CONF_modules_load
0001:00774510* _CONF_modules_load_file
0001:00774690* _CONF_modules_unload
0001:00774800* _CONF_modules_finish
0001:00774880* _CONF_module_add
0001:00774930* _CONF_modules_free
0001:00774ab0* _CONF_imodule_get_name
0001:00774ac0* _CONF_imodule_get_value
0001:00774ad0* _CONF_imodule_get_usr_data
0001:00774ae0* _CONF_imodule_set_usr_data
0001:00774af0* _CONF_imodule_get_module
0001:00774b00* _CONF_imodule_get_flags
0001:00774b10* _CONF_imodule_set_flags
0001:00774b20* _CONF_module_get_usr_data
0001:00774b30* _CONF_module_set_usr_data
0001:00774b40* _CONF_get1_default_config_file
0001:00774be0  _CONF_parse_list
Module: U:\extras\lib\libcrypto.lib(x509_req.obj)
0001:00774d70* _X509_to_X509_REQ
0001:00774e90* _X509_REQ_get_pubkey
0001:00774ed0* _X509_REQ_check_private_key
0001:007750c0* _X509_REQ_extension_nid
0001:00775110* _X509_REQ_get_extension_nids
0001:00775120* _X509_REQ_set_extension_nids
0001:00775130  _X509_REQ_get_extensions
0001:00775220* _X509_REQ_add_extensions_nid
0001:00775330  _X509_REQ_add_extensions
0001:00775440* _X509_REQ_get_attr_count
0001:00775460* _X509_REQ_get_attr_by_NID
0001:00775480* _X509_REQ_get_attr_by_OBJ
0001:007754a0* _X509_REQ_get_attr
0001:007754c0* _X509_REQ_delete_attr
0001:007754e0* _X509_REQ_add1_attr
0001:00775510* _X509_REQ_add1_attr_by_OBJ
0001:00775560* _X509_REQ_add1_attr_by_NID
0001:007755b0* _X509_REQ_add1_attr_by_txt
Module: U:\extras\lib\libcrypto.lib(asn1_gen.obj)
0001:00775e70  _ASN1_generate_v3
0001:00776a90* _ASN1_generate_nconf
Module: U:\extras\lib\libcrypto.lib(conf_lib.obj)
0001:00776ec0  _CONF_set_nconf
0001:00776f00* _CONF_set_default_method
0001:00776f30* _CONF_load
0001:00776ff0* _CONF_load_fp
0001:007770b0* _CONF_load_bio
0001:00777120  _CONF_get_section
0001:007771c0  _CONF_get_string
0001:007772f0  _CONF_free
0001:00777330* _CONF_dump_fp
0001:007773e0* _CONF_dump_bio
0001:00777430  _NCONF_new
0001:00777490  _NCONF_free
0001:007774c0* _NCONF_free_data
0001:007774f0  _NCONF_load
0001:00777560* _NCONF_load_fp
0001:00777630* _NCONF_load_bio
0001:007776a0  _NCONF_get_section
0001:00777730  _NCONF_get_string
0001:00777810* _NCONF_get_number_e
0001:00777970* _CONF_get_number
0001:00777a10* _NCONF_dump_fp
0001:00777ae0* _NCONF_dump_bio
0001:00777b50* _CONF_version
Module: U:\extras\lib\libcrypto.lib(v3_pmaps.obj)
0001:00777c20  _POLICY_MAPPING_free
0001:00777ed0* _POLICY_MAPPING_it
0001:00777e60* _POLICY_MAPPING_new
0001:00777e80  _v3_policy_mappings
0001:00777f00* _POLICY_MAPPINGS_it
Module: U:\extras\lib\libcrypto.lib(p5_pbe.obj)
0001:00777fa0  _d2i_PBEPARAM
0001:007783b0* _PBEPARAM_it
0001:00777fd0* _i2d_PBEPARAM
0001:00778000* _PBEPARAM_new
0001:00778020  _PBEPARAM_free
0001:00778060* _PKCS5_pbe_set0_algor
0001:00778310  _PKCS5_pbe_set
Module: U:\extras\lib\libcrypto.lib(p12_key.obj)
0001:00778430* _PKCS12_key_gen_uni
0001:00778be0  _PKCS12_key_gen_asc
Module: U:\extras\lib\libcrypto.lib(p5_pbev2.obj)
0001:00778d00  _d2i_PBE2PARAM
0001:00779af0* _PBE2PARAM_it
0001:00778d30* _i2d_PBE2PARAM
0001:00778d60* _PBE2PARAM_new
0001:00778d80  _PBE2PARAM_free
0001:00778da0  _d2i_PBKDF2PARAM
0001:00779b20* _PBKDF2PARAM_it
0001:00778dd0* _i2d_PBKDF2PARAM
0001:00778e00* _PBKDF2PARAM_new
0001:00778e20  _PBKDF2PARAM_free
0001:00778e60* _PKCS5_pbe2_set_iv
0001:00779500  _PKCS5_pbe2_set
Module: U:\extras\lib\libcrypto.lib(bn_exp2.obj)
0001:00779c00  _BN_mod_exp2_mont
Module: U:\extras\lib\libcrypto.lib(pk7_doit.obj)
0001:0077a9d0  _PKCS7_dataInit
0001:0077b200* _PKCS7_dataDecode
0001:0077b9a0* _PKCS7_SIGNER_INFO_sign
0001:0077bbe0  _PKCS7_dataFinal
0001:0077c4f0* _PKCS7_signatureVerify
0001:0077c970* _PKCS7_dataVerify
0001:0077cb50* _PKCS7_get_issuer_and_serial
0001:0077cbc0  _PKCS7_get_signed_attribute
0001:0077cc60* _PKCS7_get_attribute
0001:0077cd00* _PKCS7_digest_from_attributes
0001:0077cdb0* _PKCS7_set_signed_attributes
0001:0077ce50* _PKCS7_set_attributes
0001:0077cef0  _PKCS7_add_signed_attribute
0001:0077cf20* _PKCS7_add_attribute
Module: U:\extras\lib\libcrypto.lib(tasn_prn.obj)
0001:0077d080* _ASN1_PCTX_new
0001:0077d100* _ASN1_PCTX_free
0001:0077d110* _ASN1_PCTX_get_flags
0001:0077d120* _ASN1_PCTX_set_flags
0001:0077d130* _ASN1_PCTX_get_nm_flags
0001:0077d140* _ASN1_PCTX_set_nm_flags
0001:0077d150* _ASN1_PCTX_get_cert_flags
0001:0077d160* _ASN1_PCTX_set_cert_flags
0001:0077d170* _ASN1_PCTX_get_oid_flags
0001:0077d180* _ASN1_PCTX_set_oid_flags
0001:0077d190* _ASN1_PCTX_get_str_flags
0001:0077d1a0* _ASN1_PCTX_set_str_flags
0001:0077d1f0* _asn1_template_print_ctx
0001:0077dd80  _ASN1_item_print
0002:0000a900* _default_pctx
Module: U:\extras\lib\libcrypto.lib(ec2_smpl.obj)
0001:0077de10* _ec_GF2m_simple_is_at_infinity
0001:0077de30* _ec_GF2m_simple_points_make_affine
0001:0077de90* _ec_GF2m_simple_field_div
0001:0077dec0* _ec_GF2m_simple_field_sqr
0001:0077def0* _ec_GF2m_simple_field_mul
0001:0077df20* _ec_GF2m_simple_point_copy
0001:0077df90* _ec_GF2m_simple_group_get_curve
0001:0077e020* _ec_GF2m_simple_point_set_to_infinity
0001:0077e050* _ec_GF2m_simple_make_affine
0001:0077e180* _ec_GF2m_simple_cmp
0001:0077e390* _ec_GF2m_simple_is_on_curve
0001:0077e570* _ec_GF2m_simple_invert
0001:0077e5f0* _ec_GF2m_simple_add
0001:0077eaf0* _ec_GF2m_simple_dbl
0001:0077eb40* _ec_GF2m_simple_oct2point
0001:0077efe0* _ec_GF2m_simple_group_get_degree
0001:0077f000* _ec_GF2m_simple_point2oct
0001:0077f5c0* _ec_GF2m_simple_group_check_discriminant
0001:0077f6b0* _ec_GF2m_simple_set_compressed_coordinates
0001:0077f9e0* _ec_GF2m_simple_point_get_affine_coordinates
0001:0077fb30* _ec_GF2m_simple_point_set_affine_coordinates
0001:0077fc30* _ec_GF2m_simple_point_clear_finish
0001:0077fc70* _ec_GF2m_simple_group_clear_finish
0001:0077fcd0* _ec_GF2m_simple_point_finish
0001:0077fd00* _ec_GF2m_simple_group_finish
0001:0077fd40* _ec_GF2m_simple_point_init
0001:0077fd80* _ec_GF2m_simple_group_init
0001:0077fdc0  _ec_GF2m_simple_group_set_curve
0001:0077ff90* _ec_GF2m_simple_group_copy
0001:00780140  _EC_GF2m_simple_method
Module: U:\extras\lib\libcrypto.lib(x509_att.obj)
0001:007801f0  _X509at_get_attr_count
0001:00780200  _X509at_get_attr_by_NID
0001:007802b0  _X509at_get_attr_by_OBJ
0001:00780340  _X509at_get_attr
0001:00780390  _X509at_delete_attr
0001:007803f0  _X509at_add1_attr
0001:007804e0  _X509at_get0_data_by_OBJ
0001:00780740* _X509_ATTRIBUTE_set1_object
0001:00780790* _X509_ATTRIBUTE_set1_data
0001:00780990* _X509_ATTRIBUTE_create_by_OBJ
0001:00780a80  _X509at_add1_attr_by_txt
0001:00780c90  _X509at_add1_attr_by_OBJ
0001:00780e30  _X509at_add1_attr_by_NID
0001:00781020* _X509_ATTRIBUTE_create_by_txt
0001:00781160* _X509_ATTRIBUTE_create_by_NID
0001:00781280* _X509_ATTRIBUTE_count
0001:007812b0* _X509_ATTRIBUTE_get0_object
0001:007812d0* _X509_ATTRIBUTE_get0_data
0001:00781390* _X509_ATTRIBUTE_get0_type
Module: U:\extras\lib\libcrypto.lib(v3_bitst.obj)
0001:00781450* _v2i_ASN1_BIT_STRING
0001:00781650* _i2v_ASN1_BIT_STRING
0001:007816c0  _v3_nscert
0001:00781700  _v3_key_usage
Module: U:\extras\lib\libcrypto.lib(v3_ia5.obj)
0001:00781ab0  _v3_ns_ia5_list
Module: U:\extras\lib\libcrypto.lib(v3_skey.obj)
0001:00781c70* _i2s_ASN1_OCTET_STRING
0001:00781eb0* _s2i_ASN1_OCTET_STRING
0001:00781f30  _v3_skey_id
Module: U:\extras\lib\libcrypto.lib(v3_pku.obj)
0001:00782060* _d2i_PKEY_USAGE_PERIOD
0001:00782150* _PKEY_USAGE_PERIOD_it
0001:00782090* _i2d_PKEY_USAGE_PERIOD
0001:007820c0* _PKEY_USAGE_PERIOD_new
0001:007820e0* _PKEY_USAGE_PERIOD_free
0001:00782100  _v3_pkey_usage_period
Module: U:\extras\lib\libcrypto.lib(v3_int.obj)
0001:007821d0  _v3_crl_num
0001:00782210  _v3_delta_crl
0001:00782250  _v3_inhibit_anyp
Module: U:\extras\lib\libcrypto.lib(v3_akey.obj)
0001:00782780  _v3_akey_id
Module: U:\extras\lib\libcrypto.lib(v3_extku.obj)
0001:007829b0* _d2i_EXTENDED_KEY_USAGE
0001:00782ae0* _EXTENDED_KEY_USAGE_it
0001:007829e0* _i2d_EXTENDED_KEY_USAGE
0001:00782a10* _EXTENDED_KEY_USAGE_new
0001:00782a30* _EXTENDED_KEY_USAGE_free
0001:00782a50  _v3_ext_ku
0001:00782a90  _v3_ocsp_accresp
Module: U:\extras\lib\libcrypto.lib(v3_enum.obj)
0001:00782b20* _i2s_ASN1_ENUMERATED_TABLE
0001:00782b90  _v3_crl_reason
Module: U:\extras\lib\libcrypto.lib(v3_ocsp.obj)
0001:007832b0  _v3_ocsp_crlid
0001:007832f0  _v3_ocsp_acutoff
0001:00783330  _v3_crl_invdate
0001:00783370  _v3_crl_hold
0001:007833b0  _v3_ocsp_nonce
0001:007833f0  _v3_ocsp_nocheck
0001:00783430  _v3_ocsp_serviceloc
Module: U:\extras\lib\libcrypto.lib(v3_sxnet.obj)
0001:00783580* _d2i_SXNETID
0001:00783dc0* _SXNETID_it
0001:007835b0* _i2d_SXNETID
0001:007835e0* _SXNETID_new
0001:00783600* _SXNETID_free
0001:00783620* _d2i_SXNET
0001:00783df0* _SXNET_it
0001:00783650* _i2d_SXNET
0001:00783680* _SXNET_new
0001:007836a0* _SXNET_free
0001:007836e0* _SXNET_add_id_INTEGER
0001:00783980* _SXNET_add_id_ulong
0001:00783a20* _SXNET_add_id_asc
0001:00783b70* _SXNET_get_id_asc
0001:00783c30* _SXNET_get_id_ulong
0001:00783d10* _SXNET_get_id_INTEGER
0001:00783d80  _v3_sxnet
Module: U:\extras\lib\libcrypto.lib(v3_pci.obj)
0001:00784af0  _v3_pci
Module: U:\extras\lib\libcrypto.lib(bn_sqr.obj)
0001:00784b30* _bn_sqr_normal
0001:00784c70* _bn_sqr_recursive
0001:00784f30  _BN_sqr
Module: U:\extras\lib\libcrypto.lib(x86-mont.obj)
0001:007851e0  _bn_mul_mont
Module: U:\extras\lib\libcrypto.lib(bn_recp.obj)
0001:00785780  _BN_RECP_CTX_init
0001:007857d0* _BN_RECP_CTX_new
0001:00785820  _BN_RECP_CTX_free
0001:00785860  _BN_RECP_CTX_set
0001:007858c0  _BN_mod_mul_reciprocal
0001:00785c80* _BN_div_recp
0001:007860c0* _BN_reciprocal
Module: U:\extras\lib\libcrypto.lib(bn_prime.obj)
0001:007867e0  _BN_GENCB_call
0001:00786870  _BN_generate_prime_ex
0001:00786f40  _BN_is_prime_ex
0001:00786f60  _BN_is_prime_fasttest_ex
Module: U:\extras\lib\libcrypto.lib(x_pkey.obj)
0001:00788470* _i2d_X509_PKEY
0001:00788490* _d2i_X509_PKEY
0001:00788980  _X509_PKEY_new
0001:00788a60  _X509_PKEY_free
Module: U:\extras\lib\libcrypto.lib(nsseq.obj)
0001:00788b40  _d2i_NETSCAPE_CERT_SEQUENCE
0001:00788c00* _NETSCAPE_CERT_SEQUENCE_it
0001:00788b70  _i2d_NETSCAPE_CERT_SEQUENCE
0001:00788ba0* _NETSCAPE_CERT_SEQUENCE_new
0001:00788bc0* _NETSCAPE_CERT_SEQUENCE_free
Module: U:\extras\lib\libcrypto.lib(ecp_nist.obj)
0001:00788ca0* _ec_GFp_nist_field_sqr
0001:00788db0* _ec_GFp_nist_field_mul
0001:00788ec0* _ec_GFp_nist_group_set_curve
0001:00789070* _ec_GFp_nist_group_copy
0001:00789090  _EC_GFp_nist_method
Module: U:\extras\lib\libcrypto.lib(ecp_mont.obj)
0001:00789160* _ec_GFp_mont_field_set_to_one
0001:007891d0* _ec_GFp_mont_field_decode
0001:00789250* _ec_GFp_mont_field_encode
0001:007892d0* _ec_GFp_mont_field_sqr
0001:00789350* _ec_GFp_mont_field_mul
0001:007893e0* _ec_GFp_mont_group_set_curve
0001:007895a0* _ec_GFp_mont_group_copy
0001:00789690* _ec_GFp_mont_group_clear_finish
0001:007896e0* _ec_GFp_mont_group_finish
0001:00789730* _ec_GFp_mont_group_init
0001:00789760  _EC_GFp_mont_method
Module: U:\extras\lib\libcrypto.lib(tb_ecdh.obj)
0001:00789830* _ENGINE_unregister_ECDH
0001:00789850* _ENGINE_register_ECDH
0001:007898b0* _ENGINE_register_all_ECDH
0001:00789910* _ENGINE_set_default_ECDH
0001:00789970  _ENGINE_get_default_ECDH
0001:00789990  _ENGINE_get_ECDH
0001:007899a0* _ENGINE_set_ECDH
Module: U:\extras\lib\libcrypto.lib(ech_ossl.obj)
0001:00789f50  _ECDH_OpenSSL
Module: U:\extras\lib\libcrypto.lib(tb_ecdsa.obj)
0001:00789f90* _ENGINE_unregister_ECDSA
0001:00789fb0* _ENGINE_register_ECDSA
0001:0078a010* _ENGINE_register_all_ECDSA
0001:0078a070* _ENGINE_set_default_ECDSA
0001:0078a0d0  _ENGINE_get_default_ECDSA
0001:0078a0f0  _ENGINE_get_ECDSA
0001:0078a100* _ENGINE_set_ECDSA
Module: U:\extras\lib\libcrypto.lib(ecs_ossl.obj)
0001:0078b070  _ECDSA_OpenSSL
Module: U:\extras\lib\libcrypto.lib(p12_p8d.obj)
0001:0078b090  _PKCS8_decrypt
Module: U:\extras\lib\libcrypto.lib(pem_pk8.obj)
0001:0078b420* _PEM_write_bio_PKCS8PrivateKey_nid
0001:0078b470  _PEM_write_bio_PKCS8PrivateKey
0001:0078b4c0* _i2d_PKCS8PrivateKey_bio
0001:0078b510* _i2d_PKCS8PrivateKey_nid_bio
0001:0078b560* _d2i_PKCS8PrivateKey_bio
0001:0078b6c0* _i2d_PKCS8PrivateKey_fp
0001:0078b770* _i2d_PKCS8PrivateKey_nid_fp
0001:0078b820* _PEM_write_PKCS8PrivateKey_nid
0001:0078b8d0* _PEM_write_PKCS8PrivateKey
0001:0078b980* _d2i_PKCS8PrivateKey_fp
0001:0078ba10* _PEM_read_bio_PKCS8
0001:0078ba50* _PEM_read_PKCS8
0001:0078ba90* _PEM_write_bio_PKCS8
0001:0078baf0* _PEM_write_PKCS8
0001:0078bb50* _PEM_read_bio_PKCS8_PRIV_KEY_INFO
0001:0078bb90* _PEM_read_PKCS8_PRIV_KEY_INFO
0001:0078bbd0* _PEM_write_bio_PKCS8_PRIV_KEY_INFO
0001:0078bc30* _PEM_write_PKCS8_PRIV_KEY_INFO
Module: U:\extras\lib\libcrypto.lib(cfb128.obj)
0001:0078c040  _CRYPTO_cfb128_encrypt
0001:0078c490  _CRYPTO_cfb128_1_encrypt
0001:0078c540  _CRYPTO_cfb128_8_encrypt
Module: U:\extras\lib\libcrypto.lib(ofb128.obj)
0001:0078c5a0  _CRYPTO_ofb128_encrypt
Module: U:\extras\lib\libcrypto.lib(ui_openssl.obj)
0001:0078ce30  _UI_OpenSSL
Module: U:\extras\lib\libcrypto.lib(cms_asn1.obj)
0001:0078d010  _CMS_IssuerAndSerialNumber_it
0001:0078d050* _CMS_OtherCertificateFormat_it
0001:0078d090  _CMS_CertificateChoices_it
0001:0078d0d0* _CMS_SignerIdentifier_it
0001:0078d110* _CMS_EncapsulatedContentInfo_it
0001:0078d140  _CMS_SignerInfo_it
0001:0078d180* _CMS_OtherRevocationInfoFormat_it
0001:0078d1c0  _CMS_RevocationInfoChoice_it
0001:0078d1f0  _CMS_SignedData_it
0001:0078d220* _CMS_OriginatorInfo_it
0001:0078d260* _CMS_EncryptedContentInfo_it
0001:0078d2a0  _CMS_KeyTransRecipientInfo_it
0001:0078d2e0  _CMS_OtherKeyAttribute_it
0001:0078d320* _CMS_RecipientKeyIdentifier_it
0001:0078d360* _CMS_KeyAgreeRecipientIdentifier_it
0001:0078d3a0* _CMS_RecipientEncryptedKey_it
0001:0078d3e0* _CMS_OriginatorPublicKey_it
0001:0078d420* _CMS_OriginatorIdentifierOrKey_it
0001:0078d460* _CMS_KeyAgreeRecipientInfo_it
0001:0078d490* _CMS_KEKIdentifier_it
0001:0078d4d0  _CMS_KEKRecipientInfo_it
0001:0078d510* _CMS_PasswordRecipientInfo_it
0001:0078d550* _CMS_OtherRecipientInfo_it
0001:0078d580  _CMS_RecipientInfo_it
0001:0078d5b0  _CMS_EnvelopedData_it
0001:0078d5e0  _CMS_DigestedData_it
0001:0078d610  _CMS_EncryptedData_it
0001:0078d650* _CMS_AuthenticatedData_it
0001:0078d680  _CMS_CompressedData_it
0001:0078d6b0  _CMS_ContentInfo_it
0001:0078d6e0  _CMS_Attributes_Sign_it
0001:0078d720  _CMS_Attributes_Verify_it
0001:0078d750* _CMS_ReceiptsFrom_it
0001:0078d780* _CMS_ReceiptRequest_it
0001:0078d7b0* _CMS_Receipt_it
Module: U:\extras\lib\libcrypto.lib(cms_att.obj)
0001:0078e730  _CMS_signed_get_attr_count
0001:0078e750  _CMS_signed_get_attr_by_NID
0001:0078e770* _CMS_signed_get_attr_by_OBJ
0001:0078e790* _CMS_signed_get_attr
0001:0078e7b0* _CMS_signed_delete_attr
0001:0078e7d0* _CMS_signed_add1_attr
0001:0078e800* _CMS_signed_add1_attr_by_OBJ
0001:0078e840  _CMS_signed_add1_attr_by_NID
0001:0078e880* _CMS_signed_add1_attr_by_txt
0001:0078e8c0  _CMS_signed_get0_data_by_OBJ
0001:0078e8e0* _CMS_unsigned_get_attr_count
0001:0078e900* _CMS_unsigned_get_attr_by_NID
0001:0078e920* _CMS_unsigned_get_attr_by_OBJ
0001:0078e940* _CMS_unsigned_get_attr
0001:0078e960* _CMS_unsigned_delete_attr
0001:0078e980* _CMS_unsigned_add1_attr
0001:0078e9b0* _CMS_unsigned_add1_attr_by_OBJ
0001:0078e9f0* _CMS_unsigned_add1_attr_by_NID
0001:0078ea30* _CMS_unsigned_add1_attr_by_txt
0001:0078ea70* _CMS_unsigned_get0_data_by_OBJ
Module: U:\extras\lib\libcrypto.lib(cms_lib.obj)
0001:0078ea90  _d2i_CMS_ContentInfo
0001:0078eac0  _i2d_CMS_ContentInfo
0001:0078eaf0  _CMS_ContentInfo_new
0001:0078eb10  _CMS_ContentInfo_free
0001:0078eb30* _CMS_ContentInfo_print_ctx
0001:0078eb70* _CMS_get0_type
0001:0078eb90  _CMS_get0_content
0001:0078ec70  _CMS_dataFinal
0001:0078ee40* _cms_content_bio
0001:0078eed0* _priv_cms_Data_create
0001:0078ef60  _CMS_dataInit
0001:0078f120  _CMS_get0_eContentType
0001:0078f1d0* _CMS_set1_eContentType
0001:0078f2e0* _CMS_is_detached
0001:0078f320* _CMS_set_detached
0001:0078f3e0  _cms_DigestAlgorithm_set
0001:0078f430  _cms_DigestAlgorithm_init_bio
0001:0078f540  _cms_DigestAlgorithm_find_ctx
0001:0078f660* _CMS_add0_CertificateChoices
0001:0078f740* _CMS_add0_cert
0001:0078f910  _CMS_add1_cert
0001:0078f970* _CMS_add0_RevocationInfoChoice
0001:0078fa50* _CMS_add0_crl
0001:0078fb50* _CMS_add1_crl
0001:0078fc70* _CMS_get1_certs
0001:0078fdb0* _CMS_get1_crls
Module: U:\extras\lib\libcrypto.lib(cms_enc.obj)
0001:0078ff10  _cms_EncryptedContent_init_bio
0001:007903e0  _cms_EncryptedContent_init
0001:00790510* _CMS_EncryptedData_set1_key
0001:00790780  _cms_EncryptedData_init_bio
Module: U:\extras\lib\libcrypto.lib(aes_wrap.obj)
0001:007907b0  _AES_wrap_key
0001:00790940  _AES_unwrap_key
Module: U:\extras\lib\libcrypto.lib(dso_lib.obj)
0001:00790b00* _DSO_set_default_method
0001:00790b10* _DSO_get_default_method
0001:00790b20* _DSO_get_method
0001:00790b30* _DSO_set_method
0001:00790b60* _DSO_new_method
0001:00790c90* _DSO_new
0001:00790cb0  _DSO_free
0001:00790e30* _DSO_flags
0001:00790e50* _DSO_up_ref
0001:00790ed0* _DSO_bind_var
0001:00790fa0  _DSO_bind_func
0001:00791070* _DSO_ctrl
0001:00791170* _DSO_set_name_converter
0001:007911d0* _DSO_get_filename
0001:00791220* _DSO_set_filename
0001:00791360  _DSO_load
0001:00791570* _DSO_merge
0001:00791600* _DSO_convert_filename
0001:00791760* _DSO_get_loaded_filename
0001:007917b0* _DSO_pathbyaddr
0001:00791830* _DSO_global_lookup
Module: U:\extras\lib\libcrypto.lib(x509rset.obj)
0001:007918b0* _X509_REQ_set_version
0001:007918e0  _X509_REQ_set_subject_name
0001:00791910  _X509_REQ_set_pubkey
Module: U:\extras\lib\libcrypto.lib(conf_def.obj)
0001:00792cc0  _NCONF_default
0001:00792cd0* _NCONF_WIN32
0001:00792ce0* _CONF_def_version
Module: U:\extras\lib\libcrypto.lib(conf_api.obj)
0001:00792eb0  __CONF_get_section
0001:00792f00  __CONF_get_section_values
0001:00792f50  __CONF_add_string
0001:00792ff0  __CONF_get_string
0001:007930d0  __CONF_new_data
0001:00793130  __CONF_free_data
0001:007931c0  __CONF_new_section
Module: U:\extras\lib\libcrypto.lib(asn_pack.obj)
0001:00793370* _ASN1_seq_unpack
0001:00793400* _ASN1_seq_pack
0001:00793530* _ASN1_unpack_string
0001:007935a0* _ASN1_pack_string
0001:007936d0  _ASN1_item_pack
0001:007937f0  _ASN1_item_unpack
Module: U:\extras\lib\libcrypto.lib(p12_utl.obj)
0001:00793890  _OPENSSL_asc2uni
0001:00793930* _OPENSSL_uni2asc
0001:007939c0* _i2d_PKCS12_bio
0001:007939f0* _i2d_PKCS12_fp
0001:00793a20* _d2i_PKCS12_bio
0001:00793a50* _d2i_PKCS12_fp
0001:00793a80* _PKCS12_x5092certbag
0001:00793ab0* _PKCS12_x509crl2certbag
0001:00793ae0* _PKCS12_certbag2x509
0001:00793b30* _PKCS12_certbag2x509crl
Module: U:\extras\lib\libcrypto.lib(bio_md.obj)
0001:00793fb0  _BIO_f_md
Module: U:\extras\lib\libcrypto.lib(bio_enc.obj)
0001:00794a10  _BIO_f_cipher
0001:00794a20* _BIO_set_cipher
Module: U:\extras\lib\libcrypto.lib(bss_null.obj)
0001:00794ba0  _BIO_s_null
Module: U:\extras\lib\libcrypto.lib(pk7_attr.obj)
0001:00794c00* _PKCS7_add_attrib_smimecap
0001:00794ca0* _PKCS7_get_smimecap
0001:00794d10* _PKCS7_simple_smimecap
0001:00794e10* _PKCS7_add_attrib_content_type
0001:00794e80  _PKCS7_add0_attrib_signing_time
0001:00794f00  _PKCS7_add1_attrib_digest
Module: U:\extras\lib\libcrypto.lib(bn_gf2m.obj)
0001:00795150  _BN_GF2m_add
0001:00795260  _BN_GF2m_mod_arr
0001:007955d0* _BN_GF2m_mod
0001:00795730  _BN_GF2m_mod_sqr_arr
0001:007958d0  _BN_GF2m_mod_mul_arr
0001:00795b50* _BN_GF2m_mod_mul
0001:00795cc0* _BN_GF2m_mod_sqr
0001:00795e20* _BN_GF2m_mod_inv
0001:00796120* _BN_GF2m_mod_inv_arr
0001:007961c0  _BN_GF2m_mod_div
0001:00796390* _BN_GF2m_mod_div_arr
0001:00796470* _BN_GF2m_mod_exp_arr
0001:007965e0* _BN_GF2m_mod_exp
0001:00796750  _BN_GF2m_mod_sqrt_arr
0001:007967f0* _BN_GF2m_mod_sqrt
0001:007969d0  _BN_GF2m_mod_solve_quad_arr
0001:00796de0* _BN_GF2m_mod_solve_quad
0001:00796f40  _BN_GF2m_poly2arr
0001:00797000* _BN_GF2m_arr2poly
Module: U:\extras\lib\libcrypto.lib(ec2_mult.obj)
0001:00797a80  _ec_GF2m_simple_mul
0001:00797cf0  _ec_GF2m_precompute_mult
0001:00797d00  _ec_GF2m_have_precompute_mult
Module: U:\extras\lib\libcrypto.lib(f_string.obj)
0001:00797d30  _i2a_ASN1_STRING
0001:00797e70* _a2i_ASN1_STRING
Module: U:\extras\lib\libcrypto.lib(f_int.obj)
0001:00798240  _i2a_ASN1_INTEGER
0001:007983b0* _a2i_ASN1_INTEGER
Module: U:\extras\lib\libcrypto.lib(bn_nist.obj)
0001:007987a0  _BN_get0_nist_prime_192
0001:007987b0  _BN_get0_nist_prime_224
0001:007987c0  _BN_get0_nist_prime_256
0001:007987d0  _BN_get0_nist_prime_384
0001:007987e0  _BN_get0_nist_prime_521
0001:007987f0  _BN_nist_mod_192
0001:00798b80  _BN_nist_mod_224
0001:00799090  _BN_nist_mod_256
0001:007998a0  _BN_nist_mod_384
0001:0079a210  _BN_nist_mod_521
Module: U:\extras\lib\libcrypto.lib(ecp_smpl.obj)
0001:0079ac90  _ec_GFp_simple_is_at_infinity
0001:0079acb0* _ec_GFp_simple_field_sqr
0001:0079ace0* _ec_GFp_simple_field_mul
0001:0079ad10  _ec_GFp_simple_point_copy
0001:0079ad80  _ec_GFp_simple_group_copy
0001:0079ae00  _ec_GFp_simple_point_set_to_infinity
0001:0079ae30  _ec_GFp_simple_get_Jprojective_coordinates_GFp
0001:0079afe0  _ec_GFp_simple_group_get_curve
0001:0079b170  _ec_GFp_simple_point_clear_finish
0001:0079b1b0  _ec_GFp_simple_group_clear_finish
0001:0079b200  _ec_GFp_simple_points_make_affine
0001:0079b790  _ec_GFp_simple_point_get_affine_coordinates
0001:0079bb80  _ec_GFp_simple_make_affine
0001:0079bcd0  _ec_GFp_simple_cmp
0001:0079c080  _ec_GFp_simple_is_on_curve
0001:0079c430  _ec_GFp_simple_invert
0001:0079c480  _ec_GFp_simple_dbl
0001:0079cae0  _ec_GFp_simple_add
0001:0079d270  _ec_GFp_simple_group_get_degree
0001:0079d280  _ec_GFp_simple_oct2point
0001:0079d6e0  _ec_GFp_simple_point2oct
0001:0079dc30  _ec_GFp_simple_set_Jprojective_coordinates_GFp
0001:0079de40  _ec_GFp_simple_set_compressed_coordinates
0001:0079e3f0  _ec_GFp_simple_point_set_affine_coordinates
0001:0079e480  _ec_GFp_simple_point_finish
0001:0079e4b0  _ec_GFp_simple_group_finish
0001:0079e4f0  _ec_GFp_simple_point_init
0001:0079e530  _ec_GFp_simple_group_init
0001:0079e570  _ec_GFp_simple_group_check_discriminant
0001:0079e830  _ec_GFp_simple_group_set_curve
0001:0079ea60* _EC_GFp_simple_method
Module: U:\extras\lib\libcrypto.lib(p12_decr.obj)
0001:0079eb30* _PKCS12_pbe_crypt
0001:0079ed10  _PKCS12_item_decrypt_d2i
0001:0079ee50  _PKCS12_item_i2d_encrypt
Module: U:\extras\lib\libcrypto.lib(p12_p8e.obj)
0001:0079eff0  _PKCS8_encrypt
Module: U:\extras\lib\libcrypto.lib(cms_io.obj)
0001:0079f190  _CMS_stream
0001:0079f220* _d2i_CMS_bio
0001:0079f250* _i2d_CMS_bio
0001:0079f280* _PEM_read_bio_CMS
0001:0079f2c0* _PEM_read_CMS
0001:0079f300* _PEM_write_bio_CMS
0001:0079f360* _PEM_write_CMS
0001:0079f3c0* _BIO_new_CMS
0001:0079f3f0* _i2d_CMS_bio_stream
0001:0079f430* _PEM_write_bio_CMS_stream
0001:0079f470* _SMIME_write_CMS
0001:0079f4f0* _SMIME_read_CMS
Module: U:\extras\lib\libcrypto.lib(cms_dd.obj)
0001:0079f520* _cms_DigestedData_create
0001:0079f5a0  _cms_DigestedData_init_bio
0001:0079f5d0  _cms_DigestedData_do_final
Module: U:\extras\lib\libcrypto.lib(cms_cd.obj)
0001:0079f740* _cms_CompressedData_create
0001:0079f820  _cms_CompressedData_init_bio
Module: U:\extras\lib\libcrypto.lib(dso_openssl.obj)
0001:0079f910  _DSO_METHOD_openssl
Module: U:\extras\lib\libcrypto.lib(a_set.obj)
0001:0079f970  _i2d_ASN1_SET
0001:0079fce0  _d2i_ASN1_SET
Module: U:\extras\lib\libcrypto.lib(p12_asn.obj)
0001:007a0010* _d2i_PKCS12
0001:007a02a0  _PKCS12_it
0001:007a0040* _i2d_PKCS12
0001:007a0070* _PKCS12_new
0001:007a0090* _PKCS12_free
0001:007a00b0* _d2i_PKCS12_MAC_DATA
0001:007a02d0* _PKCS12_MAC_DATA_it
0001:007a00e0* _i2d_PKCS12_MAC_DATA
0001:007a0110* _PKCS12_MAC_DATA_new
0001:007a0130* _PKCS12_MAC_DATA_free
0001:007a0150* _d2i_PKCS12_BAGS
0001:007a0300* _PKCS12_BAGS_it
0001:007a0180* _i2d_PKCS12_BAGS
0001:007a01b0  _PKCS12_BAGS_new
0001:007a01d0* _PKCS12_BAGS_free
0001:007a01f0* _d2i_PKCS12_SAFEBAG
0001:007a0330* _PKCS12_SAFEBAG_it
0001:007a0220* _i2d_PKCS12_SAFEBAG
0001:007a0250  _PKCS12_SAFEBAG_new
0001:007a0270* _PKCS12_SAFEBAG_free
0001:007a0360  _PKCS12_SAFEBAGS_it
0001:007a0390  _PKCS12_AUTHSAFES_it
Module: U:\extras\lib\libcrypto.lib(p12_add.obj)
0001:007a0710  _PKCS12_item_pack_safebag
0001:007a0800* _PKCS12_MAKE_KEYBAG
0001:007a0860* _PKCS12_MAKE_SHKEYBAG
0001:007a0950* _PKCS12_pack_p7data
0001:007a0a50* _PKCS12_unpack_p7data
0001:007a0ac0* _PKCS12_pack_p7encdata
0001:007a0cb0* _PKCS12_unpack_p7encdata
0001:007a0d10* _PKCS12_decrypt_skey
0001:007a0d30* _PKCS12_pack_authsafes
0001:007a0d70* _PKCS12_unpack_authsafes
Module: U:\extras\lib\libcrypto.lib(bn_sqrt.obj)
0001:007a0e10  _BN_mod_sqrt
Module: U:\extras\lib\libcrypto.lib(bn_kron.obj)
0001:007a1810  _BN_kronecker
Module: U:\extras\lib\libcrypto.lib(bio_ndef.obj)
0001:007a1d40  _BIO_new_NDEF
Module: U:\extras\lib\libcrypto.lib(asn_mime.obj)
0001:007a2d10  _SMIME_read_ASN1
0001:007a3440* _SMIME_crlf_copy
0001:007a35e0  _i2d_ASN1_bio_stream
0001:007a36f0  _PEM_write_bio_ASN1_stream
0001:007a3b10  _SMIME_write_ASN1
0001:007a44d0* _SMIME_text
Module: U:\extras\lib\libcrypto.lib(dso_null.obj)
0001:007a46c0  _DSO_METHOD_null
Module: U:\extras\lib\libcrypto.lib(bio_asn1.obj)
0001:007a4f00  _BIO_f_asn1
0001:007a4f10  _BIO_asn1_set_prefix
0001:007a4f50* _BIO_asn1_get_prefix
0001:007a4fa0  _BIO_asn1_set_suffix
0001:007a4fe0* _BIO_asn1_get_suffix
Module: U:\extras\lib\libcrypto.lib(bio_b64.obj)
0001:007a6420  _BIO_f_base64


                        +----------------------+
                        |   Imported Symbols   |
                        +----------------------+

Symbol                              Module
======                              ======

___libc_ForkRegisterModule          libc063
___init_dll                         libc063
___libc_Back_termDll                libc063
___libc_ForkDeregisterModule        libc063
__atfork_callback                   libc063
___moddi3                           libc063
___divdi3                           libc063
___libc_GLocaleCtype                libc063
___umoddi3                          libc063
_strlcat                            libc063
__alloca                            libc063
DosGetInfoBlocks                    doscalls
DosCreateMutexSem                   doscalls
DosCloseMutexSem                    doscalls
DosSleep                            doscalls
DosRequestMutexSem                  doscalls
DosQueryMutexSem                    doscalls
DosReleaseMutexSem                  doscalls
___udivdi3                          libc063
DosClose                            doscalls
DosForceDelete                      doscalls
DosSetFilePtr                       doscalls
DosRead                             doscalls
DosWrite                            doscalls
DosSetFileSize                      doscalls
DosResetBuffer                      doscalls
DosQueryFileInfo                    doscalls
DosSetFileLocks                     doscalls
UniCreateUconvObject                uconv
UniFreeUconvObject                  uconv
UniStrToUcs                         uconv
UniStrFromUcs                       uconv
DosScanEnv                          doscalls
DosQueryCurrentDisk                 doscalls
DosQueryPathInfo                    doscalls
DosOpen                             doscalls
DosDelete                           doscalls
DosLoadModule                       doscalls
DosQueryProcAddr                    doscalls
DosFreeModule                       doscalls
DosQuerySysInfo                     doscalls
DosGetDateTime                      doscalls
___stderrp                          libc063
__errno                             libc063
_strlcpy                            libc063
_getgrnam_r                         libc063
_getgrgid_r                         libc063
_getpwnam_r                         libc063
_getpwuid_r                         libc063
_initgroups                         libc063
_gethostbyname                      tcpip32
_hstrerror                          tcpip32
_inet_aton                          tcpip32
_tcp_h_errno1                       tcpip32
_getprotobyname                     tcpip32
_inet_ntoa                          tcpip32
_inet_ntop                          tcpip32
_inet_pton                          tcpip32
_getservbyname                      tcpip32
_getservbyport                      tcpip32
_getprotobynumber                   tcpip32
_gethostname                        tcpip32
_inet_addr                          tcpip32
_gethostbyaddr                      tcpip32
DosQueryFSInfo                      doscalls
___stdinp                           libc063
___stdoutp                          libc063
__exit                              libc063
___fixunsdfdi                       libc063
DosAllocThreadLocalMemory           doscalls
DosFreeThreadLocalMemory            doscalls
___threadid                         libc063
_isspace                            libc063
___flt_rounds                       libc063
__assert                            libc063
__CRT_term                          libc063
__CRT_init                          libc063
__std_getenv                        libc063
__std_memcpy                        libc063
__std_floor                         libc063
__std_malloc                        libc063
__std_strdup                        libc063
__std_time                          libc063
__std_strftime                      libc063
__std_free                          libc063
__std_strnicmp                      libc063
__std_sin                           libc063
__std_cos                           libc063
__std_atan2                         libc063
__std_sqrt                          libc063
__std_acos                          libc063
__std_realloc                       libc063
__std_strchr                        libc063
__std_calloc                        libc063
__std_strtoll                       libc063
__std_strtod                        libc063
__std_strtol                        libc063
__std_stricmp                       libc063
__std_memset                        libc063
__std_pow                           libc063
__std_printf                        libc063
__std_setlocale                     libc063
__std_putchar                       libc063
__std_strcmp                        libc063
__std_strncat                       libc063
__std_strcpy                        libc063
__std_strncmp                       libc063
__std_memmove                       libc063
__std_strncpy                       libc063
__std_sprintf                       libc063
__std_localtime                     libc063
__std_qsort                         libc063
__std_memchr                        libc063
__std_dup                           libc063
__std_fwrite                        libc063
__std_exit                          libc063
___signbit                          libc063
__std_abort                         libc063
__std_fprintf                       libc063
__std_stat                          libc063
__std_strstr                        libc063
__std_opendir                       libc063
__std_readdir                       libc063
__std_closedir                      libc063
__std_strtoull                      libc063
__std_fputc                         libc063
__std_strrchr                       libc063
__std_lseek                         libc063
__std_read                          libc063
__std_mktime                        libc063
__std_write                         libc063
__std_mkstemp                       libc063
__std_unlink                        libc063
__std_dup2                          libc063
__std_close                         libc063
__std_strerror                      libc063
__std_access                        libc063
__std_utimes                        libc063
__std_vasprintf                     libc063
__std_gmtime                        libc063
__std_asctime                       libc063
__std_strcspn                       libc063
__std_ctime                         libc063
__std_atoi                          libc063
__std_finite                        libc063
__std_strpbrk                       libc063
___libc_FH                          libc063
__libsocket_set_errno               tcpip32
__libsocket_getsockname             tcpip32
__libsocket_sock_errno              tcpip32
__std_sscanf                        libc063
__std_gmtime_r                      libc063
__libsocket_send                    tcpip32
__libsocket_recv                    tcpip32
__libsocket_accept                  tcpip32
___libc_TcpipAllocFH44              libc063
__libsocket_soclose                 tcpip32
__libsocket_socket                  tcpip32
__libsocket_bind                    tcpip32
__libsocket_listen                  tcpip32
__std_isinf                         libc063
__std_isnan                         libc063
__std_localtime_r                   libc063
__std_getuid                        libc063
__std_getgid                        libc063
__std_getgroups                     libc063
__std_strtok_r                      libc063
__std_sigsetjmp                     libc063
__std_strtok                        libc063
__std_kill                          libc063
__std_getpid                        libc063
__std_getppid                       libc063
__std_geteuid                       libc063
__std_getegid                       libc063
__std_setuid                        libc063
__std_setgid                        libc063
__std_seteuid                       libc063
__std_setegid                       libc063
__std_getlogin                      libc063
__std_getpgrp                       libc063
__std_setsid                        libc063
__std_setpgid                       libc063
__std_getpgid                       libc063
__std_getsid                        libc063
__std_uname                         libc063
__std_times                         libc063
__std_ttyname                       libc063
__std_isatty                        libc063
__std_mkfifo                        libc063
__std_mknod                         libc063
__std_sysconf                       libc063
__std_getrlimit                     libc063
__std_gettimeofday                  libc063
__std_fstat                         libc063
__std_flock                         libc063
__std_fcntl                         libc063
__std_readdir_r                     libc063
__std_pread                         libc063
__std_pwrite                        libc063
__std_ftruncate                     libc063
__std_timezone                      libc063
__std_strcat                        libc063
__std_open                          libc063
__std_select                        libc063
__libsocket_getpeername             tcpip32
__libsocket_connect                 tcpip32
__libsocket_recvfrom                tcpip32
__libsocket_sendto                  tcpip32
__libsocket_getsockopt              tcpip32
__libsocket_setsockopt              tcpip32
__libsocket_socketpair              tcpip32
___libc_FHClose                     libc063
__libsocket_shutdown                tcpip32
__std_readlink                      libc063
__std_strtoul                       libc063
__std_putenv                        libc063
__std_tzset                         libc063
__std_unsetenv                      libc063
__std_umask                         libc063
__std_environ                       libc063
__std_sleep                         libc063
__std_usleep                        libc063
__std_nanosleep                     libc063
__std_getloadavg                    libc063
__std_strptime                      libc063
__std_glob                          libc063
__std_globfree                      libc063
__std_dlopen                        libc063
__std_dlsym                         libc063
__std_dlclose                       libc063
__std_dlerror                       libc063
__std_mblen                         libc063
__std_nice                          libc063
__std_fnmatch                       libc063
__std_fclose                        libc063
__std_localeconv                    libc063
__std_nl_langinfo                   libc063
__std_getc                          libc063
__std_fileno                        libc063
__std_symlink                       libc063
__std_link                          libc063
__std_popen                         libc063
__std_pclose                        libc063
__std_ceil                          libc063
__std_asinh                         libc063
__std_acosh                         libc063
__std_atanh                         libc063
__std_log1p                         libc063
__std_expm1                         libc063
__std_tan                           libc063
__std_asin                          libc063
__std_atan                          libc063
__std_sinh                          libc063
__std_cosh                          libc063
__std_tanh                          libc063
__std_exp                           libc063
__std_log                           libc063
__std_log10                         libc063
__std_hypot                         libc063
__std_fmod                          libc063
__std_rand_r                        libc063
__std_strcoll                       libc063
__std_ctime_r                       libc063
__getprogname                       libc063
__std_vsnprintf                     libc063
__std_writev                        libc063
__std_getdtablesize                 libc063
__std_strspn                        libc063
__std_ftok                          libc063
__std_waitpid                       libc063
__std_fork                          libc063
__std_execle                        libc063
__std_execl                         libc063
__std_chdir                         libc063
__std_perror                        libc063
__std_pipe                          libc063
__std_fopen                         libc063
__std_fseek                         libc063
__std_ftell                         libc063
__std_clearerr                      libc063
__std_fread                         libc063
__std_remove                        libc063
__std_rename                        libc063
__std_chmod                         libc063
__std_fdopen                        libc063
__std_putc                          libc063
__std_atof                          libc063
__std_atol                          libc063
__std_getcwd                        libc063
__std_lstat                         libc063
__std_utime                         libc063
__std_lchown                        libc063
__std_chown                         libc063
__std_creat                         libc063
__std_mkdir                         libc063
__std_rmdir                         libc063
__std_asctime_r                     libc063
__std_fputs                         libc063
___strnlen                          libc063
__std_vsprintf                      libc063
__std_setmode                       libc063
__std_fflush                        libc063
__std_rewind                        libc063
__std_setvbuf                       libc063
__std_rewinddir                     libc063
__std_signal                        libc063
__std_sigemptyset                   libc063
__std_sigaddset                     libc063
__std_sigprocmask                   libc063
__std_setitimer                     libc063
__std_snprintf                      libc063
__std_siglongjmp                    libc063
DosTrueGetMessage                   msg
___ctordtorInit1                    libc063
___ctordtorTerm1                    libc063
__std_vfprintf                      libc063
__std_iconv                         libc063
__std_iconv_open                    libc063
__std_iconv_close                   libc063
__std_strlen                        libc063
__std_puts                          libc063
__std_memcmp                        libc063
DosEnterCritSec                     doscalls
DosExitCritSec                      doscalls
__gettid                            libc063
DosSetPriority                      doscalls
__endthread                         libc063
__beginthread                       libc063
DosWaitThread                       doscalls
DosCloseEventSem                    doscalls
DosPostEventSem                     doscalls
DosCreateEventSem                   doscalls
DosWaitEventSem                     doscalls
__std_ftime                         libc063
__std_fgets                         libc063
DosQueryModuleHandle                doscalls
DosTmrQueryTime                     doscalls
DosAllocMem                         doscalls
DosFreeMem                          doscalls
___register_frame_table             libc063
___deregister_frame                 libc063
__std_sigaction                     libc063
__std_tcsetattr                     libc063
__std_tcgetattr                     libc063


                        +--------------------+
                        |   Libraries Used   |
                        +--------------------+

U:\extras\lib\libz.lib
U:\extras\lib\xmlrpc.lib
U:\extras\lib\libssl.lib
U:\extras\lib\libcrypto.lib
U:\extras\lib\pthread.lib
U:\extras\lib\expat.lib
U:\extras\lib\poll.lib
U:\extras\lib\xml2.lib
U:\usr\lib\libc_alias.lib
U:\usr\lib\libc_dll.lib
U:\usr\lib\libos2.lib
U:\usr\lib\gcc-lib\i386-pc-os2-emx\3.3.5\libgcc_so_d.lib
U:\usr\lib\libend.lib


                        +-----------------------+
                        |   Linker Statistics   |
                        +-----------------------+

Stack size:  0000 (0.)
Memory size:  007ca920 (8169760.)
Link time: 00:01.36
